Archive member included because of file (symbol)

c:/program files/microchip/xc32/v1.33/bin/bin/../../lib/gcc/pic32mx/4.5.2/../../../../pic32mx/lib\libmchp_peripheral_32MX795F512H.a(soft_reset_lib.o)
                              build/ChaletDuinoV2_795F512H_/debug/Source/exceptions.o (SoftReset)
c:/program files/microchip/xc32/v1.33/bin/bin/../../lib/gcc/pic32mx/4.5.2/../../../../pic32mx/lib\libmchp_peripheral_32MX795F512H.a(pcache.o)
                              build/ChaletDuinoV2_795F512H_/debug/Source/main.o (CheKseg0CacheOn)
c:/program files/microchip/xc32/v1.33/bin/bin/../../lib/gcc/pic32mx/4.5.2/../../../../pic32mx/lib\libmchp_peripheral_32MX795F512H.a(int_configure_system_lib.o)
                              build/ChaletDuinoV2_795F512H_/debug/Source/main.o (INTConfigureSystem)
c:/program files/microchip/xc32/v1.33/bin/bin/../../lib/gcc/pic32mx/4.5.2/../../../../pic32mx/lib\libmchp_peripheral_32MX795F512H.a(int_enable_interrupts_lib.o)
                              build/ChaletDuinoV2_795F512H_/debug/Source/main.o (INTEnableInterrupts)
c:/program files/microchip/xc32/v1.33/bin/bin/../../lib/gcc/pic32mx/4.5.2/../../../../pic32mx/lib\libmchp_peripheral_32MX795F512H.a(int_disable_interrupts_lib.o)
                              build/ChaletDuinoV2_795F512H_/debug/Source/main.o (INTDisableInterrupts)
c:/program files/microchip/xc32/v1.33/bin/bin/../../lib/gcc/pic32mx/4.5.2/../../../../pic32mx/lib\libmchp_peripheral_32MX795F512H.a(int_restore_interrupts_lib.o)
                              build/ChaletDuinoV2_795F512H_/debug/Source/main.o (INTRestoreInterrupts)
c:/program files/microchip/xc32/v1.33/bin/bin/../../lib/gcc/pic32mx/4.5.2/../../../../pic32mx/lib\libpic32.a(memcmp.o)
                              build/ChaletDuinoV2_795F512H_/debug/Source/winc3400_142/driver/source/m2m_flash.o (memcmp)
c:/program files/microchip/xc32/v1.33/bin/bin/../../lib/gcc/pic32mx/4.5.2/../../../../pic32mx/lib\libpic32.a(memcpy.o)
                              build/ChaletDuinoV2_795F512H_/debug/Source/winc3400_142/driver/source/m2m_ssl.o (memcpy)
c:/program files/microchip/xc32/v1.33/bin/bin/../../lib/gcc/pic32mx/4.5.2/../../../../pic32mx/lib\libpic32.a(memset.o)
                              build/ChaletDuinoV2_795F512H_/debug/Source/winc3400_142/driver/source/m2m_hif.o (memset)
c:/program files/microchip/xc32/v1.33/bin/bin/../../lib/gcc/pic32mx/4.5.2/../../../../pic32mx/lib\libpic32.a(strcpy.o)
                              build/ChaletDuinoV2_795F512H_/debug/Source/Terminal.o (strcpy)
c:/program files/microchip/xc32/v1.33/bin/bin/../../lib/gcc/pic32mx/4.5.2/../../../../pic32mx/lib\libpic32.a(strlen.o)
                              build/ChaletDuinoV2_795F512H_/debug/Source/winc3400_142/driver/source/m2m_ota.o (strlen)
c:/program files/microchip/xc32/v1.33/bin/bin/../../lib/gcc/pic32mx/4.5.2/../../../../pic32mx/lib\libpic32.a(default-bootstrap-exception-handler.o)
                              c:/program files/microchip/xc32/v1.33/bin/bin/../../lib/gcc/pic32mx/4.5.2/../../../../pic32mx/lib/./proc/32MX795F512H/crt0_mips32r2.o (_bootstrap_exception_handler)
c:/program files/microchip/xc32/v1.33/bin/bin/../../lib/gcc/pic32mx/4.5.2/../../../../pic32mx/lib\libpic32.a(default-on-reset.o)
                              c:/program files/microchip/xc32/v1.33/bin/bin/../../lib/gcc/pic32mx/4.5.2/../../../../pic32mx/lib/./proc/32MX795F512H/crt0_mips32r2.o (_on_reset)
c:/program files/microchip/xc32/v1.33/bin/bin/../../lib/gcc/pic32mx/4.5.2/../../../../pic32mx/lib\libpic32.a(default-on-bootstrap.o)
                              c:/program files/microchip/xc32/v1.33/bin/bin/../../lib/gcc/pic32mx/4.5.2/../../../../pic32mx/lib/./proc/32MX795F512H/crt0_mips32r2.o (_on_bootstrap)
c:/program files/microchip/xc32/v1.33/bin/bin/../../lib/gcc/pic32mx/4.5.2/../../../../pic32mx/lib\libpic32.a(default-nmi-handler.o)
                              c:/program files/microchip/xc32/v1.33/bin/bin/../../lib/gcc/pic32mx/4.5.2/../../../../pic32mx/lib/./proc/32MX795F512H/crt0_mips32r2.o (_nmi_handler)
c:/program files/microchip/xc32/v1.33/bin/bin/../../lib/gcc/pic32mx/4.5.2/../../../../pic32mx/lib\libpic32.a(close.o)
                              build/ChaletDuinoV2_795F512H_/debug/Source/WiFiCtrl.o (close)
c:/program files/microchip/xc32/v1.33/bin/bin/../../lib/gcc/pic32mx/4.5.2/../../../../pic32mx/lib\libpic32.a(general-exception.o)
                              c:/program files/microchip/xc32/v1.33/bin/bin/../../lib/gcc/pic32mx/4.5.2/../../../../pic32mx/lib/./proc/32MX795F512H/crt0_mips32r2.o (_general_exception_context)
c:/program files/microchip/xc32/v1.33/bin/bin/../../lib/gcc/pic32mx/4.5.2/../../../../pic32mx/lib\libpic32.a(vector0.o)
                              c:/program files/microchip/xc32/v1.33/bin/bin/../../lib/gcc/pic32mx/4.5.2/../../../../pic32mx/lib/./proc/32MX795F512H\default_isr_vectors.o (__vector_dispatch_0)
c:/program files/microchip/xc32/v1.33/bin/bin/../../lib/gcc/pic32mx/4.5.2/../../../../pic32mx/lib\libpic32.a(vector1.o)
                              c:/program files/microchip/xc32/v1.33/bin/bin/../../lib/gcc/pic32mx/4.5.2/../../../../pic32mx/lib/./proc/32MX795F512H\default_isr_vectors.o (__vector_dispatch_1)
c:/program files/microchip/xc32/v1.33/bin/bin/../../lib/gcc/pic32mx/4.5.2/../../../../pic32mx/lib\libpic32.a(vector2.o)
                              c:/program files/microchip/xc32/v1.33/bin/bin/../../lib/gcc/pic32mx/4.5.2/../../../../pic32mx/lib/./proc/32MX795F512H\default_isr_vectors.o (__vector_dispatch_2)
c:/program files/microchip/xc32/v1.33/bin/bin/../../lib/gcc/pic32mx/4.5.2/../../../../pic32mx/lib\libpic32.a(vector5.o)
                              c:/program files/microchip/xc32/v1.33/bin/bin/../../lib/gcc/pic32mx/4.5.2/../../../../pic32mx/lib/./proc/32MX795F512H\default_isr_vectors.o (__vector_dispatch_5)
c:/program files/microchip/xc32/v1.33/bin/bin/../../lib/gcc/pic32mx/4.5.2/../../../../pic32mx/lib\libpic32.a(vector6.o)
                              c:/program files/microchip/xc32/v1.33/bin/bin/../../lib/gcc/pic32mx/4.5.2/../../../../pic32mx/lib/./proc/32MX795F512H\default_isr_vectors.o (__vector_dispatch_6)
c:/program files/microchip/xc32/v1.33/bin/bin/../../lib/gcc/pic32mx/4.5.2/../../../../pic32mx/lib\libpic32.a(vector8.o)
                              c:/program files/microchip/xc32/v1.33/bin/bin/../../lib/gcc/pic32mx/4.5.2/../../../../pic32mx/lib/./proc/32MX795F512H\default_isr_vectors.o (__vector_dispatch_8)
c:/program files/microchip/xc32/v1.33/bin/bin/../../lib/gcc/pic32mx/4.5.2/../../../../pic32mx/lib\libpic32.a(vector9.o)
                              c:/program files/microchip/xc32/v1.33/bin/bin/../../lib/gcc/pic32mx/4.5.2/../../../../pic32mx/lib/./proc/32MX795F512H\default_isr_vectors.o (__vector_dispatch_9)
c:/program files/microchip/xc32/v1.33/bin/bin/../../lib/gcc/pic32mx/4.5.2/../../../../pic32mx/lib\libpic32.a(vector10.o)
                              c:/program files/microchip/xc32/v1.33/bin/bin/../../lib/gcc/pic32mx/4.5.2/../../../../pic32mx/lib/./proc/32MX795F512H\default_isr_vectors.o (__vector_dispatch_10)
c:/program files/microchip/xc32/v1.33/bin/bin/../../lib/gcc/pic32mx/4.5.2/../../../../pic32mx/lib\libpic32.a(vector11.o)
                              c:/program files/microchip/xc32/v1.33/bin/bin/../../lib/gcc/pic32mx/4.5.2/../../../../pic32mx/lib/./proc/32MX795F512H\default_isr_vectors.o (__vector_dispatch_11)
c:/program files/microchip/xc32/v1.33/bin/bin/../../lib/gcc/pic32mx/4.5.2/../../../../pic32mx/lib\libpic32.a(vector12.o)
                              c:/program files/microchip/xc32/v1.33/bin/bin/../../lib/gcc/pic32mx/4.5.2/../../../../pic32mx/lib/./proc/32MX795F512H\default_isr_vectors.o (__vector_dispatch_12)
c:/program files/microchip/xc32/v1.33/bin/bin/../../lib/gcc/pic32mx/4.5.2/../../../../pic32mx/lib\libpic32.a(vector13.o)
                              c:/program files/microchip/xc32/v1.33/bin/bin/../../lib/gcc/pic32mx/4.5.2/../../../../pic32mx/lib/./proc/32MX795F512H\default_isr_vectors.o (__vector_dispatch_13)
c:/program files/microchip/xc32/v1.33/bin/bin/../../lib/gcc/pic32mx/4.5.2/../../../../pic32mx/lib\libpic32.a(vector14.o)
                              c:/program files/microchip/xc32/v1.33/bin/bin/../../lib/gcc/pic32mx/4.5.2/../../../../pic32mx/lib/./proc/32MX795F512H\default_isr_vectors.o (__vector_dispatch_14)
c:/program files/microchip/xc32/v1.33/bin/bin/../../lib/gcc/pic32mx/4.5.2/../../../../pic32mx/lib\libpic32.a(vector16.o)
                              c:/program files/microchip/xc32/v1.33/bin/bin/../../lib/gcc/pic32mx/4.5.2/../../../../pic32mx/lib/./proc/32MX795F512H\default_isr_vectors.o (__vector_dispatch_16)
c:/program files/microchip/xc32/v1.33/bin/bin/../../lib/gcc/pic32mx/4.5.2/../../../../pic32mx/lib\libpic32.a(vector17.o)
                              c:/program files/microchip/xc32/v1.33/bin/bin/../../lib/gcc/pic32mx/4.5.2/../../../../pic32mx/lib/./proc/32MX795F512H\default_isr_vectors.o (__vector_dispatch_17)
c:/program files/microchip/xc32/v1.33/bin/bin/../../lib/gcc/pic32mx/4.5.2/../../../../pic32mx/lib\libpic32.a(vector18.o)
                              c:/program files/microchip/xc32/v1.33/bin/bin/../../lib/gcc/pic32mx/4.5.2/../../../../pic32mx/lib/./proc/32MX795F512H\default_isr_vectors.o (__vector_dispatch_18)
c:/program files/microchip/xc32/v1.33/bin/bin/../../lib/gcc/pic32mx/4.5.2/../../../../pic32mx/lib\libpic32.a(vector19.o)
                              c:/program files/microchip/xc32/v1.33/bin/bin/../../lib/gcc/pic32mx/4.5.2/../../../../pic32mx/lib/./proc/32MX795F512H\default_isr_vectors.o (__vector_dispatch_19)
c:/program files/microchip/xc32/v1.33/bin/bin/../../lib/gcc/pic32mx/4.5.2/../../../../pic32mx/lib\libpic32.a(vector20.o)
                              c:/program files/microchip/xc32/v1.33/bin/bin/../../lib/gcc/pic32mx/4.5.2/../../../../pic32mx/lib/./proc/32MX795F512H\default_isr_vectors.o (__vector_dispatch_20)
c:/program files/microchip/xc32/v1.33/bin/bin/../../lib/gcc/pic32mx/4.5.2/../../../../pic32mx/lib\libpic32.a(vector21.o)
                              c:/program files/microchip/xc32/v1.33/bin/bin/../../lib/gcc/pic32mx/4.5.2/../../../../pic32mx/lib/./proc/32MX795F512H\default_isr_vectors.o (__vector_dispatch_21)
c:/program files/microchip/xc32/v1.33/bin/bin/../../lib/gcc/pic32mx/4.5.2/../../../../pic32mx/lib\libpic32.a(vector22.o)
                              c:/program files/microchip/xc32/v1.33/bin/bin/../../lib/gcc/pic32mx/4.5.2/../../../../pic32mx/lib/./proc/32MX795F512H\default_isr_vectors.o (__vector_dispatch_22)
c:/program files/microchip/xc32/v1.33/bin/bin/../../lib/gcc/pic32mx/4.5.2/../../../../pic32mx/lib\libpic32.a(vector23.o)
                              c:/program files/microchip/xc32/v1.33/bin/bin/../../lib/gcc/pic32mx/4.5.2/../../../../pic32mx/lib/./proc/32MX795F512H\default_isr_vectors.o (__vector_dispatch_23)
c:/program files/microchip/xc32/v1.33/bin/bin/../../lib/gcc/pic32mx/4.5.2/../../../../pic32mx/lib\libpic32.a(vector24.o)
                              c:/program files/microchip/xc32/v1.33/bin/bin/../../lib/gcc/pic32mx/4.5.2/../../../../pic32mx/lib/./proc/32MX795F512H\default_isr_vectors.o (__vector_dispatch_24)
c:/program files/microchip/xc32/v1.33/bin/bin/../../lib/gcc/pic32mx/4.5.2/../../../../pic32mx/lib\libpic32.a(vector25.o)
                              c:/program files/microchip/xc32/v1.33/bin/bin/../../lib/gcc/pic32mx/4.5.2/../../../../pic32mx/lib/./proc/32MX795F512H\default_isr_vectors.o (__vector_dispatch_25)
c:/program files/microchip/xc32/v1.33/bin/bin/../../lib/gcc/pic32mx/4.5.2/../../../../pic32mx/lib\libpic32.a(vector26.o)
                              c:/program files/microchip/xc32/v1.33/bin/bin/../../lib/gcc/pic32mx/4.5.2/../../../../pic32mx/lib/./proc/32MX795F512H\default_isr_vectors.o (__vector_dispatch_26)
c:/program files/microchip/xc32/v1.33/bin/bin/../../lib/gcc/pic32mx/4.5.2/../../../../pic32mx/lib\libpic32.a(vector27.o)
                              c:/program files/microchip/xc32/v1.33/bin/bin/../../lib/gcc/pic32mx/4.5.2/../../../../pic32mx/lib/./proc/32MX795F512H\default_isr_vectors.o (__vector_dispatch_27)
c:/program files/microchip/xc32/v1.33/bin/bin/../../lib/gcc/pic32mx/4.5.2/../../../../pic32mx/lib\libpic32.a(vector28.o)
                              c:/program files/microchip/xc32/v1.33/bin/bin/../../lib/gcc/pic32mx/4.5.2/../../../../pic32mx/lib/./proc/32MX795F512H\default_isr_vectors.o (__vector_dispatch_28)
c:/program files/microchip/xc32/v1.33/bin/bin/../../lib/gcc/pic32mx/4.5.2/../../../../pic32mx/lib\libpic32.a(vector29.o)
                              c:/program files/microchip/xc32/v1.33/bin/bin/../../lib/gcc/pic32mx/4.5.2/../../../../pic32mx/lib/./proc/32MX795F512H\default_isr_vectors.o (__vector_dispatch_29)
c:/program files/microchip/xc32/v1.33/bin/bin/../../lib/gcc/pic32mx/4.5.2/../../../../pic32mx/lib\libpic32.a(vector30.o)
                              c:/program files/microchip/xc32/v1.33/bin/bin/../../lib/gcc/pic32mx/4.5.2/../../../../pic32mx/lib/./proc/32MX795F512H\default_isr_vectors.o (__vector_dispatch_30)
c:/program files/microchip/xc32/v1.33/bin/bin/../../lib/gcc/pic32mx/4.5.2/../../../../pic32mx/lib\libpic32.a(vector31.o)
                              c:/program files/microchip/xc32/v1.33/bin/bin/../../lib/gcc/pic32mx/4.5.2/../../../../pic32mx/lib/./proc/32MX795F512H\default_isr_vectors.o (__vector_dispatch_31)
c:/program files/microchip/xc32/v1.33/bin/bin/../../lib/gcc/pic32mx/4.5.2/../../../../pic32mx/lib\libpic32.a(vector32.o)
                              c:/program files/microchip/xc32/v1.33/bin/bin/../../lib/gcc/pic32mx/4.5.2/../../../../pic32mx/lib/./proc/32MX795F512H\default_isr_vectors.o (__vector_dispatch_32)
c:/program files/microchip/xc32/v1.33/bin/bin/../../lib/gcc/pic32mx/4.5.2/../../../../pic32mx/lib\libpic32.a(vector33.o)
                              c:/program files/microchip/xc32/v1.33/bin/bin/../../lib/gcc/pic32mx/4.5.2/../../../../pic32mx/lib/./proc/32MX795F512H\default_isr_vectors.o (__vector_dispatch_33)
c:/program files/microchip/xc32/v1.33/bin/bin/../../lib/gcc/pic32mx/4.5.2/../../../../pic32mx/lib\libpic32.a(vector34.o)
                              c:/program files/microchip/xc32/v1.33/bin/bin/../../lib/gcc/pic32mx/4.5.2/../../../../pic32mx/lib/./proc/32MX795F512H\default_isr_vectors.o (__vector_dispatch_34)
c:/program files/microchip/xc32/v1.33/bin/bin/../../lib/gcc/pic32mx/4.5.2/../../../../pic32mx/lib\libpic32.a(vector35.o)
                              c:/program files/microchip/xc32/v1.33/bin/bin/../../lib/gcc/pic32mx/4.5.2/../../../../pic32mx/lib/./proc/32MX795F512H\default_isr_vectors.o (__vector_dispatch_35)
c:/program files/microchip/xc32/v1.33/bin/bin/../../lib/gcc/pic32mx/4.5.2/../../../../pic32mx/lib\libpic32.a(vector36.o)
                              c:/program files/microchip/xc32/v1.33/bin/bin/../../lib/gcc/pic32mx/4.5.2/../../../../pic32mx/lib/./proc/32MX795F512H\default_isr_vectors.o (__vector_dispatch_36)
c:/program files/microchip/xc32/v1.33/bin/bin/../../lib/gcc/pic32mx/4.5.2/../../../../pic32mx/lib\libpic32.a(vector37.o)
                              c:/program files/microchip/xc32/v1.33/bin/bin/../../lib/gcc/pic32mx/4.5.2/../../../../pic32mx/lib/./proc/32MX795F512H\default_isr_vectors.o (__vector_dispatch_37)
c:/program files/microchip/xc32/v1.33/bin/bin/../../lib/gcc/pic32mx/4.5.2/../../../../pic32mx/lib\libpic32.a(vector38.o)
                              c:/program files/microchip/xc32/v1.33/bin/bin/../../lib/gcc/pic32mx/4.5.2/../../../../pic32mx/lib/./proc/32MX795F512H\default_isr_vectors.o (__vector_dispatch_38)
c:/program files/microchip/xc32/v1.33/bin/bin/../../lib/gcc/pic32mx/4.5.2/../../../../pic32mx/lib\libpic32.a(vector39.o)
                              c:/program files/microchip/xc32/v1.33/bin/bin/../../lib/gcc/pic32mx/4.5.2/../../../../pic32mx/lib/./proc/32MX795F512H\default_isr_vectors.o (__vector_dispatch_39)
c:/program files/microchip/xc32/v1.33/bin/bin/../../lib/gcc/pic32mx/4.5.2/../../../../pic32mx/lib\libpic32.a(vector40.o)
                              c:/program files/microchip/xc32/v1.33/bin/bin/../../lib/gcc/pic32mx/4.5.2/../../../../pic32mx/lib/./proc/32MX795F512H\default_isr_vectors.o (__vector_dispatch_40)
c:/program files/microchip/xc32/v1.33/bin/bin/../../lib/gcc/pic32mx/4.5.2/../../../../pic32mx/lib\libpic32.a(vector41.o)
                              c:/program files/microchip/xc32/v1.33/bin/bin/../../lib/gcc/pic32mx/4.5.2/../../../../pic32mx/lib/./proc/32MX795F512H\default_isr_vectors.o (__vector_dispatch_41)
c:/program files/microchip/xc32/v1.33/bin/bin/../../lib/gcc/pic32mx/4.5.2/../../../../pic32mx/lib\libpic32.a(vector42.o)
                              c:/program files/microchip/xc32/v1.33/bin/bin/../../lib/gcc/pic32mx/4.5.2/../../../../pic32mx/lib/./proc/32MX795F512H\default_isr_vectors.o (__vector_dispatch_42)
c:/program files/microchip/xc32/v1.33/bin/bin/../../lib/gcc/pic32mx/4.5.2/../../../../pic32mx/lib\libpic32.a(vector43.o)
                              c:/program files/microchip/xc32/v1.33/bin/bin/../../lib/gcc/pic32mx/4.5.2/../../../../pic32mx/lib/./proc/32MX795F512H\default_isr_vectors.o (__vector_dispatch_43)
c:/program files/microchip/xc32/v1.33/bin/bin/../../lib/gcc/pic32mx/4.5.2/../../../../pic32mx/lib\libpic32.a(vector44.o)
                              c:/program files/microchip/xc32/v1.33/bin/bin/../../lib/gcc/pic32mx/4.5.2/../../../../pic32mx/lib/./proc/32MX795F512H\default_isr_vectors.o (__vector_dispatch_44)
c:/program files/microchip/xc32/v1.33/bin/bin/../../lib/gcc/pic32mx/4.5.2/../../../../pic32mx/lib\libpic32.a(vector45.o)
                              c:/program files/microchip/xc32/v1.33/bin/bin/../../lib/gcc/pic32mx/4.5.2/../../../../pic32mx/lib/./proc/32MX795F512H\default_isr_vectors.o (__vector_dispatch_45)
c:/program files/microchip/xc32/v1.33/bin/bin/../../lib/gcc/pic32mx/4.5.2/../../../../pic32mx/lib\libpic32.a(vector46.o)
                              c:/program files/microchip/xc32/v1.33/bin/bin/../../lib/gcc/pic32mx/4.5.2/../../../../pic32mx/lib/./proc/32MX795F512H\default_isr_vectors.o (__vector_dispatch_46)
c:/program files/microchip/xc32/v1.33/bin/bin/../../lib/gcc/pic32mx/4.5.2/../../../../pic32mx/lib\libpic32.a(vector47.o)
                              c:/program files/microchip/xc32/v1.33/bin/bin/../../lib/gcc/pic32mx/4.5.2/../../../../pic32mx/lib/./proc/32MX795F512H\default_isr_vectors.o (__vector_dispatch_47)
c:/program files/microchip/xc32/v1.33/bin/bin/../../lib/gcc/pic32mx/4.5.2/../../../../pic32mx/lib\libpic32.a(vector48.o)
                              c:/program files/microchip/xc32/v1.33/bin/bin/../../lib/gcc/pic32mx/4.5.2/../../../../pic32mx/lib/./proc/32MX795F512H\default_isr_vectors.o (__vector_dispatch_48)
c:/program files/microchip/xc32/v1.33/bin/bin/../../lib/gcc/pic32mx/4.5.2/../../../../pic32mx/lib\libpic32.a(vector49.o)
                              c:/program files/microchip/xc32/v1.33/bin/bin/../../lib/gcc/pic32mx/4.5.2/../../../../pic32mx/lib/./proc/32MX795F512H\default_isr_vectors.o (__vector_dispatch_49)
c:/program files/microchip/xc32/v1.33/bin/bin/../../lib/gcc/pic32mx/4.5.2/../../../../pic32mx/lib\libpic32.a(vector50.o)
                              c:/program files/microchip/xc32/v1.33/bin/bin/../../lib/gcc/pic32mx/4.5.2/../../../../pic32mx/lib/./proc/32MX795F512H\default_isr_vectors.o (__vector_dispatch_50)
c:/program files/microchip/xc32/v1.33/bin/bin/../../lib/gcc/pic32mx/4.5.2/../../../../pic32mx/lib\libpic32.a(vector51.o)
                              c:/program files/microchip/xc32/v1.33/bin/bin/../../lib/gcc/pic32mx/4.5.2/../../../../pic32mx/lib/./proc/32MX795F512H\default_isr_vectors.o (__vector_dispatch_51)
c:/program files/microchip/xc32/v1.33/bin/bin/../../lib/gcc/pic32mx/4.5.2/../../../../pic32mx/lib\libpic32.a(vector52.o)
                              c:/program files/microchip/xc32/v1.33/bin/bin/../../lib/gcc/pic32mx/4.5.2/../../../../pic32mx/lib/./proc/32MX795F512H\default_isr_vectors.o (__vector_dispatch_52)
c:/program files/microchip/xc32/v1.33/bin/bin/../../lib/gcc/pic32mx/4.5.2/../../../../pic32mx/lib\libpic32.a(vector53.o)
                              c:/program files/microchip/xc32/v1.33/bin/bin/../../lib/gcc/pic32mx/4.5.2/../../../../pic32mx/lib/./proc/32MX795F512H\default_isr_vectors.o (__vector_dispatch_53)
c:/program files/microchip/xc32/v1.33/bin/bin/../../lib/gcc/pic32mx/4.5.2/../../../../pic32mx/lib\libpic32.a(vector54.o)
                              c:/program files/microchip/xc32/v1.33/bin/bin/../../lib/gcc/pic32mx/4.5.2/../../../../pic32mx/lib/./proc/32MX795F512H\default_isr_vectors.o (__vector_dispatch_54)
c:/program files/microchip/xc32/v1.33/bin/bin/../../lib/gcc/pic32mx/4.5.2/../../../../pic32mx/lib\libpic32.a(vector55.o)
                              c:/program files/microchip/xc32/v1.33/bin/bin/../../lib/gcc/pic32mx/4.5.2/../../../../pic32mx/lib/./proc/32MX795F512H\default_isr_vectors.o (__vector_dispatch_55)
c:/program files/microchip/xc32/v1.33/bin/bin/../../lib/gcc/pic32mx/4.5.2/../../../../pic32mx/lib\libpic32.a(vector56.o)
                              c:/program files/microchip/xc32/v1.33/bin/bin/../../lib/gcc/pic32mx/4.5.2/../../../../pic32mx/lib/./proc/32MX795F512H\default_isr_vectors.o (__vector_dispatch_56)
c:/program files/microchip/xc32/v1.33/bin/bin/../../lib/gcc/pic32mx/4.5.2/../../../../pic32mx/lib\libpic32.a(vector57.o)
                              c:/program files/microchip/xc32/v1.33/bin/bin/../../lib/gcc/pic32mx/4.5.2/../../../../pic32mx/lib/./proc/32MX795F512H\default_isr_vectors.o (__vector_dispatch_57)
c:/program files/microchip/xc32/v1.33/bin/bin/../../lib/gcc/pic32mx/4.5.2/../../../../pic32mx/lib\libpic32.a(vector58.o)
                              c:/program files/microchip/xc32/v1.33/bin/bin/../../lib/gcc/pic32mx/4.5.2/../../../../pic32mx/lib/./proc/32MX795F512H\default_isr_vectors.o (__vector_dispatch_58)
c:/program files/microchip/xc32/v1.33/bin/bin/../../lib/gcc/pic32mx/4.5.2/../../../../pic32mx/lib\libpic32.a(vector59.o)
                              c:/program files/microchip/xc32/v1.33/bin/bin/../../lib/gcc/pic32mx/4.5.2/../../../../pic32mx/lib/./proc/32MX795F512H\default_isr_vectors.o (__vector_dispatch_59)
c:/program files/microchip/xc32/v1.33/bin/bin/../../lib/gcc/pic32mx/4.5.2/../../../../pic32mx/lib\libpic32.a(vector60.o)
                              c:/program files/microchip/xc32/v1.33/bin/bin/../../lib/gcc/pic32mx/4.5.2/../../../../pic32mx/lib/./proc/32MX795F512H\default_isr_vectors.o (__vector_dispatch_60)
c:/program files/microchip/xc32/v1.33/bin/bin/../../lib/gcc/pic32mx/4.5.2/../../../../pic32mx/lib\libpic32.a(vector61.o)
                              c:/program files/microchip/xc32/v1.33/bin/bin/../../lib/gcc/pic32mx/4.5.2/../../../../pic32mx/lib/./proc/32MX795F512H\default_isr_vectors.o (__vector_dispatch_61)
c:/program files/microchip/xc32/v1.33/bin/bin/../../lib/gcc/pic32mx/4.5.2/../../../../pic32mx/lib\libpic32.a(vector62.o)
                              c:/program files/microchip/xc32/v1.33/bin/bin/../../lib/gcc/pic32mx/4.5.2/../../../../pic32mx/lib/./proc/32MX795F512H\default_isr_vectors.o (__vector_dispatch_62)
c:/program files/microchip/xc32/v1.33/bin/bin/../../lib/gcc/pic32mx/4.5.2/../../../../pic32mx/lib\libpic32.a(vector63.o)
                              c:/program files/microchip/xc32/v1.33/bin/bin/../../lib/gcc/pic32mx/4.5.2/../../../../pic32mx/lib/./proc/32MX795F512H\default_isr_vectors.o (__vector_dispatch_63)
c:/program files/microchip/xc32/v1.33/bin/bin/../../lib/gcc/pic32mx/4.5.2/../../../../pic32mx/lib\libpic32.a(defaultinterrupt.o)
                              c:/program files/microchip/xc32/v1.33/bin/bin/../../lib/gcc/pic32mx/4.5.2/../../../../pic32mx/lib\libpic32.a(vector0.o) (_DefaultInterrupt)
c:/program files/microchip/xc32/v1.33/bin/bin/../../lib/gcc/pic32mx/4.5.2/../../../../pic32mx/lib\libc.a(puts.o)
                              build/ChaletDuinoV2_795F512H_/debug/Source/main.o (puts)
c:/program files/microchip/xc32/v1.33/bin/bin/../../lib/gcc/pic32mx/4.5.2/../../../../pic32mx/lib\libc.a(strncmp.o)
                              build/ChaletDuinoV2_795F512H_/debug/Source/Terminal.o (strncmp)
c:/program files/microchip/xc32/v1.33/bin/bin/../../lib/gcc/pic32mx/4.5.2/../../../../pic32mx/lib\libc.a(printf_cdnopsuxX.eo)
                              build/ChaletDuinoV2_795F512H_/debug/Source/WiFiCtrl.o (_printf_cdnopsuxX)
c:/program files/microchip/xc32/v1.33/bin/bin/../../lib/gcc/pic32mx/4.5.2/../../../../pic32mx/lib\libc.a(printf_cdnopuxX.eo)
                              build/ChaletDuinoV2_795F512H_/debug/Source/main.o (_printf_cdnopuxX)
c:/program files/microchip/xc32/v1.33/bin/bin/../../lib/gcc/pic32mx/4.5.2/../../../../pic32mx/lib\libc.a(sprintf_cdnopuxX.eo)
                              build/ChaletDuinoV2_795F512H_/debug/Source/Util.o (_sprintf_cdnopuxX)
c:/program files/microchip/xc32/v1.33/bin/bin/../../lib/gcc/pic32mx/4.5.2/../../../../pic32mx/lib\libc.a(sscanf_s.eo)
                              build/ChaletDuinoV2_795F512H_/debug/Source/Terminal.o (_sscanf_s)
c:/program files/microchip/xc32/v1.33/bin/bin/../../lib/gcc/pic32mx/4.5.2/../../../../pic32mx/lib\libc.a(_iob.o)
                              c:/program files/microchip/xc32/v1.33/bin/bin/../../lib/gcc/pic32mx/4.5.2/../../../../pic32mx/lib\libc.a(puts.o) (_iob)
c:/program files/microchip/xc32/v1.33/bin/bin/../../lib/gcc/pic32mx/4.5.2/../../../../pic32mx/lib\libc.a(_fputc_simple.o)
                              c:/program files/microchip/xc32/v1.33/bin/bin/../../lib/gcc/pic32mx/4.5.2/../../../../pic32mx/lib\libc.a(puts.o) (fputc)
c:/program files/microchip/xc32/v1.33/bin/bin/../../lib/gcc/pic32mx/4.5.2/../../../../pic32mx/lib\libc.a(doprnt_cdnopsuxX.eo)
                              c:/program files/microchip/xc32/v1.33/bin/bin/../../lib/gcc/pic32mx/4.5.2/../../../../pic32mx/lib\libc.a(printf_cdnopsuxX.eo) (_vfprintf_cdnopsuxX)
c:/program files/microchip/xc32/v1.33/bin/bin/../../lib/gcc/pic32mx/4.5.2/../../../../pic32mx/lib\libc.a(doprnt_cdnopuxX.eo)
                              c:/program files/microchip/xc32/v1.33/bin/bin/../../lib/gcc/pic32mx/4.5.2/../../../../pic32mx/lib\libc.a(printf_cdnopuxX.eo) (_vfprintf_cdnopuxX)
c:/program files/microchip/xc32/v1.33/bin/bin/../../lib/gcc/pic32mx/4.5.2/../../../../pic32mx/lib\libc.a(doscan_s.eo)
                              c:/program files/microchip/xc32/v1.33/bin/bin/../../lib/gcc/pic32mx/4.5.2/../../../../pic32mx/lib\libc.a(sscanf_s.eo) (_vfscanf_s)
c:/program files/microchip/xc32/v1.33/bin/bin/../../lib/gcc/pic32mx/4.5.2/../../../../pic32mx/lib\libc.a(_flsbuf_simple.o)
                              c:/program files/microchip/xc32/v1.33/bin/bin/../../lib/gcc/pic32mx/4.5.2/../../../../pic32mx/lib\libc.a(_fputc_simple.o) (_flsbuf)
c:/program files/microchip/xc32/v1.33/bin/bin/../../lib/gcc/pic32mx/4.5.2/../../../../pic32mx/lib\libc.a(fgetc.o)
                              c:/program files/microchip/xc32/v1.33/bin/bin/../../lib/gcc/pic32mx/4.5.2/../../../../pic32mx/lib\libc.a(doscan_s.eo) (fgetc)
c:/program files/microchip/xc32/v1.33/bin/bin/../../lib/gcc/pic32mx/4.5.2/../../../../pic32mx/lib\libc.a(atoi.o)
                              c:/program files/microchip/xc32/v1.33/bin/bin/../../lib/gcc/pic32mx/4.5.2/../../../../pic32mx/lib\libc.a(doscan_s.eo) (atoi)
c:/program files/microchip/xc32/v1.33/bin/bin/../../lib/gcc/pic32mx/4.5.2/../../../../pic32mx/lib\libc.a(ctype.o)
                              c:/program files/microchip/xc32/v1.33/bin/bin/../../lib/gcc/pic32mx/4.5.2/../../../../pic32mx/lib\libc.a(doprnt_cdnopsuxX.eo) (_ctype)
c:/program files/microchip/xc32/v1.33/bin/bin/../../lib/gcc/pic32mx/4.5.2/../../../../pic32mx/lib\libc.a(ctypef.o)
                              c:/program files/microchip/xc32/v1.33/bin/bin/../../lib/gcc/pic32mx/4.5.2/../../../../pic32mx/lib\libc.a(doscan_s.eo) (tolower)
c:/program files/microchip/xc32/v1.33/bin/bin/../../lib/gcc/pic32mx/4.5.2/../../../../pic32mx/lib\libc.a(ungetc.o)
                              c:/program files/microchip/xc32/v1.33/bin/bin/../../lib/gcc/pic32mx/4.5.2/../../../../pic32mx/lib\libc.a(doscan_s.eo) (ungetc)
c:/program files/microchip/xc32/v1.33/bin/bin/../../lib/gcc/pic32mx/4.5.2/../../../../pic32mx/lib\libc.a(filbuf.o)
                              c:/program files/microchip/xc32/v1.33/bin/bin/../../lib/gcc/pic32mx/4.5.2/../../../../pic32mx/lib\libc.a(fgetc.o) (_filbuf)
c:/program files/microchip/xc32/v1.33/bin/bin/../../lib/gcc/pic32mx/4.5.2/../../../../pic32mx/lib\libc.a(fflush.o)
                              c:/program files/microchip/xc32/v1.33/bin/bin/../../lib/gcc/pic32mx/4.5.2/../../../../pic32mx/lib\libc.a(filbuf.o) (fflush)
c:/program files/microchip/xc32/v1.33/bin/bin/../../lib/gcc/pic32mx/4.5.2/../../../../pic32mx/lib\libpic32.a(read.o)
                              c:/program files/microchip/xc32/v1.33/bin/bin/../../lib/gcc/pic32mx/4.5.2/../../../../pic32mx/lib\libc.a(filbuf.o) (read)
c:/program files/microchip/xc32/v1.33/bin/bin/../../lib/gcc/pic32mx/4.5.2/../../../../pic32mx/lib\libpic32.a(write.o)
                              c:/program files/microchip/xc32/v1.33/bin/bin/../../lib/gcc/pic32mx/4.5.2/../../../../pic32mx/lib\libc.a(_fputc_simple.o) (write)
c:/program files/microchip/xc32/v1.33/bin/bin/../../lib/gcc/pic32mx/4.5.2/../../../../pic32mx/lib\libpic32.a(xc32_uart.o)
                              c:/program files/microchip/xc32/v1.33/bin/bin/../../lib/gcc/pic32mx/4.5.2/../../../../pic32mx/lib\libpic32.a(read.o) (__XC_UART)
c:/program files/microchip/xc32/v1.33/bin/bin/../../lib/gcc/pic32mx/4.5.2\libgcc.a(_udivdi3.o)
                              c:/program files/microchip/xc32/v1.33/bin/bin/../../lib/gcc/pic32mx/4.5.2/../../../../pic32mx/lib\libc.a(doprnt_cdnopsuxX.eo) (__udivdi3)
c:/program files/microchip/xc32/v1.33/bin/bin/../../lib/gcc/pic32mx/4.5.2\libgcc.a(_umoddi3.o)
                              c:/program files/microchip/xc32/v1.33/bin/bin/../../lib/gcc/pic32mx/4.5.2/../../../../pic32mx/lib\libc.a(doprnt_cdnopsuxX.eo) (__umoddi3)

Allocating common symbols
Common symbol       size              file

mSyslogBufPtr       0x4               build/ChaletDuinoV2_795F512H_/debug/Source/Syslog.o
BootloaderRxPtr     0x4               build/ChaletDuinoV2_795F512H_/debug/Source/BootloaderProtocol.o
u8IsMacAddrValid    0x1               build/ChaletDuinoV2_795F512H_/debug/Source/WiFiCtrl.o
CurDataChunkSize    0x4               build/ChaletDuinoV2_795F512H_/debug/Source/BootloaderInterface.o
mTerminalOpened     0x4               build/ChaletDuinoV2_795F512H_/debug/Source/Terminal.o
TerminalDataPtr     0x4               build/ChaletDuinoV2_795F512H_/debug/Source/Terminal.o
gpfAppResolveCb     0x4               build/ChaletDuinoV2_795F512H_/debug/Source/winc3400_142/socket/source/socket.o
BootloaderFirmwareChunkWriteCount
                    0x4               build/ChaletDuinoV2_795F512H_/debug/Source/BootloaderInterface.o
BootloaderFlashWriteDataPtr
                    0x4               build/ChaletDuinoV2_795F512H_/debug/Source/BootloaderInterface.o
mTerminalPendingAction
                    0x4               build/ChaletDuinoV2_795F512H_/debug/Source/Terminal.o
mFrameData          0x136             build/ChaletDuinoV2_795F512H_/debug/Source/NetworkProtocol.o
mCurIPAddress       0x4               build/ChaletDuinoV2_795F512H_/debug/Source/WiFiCtrl.o
mSPIFlashHighSpeedBaudrate
                    0x1               build/ChaletDuinoV2_795F512H_/debug/Source/SPI_Flash.o
NetworkRxBuf        0x400             build/ChaletDuinoV2_795F512H_/debug/Source/WiFiCtrl.o
TerminalRxBuf       0x400             build/ChaletDuinoV2_795F512H_/debug/Source/WiFiCtrl.o
mStoredBootloaderInfo
                    0x14              build/ChaletDuinoV2_795F512H_/debug/Source/Terminal.o
TerminalWorkString  0x12c             build/ChaletDuinoV2_795F512H_/debug/Source/Terminal.o
mWifiSPIBaudrate    0x1               build/ChaletDuinoV2_795F512H_/debug/Source/winc3400_142/driver/source/nmspi.o
BootloaderRxBuf     0x400             build/ChaletDuinoV2_795F512H_/debug/Source/WiFiCtrl.o
BootloaderFlashErased
                    0x4               build/ChaletDuinoV2_795F512H_/debug/Source/BootloaderInterface.o
gpfAppSocketCb      0x4               build/ChaletDuinoV2_795F512H_/debug/Source/winc3400_142/socket/source/socket.o
BootloaderFlashWriteState
                    0x4               build/ChaletDuinoV2_795F512H_/debug/Source/BootloaderInterface.o
gstrHifCxt          0x24              build/ChaletDuinoV2_795F512H_/debug/Source/winc3400_142/driver/source/m2m_hif.o
mac_addr            0x6               build/ChaletDuinoV2_795F512H_/debug/Source/WiFiCtrl.o
BootloaderCurFlashWriteAddress
                    0x4               build/ChaletDuinoV2_795F512H_/debug/Source/BootloaderInterface.o
mSyslogLTEPassthroughEnabled
                    0x4               build/ChaletDuinoV2_795F512H_/debug/Source/Syslog.o
mHelpStringPtr      0x4               build/ChaletDuinoV2_795F512H_/debug/Source/Terminal.o
mSyslogBuffer       0x1f4             build/ChaletDuinoV2_795F512H_/debug/Source/Syslog.o
mAPPassword         0x40              build/ChaletDuinoV2_795F512H_/debug/Source/Terminal.o
ActualTemp          0x4               build/ChaletDuinoV2_795F512H_/debug/Source/main.o
addr_in             0x10              build/ChaletDuinoV2_795F512H_/debug/Source/WiFiCtrl.o
BooloaderFlashEraseState
                    0x4               build/ChaletDuinoV2_795F512H_/debug/Source/BootloaderInterface.o
param               0x18              build/ChaletDuinoV2_795F512H_/debug/Source/WiFiCtrl.o
VolDebug            0x64              build/ChaletDuinoV2_795F512H_/debug/Source/VolumeTransducer.o
mModuleIPConfig     0x14              build/ChaletDuinoV2_795F512H_/debug/Source/WiFiCtrl.o
BootloaderBuffer    0x12c             build/ChaletDuinoV2_795F512H_/debug/Source/BootloaderInterface.o
mSPIFlashBaudrate   0x1               build/ChaletDuinoV2_795F512H_/debug/Source/SPI_Flash.o
BootloaderCurFlashEraseAddress
                    0x4               build/ChaletDuinoV2_795F512H_/debug/Source/BootloaderInterface.o
TerminalPrevDataBuf
                    0x12c             build/ChaletDuinoV2_795F512H_/debug/Source/Terminal.o
BootloaderFlashWritePollCount
                    0x4               build/ChaletDuinoV2_795F512H_/debug/Source/BootloaderInterface.o
mLoraProtocolData   0x284             build/ChaletDuinoV2_795F512H_/debug/Source/NetworkProtocol.o
BootloaderInterfaceState
                    0x4               build/ChaletDuinoV2_795F512H_/debug/Source/BootloaderInterface.o
mLTEProtocolData    0x284             build/ChaletDuinoV2_795F512H_/debug/Source/NetworkProtocol.o
mUseDHCP            0x1               build/ChaletDuinoV2_795F512H_/debug/Source/Terminal.o
mDACSPIBaudrate     0x1               build/ChaletDuinoV2_795F512H_/debug/Source/DACInterface.o
DataChunkWritten    0x4               build/ChaletDuinoV2_795F512H_/debug/Source/BootloaderInterface.o
mSPIFlashOK         0x4               build/ChaletDuinoV2_795F512H_/debug/Source/SPI_Flash.o
gastrSockets        0xc0              build/ChaletDuinoV2_795F512H_/debug/Source/winc3400_142/socket/source/socket.o
mTerminalTickState  0x4               build/ChaletDuinoV2_795F512H_/debug/Source/Terminal.o
BooloaderFlashErasePollCount
                    0x4               build/ChaletDuinoV2_795F512H_/debug/Source/BootloaderInterface.o
FirmwareUploaded    0x4               build/ChaletDuinoV2_795F512H_/debug/Source/BootloaderInterface.o
mFlashSectorBuffer  0x1000            build/ChaletDuinoV2_795F512H_/debug/Source/SPI_Flash.o
CurDataChunkIndex   0x4               build/ChaletDuinoV2_795F512H_/debug/Source/BootloaderInterface.o
astTimer            0xc0              build/ChaletDuinoV2_795F512H_/debug/Source/timer.o
TerminalDataBuf     0x12c             build/ChaletDuinoV2_795F512H_/debug/Source/Terminal.o
mAPName             0x40              build/ChaletDuinoV2_795F512H_/debug/Source/Terminal.o
SyslogRxBuf         0xc8              build/ChaletDuinoV2_795F512H_/debug/Source/WiFiCtrl.o

Microchip PIC32 Memory-Usage Report

kseg0 Program-Memory Usage
section                    address  length [bytes]      (dec)  Description
-------                 ----------  -------------------------  -----------
.text                   0x9d005800        0x108e4       67812  App's exec code 
.dinit                  0x9d0160e4          0xd60        3424   
.text                   0x9d016e44         0x4844       18500  App's exec code 
.text._vfprintf_cdnopsu 0x9d01b688          0xae8        2792   
.text._vfscanf_s        0x9d01c170          0x868        2152   
.rodata                 0x9d01c9d8          0x7b8        1976  Read-only const 
.text                   0x9d01d190         0x286c       10348  App's exec code 
.rodata                 0x9d01f9fc          0x804        2052  Read-only const 
.text                   0x9d020200          0xf50        3920  App's exec code 
.rodata                 0x9d021150          0x25c         604  Read-only const 
.text                   0x9d0213ac          0x810        2064  App's exec code 
.text._filbuf           0x9d021bbc          0x188         392   
.text.read              0x9d021d44          0x174         372   
.text                   0x9d021eb8          0x2d0         720  App's exec code 
.text.fputc             0x9d022188          0x15c         348   
.text._flsbuf           0x9d0222e4          0x12c         300   
.text.fgetc             0x9d022410          0x108         264   
.rodata                 0x9d022518          0x204         516  Read-only const 
.text.general_exception 0x9d02271c           0xdc         220   
.text                   0x9d0227f8           0xd8         216  App's exec code 
.rodata                 0x9d0228d0          0x198         408  Read-only const 
.text                   0x9d022a68           0xa8         168  App's exec code 
.text.atoi              0x9d022b10           0xa8         168   
.text.range             0x9d022bb8           0xa0         160   
.text                   0x9d022c58           0x98         152  App's exec code 
.text.fflush            0x9d022cf0           0x94         148   
.text.write             0x9d022d84           0x94         148   
.text.SoftReset         0x9d022e18           0x78         120   
.text.fputs             0x9d022e90           0x78         120   
.text.strncmp           0x9d022f08           0x78         120   
.text.ungetc            0x9d022f80           0x74         116   
.text                   0x9d022ff4           0x70         112  App's exec code 
.text._sprintf_cdnopuxX 0x9d023064           0x68         104   
.text.wspace            0x9d0230cc           0x60          96   
.text                   0x9d02312c           0x58          88  App's exec code 
.text._sscanf_s         0x9d023184           0x54          84   
.rodata                 0x9d0231d8           0x50          80  Read-only const 
.text.main_entry        0x9d023228           0x4c          76   
.rodata                 0x9d023274           0x48          72  Read-only const 
.text._bootstrap_except 0x9d0232bc           0x48          72   
.text                   0x9d023304           0x44          68  App's exec code 
.text.puts              0x9d023348           0x44          68   
.text._printf_cdnopsuxX 0x9d02338c           0x40          64   
.vector_default         0x9d0233cc           0x38          56   
.rodata                 0x9d023404           0x30          48  Read-only const 
.text.INTConfigureSyste 0x9d023434           0x30          48   
.text.tolower           0x9d023464           0x24          36   
.text.toupper           0x9d023488           0x24          36   
.text                   0x9d0234ac           0x20          32  App's exec code 
.rodata                 0x9d0234cc           0x1c          28  Read-only const 
.text.INTRestoreInterru 0x9d0234e8           0x1c          28   
.rodata                 0x9d023504           0x18          24  Read-only const 
.text.CheKseg0CacheOff  0x9d02351c           0x18          24   
.text.CheKseg0CacheOn   0x9d023534           0x18          24   
.text                   0x9d02354c           0x18          24  App's exec code 
.text.isalnum           0x9d023564           0x18          24   
.text.isalpha           0x9d02357c           0x18          24   
.text.iscntrl           0x9d023594           0x18          24   
.text.isdigit           0x9d0235ac           0x18          24   
.text.isgraph           0x9d0235c4           0x18          24   
.text.islower           0x9d0235dc           0x18          24   
.text.isprint           0x9d0235f4           0x18          24   
.text.ispunct           0x9d02360c           0x18          24   
.text.isspace           0x9d023624           0x18          24   
.text.isupper           0x9d02363c           0x18          24   
.text.isxdigit          0x9d023654           0x18          24   
.text.__exception_handl 0x9d02366c            0xc          12   
.rodata                 0x9d023678            0x8           8  Read-only const 
.text.INTEnableInterrup 0x9d023680            0x8           8   
.text.INTDisableInterru 0x9d023688            0x8           8   
.text._on_reset         0x9d023690            0x8           8   
.text._on_bootstrap     0x9d023698            0x8           8   
.text.close             0x9d0236a0            0x8           8   
.text.isascii           0x9d0236a8            0x8           8   
.text.toascii           0x9d0236b0            0x8           8   
.text._tolower          0x9d0236b8            0x8           8   
.text._toupper          0x9d0236c0            0x8           8   
      Total kseg0_program_mem used  :     0x1dec8      122568  24.4% of 0x7a7ff

kseg0 Boot-Memory Usage
section                    address  length [bytes]      (dec)  Description
-------                 ----------  -------------------------  -----------
.startup                0x9d005000          0x1e8         488  C startup code 
         Total kseg0_boot_mem used  :       0x1e8         488  24.0% of 0x7f0

Exception-Memory Usage 
section                    address  length [bytes]      (dec)  Description
-------                 ----------  -------------------------  -----------
.app_excpt              0x9d004180           0x10          16  General-Exception 
.vector_0               0x9d004200            0x8           8  Interrupt Vector 0 
.vector_1               0x9d004220            0x8           8  Interrupt Vector 1 
.vector_2               0x9d004240            0x8           8  Interrupt Vector 2 
.vector_3               0x9d004260            0x8           8  Interrupt Vector 3 
.vector_4               0x9d004280            0x8           8  Interrupt Vector 4 
.vector_5               0x9d0042a0            0x8           8  Interrupt Vector 5 
.vector_6               0x9d0042c0            0x8           8  Interrupt Vector 6 
.vector_7               0x9d0042e0            0x8           8  Interrupt Vector 7 
.vector_8               0x9d004300            0x8           8  Interrupt Vector 8 
.vector_9               0x9d004320            0x8           8  Interrupt Vector 9 
.vector_10              0x9d004340            0x8           8  Interrupt Vector 10 
.vector_11              0x9d004360            0x8           8  Interrupt Vector 11 
.vector_12              0x9d004380            0x8           8  Interrupt Vector 12 
.vector_13              0x9d0043a0            0x8           8  Interrupt Vector 13 
.vector_14              0x9d0043c0            0x8           8  Interrupt Vector 14 
.vector_15              0x9d0043e0            0x8           8  Interrupt Vector 15 
.vector_16              0x9d004400            0x8           8  Interrupt Vector 16 
.vector_17              0x9d004420            0x8           8  Interrupt Vector 17 
.vector_18              0x9d004440            0x8           8  Interrupt Vector 18 
.vector_19              0x9d004460            0x8           8  Interrupt Vector 19 
.vector_20              0x9d004480            0x8           8  Interrupt Vector 20 
.vector_21              0x9d0044a0            0x8           8  Interrupt Vector 21 
.vector_22              0x9d0044c0            0x8           8  Interrupt Vector 22 
.vector_23              0x9d0044e0            0x8           8  Interrupt Vector 23 
.vector_24              0x9d004500            0x8           8  Interrupt Vector 24 
.vector_25              0x9d004520            0x8           8  Interrupt Vector 25 
.vector_26              0x9d004540            0x8           8  Interrupt Vector 26 
.vector_27              0x9d004560            0x8           8  Interrupt Vector 27 
.vector_28              0x9d004580            0x8           8  Interrupt Vector 28 
.vector_29              0x9d0045a0            0x8           8  Interrupt Vector 29 
.vector_30              0x9d0045c0            0x8           8  Interrupt Vector 30 
.vector_31              0x9d0045e0            0x8           8  Interrupt Vector 31 
.vector_32              0x9d004600            0x8           8  Interrupt Vector 32 
.vector_33              0x9d004620            0x8           8  Interrupt Vector 33 
.vector_34              0x9d004640            0x8           8  Interrupt Vector 34 
.vector_35              0x9d004660            0x8           8  Interrupt Vector 35 
.vector_36              0x9d004680            0x8           8  Interrupt Vector 36 
.vector_37              0x9d0046a0            0x8           8  Interrupt Vector 37 
.vector_38              0x9d0046c0            0x8           8  Interrupt Vector 38 
.vector_39              0x9d0046e0            0x8           8  Interrupt Vector 39 
.vector_40              0x9d004700            0x8           8  Interrupt Vector 40 
.vector_41              0x9d004720            0x8           8  Interrupt Vector 41 
.vector_42              0x9d004740            0x8           8  Interrupt Vector 42 
.vector_43              0x9d004760            0x8           8  Interrupt Vector 43 
.vector_44              0x9d004780            0x8           8  Interrupt Vector 44 
.vector_45              0x9d0047a0            0x8           8  Interrupt Vector 45 
.vector_46              0x9d0047c0            0x8           8  Interrupt Vector 46 
.vector_47              0x9d0047e0            0x8           8  Interrupt Vector 47 
.vector_48              0x9d004800            0x8           8  Interrupt Vector 48 
.vector_49              0x9d004820            0x8           8  Interrupt Vector 49 
.vector_50              0x9d004840            0x8           8  Interrupt Vector 50 
.vector_51              0x9d004860            0x8           8  Interrupt Vector 51 
.vector_52              0x9d004880            0x8           8  Interrupt Vector 52 
.vector_53              0x9d0048a0            0x8           8  Interrupt Vector 53 
.vector_54              0x9d0048c0            0x8           8  Interrupt Vector 54 
.vector_55              0x9d0048e0            0x8           8  Interrupt Vector 55 
.vector_56              0x9d004900            0x8           8  Interrupt Vector 56 
.vector_57              0x9d004920            0x8           8  Interrupt Vector 57 
.vector_58              0x9d004940            0x8           8  Interrupt Vector 58 
.vector_59              0x9d004960            0x8           8  Interrupt Vector 59 
.vector_60              0x9d004980            0x8           8  Interrupt Vector 60 
.vector_61              0x9d0049a0            0x8           8  Interrupt Vector 61 
.vector_62              0x9d0049c0            0x8           8  Interrupt Vector 62 
.vector_63              0x9d0049e0            0x8           8  Interrupt Vector 63 
          Total exception_mem used  :       0x210         528  12.9% of 0x1000

kseg1 Boot-Memory Usage
section                    address  length [bytes]      (dec)  Description
-------                 ----------  -------------------------  -----------
.reset                  0xbfc00000            0x8           8  Reset handler 
.bev_excpt              0xbfc00380           0x10          16  BEV-Exception 
         Total kseg1_boot_mem used  :        0x18          24  2.1% of 0x490
        --------------------------------------------------------------------------
         Total Program Memory used  :     0x1e2d8      123608  24.3% of 0x7c47f
        --------------------------------------------------------------------------


kseg0 Data-Memory Usage
section                    address  length [bytes]      (dec)  Description
-------                 ----------  -------------------------  -----------
reserve_data_0_kseg0    0x80000000          0x200         512   
         Total kseg0_data_mem used  :       0x200         512  100.0% of 0x200

kseg1 Data-Memory Usage
section                    address  length [bytes]      (dec)  Description
-------                 ----------  -------------------------  -----------
reserve_data_0_kseg1    0xa0000000          0x200         512   
.eh_frame               0xa0000200           0x30          48   
.sdata                  0xa0000230           0x64         100  Small init data 
.sbss                   0xa0000294          0x124         292  Small uninit data 
.bss                    0xa00003b8         0x2c84       11396  Uninitialized data 
.data                   0xa000303c          0x7a8        1960  Initialized data 
.bss                    0xa00037e4          0x800        2048  Uninitialized data 
.data                   0xa0003fe4          0x26c         620  Initialized data 
.bss                    0xa0004250           0x40          64  Uninitialized data 
.data                   0xa0004290           0x1c          28  Initialized data 
.bss                    0xa00042ac           0x18          24  Uninitialized data 
         Total kseg1_data_mem used  :      0x42c4       17092  26.1% of 0x10000
        --------------------------------------------------------------------------
            Total Data Memory used  :      0x44c4       17604  26.7% of 0x10200
        --------------------------------------------------------------------------


Dynamic Data-Memory Reservation
section                    address  length [bytes]      (dec)  Description
-------                 ----------  -------------------------  -----------
heap                    0xa00042c8           0x80         128  Reserved for heap 
stack                   0xa0004360         0xbc90       48272  Reserved for stack 

        --------------------------------------------------------------------------

Discarded input sections

 .reginfo       0x00000000       0x18 c:/program files/microchip/xc32/v1.33/bin/bin/../../lib/gcc/pic32mx/4.5.2/../../../../pic32mx/lib\software-debug-break.o
 .reginfo       0x00000000       0x18 build/ChaletDuinoV2_795F512H_/debug/Source/ChaletduinoV2Board.o
 .reginfo       0x00000000       0x18 build/ChaletDuinoV2_795F512H_/debug/Source/winc3400_142/common/source/nm_common.o
 .reginfo       0x00000000       0x18 build/ChaletDuinoV2_795F512H_/debug/Source/winc3400_142/driver/source/m2m_flash.o
 .reginfo       0x00000000       0x18 build/ChaletDuinoV2_795F512H_/debug/Source/winc3400_142/driver/source/m2m_hif.o
 .reginfo       0x00000000       0x18 build/ChaletDuinoV2_795F512H_/debug/Source/winc3400_142/driver/source/m2m_ota.o
 .reginfo       0x00000000       0x18 build/ChaletDuinoV2_795F512H_/debug/Source/winc3400_142/driver/source/m2m_periph.o
 .reginfo       0x00000000       0x18 build/ChaletDuinoV2_795F512H_/debug/Source/winc3400_142/driver/source/m2m_ssl.o
 .reginfo       0x00000000       0x18 build/ChaletDuinoV2_795F512H_/debug/Source/winc3400_142/driver/source/m2m_wifi.o
 .reginfo       0x00000000       0x18 build/ChaletDuinoV2_795F512H_/debug/Source/winc3400_142/driver/source/nmasic.o
 .reginfo       0x00000000       0x18 build/ChaletDuinoV2_795F512H_/debug/Source/winc3400_142/driver/source/nmbus.o
 .reginfo       0x00000000       0x18 build/ChaletDuinoV2_795F512H_/debug/Source/winc3400_142/driver/source/nmdrv.o
 .reginfo       0x00000000       0x18 build/ChaletDuinoV2_795F512H_/debug/Source/winc3400_142/driver/source/nmspi.o
 .reginfo       0x00000000       0x18 build/ChaletDuinoV2_795F512H_/debug/Source/winc3400_142/socket/source/inet_addr.o
 .reginfo       0x00000000       0x18 build/ChaletDuinoV2_795F512H_/debug/Source/winc3400_142/socket/source/inet_ntop.o
 .reginfo       0x00000000       0x18 build/ChaletDuinoV2_795F512H_/debug/Source/winc3400_142/socket/source/socket.o
 .reginfo       0x00000000       0x18 build/ChaletDuinoV2_795F512H_/debug/Source/winc3400_142/spi_flash/source/spi_flash.o
 .reginfo       0x00000000       0x18 build/ChaletDuinoV2_795F512H_/debug/Source/DigitalIO.o
 .reginfo       0x00000000       0x18 build/ChaletDuinoV2_795F512H_/debug/Source/NetworkProtocol.o
 .reginfo       0x00000000       0x18 build/ChaletDuinoV2_795F512H_/debug/Source/Terminal.o
 .reginfo       0x00000000       0x18 build/ChaletDuinoV2_795F512H_/debug/Source/Util.o
 .reginfo       0x00000000       0x18 build/ChaletDuinoV2_795F512H_/debug/Source/exceptions.o
 .reginfo       0x00000000       0x18 build/ChaletDuinoV2_795F512H_/debug/Source/interrupts.o
 .reginfo       0x00000000       0x18 build/ChaletDuinoV2_795F512H_/debug/Source/main.o
 .reginfo       0x00000000       0x18 build/ChaletDuinoV2_795F512H_/debug/Source/system.o
 .reginfo       0x00000000       0x18 build/ChaletDuinoV2_795F512H_/debug/Source/template.o
 .reginfo       0x00000000       0x18 build/ChaletDuinoV2_795F512H_/debug/Source/timer.o
 .reginfo       0x00000000       0x18 build/ChaletDuinoV2_795F512H_/debug/Source/WiFiCtrl.o
 .reginfo       0x00000000       0x18 build/ChaletDuinoV2_795F512H_/debug/Source/SPI.o
 .reginfo       0x00000000       0x18 build/ChaletDuinoV2_795F512H_/debug/Source/SPI_Flash.o
 .reginfo       0x00000000       0x18 build/ChaletDuinoV2_795F512H_/debug/Source/Syslog.o
 .reginfo       0x00000000       0x18 build/ChaletDuinoV2_795F512H_/debug/Source/Watchdog.o
 .reginfo       0x00000000       0x18 build/ChaletDuinoV2_795F512H_/debug/Source/BootloaderInterface.o
 .reginfo       0x00000000       0x18 build/ChaletDuinoV2_795F512H_/debug/Source/BootloaderProtocol.o
 .reginfo       0x00000000       0x18 build/ChaletDuinoV2_795F512H_/debug/Source/crc32.o
 .reginfo       0x00000000       0x18 build/ChaletDuinoV2_795F512H_/debug/Source/VolumeTransducer.o
 .reginfo       0x00000000       0x18 build/ChaletDuinoV2_795F512H_/debug/Source/DACInterface.o
 .reginfo       0x00000000       0x18 c:/program files/microchip/xc32/v1.33/bin/bin/../../lib/gcc/pic32mx/4.5.2/../../../../pic32mx/lib/./proc/32MX795F512H\processor.o
 .reginfo       0x00000000       0x18 c:/program files/microchip/xc32/v1.33/bin/bin/../../lib/gcc/pic32mx/4.5.2/../../../../pic32mx/lib\libmchp_peripheral_32MX795F512H.a(soft_reset_lib.o)
 .reginfo       0x00000000       0x18 c:/program files/microchip/xc32/v1.33/bin/bin/../../lib/gcc/pic32mx/4.5.2/../../../../pic32mx/lib\libmchp_peripheral_32MX795F512H.a(pcache.o)
 .reginfo       0x00000000       0x18 c:/program files/microchip/xc32/v1.33/bin/bin/../../lib/gcc/pic32mx/4.5.2/../../../../pic32mx/lib\libmchp_peripheral_32MX795F512H.a(int_configure_system_lib.o)
 .reginfo       0x00000000       0x18 c:/program files/microchip/xc32/v1.33/bin/bin/../../lib/gcc/pic32mx/4.5.2/../../../../pic32mx/lib\libmchp_peripheral_32MX795F512H.a(int_enable_interrupts_lib.o)
 .reginfo       0x00000000       0x18 c:/program files/microchip/xc32/v1.33/bin/bin/../../lib/gcc/pic32mx/4.5.2/../../../../pic32mx/lib\libmchp_peripheral_32MX795F512H.a(int_disable_interrupts_lib.o)
 .reginfo       0x00000000       0x18 c:/program files/microchip/xc32/v1.33/bin/bin/../../lib/gcc/pic32mx/4.5.2/../../../../pic32mx/lib\libmchp_peripheral_32MX795F512H.a(int_restore_interrupts_lib.o)
 .reginfo       0x00000000       0x18 c:/program files/microchip/xc32/v1.33/bin/bin/../../lib/gcc/pic32mx/4.5.2/../../../../pic32mx/lib/./proc/32MX795F512H\default_isr_vectors.o
 .discard       0x00000000      0x100 c:/program files/microchip/xc32/v1.33/bin/bin/../../lib/gcc/pic32mx/4.5.2/../../../../pic32mx/lib/./proc/32MX795F512H\default_isr_vectors.o
 .reginfo       0x00000000       0x18 c:/program files/microchip/xc32/v1.33/bin/bin/../../lib/gcc/pic32mx/4.5.2/../../../../pic32mx/lib\pic32_software_reset.o
 .reginfo       0x00000000       0x18 c:/program files/microchip/xc32/v1.33/bin/bin/../../lib/gcc/pic32mx/4.5.2/../../../../pic32mx/lib\libpic32.a(memcmp.o)
 .reginfo       0x00000000       0x18 c:/program files/microchip/xc32/v1.33/bin/bin/../../lib/gcc/pic32mx/4.5.2/../../../../pic32mx/lib\libpic32.a(memcpy.o)
 .reginfo       0x00000000       0x18 c:/program files/microchip/xc32/v1.33/bin/bin/../../lib/gcc/pic32mx/4.5.2/../../../../pic32mx/lib\libpic32.a(memset.o)
 .reginfo       0x00000000       0x18 c:/program files/microchip/xc32/v1.33/bin/bin/../../lib/gcc/pic32mx/4.5.2/../../../../pic32mx/lib\libpic32.a(strcpy.o)
 .reginfo       0x00000000       0x18 c:/program files/microchip/xc32/v1.33/bin/bin/../../lib/gcc/pic32mx/4.5.2/../../../../pic32mx/lib\libpic32.a(strlen.o)
 .reginfo       0x00000000       0x18 c:/program files/microchip/xc32/v1.33/bin/bin/../../lib/gcc/pic32mx/4.5.2/../../../../pic32mx/lib\libpic32.a(default-bootstrap-exception-handler.o)
 .reginfo       0x00000000       0x18 c:/program files/microchip/xc32/v1.33/bin/bin/../../lib/gcc/pic32mx/4.5.2/../../../../pic32mx/lib\libpic32.a(default-on-reset.o)
 .reginfo       0x00000000       0x18 c:/program files/microchip/xc32/v1.33/bin/bin/../../lib/gcc/pic32mx/4.5.2/../../../../pic32mx/lib\libpic32.a(default-on-bootstrap.o)
 .reginfo       0x00000000       0x18 c:/program files/microchip/xc32/v1.33/bin/bin/../../lib/gcc/pic32mx/4.5.2/../../../../pic32mx/lib\libpic32.a(default-nmi-handler.o)
 .reginfo       0x00000000       0x18 c:/program files/microchip/xc32/v1.33/bin/bin/../../lib/gcc/pic32mx/4.5.2/../../../../pic32mx/lib\libpic32.a(close.o)
 .reginfo       0x00000000       0x18 c:/program files/microchip/xc32/v1.33/bin/bin/../../lib/gcc/pic32mx/4.5.2/../../../../pic32mx/lib\libpic32.a(general-exception.o)
 .reginfo       0x00000000       0x18 c:/program files/microchip/xc32/v1.33/bin/bin/../../lib/gcc/pic32mx/4.5.2/../../../../pic32mx/lib\libpic32.a(vector0.o)
 .reginfo       0x00000000       0x18 c:/program files/microchip/xc32/v1.33/bin/bin/../../lib/gcc/pic32mx/4.5.2/../../../../pic32mx/lib\libpic32.a(vector1.o)
 .reginfo       0x00000000       0x18 c:/program files/microchip/xc32/v1.33/bin/bin/../../lib/gcc/pic32mx/4.5.2/../../../../pic32mx/lib\libpic32.a(vector2.o)
 .reginfo       0x00000000       0x18 c:/program files/microchip/xc32/v1.33/bin/bin/../../lib/gcc/pic32mx/4.5.2/../../../../pic32mx/lib\libpic32.a(vector5.o)
 .reginfo       0x00000000       0x18 c:/program files/microchip/xc32/v1.33/bin/bin/../../lib/gcc/pic32mx/4.5.2/../../../../pic32mx/lib\libpic32.a(vector6.o)
 .reginfo       0x00000000       0x18 c:/program files/microchip/xc32/v1.33/bin/bin/../../lib/gcc/pic32mx/4.5.2/../../../../pic32mx/lib\libpic32.a(vector8.o)
 .reginfo       0x00000000       0x18 c:/program files/microchip/xc32/v1.33/bin/bin/../../lib/gcc/pic32mx/4.5.2/../../../../pic32mx/lib\libpic32.a(vector9.o)
 .reginfo       0x00000000       0x18 c:/program files/microchip/xc32/v1.33/bin/bin/../../lib/gcc/pic32mx/4.5.2/../../../../pic32mx/lib\libpic32.a(vector10.o)
 .reginfo       0x00000000       0x18 c:/program files/microchip/xc32/v1.33/bin/bin/../../lib/gcc/pic32mx/4.5.2/../../../../pic32mx/lib\libpic32.a(vector11.o)
 .reginfo       0x00000000       0x18 c:/program files/microchip/xc32/v1.33/bin/bin/../../lib/gcc/pic32mx/4.5.2/../../../../pic32mx/lib\libpic32.a(vector12.o)
 .reginfo       0x00000000       0x18 c:/program files/microchip/xc32/v1.33/bin/bin/../../lib/gcc/pic32mx/4.5.2/../../../../pic32mx/lib\libpic32.a(vector13.o)
 .reginfo       0x00000000       0x18 c:/program files/microchip/xc32/v1.33/bin/bin/../../lib/gcc/pic32mx/4.5.2/../../../../pic32mx/lib\libpic32.a(vector14.o)
 .reginfo       0x00000000       0x18 c:/program files/microchip/xc32/v1.33/bin/bin/../../lib/gcc/pic32mx/4.5.2/../../../../pic32mx/lib\libpic32.a(vector16.o)
 .reginfo       0x00000000       0x18 c:/program files/microchip/xc32/v1.33/bin/bin/../../lib/gcc/pic32mx/4.5.2/../../../../pic32mx/lib\libpic32.a(vector17.o)
 .reginfo       0x00000000       0x18 c:/program files/microchip/xc32/v1.33/bin/bin/../../lib/gcc/pic32mx/4.5.2/../../../../pic32mx/lib\libpic32.a(vector18.o)
 .reginfo       0x00000000       0x18 c:/program files/microchip/xc32/v1.33/bin/bin/../../lib/gcc/pic32mx/4.5.2/../../../../pic32mx/lib\libpic32.a(vector19.o)
 .reginfo       0x00000000       0x18 c:/program files/microchip/xc32/v1.33/bin/bin/../../lib/gcc/pic32mx/4.5.2/../../../../pic32mx/lib\libpic32.a(vector20.o)
 .reginfo       0x00000000       0x18 c:/program files/microchip/xc32/v1.33/bin/bin/../../lib/gcc/pic32mx/4.5.2/../../../../pic32mx/lib\libpic32.a(vector21.o)
 .reginfo       0x00000000       0x18 c:/program files/microchip/xc32/v1.33/bin/bin/../../lib/gcc/pic32mx/4.5.2/../../../../pic32mx/lib\libpic32.a(vector22.o)
 .reginfo       0x00000000       0x18 c:/program files/microchip/xc32/v1.33/bin/bin/../../lib/gcc/pic32mx/4.5.2/../../../../pic32mx/lib\libpic32.a(vector23.o)
 .reginfo       0x00000000       0x18 c:/program files/microchip/xc32/v1.33/bin/bin/../../lib/gcc/pic32mx/4.5.2/../../../../pic32mx/lib\libpic32.a(vector24.o)
 .reginfo       0x00000000       0x18 c:/program files/microchip/xc32/v1.33/bin/bin/../../lib/gcc/pic32mx/4.5.2/../../../../pic32mx/lib\libpic32.a(vector25.o)
 .reginfo       0x00000000       0x18 c:/program files/microchip/xc32/v1.33/bin/bin/../../lib/gcc/pic32mx/4.5.2/../../../../pic32mx/lib\libpic32.a(vector26.o)
 .reginfo       0x00000000       0x18 c:/program files/microchip/xc32/v1.33/bin/bin/../../lib/gcc/pic32mx/4.5.2/../../../../pic32mx/lib\libpic32.a(vector27.o)
 .reginfo       0x00000000       0x18 c:/program files/microchip/xc32/v1.33/bin/bin/../../lib/gcc/pic32mx/4.5.2/../../../../pic32mx/lib\libpic32.a(vector28.o)
 .reginfo       0x00000000       0x18 c:/program files/microchip/xc32/v1.33/bin/bin/../../lib/gcc/pic32mx/4.5.2/../../../../pic32mx/lib\libpic32.a(vector29.o)
 .reginfo       0x00000000       0x18 c:/program files/microchip/xc32/v1.33/bin/bin/../../lib/gcc/pic32mx/4.5.2/../../../../pic32mx/lib\libpic32.a(vector30.o)
 .reginfo       0x00000000       0x18 c:/program files/microchip/xc32/v1.33/bin/bin/../../lib/gcc/pic32mx/4.5.2/../../../../pic32mx/lib\libpic32.a(vector31.o)
 .reginfo       0x00000000       0x18 c:/program files/microchip/xc32/v1.33/bin/bin/../../lib/gcc/pic32mx/4.5.2/../../../../pic32mx/lib\libpic32.a(vector32.o)
 .reginfo       0x00000000       0x18 c:/program files/microchip/xc32/v1.33/bin/bin/../../lib/gcc/pic32mx/4.5.2/../../../../pic32mx/lib\libpic32.a(vector33.o)
 .reginfo       0x00000000       0x18 c:/program files/microchip/xc32/v1.33/bin/bin/../../lib/gcc/pic32mx/4.5.2/../../../../pic32mx/lib\libpic32.a(vector34.o)
 .reginfo       0x00000000       0x18 c:/program files/microchip/xc32/v1.33/bin/bin/../../lib/gcc/pic32mx/4.5.2/../../../../pic32mx/lib\libpic32.a(vector35.o)
 .reginfo       0x00000000       0x18 c:/program files/microchip/xc32/v1.33/bin/bin/../../lib/gcc/pic32mx/4.5.2/../../../../pic32mx/lib\libpic32.a(vector36.o)
 .reginfo       0x00000000       0x18 c:/program files/microchip/xc32/v1.33/bin/bin/../../lib/gcc/pic32mx/4.5.2/../../../../pic32mx/lib\libpic32.a(vector37.o)
 .reginfo       0x00000000       0x18 c:/program files/microchip/xc32/v1.33/bin/bin/../../lib/gcc/pic32mx/4.5.2/../../../../pic32mx/lib\libpic32.a(vector38.o)
 .reginfo       0x00000000       0x18 c:/program files/microchip/xc32/v1.33/bin/bin/../../lib/gcc/pic32mx/4.5.2/../../../../pic32mx/lib\libpic32.a(vector39.o)
 .reginfo       0x00000000       0x18 c:/program files/microchip/xc32/v1.33/bin/bin/../../lib/gcc/pic32mx/4.5.2/../../../../pic32mx/lib\libpic32.a(vector40.o)
 .reginfo       0x00000000       0x18 c:/program files/microchip/xc32/v1.33/bin/bin/../../lib/gcc/pic32mx/4.5.2/../../../../pic32mx/lib\libpic32.a(vector41.o)
 .reginfo       0x00000000       0x18 c:/program files/microchip/xc32/v1.33/bin/bin/../../lib/gcc/pic32mx/4.5.2/../../../../pic32mx/lib\libpic32.a(vector42.o)
 .reginfo       0x00000000       0x18 c:/program files/microchip/xc32/v1.33/bin/bin/../../lib/gcc/pic32mx/4.5.2/../../../../pic32mx/lib\libpic32.a(vector43.o)
 .reginfo       0x00000000       0x18 c:/program files/microchip/xc32/v1.33/bin/bin/../../lib/gcc/pic32mx/4.5.2/../../../../pic32mx/lib\libpic32.a(vector44.o)
 .reginfo       0x00000000       0x18 c:/program files/microchip/xc32/v1.33/bin/bin/../../lib/gcc/pic32mx/4.5.2/../../../../pic32mx/lib\libpic32.a(vector45.o)
 .reginfo       0x00000000       0x18 c:/program files/microchip/xc32/v1.33/bin/bin/../../lib/gcc/pic32mx/4.5.2/../../../../pic32mx/lib\libpic32.a(vector46.o)
 .reginfo       0x00000000       0x18 c:/program files/microchip/xc32/v1.33/bin/bin/../../lib/gcc/pic32mx/4.5.2/../../../../pic32mx/lib\libpic32.a(vector47.o)
 .reginfo       0x00000000       0x18 c:/program files/microchip/xc32/v1.33/bin/bin/../../lib/gcc/pic32mx/4.5.2/../../../../pic32mx/lib\libpic32.a(vector48.o)
 .reginfo       0x00000000       0x18 c:/program files/microchip/xc32/v1.33/bin/bin/../../lib/gcc/pic32mx/4.5.2/../../../../pic32mx/lib\libpic32.a(vector49.o)
 .reginfo       0x00000000       0x18 c:/program files/microchip/xc32/v1.33/bin/bin/../../lib/gcc/pic32mx/4.5.2/../../../../pic32mx/lib\libpic32.a(vector50.o)
 .reginfo       0x00000000       0x18 c:/program files/microchip/xc32/v1.33/bin/bin/../../lib/gcc/pic32mx/4.5.2/../../../../pic32mx/lib\libpic32.a(vector51.o)
 .reginfo       0x00000000       0x18 c:/program files/microchip/xc32/v1.33/bin/bin/../../lib/gcc/pic32mx/4.5.2/../../../../pic32mx/lib\libpic32.a(vector52.o)
 .reginfo       0x00000000       0x18 c:/program files/microchip/xc32/v1.33/bin/bin/../../lib/gcc/pic32mx/4.5.2/../../../../pic32mx/lib\libpic32.a(vector53.o)
 .reginfo       0x00000000       0x18 c:/program files/microchip/xc32/v1.33/bin/bin/../../lib/gcc/pic32mx/4.5.2/../../../../pic32mx/lib\libpic32.a(vector54.o)
 .reginfo       0x00000000       0x18 c:/program files/microchip/xc32/v1.33/bin/bin/../../lib/gcc/pic32mx/4.5.2/../../../../pic32mx/lib\libpic32.a(vector55.o)
 .reginfo       0x00000000       0x18 c:/program files/microchip/xc32/v1.33/bin/bin/../../lib/gcc/pic32mx/4.5.2/../../../../pic32mx/lib\libpic32.a(vector56.o)
 .reginfo       0x00000000       0x18 c:/program files/microchip/xc32/v1.33/bin/bin/../../lib/gcc/pic32mx/4.5.2/../../../../pic32mx/lib\libpic32.a(vector57.o)
 .reginfo       0x00000000       0x18 c:/program files/microchip/xc32/v1.33/bin/bin/../../lib/gcc/pic32mx/4.5.2/../../../../pic32mx/lib\libpic32.a(vector58.o)
 .reginfo       0x00000000       0x18 c:/program files/microchip/xc32/v1.33/bin/bin/../../lib/gcc/pic32mx/4.5.2/../../../../pic32mx/lib\libpic32.a(vector59.o)
 .reginfo       0x00000000       0x18 c:/program files/microchip/xc32/v1.33/bin/bin/../../lib/gcc/pic32mx/4.5.2/../../../../pic32mx/lib\libpic32.a(vector60.o)
 .reginfo       0x00000000       0x18 c:/program files/microchip/xc32/v1.33/bin/bin/../../lib/gcc/pic32mx/4.5.2/../../../../pic32mx/lib\libpic32.a(vector61.o)
 .reginfo       0x00000000       0x18 c:/program files/microchip/xc32/v1.33/bin/bin/../../lib/gcc/pic32mx/4.5.2/../../../../pic32mx/lib\libpic32.a(vector62.o)
 .reginfo       0x00000000       0x18 c:/program files/microchip/xc32/v1.33/bin/bin/../../lib/gcc/pic32mx/4.5.2/../../../../pic32mx/lib\libpic32.a(vector63.o)
 .reginfo       0x00000000       0x18 c:/program files/microchip/xc32/v1.33/bin/bin/../../lib/gcc/pic32mx/4.5.2/../../../../pic32mx/lib\libpic32.a(defaultinterrupt.o)
 .reginfo       0x00000000       0x18 c:/program files/microchip/xc32/v1.33/bin/bin/../../lib/gcc/pic32mx/4.5.2/../../../../pic32mx/lib\libc.a(puts.o)
 .reginfo       0x00000000       0x18 c:/program files/microchip/xc32/v1.33/bin/bin/../../lib/gcc/pic32mx/4.5.2/../../../../pic32mx/lib\libc.a(strncmp.o)
 .reginfo       0x00000000       0x18 c:/program files/microchip/xc32/v1.33/bin/bin/../../lib/gcc/pic32mx/4.5.2/../../../../pic32mx/lib\libc.a(printf_cdnopsuxX.eo)
 .reginfo       0x00000000       0x18 c:/program files/microchip/xc32/v1.33/bin/bin/../../lib/gcc/pic32mx/4.5.2/../../../../pic32mx/lib\libc.a(sprintf_cdnopuxX.eo)
 .reginfo       0x00000000       0x18 c:/program files/microchip/xc32/v1.33/bin/bin/../../lib/gcc/pic32mx/4.5.2/../../../../pic32mx/lib\libc.a(sscanf_s.eo)
 .reginfo       0x00000000       0x18 c:/program files/microchip/xc32/v1.33/bin/bin/../../lib/gcc/pic32mx/4.5.2/../../../../pic32mx/lib\libc.a(_iob.o)
 .reginfo       0x00000000       0x18 c:/program files/microchip/xc32/v1.33/bin/bin/../../lib/gcc/pic32mx/4.5.2/../../../../pic32mx/lib\libc.a(_fputc_simple.o)
 .reginfo       0x00000000       0x18 c:/program files/microchip/xc32/v1.33/bin/bin/../../lib/gcc/pic32mx/4.5.2/../../../../pic32mx/lib\libc.a(doprnt_cdnopsuxX.eo)
 .reginfo       0x00000000       0x18 c:/program files/microchip/xc32/v1.33/bin/bin/../../lib/gcc/pic32mx/4.5.2/../../../../pic32mx/lib\libc.a(doscan_s.eo)
 .reginfo       0x00000000       0x18 c:/program files/microchip/xc32/v1.33/bin/bin/../../lib/gcc/pic32mx/4.5.2/../../../../pic32mx/lib\libc.a(_flsbuf_simple.o)
 .reginfo       0x00000000       0x18 c:/program files/microchip/xc32/v1.33/bin/bin/../../lib/gcc/pic32mx/4.5.2/../../../../pic32mx/lib\libc.a(fgetc.o)
 .reginfo       0x00000000       0x18 c:/program files/microchip/xc32/v1.33/bin/bin/../../lib/gcc/pic32mx/4.5.2/../../../../pic32mx/lib\libc.a(atoi.o)
 .reginfo       0x00000000       0x18 c:/program files/microchip/xc32/v1.33/bin/bin/../../lib/gcc/pic32mx/4.5.2/../../../../pic32mx/lib\libc.a(ctype.o)
 .reginfo       0x00000000       0x18 c:/program files/microchip/xc32/v1.33/bin/bin/../../lib/gcc/pic32mx/4.5.2/../../../../pic32mx/lib\libc.a(ctypef.o)
 .reginfo       0x00000000       0x18 c:/program files/microchip/xc32/v1.33/bin/bin/../../lib/gcc/pic32mx/4.5.2/../../../../pic32mx/lib\libc.a(ungetc.o)
 .reginfo       0x00000000       0x18 c:/program files/microchip/xc32/v1.33/bin/bin/../../lib/gcc/pic32mx/4.5.2/../../../../pic32mx/lib\libc.a(filbuf.o)
 .reginfo       0x00000000       0x18 c:/program files/microchip/xc32/v1.33/bin/bin/../../lib/gcc/pic32mx/4.5.2/../../../../pic32mx/lib\libc.a(fflush.o)
 .reginfo       0x00000000       0x18 c:/program files/microchip/xc32/v1.33/bin/bin/../../lib/gcc/pic32mx/4.5.2/../../../../pic32mx/lib\libpic32.a(read.o)
 .reginfo       0x00000000       0x18 c:/program files/microchip/xc32/v1.33/bin/bin/../../lib/gcc/pic32mx/4.5.2/../../../../pic32mx/lib\libpic32.a(write.o)
 .reginfo       0x00000000       0x18 c:/program files/microchip/xc32/v1.33/bin/bin/../../lib/gcc/pic32mx/4.5.2/../../../../pic32mx/lib\libpic32.a(xc32_uart.o)
 .reginfo       0x00000000       0x18 c:/program files/microchip/xc32/v1.33/bin/bin/../../lib/gcc/pic32mx/4.5.2\libgcc.a(_udivdi3.o)
 .reginfo       0x00000000       0x18 c:/program files/microchip/xc32/v1.33/bin/bin/../../lib/gcc/pic32mx/4.5.2\libgcc.a(_umoddi3.o)

Memory Configuration

Name             Origin             Length             Attributes
kseg0_data_mem   0x80000000         0x00000200
kseg1_data_mem   0xa0000000         0x00010000         w !x
kseg0_boot_mem   0x9d005000         0x000007f0
kseg1_boot_mem   0xbfc00000         0x00000490
kseg0_program_mem 0x9d005800         0x0007a7ff         xr
exception_mem    0x9d004000         0x00001000
debug_exec_mem   0xbfc02000         0x00000ff0
config3          0xbfc02ff0         0x00000004
config2          0xbfc02ff4         0x00000004
config1          0xbfc02ff8         0x00000004
config0          0xbfc02ffc         0x00000004
sfrs             0xbf800000         0x00100000
configsfrs       0xbfc02ff0         0x00000010
*default*        0x00000000         0xffffffff

Linker script and memory map


reserve_data_0_kseg0
                0x80000000      0x200
                0x80000000        0x2 SHORT 0x0
                0x000001fd                . = 0x1fd
 *fill*         0x80000002      0x1fb 
                0x80000200                . = ALIGN (0x4)
 *fill*         0x800001fd        0x3 

reserve_data_0_kseg1
                0xa0000000      0x200
                0xa0000000        0x2 SHORT 0x0
                0x000001fd                . = 0x1fd
 *fill*         0xa0000002      0x1fb 
                0xa0000200                . = ALIGN (0x4)
 *fill*         0xa00001fd        0x3 

reserve_boot_0x1fc02000_kseg0
                0x9fc02000      0xff0
                0x9fc02000        0x2 SHORT 0x0
                0x00000500                . = 0x500
 *fill*         0x9fc02002      0x4fe 
                0x9fc02500                . = ALIGN (0x4)
                0x9fc02500        0x2 SHORT 0x0
                0x00000ff0                . = 0xff0
 *fill*         0x9fc02502      0xaee 
                0x9fc02ff0                . = ALIGN (0x4)

reserve_boot_0x1fc02000_kseg1
                0xbfc02000      0xff0
                0xbfc02000        0x2 SHORT 0x0
                0x00000500                . = 0x500
 *fill*         0xbfc02002      0x4fe 
                0xbfc02500                . = ALIGN (0x4)
                0xbfc02500        0x2 SHORT 0x0
                0x00000ff0                . = 0xff0
 *fill*         0xbfc02502      0xaee 
                0xbfc02ff0                . = ALIGN (0x4)
LOAD c:/program files/microchip/xc32/v1.33/bin/bin/../../lib/gcc/pic32mx/4.5.2/../../../../pic32mx/lib/./proc/32MX795F512H/crt0_mips32r2.o
LOAD c:/program files/microchip/xc32/v1.33/bin/bin/../../lib/gcc/pic32mx/4.5.2/../../../../pic32mx/lib\software-debug-break.o
LOAD build/ChaletDuinoV2_795F512H_/debug/Source/ChaletduinoV2Board.o
LOAD build/ChaletDuinoV2_795F512H_/debug/Source/winc3400_142/common/source/nm_common.o
LOAD build/ChaletDuinoV2_795F512H_/debug/Source/winc3400_142/driver/source/m2m_flash.o
LOAD build/ChaletDuinoV2_795F512H_/debug/Source/winc3400_142/driver/source/m2m_hif.o
LOAD build/ChaletDuinoV2_795F512H_/debug/Source/winc3400_142/driver/source/m2m_ota.o
LOAD build/ChaletDuinoV2_795F512H_/debug/Source/winc3400_142/driver/source/m2m_periph.o
LOAD build/ChaletDuinoV2_795F512H_/debug/Source/winc3400_142/driver/source/m2m_ssl.o
LOAD build/ChaletDuinoV2_795F512H_/debug/Source/winc3400_142/driver/source/m2m_wifi.o
LOAD build/ChaletDuinoV2_795F512H_/debug/Source/winc3400_142/driver/source/nmasic.o
LOAD build/ChaletDuinoV2_795F512H_/debug/Source/winc3400_142/driver/source/nmbus.o
LOAD build/ChaletDuinoV2_795F512H_/debug/Source/winc3400_142/driver/source/nmdrv.o
LOAD build/ChaletDuinoV2_795F512H_/debug/Source/winc3400_142/driver/source/nmspi.o
LOAD build/ChaletDuinoV2_795F512H_/debug/Source/winc3400_142/socket/source/inet_addr.o
LOAD build/ChaletDuinoV2_795F512H_/debug/Source/winc3400_142/socket/source/inet_ntop.o
LOAD build/ChaletDuinoV2_795F512H_/debug/Source/winc3400_142/socket/source/socket.o
LOAD build/ChaletDuinoV2_795F512H_/debug/Source/winc3400_142/spi_flash/source/spi_flash.o
LOAD build/ChaletDuinoV2_795F512H_/debug/Source/DigitalIO.o
LOAD build/ChaletDuinoV2_795F512H_/debug/Source/NetworkProtocol.o
LOAD build/ChaletDuinoV2_795F512H_/debug/Source/Terminal.o
LOAD build/ChaletDuinoV2_795F512H_/debug/Source/Util.o
LOAD build/ChaletDuinoV2_795F512H_/debug/Source/exceptions.o
LOAD build/ChaletDuinoV2_795F512H_/debug/Source/interrupts.o
LOAD build/ChaletDuinoV2_795F512H_/debug/Source/main.o
LOAD build/ChaletDuinoV2_795F512H_/debug/Source/system.o
LOAD build/ChaletDuinoV2_795F512H_/debug/Source/template.o
LOAD build/ChaletDuinoV2_795F512H_/debug/Source/timer.o
LOAD build/ChaletDuinoV2_795F512H_/debug/Source/WiFiCtrl.o
LOAD build/ChaletDuinoV2_795F512H_/debug/Source/SPI.o
LOAD build/ChaletDuinoV2_795F512H_/debug/Source/SPI_Flash.o
LOAD build/ChaletDuinoV2_795F512H_/debug/Source/Syslog.o
LOAD build/ChaletDuinoV2_795F512H_/debug/Source/Watchdog.o
LOAD build/ChaletDuinoV2_795F512H_/debug/Source/BootloaderInterface.o
LOAD build/ChaletDuinoV2_795F512H_/debug/Source/BootloaderProtocol.o
LOAD build/ChaletDuinoV2_795F512H_/debug/Source/crc32.o
LOAD build/ChaletDuinoV2_795F512H_/debug/Source/VolumeTransducer.o
LOAD build/ChaletDuinoV2_795F512H_/debug/Source/DACInterface.o
                0x00000001                __MPLAB_BUILD = 0x1
                0x00000400                PROVIDE (_min_stack_size, 0x400)
LOAD c:/program files/microchip/xc32/v1.33/bin/bin/../../lib/gcc/pic32mx/4.5.2/../../../../pic32mx/lib/./proc/32MX795F512H\processor.o
START GROUP
LOAD c:/program files/microchip/xc32/v1.33/bin/bin/../../lib/gcc/pic32mx/4.5.2/../../../../pic32mx/lib\libmchp_peripheral.a
END GROUP
START GROUP
LOAD c:/program files/microchip/xc32/v1.33/bin/bin/../../lib/gcc/pic32mx/4.5.2/../../../../pic32mx/lib\libmchp_peripheral_32MX795F512H.a
END GROUP
                0x00000001                PROVIDE (_vector_spacing, 0x1)
                0x9d004000                _ebase_address = 0x9d004000
                0xbfc00000                _RESET_ADDR = 0xbfc00000
                0xbfc00380                _BEV_EXCPT_ADDR = 0xbfc00380
                0xbfc00480                _DBG_EXCPT_ADDR = 0xbfc00480
                0xbfc02000                _DBG_CODE_ADDR = 0xbfc02000
                0x00000ff0                _DBG_CODE_SIZE = 0xff0
                0x9d004180                _GEN_EXCPT_ADDR = (_ebase_address + 0x180)

.config_BFC02FF0
 *(.config_BFC02FF0)

.config_BFC02FF4
                0xbfc02ff4        0x4
 *(.config_BFC02FF4)
 .config_BFC02FF4
                0xbfc02ff4        0x4 build/ChaletDuinoV2_795F512H_/debug/Source/main.o

.config_BFC02FF8
                0xbfc02ff8        0x4
 *(.config_BFC02FF8)
 .config_BFC02FF8
                0xbfc02ff8        0x4 build/ChaletDuinoV2_795F512H_/debug/Source/main.o

.config_BFC02FFC
                0xbfc02ffc        0x4
 *(.config_BFC02FFC)
 .config_BFC02FFC
                0xbfc02ffc        0x4 build/ChaletDuinoV2_795F512H_/debug/Source/main.o
                0xbfc02000                PROVIDE (_DBG_CODE_ADDR, 0xbfc02000)
                0x00000ff0                PROVIDE (_DBG_CODE_SIZE, 0xff0)

.reset          0xbfc00000        0x8
 *(.reset)
 .reset         0xbfc00000        0x8 c:/program files/microchip/xc32/v1.33/bin/bin/../../lib/gcc/pic32mx/4.5.2/../../../../pic32mx/lib/./proc/32MX795F512H/crt0_mips32r2.o
                0xbfc00000                _reset

.bev_excpt      0xbfc00380       0x10
 *(.bev_handler)
 .bev_handler   0xbfc00380       0x10 c:/program files/microchip/xc32/v1.33/bin/bin/../../lib/gcc/pic32mx/4.5.2/../../../../pic32mx/lib/./proc/32MX795F512H/crt0_mips32r2.o

.dbg_excpt      0xbfc00480        0x0
                0xbfc00480                . = (. + DEFINED (_DEBUGGER)?0x8:0x0)

.dbg_code       0xbfc02000        0x0
                0xbfc02000                . = (. + DEFINED (_DEBUGGER)?_DBG_CODE_SIZE:0x0)

.app_excpt      0x9d004180       0x10
 *(.gen_handler)
 .gen_handler   0x9d004180       0x10 c:/program files/microchip/xc32/v1.33/bin/bin/../../lib/gcc/pic32mx/4.5.2/../../../../pic32mx/lib/./proc/32MX795F512H/crt0_mips32r2.o

.vector_0       0x9d004200        0x8
 *(.vector_0)
 .vector_0      0x9d004200        0x8 c:/program files/microchip/xc32/v1.33/bin/bin/../../lib/gcc/pic32mx/4.5.2/../../../../pic32mx/lib\libpic32.a(vector0.o)
                0x9d004200                __vector_dispatch_0
                0x00000001                ASSERT (((_vector_spacing == 0x0) || (SIZEOF (.vector_0) <= (_vector_spacing << 0x5))), function at exception vector 0 too large)

.vector_1       0x9d004220        0x8
 *(.vector_1)
 .vector_1      0x9d004220        0x8 c:/program files/microchip/xc32/v1.33/bin/bin/../../lib/gcc/pic32mx/4.5.2/../../../../pic32mx/lib\libpic32.a(vector1.o)
                0x9d004220                __vector_dispatch_1
                0x00000001                ASSERT (((_vector_spacing == 0x0) || (SIZEOF (.vector_1) <= (_vector_spacing << 0x5))), function at exception vector 1 too large)

.vector_2       0x9d004240        0x8
 *(.vector_2)
 .vector_2      0x9d004240        0x8 c:/program files/microchip/xc32/v1.33/bin/bin/../../lib/gcc/pic32mx/4.5.2/../../../../pic32mx/lib\libpic32.a(vector2.o)
                0x9d004240                __vector_dispatch_2
                0x00000001                ASSERT (((_vector_spacing == 0x0) || (SIZEOF (.vector_2) <= (_vector_spacing << 0x5))), function at exception vector 2 too large)

.vector_3       0x9d004260        0x8
 *(.vector_3)
 .vector_3      0x9d004260        0x8 build/ChaletDuinoV2_795F512H_/debug/Source/winc3400_142/common/source/nm_common.o
                0x9d004260                __vector_dispatch_3
                0x00000001                ASSERT (((_vector_spacing == 0x0) || (SIZEOF (.vector_3) <= (_vector_spacing << 0x5))), function at exception vector 3 too large)

.vector_4       0x9d004280        0x8
 *(.vector_4)
 .vector_4      0x9d004280        0x8 build/ChaletDuinoV2_795F512H_/debug/Source/timer.o
                0x9d004280                __vector_dispatch_4
                0x00000001                ASSERT (((_vector_spacing == 0x0) || (SIZEOF (.vector_4) <= (_vector_spacing << 0x5))), function at exception vector 4 too large)

.vector_5       0x9d0042a0        0x8
 *(.vector_5)
 .vector_5      0x9d0042a0        0x8 c:/program files/microchip/xc32/v1.33/bin/bin/../../lib/gcc/pic32mx/4.5.2/../../../../pic32mx/lib\libpic32.a(vector5.o)
                0x9d0042a0                __vector_dispatch_5
                0x00000001                ASSERT (((_vector_spacing == 0x0) || (SIZEOF (.vector_5) <= (_vector_spacing << 0x5))), function at exception vector 5 too large)

.vector_6       0x9d0042c0        0x8
 *(.vector_6)
 .vector_6      0x9d0042c0        0x8 c:/program files/microchip/xc32/v1.33/bin/bin/../../lib/gcc/pic32mx/4.5.2/../../../../pic32mx/lib\libpic32.a(vector6.o)
                0x9d0042c0                __vector_dispatch_6
                0x00000001                ASSERT (((_vector_spacing == 0x0) || (SIZEOF (.vector_6) <= (_vector_spacing << 0x5))), function at exception vector 6 too large)

.vector_7       0x9d0042e0        0x8
 *(.vector_7)
 .vector_7      0x9d0042e0        0x8 build/ChaletDuinoV2_795F512H_/debug/Source/VolumeTransducer.o
                0x9d0042e0                __vector_dispatch_7
                0x00000001                ASSERT (((_vector_spacing == 0x0) || (SIZEOF (.vector_7) <= (_vector_spacing << 0x5))), function at exception vector 7 too large)

.vector_8       0x9d004300        0x8
 *(.vector_8)
 .vector_8      0x9d004300        0x8 c:/program files/microchip/xc32/v1.33/bin/bin/../../lib/gcc/pic32mx/4.5.2/../../../../pic32mx/lib\libpic32.a(vector8.o)
                0x9d004300                __vector_dispatch_8
                0x00000001                ASSERT (((_vector_spacing == 0x0) || (SIZEOF (.vector_8) <= (_vector_spacing << 0x5))), function at exception vector 8 too large)

.vector_9       0x9d004320        0x8
 *(.vector_9)
 .vector_9      0x9d004320        0x8 c:/program files/microchip/xc32/v1.33/bin/bin/../../lib/gcc/pic32mx/4.5.2/../../../../pic32mx/lib\libpic32.a(vector9.o)
                0x9d004320                __vector_dispatch_9
                0x00000001                ASSERT (((_vector_spacing == 0x0) || (SIZEOF (.vector_9) <= (_vector_spacing << 0x5))), function at exception vector 9 too large)

.vector_10      0x9d004340        0x8
 *(.vector_10)
 .vector_10     0x9d004340        0x8 c:/program files/microchip/xc32/v1.33/bin/bin/../../lib/gcc/pic32mx/4.5.2/../../../../pic32mx/lib\libpic32.a(vector10.o)
                0x9d004340                __vector_dispatch_10
                0x00000001                ASSERT (((_vector_spacing == 0x0) || (SIZEOF (.vector_10) <= (_vector_spacing << 0x5))), function at exception vector 10 too large)

.vector_11      0x9d004360        0x8
 *(.vector_11)
 .vector_11     0x9d004360        0x8 c:/program files/microchip/xc32/v1.33/bin/bin/../../lib/gcc/pic32mx/4.5.2/../../../../pic32mx/lib\libpic32.a(vector11.o)
                0x9d004360                __vector_dispatch_11
                0x00000001                ASSERT (((_vector_spacing == 0x0) || (SIZEOF (.vector_11) <= (_vector_spacing << 0x5))), function at exception vector 11 too large)

.vector_12      0x9d004380        0x8
 *(.vector_12)
 .vector_12     0x9d004380        0x8 c:/program files/microchip/xc32/v1.33/bin/bin/../../lib/gcc/pic32mx/4.5.2/../../../../pic32mx/lib\libpic32.a(vector12.o)
                0x9d004380                __vector_dispatch_12
                0x00000001                ASSERT (((_vector_spacing == 0x0) || (SIZEOF (.vector_12) <= (_vector_spacing << 0x5))), function at exception vector 12 too large)

.vector_13      0x9d0043a0        0x8
 *(.vector_13)
 .vector_13     0x9d0043a0        0x8 c:/program files/microchip/xc32/v1.33/bin/bin/../../lib/gcc/pic32mx/4.5.2/../../../../pic32mx/lib\libpic32.a(vector13.o)
                0x9d0043a0                __vector_dispatch_13
                0x00000001                ASSERT (((_vector_spacing == 0x0) || (SIZEOF (.vector_13) <= (_vector_spacing << 0x5))), function at exception vector 13 too large)

.vector_14      0x9d0043c0        0x8
 *(.vector_14)
 .vector_14     0x9d0043c0        0x8 c:/program files/microchip/xc32/v1.33/bin/bin/../../lib/gcc/pic32mx/4.5.2/../../../../pic32mx/lib\libpic32.a(vector14.o)
                0x9d0043c0                __vector_dispatch_14
                0x00000001                ASSERT (((_vector_spacing == 0x0) || (SIZEOF (.vector_14) <= (_vector_spacing << 0x5))), function at exception vector 14 too large)

.vector_15      0x9d0043e0        0x8
 *(.vector_15)
 .vector_15     0x9d0043e0        0x8 build/ChaletDuinoV2_795F512H_/debug/Source/VolumeTransducer.o
                0x9d0043e0                __vector_dispatch_15
                0x00000001                ASSERT (((_vector_spacing == 0x0) || (SIZEOF (.vector_15) <= (_vector_spacing << 0x5))), function at exception vector 15 too large)

.vector_16      0x9d004400        0x8
 *(.vector_16)
 .vector_16     0x9d004400        0x8 c:/program files/microchip/xc32/v1.33/bin/bin/../../lib/gcc/pic32mx/4.5.2/../../../../pic32mx/lib\libpic32.a(vector16.o)
                0x9d004400                __vector_dispatch_16
                0x00000001                ASSERT (((_vector_spacing == 0x0) || (SIZEOF (.vector_16) <= (_vector_spacing << 0x5))), function at exception vector 16 too large)

.vector_17      0x9d004420        0x8
 *(.vector_17)
 .vector_17     0x9d004420        0x8 c:/program files/microchip/xc32/v1.33/bin/bin/../../lib/gcc/pic32mx/4.5.2/../../../../pic32mx/lib\libpic32.a(vector17.o)
                0x9d004420                __vector_dispatch_17
                0x00000001                ASSERT (((_vector_spacing == 0x0) || (SIZEOF (.vector_17) <= (_vector_spacing << 0x5))), function at exception vector 17 too large)

.vector_18      0x9d004440        0x8
 *(.vector_18)
 .vector_18     0x9d004440        0x8 c:/program files/microchip/xc32/v1.33/bin/bin/../../lib/gcc/pic32mx/4.5.2/../../../../pic32mx/lib\libpic32.a(vector18.o)
                0x9d004440                __vector_dispatch_18
                0x00000001                ASSERT (((_vector_spacing == 0x0) || (SIZEOF (.vector_18) <= (_vector_spacing << 0x5))), function at exception vector 18 too large)

.vector_19      0x9d004460        0x8
 *(.vector_19)
 .vector_19     0x9d004460        0x8 c:/program files/microchip/xc32/v1.33/bin/bin/../../lib/gcc/pic32mx/4.5.2/../../../../pic32mx/lib\libpic32.a(vector19.o)
                0x9d004460                __vector_dispatch_19
                0x00000001                ASSERT (((_vector_spacing == 0x0) || (SIZEOF (.vector_19) <= (_vector_spacing << 0x5))), function at exception vector 19 too large)

.vector_20      0x9d004480        0x8
 *(.vector_20)
 .vector_20     0x9d004480        0x8 c:/program files/microchip/xc32/v1.33/bin/bin/../../lib/gcc/pic32mx/4.5.2/../../../../pic32mx/lib\libpic32.a(vector20.o)
                0x9d004480                __vector_dispatch_20
                0x00000001                ASSERT (((_vector_spacing == 0x0) || (SIZEOF (.vector_20) <= (_vector_spacing << 0x5))), function at exception vector 20 too large)

.vector_21      0x9d0044a0        0x8
 *(.vector_21)
 .vector_21     0x9d0044a0        0x8 c:/program files/microchip/xc32/v1.33/bin/bin/../../lib/gcc/pic32mx/4.5.2/../../../../pic32mx/lib\libpic32.a(vector21.o)
                0x9d0044a0                __vector_dispatch_21
                0x00000001                ASSERT (((_vector_spacing == 0x0) || (SIZEOF (.vector_21) <= (_vector_spacing << 0x5))), function at exception vector 21 too large)

.vector_22      0x9d0044c0        0x8
 *(.vector_22)
 .vector_22     0x9d0044c0        0x8 c:/program files/microchip/xc32/v1.33/bin/bin/../../lib/gcc/pic32mx/4.5.2/../../../../pic32mx/lib\libpic32.a(vector22.o)
                0x9d0044c0                __vector_dispatch_22
                0x00000001                ASSERT (((_vector_spacing == 0x0) || (SIZEOF (.vector_22) <= (_vector_spacing << 0x5))), function at exception vector 22 too large)

.vector_23      0x9d0044e0        0x8
 *(.vector_23)
 .vector_23     0x9d0044e0        0x8 c:/program files/microchip/xc32/v1.33/bin/bin/../../lib/gcc/pic32mx/4.5.2/../../../../pic32mx/lib\libpic32.a(vector23.o)
                0x9d0044e0                __vector_dispatch_23
                0x00000001                ASSERT (((_vector_spacing == 0x0) || (SIZEOF (.vector_23) <= (_vector_spacing << 0x5))), function at exception vector 23 too large)

.vector_24      0x9d004500        0x8
 *(.vector_24)
 .vector_24     0x9d004500        0x8 c:/program files/microchip/xc32/v1.33/bin/bin/../../lib/gcc/pic32mx/4.5.2/../../../../pic32mx/lib\libpic32.a(vector24.o)
                0x9d004500                __vector_dispatch_24
                0x00000001                ASSERT (((_vector_spacing == 0x0) || (SIZEOF (.vector_24) <= (_vector_spacing << 0x5))), function at exception vector 24 too large)

.vector_25      0x9d004520        0x8
 *(.vector_25)
 .vector_25     0x9d004520        0x8 c:/program files/microchip/xc32/v1.33/bin/bin/../../lib/gcc/pic32mx/4.5.2/../../../../pic32mx/lib\libpic32.a(vector25.o)
                0x9d004520                __vector_dispatch_25
                0x00000001                ASSERT (((_vector_spacing == 0x0) || (SIZEOF (.vector_25) <= (_vector_spacing << 0x5))), function at exception vector 25 too large)

.vector_26      0x9d004540        0x8
 *(.vector_26)
 .vector_26     0x9d004540        0x8 c:/program files/microchip/xc32/v1.33/bin/bin/../../lib/gcc/pic32mx/4.5.2/../../../../pic32mx/lib\libpic32.a(vector26.o)
                0x9d004540                __vector_dispatch_26
                0x00000001                ASSERT (((_vector_spacing == 0x0) || (SIZEOF (.vector_26) <= (_vector_spacing << 0x5))), function at exception vector 26 too large)

.vector_27      0x9d004560        0x8
 *(.vector_27)
 .vector_27     0x9d004560        0x8 c:/program files/microchip/xc32/v1.33/bin/bin/../../lib/gcc/pic32mx/4.5.2/../../../../pic32mx/lib\libpic32.a(vector27.o)
                0x9d004560                __vector_dispatch_27
                0x00000001                ASSERT (((_vector_spacing == 0x0) || (SIZEOF (.vector_27) <= (_vector_spacing << 0x5))), function at exception vector 27 too large)

.vector_28      0x9d004580        0x8
 *(.vector_28)
 .vector_28     0x9d004580        0x8 c:/program files/microchip/xc32/v1.33/bin/bin/../../lib/gcc/pic32mx/4.5.2/../../../../pic32mx/lib\libpic32.a(vector28.o)
                0x9d004580                __vector_dispatch_28
                0x00000001                ASSERT (((_vector_spacing == 0x0) || (SIZEOF (.vector_28) <= (_vector_spacing << 0x5))), function at exception vector 28 too large)

.vector_29      0x9d0045a0        0x8
 *(.vector_29)
 .vector_29     0x9d0045a0        0x8 c:/program files/microchip/xc32/v1.33/bin/bin/../../lib/gcc/pic32mx/4.5.2/../../../../pic32mx/lib\libpic32.a(vector29.o)
                0x9d0045a0                __vector_dispatch_29
                0x00000001                ASSERT (((_vector_spacing == 0x0) || (SIZEOF (.vector_29) <= (_vector_spacing << 0x5))), function at exception vector 29 too large)

.vector_30      0x9d0045c0        0x8
 *(.vector_30)
 .vector_30     0x9d0045c0        0x8 c:/program files/microchip/xc32/v1.33/bin/bin/../../lib/gcc/pic32mx/4.5.2/../../../../pic32mx/lib\libpic32.a(vector30.o)
                0x9d0045c0                __vector_dispatch_30
                0x00000001                ASSERT (((_vector_spacing == 0x0) || (SIZEOF (.vector_30) <= (_vector_spacing << 0x5))), function at exception vector 30 too large)

.vector_31      0x9d0045e0        0x8
 *(.vector_31)
 .vector_31     0x9d0045e0        0x8 c:/program files/microchip/xc32/v1.33/bin/bin/../../lib/gcc/pic32mx/4.5.2/../../../../pic32mx/lib\libpic32.a(vector31.o)
                0x9d0045e0                __vector_dispatch_31
                0x00000001                ASSERT (((_vector_spacing == 0x0) || (SIZEOF (.vector_31) <= (_vector_spacing << 0x5))), function at exception vector 31 too large)

.vector_32      0x9d004600        0x8
 *(.vector_32)
 .vector_32     0x9d004600        0x8 c:/program files/microchip/xc32/v1.33/bin/bin/../../lib/gcc/pic32mx/4.5.2/../../../../pic32mx/lib\libpic32.a(vector32.o)
                0x9d004600                __vector_dispatch_32
                0x00000001                ASSERT (((_vector_spacing == 0x0) || (SIZEOF (.vector_32) <= (_vector_spacing << 0x5))), function at exception vector 32 too large)

.vector_33      0x9d004620        0x8
 *(.vector_33)
 .vector_33     0x9d004620        0x8 c:/program files/microchip/xc32/v1.33/bin/bin/../../lib/gcc/pic32mx/4.5.2/../../../../pic32mx/lib\libpic32.a(vector33.o)
                0x9d004620                __vector_dispatch_33
                0x00000001                ASSERT (((_vector_spacing == 0x0) || (SIZEOF (.vector_33) <= (_vector_spacing << 0x5))), function at exception vector 33 too large)

.vector_34      0x9d004640        0x8
 *(.vector_34)
 .vector_34     0x9d004640        0x8 c:/program files/microchip/xc32/v1.33/bin/bin/../../lib/gcc/pic32mx/4.5.2/../../../../pic32mx/lib\libpic32.a(vector34.o)
                0x9d004640                __vector_dispatch_34
                0x00000001                ASSERT (((_vector_spacing == 0x0) || (SIZEOF (.vector_34) <= (_vector_spacing << 0x5))), function at exception vector 34 too large)

.vector_35      0x9d004660        0x8
 *(.vector_35)
 .vector_35     0x9d004660        0x8 c:/program files/microchip/xc32/v1.33/bin/bin/../../lib/gcc/pic32mx/4.5.2/../../../../pic32mx/lib\libpic32.a(vector35.o)
                0x9d004660                __vector_dispatch_35
                0x00000001                ASSERT (((_vector_spacing == 0x0) || (SIZEOF (.vector_35) <= (_vector_spacing << 0x5))), function at exception vector 35 too large)

.vector_36      0x9d004680        0x8
 *(.vector_36)
 .vector_36     0x9d004680        0x8 c:/program files/microchip/xc32/v1.33/bin/bin/../../lib/gcc/pic32mx/4.5.2/../../../../pic32mx/lib\libpic32.a(vector36.o)
                0x9d004680                __vector_dispatch_36
                0x00000001                ASSERT (((_vector_spacing == 0x0) || (SIZEOF (.vector_36) <= (_vector_spacing << 0x5))), function at exception vector 36 too large)

.vector_37      0x9d0046a0        0x8
 *(.vector_37)
 .vector_37     0x9d0046a0        0x8 c:/program files/microchip/xc32/v1.33/bin/bin/../../lib/gcc/pic32mx/4.5.2/../../../../pic32mx/lib\libpic32.a(vector37.o)
                0x9d0046a0                __vector_dispatch_37
                0x00000001                ASSERT (((_vector_spacing == 0x0) || (SIZEOF (.vector_37) <= (_vector_spacing << 0x5))), function at exception vector 37 too large)

.vector_38      0x9d0046c0        0x8
 *(.vector_38)
 .vector_38     0x9d0046c0        0x8 c:/program files/microchip/xc32/v1.33/bin/bin/../../lib/gcc/pic32mx/4.5.2/../../../../pic32mx/lib\libpic32.a(vector38.o)
                0x9d0046c0                __vector_dispatch_38
                0x00000001                ASSERT (((_vector_spacing == 0x0) || (SIZEOF (.vector_38) <= (_vector_spacing << 0x5))), function at exception vector 38 too large)

.vector_39      0x9d0046e0        0x8
 *(.vector_39)
 .vector_39     0x9d0046e0        0x8 c:/program files/microchip/xc32/v1.33/bin/bin/../../lib/gcc/pic32mx/4.5.2/../../../../pic32mx/lib\libpic32.a(vector39.o)
                0x9d0046e0                __vector_dispatch_39
                0x00000001                ASSERT (((_vector_spacing == 0x0) || (SIZEOF (.vector_39) <= (_vector_spacing << 0x5))), function at exception vector 39 too large)

.vector_40      0x9d004700        0x8
 *(.vector_40)
 .vector_40     0x9d004700        0x8 c:/program files/microchip/xc32/v1.33/bin/bin/../../lib/gcc/pic32mx/4.5.2/../../../../pic32mx/lib\libpic32.a(vector40.o)
                0x9d004700                __vector_dispatch_40
                0x00000001                ASSERT (((_vector_spacing == 0x0) || (SIZEOF (.vector_40) <= (_vector_spacing << 0x5))), function at exception vector 40 too large)

.vector_41      0x9d004720        0x8
 *(.vector_41)
 .vector_41     0x9d004720        0x8 c:/program files/microchip/xc32/v1.33/bin/bin/../../lib/gcc/pic32mx/4.5.2/../../../../pic32mx/lib\libpic32.a(vector41.o)
                0x9d004720                __vector_dispatch_41
                0x00000001                ASSERT (((_vector_spacing == 0x0) || (SIZEOF (.vector_41) <= (_vector_spacing << 0x5))), function at exception vector 41 too large)

.vector_42      0x9d004740        0x8
 *(.vector_42)
 .vector_42     0x9d004740        0x8 c:/program files/microchip/xc32/v1.33/bin/bin/../../lib/gcc/pic32mx/4.5.2/../../../../pic32mx/lib\libpic32.a(vector42.o)
                0x9d004740                __vector_dispatch_42
                0x00000001                ASSERT (((_vector_spacing == 0x0) || (SIZEOF (.vector_42) <= (_vector_spacing << 0x5))), function at exception vector 42 too large)

.vector_43      0x9d004760        0x8
 *(.vector_43)
 .vector_43     0x9d004760        0x8 c:/program files/microchip/xc32/v1.33/bin/bin/../../lib/gcc/pic32mx/4.5.2/../../../../pic32mx/lib\libpic32.a(vector43.o)
                0x9d004760                __vector_dispatch_43
                0x00000001                ASSERT (((_vector_spacing == 0x0) || (SIZEOF (.vector_43) <= (_vector_spacing << 0x5))), function at exception vector 43 too large)

.vector_44      0x9d004780        0x8
 *(.vector_44)
 .vector_44     0x9d004780        0x8 c:/program files/microchip/xc32/v1.33/bin/bin/../../lib/gcc/pic32mx/4.5.2/../../../../pic32mx/lib\libpic32.a(vector44.o)
                0x9d004780                __vector_dispatch_44
                0x00000001                ASSERT (((_vector_spacing == 0x0) || (SIZEOF (.vector_44) <= (_vector_spacing << 0x5))), function at exception vector 44 too large)

.vector_45      0x9d0047a0        0x8
 *(.vector_45)
 .vector_45     0x9d0047a0        0x8 c:/program files/microchip/xc32/v1.33/bin/bin/../../lib/gcc/pic32mx/4.5.2/../../../../pic32mx/lib\libpic32.a(vector45.o)
                0x9d0047a0                __vector_dispatch_45
                0x00000001                ASSERT (((_vector_spacing == 0x0) || (SIZEOF (.vector_45) <= (_vector_spacing << 0x5))), function at exception vector 45 too large)

.vector_46      0x9d0047c0        0x8
 *(.vector_46)
 .vector_46     0x9d0047c0        0x8 c:/program files/microchip/xc32/v1.33/bin/bin/../../lib/gcc/pic32mx/4.5.2/../../../../pic32mx/lib\libpic32.a(vector46.o)
                0x9d0047c0                __vector_dispatch_46
                0x00000001                ASSERT (((_vector_spacing == 0x0) || (SIZEOF (.vector_46) <= (_vector_spacing << 0x5))), function at exception vector 46 too large)

.vector_47      0x9d0047e0        0x8
 *(.vector_47)
 .vector_47     0x9d0047e0        0x8 c:/program files/microchip/xc32/v1.33/bin/bin/../../lib/gcc/pic32mx/4.5.2/../../../../pic32mx/lib\libpic32.a(vector47.o)
                0x9d0047e0                __vector_dispatch_47
                0x00000001                ASSERT (((_vector_spacing == 0x0) || (SIZEOF (.vector_47) <= (_vector_spacing << 0x5))), function at exception vector 47 too large)

.vector_48      0x9d004800        0x8
 *(.vector_48)
 .vector_48     0x9d004800        0x8 c:/program files/microchip/xc32/v1.33/bin/bin/../../lib/gcc/pic32mx/4.5.2/../../../../pic32mx/lib\libpic32.a(vector48.o)
                0x9d004800                __vector_dispatch_48
                0x00000001                ASSERT (((_vector_spacing == 0x0) || (SIZEOF (.vector_48) <= (_vector_spacing << 0x5))), function at exception vector 48 too large)

.vector_49      0x9d004820        0x8
 *(.vector_49)
 .vector_49     0x9d004820        0x8 c:/program files/microchip/xc32/v1.33/bin/bin/../../lib/gcc/pic32mx/4.5.2/../../../../pic32mx/lib\libpic32.a(vector49.o)
                0x9d004820                __vector_dispatch_49
                0x00000001                ASSERT (((_vector_spacing == 0x0) || (SIZEOF (.vector_49) <= (_vector_spacing << 0x5))), function at exception vector 49 too large)

.vector_50      0x9d004840        0x8
 *(.vector_50)
 .vector_50     0x9d004840        0x8 c:/program files/microchip/xc32/v1.33/bin/bin/../../lib/gcc/pic32mx/4.5.2/../../../../pic32mx/lib\libpic32.a(vector50.o)
                0x9d004840                __vector_dispatch_50
                0x00000001                ASSERT (((_vector_spacing == 0x0) || (SIZEOF (.vector_50) <= (_vector_spacing << 0x5))), function at exception vector 50 too large)

.vector_51      0x9d004860        0x8
 *(.vector_51)
 .vector_51     0x9d004860        0x8 c:/program files/microchip/xc32/v1.33/bin/bin/../../lib/gcc/pic32mx/4.5.2/../../../../pic32mx/lib\libpic32.a(vector51.o)
                0x9d004860                __vector_dispatch_51
                0x00000001                ASSERT (((_vector_spacing == 0x0) || (SIZEOF (.vector_51) <= (_vector_spacing << 0x5))), function at exception vector 51 too large)

.vector_52      0x9d004880        0x8
 *(.vector_52)
 .vector_52     0x9d004880        0x8 c:/program files/microchip/xc32/v1.33/bin/bin/../../lib/gcc/pic32mx/4.5.2/../../../../pic32mx/lib\libpic32.a(vector52.o)
                0x9d004880                __vector_dispatch_52
                0x00000001                ASSERT (((_vector_spacing == 0x0) || (SIZEOF (.vector_52) <= (_vector_spacing << 0x5))), function at exception vector 52 too large)

.vector_53      0x9d0048a0        0x8
 *(.vector_53)
 .vector_53     0x9d0048a0        0x8 c:/program files/microchip/xc32/v1.33/bin/bin/../../lib/gcc/pic32mx/4.5.2/../../../../pic32mx/lib\libpic32.a(vector53.o)
                0x9d0048a0                __vector_dispatch_53
                0x00000001                ASSERT (((_vector_spacing == 0x0) || (SIZEOF (.vector_53) <= (_vector_spacing << 0x5))), function at exception vector 53 too large)

.vector_54      0x9d0048c0        0x8
 *(.vector_54)
 .vector_54     0x9d0048c0        0x8 c:/program files/microchip/xc32/v1.33/bin/bin/../../lib/gcc/pic32mx/4.5.2/../../../../pic32mx/lib\libpic32.a(vector54.o)
                0x9d0048c0                __vector_dispatch_54
                0x00000001                ASSERT (((_vector_spacing == 0x0) || (SIZEOF (.vector_54) <= (_vector_spacing << 0x5))), function at exception vector 54 too large)

.vector_55      0x9d0048e0        0x8
 *(.vector_55)
 .vector_55     0x9d0048e0        0x8 c:/program files/microchip/xc32/v1.33/bin/bin/../../lib/gcc/pic32mx/4.5.2/../../../../pic32mx/lib\libpic32.a(vector55.o)
                0x9d0048e0                __vector_dispatch_55
                0x00000001                ASSERT (((_vector_spacing == 0x0) || (SIZEOF (.vector_55) <= (_vector_spacing << 0x5))), function at exception vector 55 too large)

.vector_56      0x9d004900        0x8
 *(.vector_56)
 .vector_56     0x9d004900        0x8 c:/program files/microchip/xc32/v1.33/bin/bin/../../lib/gcc/pic32mx/4.5.2/../../../../pic32mx/lib\libpic32.a(vector56.o)
                0x9d004900                __vector_dispatch_56
                0x00000001                ASSERT (((_vector_spacing == 0x0) || (SIZEOF (.vector_56) <= (_vector_spacing << 0x5))), function at exception vector 56 too large)

.vector_57      0x9d004920        0x8
 *(.vector_57)
 .vector_57     0x9d004920        0x8 c:/program files/microchip/xc32/v1.33/bin/bin/../../lib/gcc/pic32mx/4.5.2/../../../../pic32mx/lib\libpic32.a(vector57.o)
                0x9d004920                __vector_dispatch_57
                0x00000001                ASSERT (((_vector_spacing == 0x0) || (SIZEOF (.vector_57) <= (_vector_spacing << 0x5))), function at exception vector 57 too large)

.vector_58      0x9d004940        0x8
 *(.vector_58)
 .vector_58     0x9d004940        0x8 c:/program files/microchip/xc32/v1.33/bin/bin/../../lib/gcc/pic32mx/4.5.2/../../../../pic32mx/lib\libpic32.a(vector58.o)
                0x9d004940                __vector_dispatch_58
                0x00000001                ASSERT (((_vector_spacing == 0x0) || (SIZEOF (.vector_58) <= (_vector_spacing << 0x5))), function at exception vector 58 too large)

.vector_59      0x9d004960        0x8
 *(.vector_59)
 .vector_59     0x9d004960        0x8 c:/program files/microchip/xc32/v1.33/bin/bin/../../lib/gcc/pic32mx/4.5.2/../../../../pic32mx/lib\libpic32.a(vector59.o)
                0x9d004960                __vector_dispatch_59
                0x00000001                ASSERT (((_vector_spacing == 0x0) || (SIZEOF (.vector_59) <= (_vector_spacing << 0x5))), function at exception vector 59 too large)

.vector_60      0x9d004980        0x8
 *(.vector_60)
 .vector_60     0x9d004980        0x8 c:/program files/microchip/xc32/v1.33/bin/bin/../../lib/gcc/pic32mx/4.5.2/../../../../pic32mx/lib\libpic32.a(vector60.o)
                0x9d004980                __vector_dispatch_60
                0x00000001                ASSERT (((_vector_spacing == 0x0) || (SIZEOF (.vector_60) <= (_vector_spacing << 0x5))), function at exception vector 60 too large)

.vector_61      0x9d0049a0        0x8
 *(.vector_61)
 .vector_61     0x9d0049a0        0x8 c:/program files/microchip/xc32/v1.33/bin/bin/../../lib/gcc/pic32mx/4.5.2/../../../../pic32mx/lib\libpic32.a(vector61.o)
                0x9d0049a0                __vector_dispatch_61
                0x00000001                ASSERT (((_vector_spacing == 0x0) || (SIZEOF (.vector_61) <= (_vector_spacing << 0x5))), function at exception vector 61 too large)

.vector_62      0x9d0049c0        0x8
 *(.vector_62)
 .vector_62     0x9d0049c0        0x8 c:/program files/microchip/xc32/v1.33/bin/bin/../../lib/gcc/pic32mx/4.5.2/../../../../pic32mx/lib\libpic32.a(vector62.o)
                0x9d0049c0                __vector_dispatch_62
                0x00000001                ASSERT (((_vector_spacing == 0x0) || (SIZEOF (.vector_62) <= (_vector_spacing << 0x5))), function at exception vector 62 too large)

.vector_63      0x9d0049e0        0x8
 *(.vector_63)
 .vector_63     0x9d0049e0        0x8 c:/program files/microchip/xc32/v1.33/bin/bin/../../lib/gcc/pic32mx/4.5.2/../../../../pic32mx/lib\libpic32.a(vector63.o)
                0x9d0049e0                __vector_dispatch_63
                0x00000001                ASSERT (((_vector_spacing == 0x0) || (SIZEOF (.vector_63) <= (_vector_spacing << 0x5))), function at exception vector 63 too large)

.startup        0x9d005000      0x1e8
 *(.startup)
 *(.reset.startup)
 .reset.startup
                0x9d005000      0x1e8 c:/program files/microchip/xc32/v1.33/bin/bin/../../lib/gcc/pic32mx/4.5.2/../../../../pic32mx/lib/./proc/32MX795F512H/crt0_mips32r2.o

.text           0x9d005800        0x0
 *(.stub .gnu.linkonce.t.*)
 *(.text.*personality*)
 *(.mips16.fn.*)
 *(.mips16.call.*)
 *(.gnu.warning)
                0x9d005800                . = ALIGN (0x4)

.init           0x9d005800        0x0
 *crti.o(.init)
 *crtbegin.o(.init)
 *(EXCLUDE_FILE(*crtn.o *crtend?.o *crtend.o) .init)
 *crtend.o(.init)
 *crtn.o(.init)
                0x9d005800                . = ALIGN (0x4)

.fini           0x9d005800        0x0
 *(.fini)
                0x9d005800                . = ALIGN (0x4)

.preinit_array  0x9d005800        0x0
                0x9d005800                PROVIDE (__preinit_array_start, .)
 *(.preinit_array)
                0x9d005800                PROVIDE (__preinit_array_end, .)
                0x9d005800                . = ALIGN (0x4)

.init_array     0x9d005800        0x0
                0x9d005800                PROVIDE (__init_array_start, .)
 *(SORT(.init_array.*))
 *(.init_array)
                0x9d005800                PROVIDE (__init_array_end, .)
                0x9d005800                . = ALIGN (0x4)

.fini_array     0x9d005800        0x0
                0x9d005800                PROVIDE (__fini_array_start, .)
 *(SORT(.fini_array.*))
 *(.fini_array)
                0x9d005800                PROVIDE (__fini_array_end, .)
                0x9d005800                . = ALIGN (0x4)

.ctors          0x9d005800        0x0
 *crtbegin.o(.ctors)
 *crtbegin?.o(.ctors)
 *(EXCLUDE_FILE(*crtend?.o *crtend.o) .ctors)
 *(SORT(.ctors.*))
 *(.ctors)
                0x9d005800                . = ALIGN (0x4)

.dtors          0x9d005800        0x0
 *crtbegin.o(.dtors)
 *crtbegin?.o(.dtors)
 *(EXCLUDE_FILE(*crtend?.o *crtend.o) .dtors)
 *(SORT(.dtors.*))
 *(.dtors)
                0x9d005800                . = ALIGN (0x4)

.rodata         0x9d005800        0x0
 *(.gnu.linkonce.r.*)
 *(.rodata1)
                0x9d005800                . = ALIGN (0x4)

.sdata2         0x9d0051e8        0x0
 *(.sdata2 .sdata2.* .gnu.linkonce.s2.*)
                0x9d0051e8                . = ALIGN (0x4)

.sbss2          0x9d0051e8        0x0
 *(.sbss2 .sbss2.* .gnu.linkonce.sb2.*)
                0x9d0051e8                . = ALIGN (0x4)

.eh_frame_hdr
 *(.eh_frame_hdr)
                0x9d0051e8                . = ALIGN (0x4)

.eh_frame
 *(.eh_frame)
                0x9d0051e8                . = ALIGN (0x4)

.gcc_except_table
 *(.gcc_except_table .gcc_except_table.*)
                0x9d0051e8                . = ALIGN (0x4)

.dbg_data       0xa0000200        0x0
                0xa0000200                . = (. + DEFINED (_DEBUGGER)?0x200:0x0)

.jcr            0xa0000200        0x0
 *(.jcr)
                0xa0000200                . = ALIGN (0x4)

.eh_frame       0xa0000200       0x30
 *(.eh_frame)
 .eh_frame      0xa0000200       0x20 c:/program files/microchip/xc32/v1.33/bin/bin/../../lib/gcc/pic32mx/4.5.2\libgcc.a(_udivdi3.o)
 .eh_frame      0xa0000220       0x10 c:/program files/microchip/xc32/v1.33/bin/bin/../../lib/gcc/pic32mx/4.5.2\libgcc.a(_umoddi3.o)
                0xa0000230                . = ALIGN (0x4)

.gcc_except_table
 *(.gcc_except_table .gcc_except_table.*)
                0xa0000230                . = ALIGN (0x4)

.persist        0xa0000230        0x0
                0xa0000230                _persist_begin = .
 *(.persist .persist.*)
 *(.pbss .pbss.*)
                0xa0000230                . = ALIGN (0x4)
                0xa0000230                _persist_end = .

.data           0xa0000230        0x0
 *(.gnu.linkonce.d.*)
 *(.data1)
                0xa0000230                . = ALIGN (0x4)
                0xa0000230                . = .
                0xa0008220                _gp = (ALIGN (0x10) + 0x7ff0)

.got            0xa0000230        0x0
 *(.got.plt)
 *(.got)
                0xa0000230                . = ALIGN (0x4)

.sdata          0xa0000230       0x64
                0xa0000230                _sdata_begin = .
 *(.sdata .sdata.* .gnu.linkonce.s.*)
 .sdata         0xa0000230        0x4 build/ChaletDuinoV2_795F512H_/debug/Source/winc3400_142/driver/source/m2m_ssl.o
 .sdata         0xa0000234        0x4 build/ChaletDuinoV2_795F512H_/debug/Source/winc3400_142/driver/source/m2m_wifi.o
 .sdata         0xa0000238        0x4 build/ChaletDuinoV2_795F512H_/debug/Source/winc3400_142/driver/source/nmbus.o
                0xa0000238                egstrNmBusCapabilities
 .sdata         0xa000023c        0x1 build/ChaletDuinoV2_795F512H_/debug/Source/NetworkProtocol.o
 *fill*         0xa000023d        0x3 
 .sdata         0xa0000240        0xc build/ChaletDuinoV2_795F512H_/debug/Source/Terminal.o
                0xa0000248                mBootloaderMagicWord
 .sdata         0xa000024c        0x8 build/ChaletDuinoV2_795F512H_/debug/Source/main.o
 .sdata         0xa0000254       0x10 build/ChaletDuinoV2_795F512H_/debug/Source/WiFiCtrl.o
                0xa000025b                TerminalSocket
                0xa000025c                TerminalServerSocket
                0xa000025d                SyslogSocket
                0xa000025e                SyslogServerSocket
                0xa000025f                NetworkSocket
                0xa0000260                NetworkServerSocket
                0xa0000261                BootloaderSocket
                0xa0000262                BootloaderServerSocket
 .sdata         0xa0000264        0x8 build/ChaletDuinoV2_795F512H_/debug/Source/Syslog.o
 .sdata         0xa000026c        0x8 build/ChaletDuinoV2_795F512H_/debug/Source/BootloaderInterface.o
 .sdata         0xa0000274       0x18 build/ChaletDuinoV2_795F512H_/debug/Source/BootloaderProtocol.o
                0xa000027c                BtldrComputedCRC
                0xa0000280                BootloaderState
                0xa0000284                BootloaderDataStartPtr
 .sdata         0xa000028c        0x4 c:/program files/microchip/xc32/v1.33/bin/bin/../../lib/gcc/pic32mx/4.5.2/../../../../pic32mx/lib\libc.a(_iob.o)
                0xa000028c                _Files
 .sdata         0xa0000290        0x4 c:/program files/microchip/xc32/v1.33/bin/bin/../../lib/gcc/pic32mx/4.5.2/../../../../pic32mx/lib\libpic32.a(xc32_uart.o)
                0xa0000290                __XC_UART
                0xa0000294                . = ALIGN (0x4)
                0xa0000294                _sdata_end = .

.lit8
 *(.lit8)

.lit4
 *(.lit4)
                0xa0000294                . = ALIGN (0x4)
                0xa0000294                _data_end = .
                0xa0000294                _bss_begin = .

.sbss           0xa0000294      0x124
                0xa0000294                _sbss_begin = .
 *(.dynsbss)
 *(.sbss .sbss.* .gnu.linkonce.sb.*)
 .sbss          0xa0000294        0x1 build/ChaletDuinoV2_795F512H_/debug/Source/winc3400_142/driver/source/m2m_hif.o
 *fill*         0xa0000295        0x3 
 .sbss          0xa0000298        0x4 build/ChaletDuinoV2_795F512H_/debug/Source/winc3400_142/driver/source/m2m_ota.o
 .sbss          0xa000029c        0x8 build/ChaletDuinoV2_795F512H_/debug/Source/winc3400_142/driver/source/m2m_ssl.o
 .sbss          0xa00002a4       0x14 build/ChaletDuinoV2_795F512H_/debug/Source/winc3400_142/driver/source/m2m_wifi.o
 .sbss          0xa00002b8        0x4 build/ChaletDuinoV2_795F512H_/debug/Source/winc3400_142/driver/source/nmasic.o
 .sbss          0xa00002bc        0x4 build/ChaletDuinoV2_795F512H_/debug/Source/winc3400_142/driver/source/nmdrv.o
 .sbss          0xa00002c0        0x1 build/ChaletDuinoV2_795F512H_/debug/Source/winc3400_142/driver/source/nmspi.o
 *fill*         0xa00002c1        0x3 
 .sbss          0xa00002c4       0x10 build/ChaletDuinoV2_795F512H_/debug/Source/winc3400_142/socket/source/socket.o
                0xa00002c4                gu16SessionID
                0xa00002c6                gbSocketInit
 .sbss          0xa00002d4        0x4 build/ChaletDuinoV2_795F512H_/debug/Source/winc3400_142/spi_flash/source/spi_flash.o
 .sbss          0xa00002d8        0xc build/ChaletDuinoV2_795F512H_/debug/Source/exceptions.o
 .sbss          0xa00002e4       0x1c build/ChaletDuinoV2_795F512H_/debug/Source/WiFiCtrl.o
                0xa00002e4                gu32HostIp
                0xa00002e8                gu8RetryCount
                0xa00002f8                mWiFiInitOK
                0xa00002fc                mWiFiState
 .sbss          0xa0000300        0x4 build/ChaletDuinoV2_795F512H_/debug/Source/Watchdog.o
                0xa0000300                WatchdogTriggered
 .sbss          0xa0000304       0x18 build/ChaletDuinoV2_795F512H_/debug/Source/BootloaderProtocol.o
                0xa0000304                BootloaderHeader
                0xa0000308                BootloaderDataSize
                0xa000030c                BootloaderDataCtr
                0xa0000310                BootloaderBufPtr
                0xa0000314                BootloaderCRC
                0xa0000318                BootloaderCommand
 .sbss          0xa000031c        0x1 build/ChaletDuinoV2_795F512H_/debug/Source/crc32.o
 *fill*         0xa000031d        0x3 
 .sbss          0xa0000320       0x10 build/ChaletDuinoV2_795F512H_/debug/Source/VolumeTransducer.o
                0xa0000320                mDebouncingBureau
                0xa0000324                mDebouncingCuisine
                0xa0000328                mBureauVolume
                0xa000032c                mCuisineVolume
 .sbss          0xa0000330        0x1 c:/program files/microchip/xc32/v1.33/bin/bin/../../lib/gcc/pic32mx/4.5.2/../../../../pic32mx/lib\libc.a(_iob.o)
                0xa0000330                _outdone
 *(.scommon)
 .scommon       0xa0000331        0x1 build/ChaletDuinoV2_795F512H_/debug/Source/winc3400_142/driver/source/nmspi.o
                0xa0000331                mWifiSPIBaudrate
 *fill*         0xa0000332        0x2 
 .scommon       0xa0000334        0x8 build/ChaletDuinoV2_795F512H_/debug/Source/winc3400_142/socket/source/socket.o
                0xa0000334                gpfAppResolveCb
                0xa0000338                gpfAppSocketCb
 .scommon       0xa000033c       0x18 build/ChaletDuinoV2_795F512H_/debug/Source/Terminal.o
                0xa000033c                mTerminalOpened
                0xa0000340                TerminalDataPtr
                0xa0000344                mTerminalPendingAction
                0xa0000348                mHelpStringPtr
                0xa000034c                mUseDHCP
                0xa0000350                mTerminalTickState
 .scommon       0xa0000354        0x4 build/ChaletDuinoV2_795F512H_/debug/Source/main.o
                0xa0000354                ActualTemp
 .scommon       0xa0000358        0xe build/ChaletDuinoV2_795F512H_/debug/Source/WiFiCtrl.o
                0xa0000358                u8IsMacAddrValid
                0xa000035c                mCurIPAddress
                0xa0000360                mac_addr
 *fill*         0xa0000366        0x2 
 .scommon       0xa0000368        0x8 build/ChaletDuinoV2_795F512H_/debug/Source/SPI_Flash.o
                0xa0000368                mSPIFlashHighSpeedBaudrate
                0xa0000369                mSPIFlashBaudrate
                0xa000036c                mSPIFlashOK
 .scommon       0xa0000370        0x8 build/ChaletDuinoV2_795F512H_/debug/Source/Syslog.o
                0xa0000370                mSyslogBufPtr
                0xa0000374                mSyslogLTEPassthroughEnabled
 .scommon       0xa0000378       0x38 build/ChaletDuinoV2_795F512H_/debug/Source/BootloaderInterface.o
                0xa0000378                CurDataChunkSize
                0xa000037c                BootloaderFirmwareChunkWriteCount
                0xa0000380                BootloaderFlashWriteDataPtr
                0xa0000384                BootloaderFlashErased
                0xa0000388                BootloaderFlashWriteState
                0xa000038c                BootloaderCurFlashWriteAddress
                0xa0000390                BooloaderFlashEraseState
                0xa0000394                BootloaderCurFlashEraseAddress
                0xa0000398                BootloaderFlashWritePollCount
                0xa000039c                BootloaderInterfaceState
                0xa00003a0                DataChunkWritten
                0xa00003a4                BooloaderFlashErasePollCount
                0xa00003a8                FirmwareUploaded
                0xa00003ac                CurDataChunkIndex
 .scommon       0xa00003b0        0x4 build/ChaletDuinoV2_795F512H_/debug/Source/BootloaderProtocol.o
                0xa00003b0                BootloaderRxPtr
 .scommon       0xa00003b4        0x1 build/ChaletDuinoV2_795F512H_/debug/Source/DACInterface.o
                0xa00003b4                mDACSPIBaudrate
                0xa00003b5                _sbss_end = .
                0xa00003b8                . = ALIGN (0x4)
 *fill*         0xa00003b5        0x3 

.bss            0xa00003b8     0x2c84
 *(.dynbss)
 *(COMMON)
 COMMON         0xa00003b8       0x24 build/ChaletDuinoV2_795F512H_/debug/Source/winc3400_142/driver/source/m2m_hif.o
                0xa00003b8                gstrHifCxt
 COMMON         0xa00003dc       0xc0 build/ChaletDuinoV2_795F512H_/debug/Source/winc3400_142/socket/source/socket.o
                0xa00003dc                gastrSockets
 COMMON         0xa000049c      0x640 build/ChaletDuinoV2_795F512H_/debug/Source/NetworkProtocol.o
                0xa000049c                mFrameData
                0xa00005d4                mLoraProtocolData
                0xa0000858                mLTEProtocolData
 COMMON         0xa0000adc      0x418 build/ChaletDuinoV2_795F512H_/debug/Source/Terminal.o
                0xa0000adc                mStoredBootloaderInfo
                0xa0000af0                TerminalWorkString
                0xa0000c1c                mAPPassword
                0xa0000c5c                TerminalPrevDataBuf
                0xa0000d88                TerminalDataBuf
                0xa0000eb4                mAPName
 COMMON         0xa0000ef4       0xc0 build/ChaletDuinoV2_795F512H_/debug/Source/timer.o
                0xa0000ef4                astTimer
 COMMON         0xa0000fb4      0xd04 build/ChaletDuinoV2_795F512H_/debug/Source/WiFiCtrl.o
                0xa0000fb4                NetworkRxBuf
                0xa00013b4                TerminalRxBuf
                0xa00017b4                BootloaderRxBuf
                0xa0001bb4                addr_in
                0xa0001bc4                param
                0xa0001bdc                mModuleIPConfig
                0xa0001bf0                SyslogRxBuf
 COMMON         0xa0001cb8     0x1000 build/ChaletDuinoV2_795F512H_/debug/Source/SPI_Flash.o
                0xa0001cb8                mFlashSectorBuffer
 COMMON         0xa0002cb8      0x1f4 build/ChaletDuinoV2_795F512H_/debug/Source/Syslog.o
                0xa0002cb8                mSyslogBuffer
 COMMON         0xa0002eac      0x12c build/ChaletDuinoV2_795F512H_/debug/Source/BootloaderInterface.o
                0xa0002eac                BootloaderBuffer
 COMMON         0xa0002fd8       0x64 build/ChaletDuinoV2_795F512H_/debug/Source/VolumeTransducer.o
                0xa0002fd8                VolDebug
                0xa000303c                . = ALIGN ((. != 0x0)?0x4:0x1)
                0xa000303c                . = ALIGN (0x4)
                0xa000303c                _end = .
                0xa000303c                _bss_end = .
                0x00010000                _bmxdudba_address = 0x10000
                0x00010000                _bmxdupba_address = 0x10000

/DISCARD/
 *(.pdr)
 *(.rel.dyn)
 *(.note.GNU-stack)
 *(.note.GNU-stack)
 *(.gnu_debuglink)
 *(.gnu.lto_*)
 *(.discard)

.gptab.sdata
 *(.gptab.data)
 *(.gptab.sdata)

.gptab.sbss
 *(.gptab.bss)
 *(.gptab.sbss)

.mdebug.abi32   0xa000303c        0x0
 *(.mdebug.abi32)
 .mdebug.abi32  0xa000303c        0x0 c:/program files/microchip/xc32/v1.33/bin/bin/../../lib/gcc/pic32mx/4.5.2/../../../../pic32mx/lib\software-debug-break.o
 .mdebug.abi32  0xa000303c        0x0 build/ChaletDuinoV2_795F512H_/debug/Source/ChaletduinoV2Board.o
 .mdebug.abi32  0xa000303c        0x0 build/ChaletDuinoV2_795F512H_/debug/Source/winc3400_142/common/source/nm_common.o
 .mdebug.abi32  0xa000303c        0x0 build/ChaletDuinoV2_795F512H_/debug/Source/winc3400_142/driver/source/m2m_flash.o
 .mdebug.abi32  0xa000303c        0x0 build/ChaletDuinoV2_795F512H_/debug/Source/winc3400_142/driver/source/m2m_hif.o
 .mdebug.abi32  0xa000303c        0x0 build/ChaletDuinoV2_795F512H_/debug/Source/winc3400_142/driver/source/m2m_ota.o
 .mdebug.abi32  0xa000303c        0x0 build/ChaletDuinoV2_795F512H_/debug/Source/winc3400_142/driver/source/m2m_periph.o
 .mdebug.abi32  0xa000303c        0x0 build/ChaletDuinoV2_795F512H_/debug/Source/winc3400_142/driver/source/m2m_ssl.o
 .mdebug.abi32  0xa000303c        0x0 build/ChaletDuinoV2_795F512H_/debug/Source/winc3400_142/driver/source/m2m_wifi.o
 .mdebug.abi32  0xa000303c        0x0 build/ChaletDuinoV2_795F512H_/debug/Source/winc3400_142/driver/source/nmasic.o
 .mdebug.abi32  0xa000303c        0x0 build/ChaletDuinoV2_795F512H_/debug/Source/winc3400_142/driver/source/nmbus.o
 .mdebug.abi32  0xa000303c        0x0 build/ChaletDuinoV2_795F512H_/debug/Source/winc3400_142/driver/source/nmdrv.o
 .mdebug.abi32  0xa000303c        0x0 build/ChaletDuinoV2_795F512H_/debug/Source/winc3400_142/driver/source/nmspi.o
 .mdebug.abi32  0xa000303c        0x0 build/ChaletDuinoV2_795F512H_/debug/Source/winc3400_142/socket/source/inet_addr.o
 .mdebug.abi32  0xa000303c        0x0 build/ChaletDuinoV2_795F512H_/debug/Source/winc3400_142/socket/source/inet_ntop.o
 .mdebug.abi32  0xa000303c        0x0 build/ChaletDuinoV2_795F512H_/debug/Source/winc3400_142/socket/source/socket.o
 .mdebug.abi32  0xa000303c        0x0 build/ChaletDuinoV2_795F512H_/debug/Source/winc3400_142/spi_flash/source/spi_flash.o
 .mdebug.abi32  0xa000303c        0x0 build/ChaletDuinoV2_795F512H_/debug/Source/DigitalIO.o
 .mdebug.abi32  0xa000303c        0x0 build/ChaletDuinoV2_795F512H_/debug/Source/NetworkProtocol.o
 .mdebug.abi32  0xa000303c        0x0 build/ChaletDuinoV2_795F512H_/debug/Source/Terminal.o
 .mdebug.abi32  0xa000303c        0x0 build/ChaletDuinoV2_795F512H_/debug/Source/Util.o
 .mdebug.abi32  0xa000303c        0x0 build/ChaletDuinoV2_795F512H_/debug/Source/exceptions.o
 .mdebug.abi32  0xa000303c        0x0 build/ChaletDuinoV2_795F512H_/debug/Source/interrupts.o
 .mdebug.abi32  0xa000303c        0x0 build/ChaletDuinoV2_795F512H_/debug/Source/main.o
 .mdebug.abi32  0xa000303c        0x0 build/ChaletDuinoV2_795F512H_/debug/Source/system.o
 .mdebug.abi32  0xa000303c        0x0 build/ChaletDuinoV2_795F512H_/debug/Source/template.o
 .mdebug.abi32  0xa000303c        0x0 build/ChaletDuinoV2_795F512H_/debug/Source/timer.o
 .mdebug.abi32  0xa000303c        0x0 build/ChaletDuinoV2_795F512H_/debug/Source/WiFiCtrl.o
 .mdebug.abi32  0xa000303c        0x0 build/ChaletDuinoV2_795F512H_/debug/Source/SPI.o
 .mdebug.abi32  0xa000303c        0x0 build/ChaletDuinoV2_795F512H_/debug/Source/SPI_Flash.o
 .mdebug.abi32  0xa000303c        0x0 build/ChaletDuinoV2_795F512H_/debug/Source/Syslog.o
 .mdebug.abi32  0xa000303c        0x0 build/ChaletDuinoV2_795F512H_/debug/Source/Watchdog.o
 .mdebug.abi32  0xa000303c        0x0 build/ChaletDuinoV2_795F512H_/debug/Source/BootloaderInterface.o
 .mdebug.abi32  0xa000303c        0x0 build/ChaletDuinoV2_795F512H_/debug/Source/BootloaderProtocol.o
 .mdebug.abi32  0xa000303c        0x0 build/ChaletDuinoV2_795F512H_/debug/Source/crc32.o
 .mdebug.abi32  0xa000303c        0x0 build/ChaletDuinoV2_795F512H_/debug/Source/VolumeTransducer.o
 .mdebug.abi32  0xa000303c        0x0 build/ChaletDuinoV2_795F512H_/debug/Source/DACInterface.o
 .mdebug.abi32  0xa000303c        0x0 c:/program files/microchip/xc32/v1.33/bin/bin/../../lib/gcc/pic32mx/4.5.2/../../../../pic32mx/lib\libmchp_peripheral_32MX795F512H.a(soft_reset_lib.o)
 .mdebug.abi32  0xa000303c        0x0 c:/program files/microchip/xc32/v1.33/bin/bin/../../lib/gcc/pic32mx/4.5.2/../../../../pic32mx/lib\libmchp_peripheral_32MX795F512H.a(pcache.o)
 .mdebug.abi32  0xa000303c        0x0 c:/program files/microchip/xc32/v1.33/bin/bin/../../lib/gcc/pic32mx/4.5.2/../../../../pic32mx/lib\libmchp_peripheral_32MX795F512H.a(int_configure_system_lib.o)
 .mdebug.abi32  0xa000303c        0x0 c:/program files/microchip/xc32/v1.33/bin/bin/../../lib/gcc/pic32mx/4.5.2/../../../../pic32mx/lib\libmchp_peripheral_32MX795F512H.a(int_enable_interrupts_lib.o)
 .mdebug.abi32  0xa000303c        0x0 c:/program files/microchip/xc32/v1.33/bin/bin/../../lib/gcc/pic32mx/4.5.2/../../../../pic32mx/lib\libmchp_peripheral_32MX795F512H.a(int_disable_interrupts_lib.o)
 .mdebug.abi32  0xa000303c        0x0 c:/program files/microchip/xc32/v1.33/bin/bin/../../lib/gcc/pic32mx/4.5.2/../../../../pic32mx/lib\libmchp_peripheral_32MX795F512H.a(int_restore_interrupts_lib.o)
 .mdebug.abi32  0xa000303c        0x0 c:/program files/microchip/xc32/v1.33/bin/bin/../../lib/gcc/pic32mx/4.5.2/../../../../pic32mx/lib\libpic32.a(default-bootstrap-exception-handler.o)
 .mdebug.abi32  0xa000303c        0x0 c:/program files/microchip/xc32/v1.33/bin/bin/../../lib/gcc/pic32mx/4.5.2/../../../../pic32mx/lib\libpic32.a(default-on-reset.o)
 .mdebug.abi32  0xa000303c        0x0 c:/program files/microchip/xc32/v1.33/bin/bin/../../lib/gcc/pic32mx/4.5.2/../../../../pic32mx/lib\libpic32.a(default-on-bootstrap.o)
 .mdebug.abi32  0xa000303c        0x0 c:/program files/microchip/xc32/v1.33/bin/bin/../../lib/gcc/pic32mx/4.5.2/../../../../pic32mx/lib\libpic32.a(close.o)
 .mdebug.abi32  0xa000303c        0x0 c:/program files/microchip/xc32/v1.33/bin/bin/../../lib/gcc/pic32mx/4.5.2/../../../../pic32mx/lib\libpic32.a(defaultinterrupt.o)
 .mdebug.abi32  0xa000303c        0x0 c:/program files/microchip/xc32/v1.33/bin/bin/../../lib/gcc/pic32mx/4.5.2/../../../../pic32mx/lib\libc.a(puts.o)
 .mdebug.abi32  0xa000303c        0x0 c:/program files/microchip/xc32/v1.33/bin/bin/../../lib/gcc/pic32mx/4.5.2/../../../../pic32mx/lib\libc.a(strncmp.o)
 .mdebug.abi32  0xa000303c        0x0 c:/program files/microchip/xc32/v1.33/bin/bin/../../lib/gcc/pic32mx/4.5.2/../../../../pic32mx/lib\libc.a(printf_cdnopsuxX.eo)
 .mdebug.abi32  0xa000303c        0x0 c:/program files/microchip/xc32/v1.33/bin/bin/../../lib/gcc/pic32mx/4.5.2/../../../../pic32mx/lib\libc.a(sprintf_cdnopuxX.eo)
 .mdebug.abi32  0xa000303c        0x0 c:/program files/microchip/xc32/v1.33/bin/bin/../../lib/gcc/pic32mx/4.5.2/../../../../pic32mx/lib\libc.a(sscanf_s.eo)
 .mdebug.abi32  0xa000303c        0x0 c:/program files/microchip/xc32/v1.33/bin/bin/../../lib/gcc/pic32mx/4.5.2/../../../../pic32mx/lib\libc.a(_iob.o)
 .mdebug.abi32  0xa000303c        0x0 c:/program files/microchip/xc32/v1.33/bin/bin/../../lib/gcc/pic32mx/4.5.2/../../../../pic32mx/lib\libc.a(_fputc_simple.o)
 .mdebug.abi32  0xa000303c        0x0 c:/program files/microchip/xc32/v1.33/bin/bin/../../lib/gcc/pic32mx/4.5.2/../../../../pic32mx/lib\libc.a(doprnt_cdnopsuxX.eo)
 .mdebug.abi32  0xa000303c        0x0 c:/program files/microchip/xc32/v1.33/bin/bin/../../lib/gcc/pic32mx/4.5.2/../../../../pic32mx/lib\libc.a(doscan_s.eo)
 .mdebug.abi32  0xa000303c        0x0 c:/program files/microchip/xc32/v1.33/bin/bin/../../lib/gcc/pic32mx/4.5.2/../../../../pic32mx/lib\libc.a(_flsbuf_simple.o)
 .mdebug.abi32  0xa000303c        0x0 c:/program files/microchip/xc32/v1.33/bin/bin/../../lib/gcc/pic32mx/4.5.2/../../../../pic32mx/lib\libc.a(fgetc.o)
 .mdebug.abi32  0xa000303c        0x0 c:/program files/microchip/xc32/v1.33/bin/bin/../../lib/gcc/pic32mx/4.5.2/../../../../pic32mx/lib\libc.a(atoi.o)
 .mdebug.abi32  0xa000303c        0x0 c:/program files/microchip/xc32/v1.33/bin/bin/../../lib/gcc/pic32mx/4.5.2/../../../../pic32mx/lib\libc.a(ctype.o)
 .mdebug.abi32  0xa000303c        0x0 c:/program files/microchip/xc32/v1.33/bin/bin/../../lib/gcc/pic32mx/4.5.2/../../../../pic32mx/lib\libc.a(ctypef.o)
 .mdebug.abi32  0xa000303c        0x0 c:/program files/microchip/xc32/v1.33/bin/bin/../../lib/gcc/pic32mx/4.5.2/../../../../pic32mx/lib\libc.a(ungetc.o)
 .mdebug.abi32  0xa000303c        0x0 c:/program files/microchip/xc32/v1.33/bin/bin/../../lib/gcc/pic32mx/4.5.2/../../../../pic32mx/lib\libc.a(filbuf.o)
 .mdebug.abi32  0xa000303c        0x0 c:/program files/microchip/xc32/v1.33/bin/bin/../../lib/gcc/pic32mx/4.5.2/../../../../pic32mx/lib\libc.a(fflush.o)
 .mdebug.abi32  0xa000303c        0x0 c:/program files/microchip/xc32/v1.33/bin/bin/../../lib/gcc/pic32mx/4.5.2/../../../../pic32mx/lib\libpic32.a(read.o)
 .mdebug.abi32  0xa000303c        0x0 c:/program files/microchip/xc32/v1.33/bin/bin/../../lib/gcc/pic32mx/4.5.2/../../../../pic32mx/lib\libpic32.a(write.o)
 .mdebug.abi32  0xa000303c        0x0 c:/program files/microchip/xc32/v1.33/bin/bin/../../lib/gcc/pic32mx/4.5.2/../../../../pic32mx/lib\libpic32.a(xc32_uart.o)
 .mdebug.abi32  0xa000303c        0x0 c:/program files/microchip/xc32/v1.33/bin/bin/../../lib/gcc/pic32mx/4.5.2\libgcc.a(_udivdi3.o)
 .mdebug.abi32  0xa000303c        0x0 c:/program files/microchip/xc32/v1.33/bin/bin/../../lib/gcc/pic32mx/4.5.2\libgcc.a(_umoddi3.o)

.mdebug.abiN32
 *(.mdebug.abiN32)

.mdebug.abi64
 *(.mdebug.abi64)

.mdebug.abiO64
 *(.mdebug.abiO64)

.mdebug.eabi32
 *(.mdebug.eabi32)

.mdebug.eabi64
 *(.mdebug.eabi64)

.gcc_compiled_long32
 *(.gcc_compiled_long32)

.gcc_compiled_long64
 *(.gcc_compiled_long64)

.stab
 *(.stab)

.stabstr
 *(.stabstr)

.stab.excl
 *(.stab.excl)

.stab.exclstr
 *(.stab.exclstr)

.stab.index
 *(.stab.index)

.stab.indexstr
 *(.stab.indexstr)

.comment        0x00000000      0x177
 *(.comment)
 .comment       0x00000000       0x3c c:/program files/microchip/xc32/v1.33/bin/bin/../../lib/gcc/pic32mx/4.5.2/../../../../pic32mx/lib\software-debug-break.o
                                 0x3d (size before relaxing)
 .comment       0x00000000       0x3d build/ChaletDuinoV2_795F512H_/debug/Source/ChaletduinoV2Board.o
 .comment       0x00000000       0x3d build/ChaletDuinoV2_795F512H_/debug/Source/winc3400_142/common/source/nm_common.o
 .comment       0x00000000       0x3d build/ChaletDuinoV2_795F512H_/debug/Source/winc3400_142/driver/source/m2m_flash.o
 .comment       0x00000000       0x3d build/ChaletDuinoV2_795F512H_/debug/Source/winc3400_142/driver/source/m2m_hif.o
 .comment       0x00000000       0x3d build/ChaletDuinoV2_795F512H_/debug/Source/winc3400_142/driver/source/m2m_ota.o
 .comment       0x00000000       0x3d build/ChaletDuinoV2_795F512H_/debug/Source/winc3400_142/driver/source/m2m_periph.o
 .comment       0x00000000       0x3d build/ChaletDuinoV2_795F512H_/debug/Source/winc3400_142/driver/source/m2m_ssl.o
 .comment       0x00000000       0x3d build/ChaletDuinoV2_795F512H_/debug/Source/winc3400_142/driver/source/m2m_wifi.o
 .comment       0x00000000       0x3d build/ChaletDuinoV2_795F512H_/debug/Source/winc3400_142/driver/source/nmasic.o
 .comment       0x00000000       0x3d build/ChaletDuinoV2_795F512H_/debug/Source/winc3400_142/driver/source/nmbus.o
 .comment       0x00000000       0x3d build/ChaletDuinoV2_795F512H_/debug/Source/winc3400_142/driver/source/nmdrv.o
 .comment       0x00000000       0x3d build/ChaletDuinoV2_795F512H_/debug/Source/winc3400_142/driver/source/nmspi.o
 .comment       0x00000000       0x3d build/ChaletDuinoV2_795F512H_/debug/Source/winc3400_142/socket/source/inet_addr.o
 .comment       0x00000000       0x3d build/ChaletDuinoV2_795F512H_/debug/Source/winc3400_142/socket/source/inet_ntop.o
 .comment       0x00000000       0x3d build/ChaletDuinoV2_795F512H_/debug/Source/winc3400_142/socket/source/socket.o
 .comment       0x00000000       0x3d build/ChaletDuinoV2_795F512H_/debug/Source/winc3400_142/spi_flash/source/spi_flash.o
 .comment       0x00000000       0x3d build/ChaletDuinoV2_795F512H_/debug/Source/DigitalIO.o
 .comment       0x00000000       0x3d build/ChaletDuinoV2_795F512H_/debug/Source/NetworkProtocol.o
 .comment       0x00000000       0x3d build/ChaletDuinoV2_795F512H_/debug/Source/Terminal.o
 .comment       0x00000000       0x3d build/ChaletDuinoV2_795F512H_/debug/Source/Util.o
 .comment       0x00000000       0x3d build/ChaletDuinoV2_795F512H_/debug/Source/exceptions.o
 .comment       0x00000000       0x3d build/ChaletDuinoV2_795F512H_/debug/Source/interrupts.o
 .comment       0x00000000       0x3d build/ChaletDuinoV2_795F512H_/debug/Source/main.o
 .comment       0x00000000       0x3d build/ChaletDuinoV2_795F512H_/debug/Source/system.o
 .comment       0x00000000       0x3d build/ChaletDuinoV2_795F512H_/debug/Source/template.o
 .comment       0x00000000       0x3d build/ChaletDuinoV2_795F512H_/debug/Source/timer.o
 .comment       0x00000000       0x3d build/ChaletDuinoV2_795F512H_/debug/Source/WiFiCtrl.o
 .comment       0x00000000       0x3d build/ChaletDuinoV2_795F512H_/debug/Source/SPI.o
 .comment       0x00000000       0x3d build/ChaletDuinoV2_795F512H_/debug/Source/SPI_Flash.o
 .comment       0x00000000       0x3d build/ChaletDuinoV2_795F512H_/debug/Source/Syslog.o
 .comment       0x00000000       0x3d build/ChaletDuinoV2_795F512H_/debug/Source/Watchdog.o
 .comment       0x00000000       0x3d build/ChaletDuinoV2_795F512H_/debug/Source/BootloaderInterface.o
 .comment       0x00000000       0x3d build/ChaletDuinoV2_795F512H_/debug/Source/BootloaderProtocol.o
 .comment       0x00000000       0x3d build/ChaletDuinoV2_795F512H_/debug/Source/crc32.o
 .comment       0x00000000       0x3d build/ChaletDuinoV2_795F512H_/debug/Source/VolumeTransducer.o
 .comment       0x00000000       0x3d build/ChaletDuinoV2_795F512H_/debug/Source/DACInterface.o
 .comment       0x0000003c       0x3c c:/program files/microchip/xc32/v1.33/bin/bin/../../lib/gcc/pic32mx/4.5.2/../../../../pic32mx/lib\libmchp_peripheral_32MX795F512H.a(soft_reset_lib.o)
                                 0x3d (size before relaxing)
 .comment       0x00000000       0x3d c:/program files/microchip/xc32/v1.33/bin/bin/../../lib/gcc/pic32mx/4.5.2/../../../../pic32mx/lib\libmchp_peripheral_32MX795F512H.a(pcache.o)
 .comment       0x00000000       0x3d c:/program files/microchip/xc32/v1.33/bin/bin/../../lib/gcc/pic32mx/4.5.2/../../../../pic32mx/lib\libmchp_peripheral_32MX795F512H.a(int_configure_system_lib.o)
 .comment       0x00000000       0x3d c:/program files/microchip/xc32/v1.33/bin/bin/../../lib/gcc/pic32mx/4.5.2/../../../../pic32mx/lib\libmchp_peripheral_32MX795F512H.a(int_enable_interrupts_lib.o)
 .comment       0x00000000       0x3d c:/program files/microchip/xc32/v1.33/bin/bin/../../lib/gcc/pic32mx/4.5.2/../../../../pic32mx/lib\libmchp_peripheral_32MX795F512H.a(int_disable_interrupts_lib.o)
 .comment       0x00000000       0x3d c:/program files/microchip/xc32/v1.33/bin/bin/../../lib/gcc/pic32mx/4.5.2/../../../../pic32mx/lib\libmchp_peripheral_32MX795F512H.a(int_restore_interrupts_lib.o)
 .comment       0x00000078       0x18 c:/program files/microchip/xc32/v1.33/bin/bin/../../lib/gcc/pic32mx/4.5.2/../../../../pic32mx/lib\libpic32.a(memcmp.o)
                                 0x19 (size before relaxing)
 .comment       0x00000090       0x18 c:/program files/microchip/xc32/v1.33/bin/bin/../../lib/gcc/pic32mx/4.5.2/../../../../pic32mx/lib\libpic32.a(memset.o)
                                 0x19 (size before relaxing)
 .comment       0x000000a8       0x19 c:/program files/microchip/xc32/v1.33/bin/bin/../../lib/gcc/pic32mx/4.5.2/../../../../pic32mx/lib\libpic32.a(strcpy.o)
                                 0x1a (size before relaxing)
 .comment       0x000000c1       0x19 c:/program files/microchip/xc32/v1.33/bin/bin/../../lib/gcc/pic32mx/4.5.2/../../../../pic32mx/lib\libpic32.a(strlen.o)
                                 0x1a (size before relaxing)
 .comment       0x00000000       0x3d c:/program files/microchip/xc32/v1.33/bin/bin/../../lib/gcc/pic32mx/4.5.2/../../../../pic32mx/lib\libpic32.a(default-bootstrap-exception-handler.o)
 .comment       0x00000000       0x3d c:/program files/microchip/xc32/v1.33/bin/bin/../../lib/gcc/pic32mx/4.5.2/../../../../pic32mx/lib\libpic32.a(default-on-reset.o)
 .comment       0x00000000       0x3d c:/program files/microchip/xc32/v1.33/bin/bin/../../lib/gcc/pic32mx/4.5.2/../../../../pic32mx/lib\libpic32.a(default-on-bootstrap.o)
 .comment       0x00000000       0x3d c:/program files/microchip/xc32/v1.33/bin/bin/../../lib/gcc/pic32mx/4.5.2/../../../../pic32mx/lib\libpic32.a(close.o)
 .comment       0x00000000       0x3d c:/program files/microchip/xc32/v1.33/bin/bin/../../lib/gcc/pic32mx/4.5.2/../../../../pic32mx/lib\libpic32.a(defaultinterrupt.o)
 .comment       0x00000000       0x3d c:/program files/microchip/xc32/v1.33/bin/bin/../../lib/gcc/pic32mx/4.5.2/../../../../pic32mx/lib\libc.a(puts.o)
 .comment       0x00000000       0x3d c:/program files/microchip/xc32/v1.33/bin/bin/../../lib/gcc/pic32mx/4.5.2/../../../../pic32mx/lib\libc.a(strncmp.o)
 .comment       0x00000000       0x3d c:/program files/microchip/xc32/v1.33/bin/bin/../../lib/gcc/pic32mx/4.5.2/../../../../pic32mx/lib\libc.a(printf_cdnopsuxX.eo)
 .comment       0x00000000       0x3d c:/program files/microchip/xc32/v1.33/bin/bin/../../lib/gcc/pic32mx/4.5.2/../../../../pic32mx/lib\libc.a(sprintf_cdnopuxX.eo)
 .comment       0x00000000       0x3d c:/program files/microchip/xc32/v1.33/bin/bin/../../lib/gcc/pic32mx/4.5.2/../../../../pic32mx/lib\libc.a(sscanf_s.eo)
 .comment       0x00000000       0x3d c:/program files/microchip/xc32/v1.33/bin/bin/../../lib/gcc/pic32mx/4.5.2/../../../../pic32mx/lib\libc.a(_iob.o)
 .comment       0x00000000       0x3d c:/program files/microchip/xc32/v1.33/bin/bin/../../lib/gcc/pic32mx/4.5.2/../../../../pic32mx/lib\libc.a(_fputc_simple.o)
 .comment       0x00000000       0x3d c:/program files/microchip/xc32/v1.33/bin/bin/../../lib/gcc/pic32mx/4.5.2/../../../../pic32mx/lib\libc.a(doprnt_cdnopsuxX.eo)
 .comment       0x00000000       0x3d c:/program files/microchip/xc32/v1.33/bin/bin/../../lib/gcc/pic32mx/4.5.2/../../../../pic32mx/lib\libc.a(doscan_s.eo)
 .comment       0x00000000       0x3d c:/program files/microchip/xc32/v1.33/bin/bin/../../lib/gcc/pic32mx/4.5.2/../../../../pic32mx/lib\libc.a(_flsbuf_simple.o)
 .comment       0x00000000       0x3d c:/program files/microchip/xc32/v1.33/bin/bin/../../lib/gcc/pic32mx/4.5.2/../../../../pic32mx/lib\libc.a(fgetc.o)
 .comment       0x00000000       0x3d c:/program files/microchip/xc32/v1.33/bin/bin/../../lib/gcc/pic32mx/4.5.2/../../../../pic32mx/lib\libc.a(atoi.o)
 .comment       0x000000da       0x4e c:/program files/microchip/xc32/v1.33/bin/bin/../../lib/gcc/pic32mx/4.5.2/../../../../pic32mx/lib\libc.a(ctype.o)
                                 0x8b (size before relaxing)
 .comment       0x00000128       0x4f c:/program files/microchip/xc32/v1.33/bin/bin/../../lib/gcc/pic32mx/4.5.2/../../../../pic32mx/lib\libc.a(ctypef.o)
                                 0x8c (size before relaxing)
 .comment       0x00000000       0x3d c:/program files/microchip/xc32/v1.33/bin/bin/../../lib/gcc/pic32mx/4.5.2/../../../../pic32mx/lib\libc.a(ungetc.o)
 .comment       0x00000000       0x3d c:/program files/microchip/xc32/v1.33/bin/bin/../../lib/gcc/pic32mx/4.5.2/../../../../pic32mx/lib\libc.a(filbuf.o)
 .comment       0x00000000       0x3d c:/program files/microchip/xc32/v1.33/bin/bin/../../lib/gcc/pic32mx/4.5.2/../../../../pic32mx/lib\libc.a(fflush.o)
 .comment       0x00000000       0x3d c:/program files/microchip/xc32/v1.33/bin/bin/../../lib/gcc/pic32mx/4.5.2/../../../../pic32mx/lib\libpic32.a(read.o)
 .comment       0x00000000       0x3d c:/program files/microchip/xc32/v1.33/bin/bin/../../lib/gcc/pic32mx/4.5.2/../../../../pic32mx/lib\libpic32.a(write.o)
 .comment       0x00000000       0x3d c:/program files/microchip/xc32/v1.33/bin/bin/../../lib/gcc/pic32mx/4.5.2/../../../../pic32mx/lib\libpic32.a(xc32_uart.o)
 .comment       0x00000000       0x3d c:/program files/microchip/xc32/v1.33/bin/bin/../../lib/gcc/pic32mx/4.5.2\libgcc.a(_udivdi3.o)
 .comment       0x00000000       0x3d c:/program files/microchip/xc32/v1.33/bin/bin/../../lib/gcc/pic32mx/4.5.2\libgcc.a(_umoddi3.o)

.debug
 *(.debug)

.line
 *(.line)

.debug_srcinfo
 *(.debug_srcinfo)

.debug_sfnames
 *(.debug_sfnames)

.debug_aranges  0x00000000      0x8a0
 *(.debug_aranges)
 .debug_aranges
                0x00000000       0x20 c:/program files/microchip/xc32/v1.33/bin/bin/../../lib/gcc/pic32mx/4.5.2/../../../../pic32mx/lib\software-debug-break.o
 .debug_aranges
                0x00000020       0x20 build/ChaletDuinoV2_795F512H_/debug/Source/ChaletduinoV2Board.o
 .debug_aranges
                0x00000040       0x20 build/ChaletDuinoV2_795F512H_/debug/Source/winc3400_142/common/source/nm_common.o
 .debug_aranges
                0x00000060       0x20 build/ChaletDuinoV2_795F512H_/debug/Source/winc3400_142/driver/source/m2m_flash.o
 .debug_aranges
                0x00000080       0x20 build/ChaletDuinoV2_795F512H_/debug/Source/winc3400_142/driver/source/m2m_hif.o
 .debug_aranges
                0x000000a0       0x20 build/ChaletDuinoV2_795F512H_/debug/Source/winc3400_142/driver/source/m2m_ota.o
 .debug_aranges
                0x000000c0       0x20 build/ChaletDuinoV2_795F512H_/debug/Source/winc3400_142/driver/source/m2m_periph.o
 .debug_aranges
                0x000000e0       0x20 build/ChaletDuinoV2_795F512H_/debug/Source/winc3400_142/driver/source/m2m_ssl.o
 .debug_aranges
                0x00000100       0x20 build/ChaletDuinoV2_795F512H_/debug/Source/winc3400_142/driver/source/m2m_wifi.o
 .debug_aranges
                0x00000120       0x20 build/ChaletDuinoV2_795F512H_/debug/Source/winc3400_142/driver/source/nmasic.o
 .debug_aranges
                0x00000140       0x20 build/ChaletDuinoV2_795F512H_/debug/Source/winc3400_142/driver/source/nmbus.o
 .debug_aranges
                0x00000160       0x20 build/ChaletDuinoV2_795F512H_/debug/Source/winc3400_142/driver/source/nmdrv.o
 .debug_aranges
                0x00000180       0x20 build/ChaletDuinoV2_795F512H_/debug/Source/winc3400_142/driver/source/nmspi.o
 .debug_aranges
                0x000001a0       0x20 build/ChaletDuinoV2_795F512H_/debug/Source/winc3400_142/socket/source/inet_addr.o
 .debug_aranges
                0x000001c0       0x20 build/ChaletDuinoV2_795F512H_/debug/Source/winc3400_142/socket/source/inet_ntop.o
 .debug_aranges
                0x000001e0       0x20 build/ChaletDuinoV2_795F512H_/debug/Source/winc3400_142/socket/source/socket.o
 .debug_aranges
                0x00000200       0x20 build/ChaletDuinoV2_795F512H_/debug/Source/winc3400_142/spi_flash/source/spi_flash.o
 .debug_aranges
                0x00000220       0x20 build/ChaletDuinoV2_795F512H_/debug/Source/DigitalIO.o
 .debug_aranges
                0x00000240       0x20 build/ChaletDuinoV2_795F512H_/debug/Source/NetworkProtocol.o
 .debug_aranges
                0x00000260       0x20 build/ChaletDuinoV2_795F512H_/debug/Source/Terminal.o
 .debug_aranges
                0x00000280       0x20 build/ChaletDuinoV2_795F512H_/debug/Source/Util.o
 .debug_aranges
                0x000002a0       0x20 build/ChaletDuinoV2_795F512H_/debug/Source/exceptions.o
 .debug_aranges
                0x000002c0       0x20 build/ChaletDuinoV2_795F512H_/debug/Source/main.o
 .debug_aranges
                0x000002e0       0x20 build/ChaletDuinoV2_795F512H_/debug/Source/timer.o
 .debug_aranges
                0x00000300       0x20 build/ChaletDuinoV2_795F512H_/debug/Source/WiFiCtrl.o
 .debug_aranges
                0x00000320       0x20 build/ChaletDuinoV2_795F512H_/debug/Source/SPI.o
 .debug_aranges
                0x00000340       0x20 build/ChaletDuinoV2_795F512H_/debug/Source/SPI_Flash.o
 .debug_aranges
                0x00000360       0x20 build/ChaletDuinoV2_795F512H_/debug/Source/Syslog.o
 .debug_aranges
                0x00000380       0x20 build/ChaletDuinoV2_795F512H_/debug/Source/Watchdog.o
 .debug_aranges
                0x000003a0       0x20 build/ChaletDuinoV2_795F512H_/debug/Source/BootloaderInterface.o
 .debug_aranges
                0x000003c0       0x20 build/ChaletDuinoV2_795F512H_/debug/Source/BootloaderProtocol.o
 .debug_aranges
                0x000003e0       0x20 build/ChaletDuinoV2_795F512H_/debug/Source/crc32.o
 .debug_aranges
                0x00000400       0x20 build/ChaletDuinoV2_795F512H_/debug/Source/VolumeTransducer.o
 .debug_aranges
                0x00000420       0x20 build/ChaletDuinoV2_795F512H_/debug/Source/DACInterface.o
 .debug_aranges
                0x00000440       0x20 c:/program files/microchip/xc32/v1.33/bin/bin/../../lib/gcc/pic32mx/4.5.2/../../../../pic32mx/lib\libmchp_peripheral_32MX795F512H.a(soft_reset_lib.o)
 .debug_aranges
                0x00000460       0x28 c:/program files/microchip/xc32/v1.33/bin/bin/../../lib/gcc/pic32mx/4.5.2/../../../../pic32mx/lib\libmchp_peripheral_32MX795F512H.a(pcache.o)
 .debug_aranges
                0x00000488       0x20 c:/program files/microchip/xc32/v1.33/bin/bin/../../lib/gcc/pic32mx/4.5.2/../../../../pic32mx/lib\libmchp_peripheral_32MX795F512H.a(int_configure_system_lib.o)
 .debug_aranges
                0x000004a8       0x20 c:/program files/microchip/xc32/v1.33/bin/bin/../../lib/gcc/pic32mx/4.5.2/../../../../pic32mx/lib\libmchp_peripheral_32MX795F512H.a(int_enable_interrupts_lib.o)
 .debug_aranges
                0x000004c8       0x20 c:/program files/microchip/xc32/v1.33/bin/bin/../../lib/gcc/pic32mx/4.5.2/../../../../pic32mx/lib\libmchp_peripheral_32MX795F512H.a(int_disable_interrupts_lib.o)
 .debug_aranges
                0x000004e8       0x20 c:/program files/microchip/xc32/v1.33/bin/bin/../../lib/gcc/pic32mx/4.5.2/../../../../pic32mx/lib\libmchp_peripheral_32MX795F512H.a(int_restore_interrupts_lib.o)
 .debug_aranges
                0x00000508       0x20 c:/program files/microchip/xc32/v1.33/bin/bin/../../lib/gcc/pic32mx/4.5.2/../../../../pic32mx/lib\libpic32.a(default-bootstrap-exception-handler.o)
 .debug_aranges
                0x00000528       0x20 c:/program files/microchip/xc32/v1.33/bin/bin/../../lib/gcc/pic32mx/4.5.2/../../../../pic32mx/lib\libpic32.a(default-on-reset.o)
 .debug_aranges
                0x00000548       0x20 c:/program files/microchip/xc32/v1.33/bin/bin/../../lib/gcc/pic32mx/4.5.2/../../../../pic32mx/lib\libpic32.a(default-on-bootstrap.o)
 .debug_aranges
                0x00000568       0x20 c:/program files/microchip/xc32/v1.33/bin/bin/../../lib/gcc/pic32mx/4.5.2/../../../../pic32mx/lib\libpic32.a(close.o)
 .debug_aranges
                0x00000588       0x20 c:/program files/microchip/xc32/v1.33/bin/bin/../../lib/gcc/pic32mx/4.5.2/../../../../pic32mx/lib\libpic32.a(defaultinterrupt.o)
 .debug_aranges
                0x000005a8       0x28 c:/program files/microchip/xc32/v1.33/bin/bin/../../lib/gcc/pic32mx/4.5.2/../../../../pic32mx/lib\libc.a(puts.o)
 .debug_aranges
                0x000005d0       0x20 c:/program files/microchip/xc32/v1.33/bin/bin/../../lib/gcc/pic32mx/4.5.2/../../../../pic32mx/lib\libc.a(strncmp.o)
 .debug_aranges
                0x000005f0       0x20 c:/program files/microchip/xc32/v1.33/bin/bin/../../lib/gcc/pic32mx/4.5.2/../../../../pic32mx/lib\libc.a(printf_cdnopsuxX.eo)
 .debug_aranges
                0x00000610       0x20 c:/program files/microchip/xc32/v1.33/bin/bin/../../lib/gcc/pic32mx/4.5.2/../../../../pic32mx/lib\libc.a(sprintf_cdnopuxX.eo)
 .debug_aranges
                0x00000630       0x20 c:/program files/microchip/xc32/v1.33/bin/bin/../../lib/gcc/pic32mx/4.5.2/../../../../pic32mx/lib\libc.a(sscanf_s.eo)
 .debug_aranges
                0x00000650       0x20 c:/program files/microchip/xc32/v1.33/bin/bin/../../lib/gcc/pic32mx/4.5.2/../../../../pic32mx/lib\libc.a(_fputc_simple.o)
 .debug_aranges
                0x00000670       0x20 c:/program files/microchip/xc32/v1.33/bin/bin/../../lib/gcc/pic32mx/4.5.2/../../../../pic32mx/lib\libc.a(doprnt_cdnopsuxX.eo)
 .debug_aranges
                0x00000690       0x30 c:/program files/microchip/xc32/v1.33/bin/bin/../../lib/gcc/pic32mx/4.5.2/../../../../pic32mx/lib\libc.a(doscan_s.eo)
 .debug_aranges
                0x000006c0       0x20 c:/program files/microchip/xc32/v1.33/bin/bin/../../lib/gcc/pic32mx/4.5.2/../../../../pic32mx/lib\libc.a(_flsbuf_simple.o)
 .debug_aranges
                0x000006e0       0x20 c:/program files/microchip/xc32/v1.33/bin/bin/../../lib/gcc/pic32mx/4.5.2/../../../../pic32mx/lib\libc.a(fgetc.o)
 .debug_aranges
                0x00000700       0x20 c:/program files/microchip/xc32/v1.33/bin/bin/../../lib/gcc/pic32mx/4.5.2/../../../../pic32mx/lib\libc.a(atoi.o)
 .debug_aranges
                0x00000720       0xa0 c:/program files/microchip/xc32/v1.33/bin/bin/../../lib/gcc/pic32mx/4.5.2/../../../../pic32mx/lib\libc.a(ctypef.o)
 .debug_aranges
                0x000007c0       0x20 c:/program files/microchip/xc32/v1.33/bin/bin/../../lib/gcc/pic32mx/4.5.2/../../../../pic32mx/lib\libc.a(ungetc.o)
 .debug_aranges
                0x000007e0       0x20 c:/program files/microchip/xc32/v1.33/bin/bin/../../lib/gcc/pic32mx/4.5.2/../../../../pic32mx/lib\libc.a(filbuf.o)
 .debug_aranges
                0x00000800       0x20 c:/program files/microchip/xc32/v1.33/bin/bin/../../lib/gcc/pic32mx/4.5.2/../../../../pic32mx/lib\libc.a(fflush.o)
 .debug_aranges
                0x00000820       0x20 c:/program files/microchip/xc32/v1.33/bin/bin/../../lib/gcc/pic32mx/4.5.2/../../../../pic32mx/lib\libpic32.a(read.o)
 .debug_aranges
                0x00000840       0x20 c:/program files/microchip/xc32/v1.33/bin/bin/../../lib/gcc/pic32mx/4.5.2/../../../../pic32mx/lib\libpic32.a(write.o)
 .debug_aranges
                0x00000860       0x20 c:/program files/microchip/xc32/v1.33/bin/bin/../../lib/gcc/pic32mx/4.5.2\libgcc.a(_udivdi3.o)
 .debug_aranges
                0x00000880       0x20 c:/program files/microchip/xc32/v1.33/bin/bin/../../lib/gcc/pic32mx/4.5.2\libgcc.a(_umoddi3.o)

.debug_pubnames
                0x00000000     0x2dc4
 *(.debug_pubnames)
 .debug_pubnames
                0x00000000       0x30 c:/program files/microchip/xc32/v1.33/bin/bin/../../lib/gcc/pic32mx/4.5.2/../../../../pic32mx/lib\software-debug-break.o
 .debug_pubnames
                0x00000030       0x20 build/ChaletDuinoV2_795F512H_/debug/Source/ChaletduinoV2Board.o
 .debug_pubnames
                0x00000050       0x4c build/ChaletDuinoV2_795F512H_/debug/Source/winc3400_142/common/source/nm_common.o
 .debug_pubnames
                0x0000009c       0x72 build/ChaletDuinoV2_795F512H_/debug/Source/winc3400_142/driver/source/m2m_flash.o
 .debug_pubnames
                0x0000010e      0x119 build/ChaletDuinoV2_795F512H_/debug/Source/winc3400_142/driver/source/m2m_hif.o
 .debug_pubnames
                0x00000227       0x7f build/ChaletDuinoV2_795F512H_/debug/Source/winc3400_142/driver/source/m2m_ota.o
 .debug_pubnames
                0x000002a6       0x95 build/ChaletDuinoV2_795F512H_/debug/Source/winc3400_142/driver/source/m2m_periph.o
 .debug_pubnames
                0x0000033b      0x137 build/ChaletDuinoV2_795F512H_/debug/Source/winc3400_142/driver/source/m2m_ssl.o
 .debug_pubnames
                0x00000472      0x83d build/ChaletDuinoV2_795F512H_/debug/Source/winc3400_142/driver/source/m2m_wifi.o
 .debug_pubnames
                0x00000caf      0x1f1 build/ChaletDuinoV2_795F512H_/debug/Source/winc3400_142/driver/source/nmasic.o
 .debug_pubnames
                0x00000ea0       0xe8 build/ChaletDuinoV2_795F512H_/debug/Source/winc3400_142/driver/source/nmbus.o
 .debug_pubnames
                0x00000f88       0xee build/ChaletDuinoV2_795F512H_/debug/Source/winc3400_142/driver/source/nmdrv.o
 .debug_pubnames
                0x00001076       0xe2 build/ChaletDuinoV2_795F512H_/debug/Source/winc3400_142/driver/source/nmspi.o
 .debug_pubnames
                0x00001158       0x20 build/ChaletDuinoV2_795F512H_/debug/Source/winc3400_142/socket/source/inet_addr.o
 .debug_pubnames
                0x00001178       0x20 build/ChaletDuinoV2_795F512H_/debug/Source/winc3400_142/socket/source/inet_ntop.o
 .debug_pubnames
                0x00001198      0x1ef build/ChaletDuinoV2_795F512H_/debug/Source/winc3400_142/socket/source/socket.o
 .debug_pubnames
                0x00001387       0x64 build/ChaletDuinoV2_795F512H_/debug/Source/winc3400_142/spi_flash/source/spi_flash.o
 .debug_pubnames
                0x000013eb       0x24 build/ChaletDuinoV2_795F512H_/debug/Source/DigitalIO.o
 .debug_pubnames
                0x0000140f      0x123 build/ChaletDuinoV2_795F512H_/debug/Source/NetworkProtocol.o
 .debug_pubnames
                0x00001532      0x1bf build/ChaletDuinoV2_795F512H_/debug/Source/Terminal.o
 .debug_pubnames
                0x000016f1       0xd8 build/ChaletDuinoV2_795F512H_/debug/Source/Util.o
 .debug_pubnames
                0x000017c9       0x31 build/ChaletDuinoV2_795F512H_/debug/Source/exceptions.o
 .debug_pubnames
                0x000017fa       0x61 build/ChaletDuinoV2_795F512H_/debug/Source/main.o
 .debug_pubnames
                0x0000185b       0xec build/ChaletDuinoV2_795F512H_/debug/Source/timer.o
 .debug_pubnames
                0x00001947      0x385 build/ChaletDuinoV2_795F512H_/debug/Source/WiFiCtrl.o
 .debug_pubnames
                0x00001ccc       0x25 build/ChaletDuinoV2_795F512H_/debug/Source/SPI.o
 .debug_pubnames
                0x00001cf1      0x1b0 build/ChaletDuinoV2_795F512H_/debug/Source/SPI_Flash.o
 .debug_pubnames
                0x00001ea1      0x108 build/ChaletDuinoV2_795F512H_/debug/Source/Syslog.o
 .debug_pubnames
                0x00001fa9       0x71 build/ChaletDuinoV2_795F512H_/debug/Source/Watchdog.o
 .debug_pubnames
                0x0000201a      0x404 build/ChaletDuinoV2_795F512H_/debug/Source/BootloaderInterface.o
 .debug_pubnames
                0x0000241e      0x377 build/ChaletDuinoV2_795F512H_/debug/Source/BootloaderProtocol.o
 .debug_pubnames
                0x00002795       0x2f build/ChaletDuinoV2_795F512H_/debug/Source/crc32.o
 .debug_pubnames
                0x000027c4       0xe0 build/ChaletDuinoV2_795F512H_/debug/Source/VolumeTransducer.o
 .debug_pubnames
                0x000028a4       0x42 build/ChaletDuinoV2_795F512H_/debug/Source/DACInterface.o
 .debug_pubnames
                0x000028e6       0x20 c:/program files/microchip/xc32/v1.33/bin/bin/../../lib/gcc/pic32mx/4.5.2/../../../../pic32mx/lib\libmchp_peripheral_32MX795F512H.a(soft_reset_lib.o)
 .debug_pubnames
                0x00002906       0x3b c:/program files/microchip/xc32/v1.33/bin/bin/../../lib/gcc/pic32mx/4.5.2/../../../../pic32mx/lib\libmchp_peripheral_32MX795F512H.a(pcache.o)
 .debug_pubnames
                0x00002941       0x29 c:/program files/microchip/xc32/v1.33/bin/bin/../../lib/gcc/pic32mx/4.5.2/../../../../pic32mx/lib\libmchp_peripheral_32MX795F512H.a(int_configure_system_lib.o)
 .debug_pubnames
                0x0000296a       0x2a c:/program files/microchip/xc32/v1.33/bin/bin/../../lib/gcc/pic32mx/4.5.2/../../../../pic32mx/lib\libmchp_peripheral_32MX795F512H.a(int_enable_interrupts_lib.o)
 .debug_pubnames
                0x00002994       0x2b c:/program files/microchip/xc32/v1.33/bin/bin/../../lib/gcc/pic32mx/4.5.2/../../../../pic32mx/lib\libmchp_peripheral_32MX795F512H.a(int_disable_interrupts_lib.o)
 .debug_pubnames
                0x000029bf       0x2b c:/program files/microchip/xc32/v1.33/bin/bin/../../lib/gcc/pic32mx/4.5.2/../../../../pic32mx/lib\libmchp_peripheral_32MX795F512H.a(int_restore_interrupts_lib.o)
 .debug_pubnames
                0x000029ea       0x33 c:/program files/microchip/xc32/v1.33/bin/bin/../../lib/gcc/pic32mx/4.5.2/../../../../pic32mx/lib\libpic32.a(default-bootstrap-exception-handler.o)
 .debug_pubnames
                0x00002a1d       0x20 c:/program files/microchip/xc32/v1.33/bin/bin/../../lib/gcc/pic32mx/4.5.2/../../../../pic32mx/lib\libpic32.a(default-on-reset.o)
 .debug_pubnames
                0x00002a3d       0x24 c:/program files/microchip/xc32/v1.33/bin/bin/../../lib/gcc/pic32mx/4.5.2/../../../../pic32mx/lib\libpic32.a(default-on-bootstrap.o)
 .debug_pubnames
                0x00002a61       0x1c c:/program files/microchip/xc32/v1.33/bin/bin/../../lib/gcc/pic32mx/4.5.2/../../../../pic32mx/lib\libpic32.a(close.o)
 .debug_pubnames
                0x00002a7d       0x28 c:/program files/microchip/xc32/v1.33/bin/bin/../../lib/gcc/pic32mx/4.5.2/../../../../pic32mx/lib\libpic32.a(defaultinterrupt.o)
 .debug_pubnames
                0x00002aa5       0x25 c:/program files/microchip/xc32/v1.33/bin/bin/../../lib/gcc/pic32mx/4.5.2/../../../../pic32mx/lib\libc.a(puts.o)
 .debug_pubnames
                0x00002aca       0x1e c:/program files/microchip/xc32/v1.33/bin/bin/../../lib/gcc/pic32mx/4.5.2/../../../../pic32mx/lib\libc.a(strncmp.o)
 .debug_pubnames
                0x00002ae8       0x28 c:/program files/microchip/xc32/v1.33/bin/bin/../../lib/gcc/pic32mx/4.5.2/../../../../pic32mx/lib\libc.a(printf_cdnopsuxX.eo)
 .debug_pubnames
                0x00002b10       0x28 c:/program files/microchip/xc32/v1.33/bin/bin/../../lib/gcc/pic32mx/4.5.2/../../../../pic32mx/lib\libc.a(sprintf_cdnopuxX.eo)
 .debug_pubnames
                0x00002b38       0x20 c:/program files/microchip/xc32/v1.33/bin/bin/../../lib/gcc/pic32mx/4.5.2/../../../../pic32mx/lib\libc.a(sscanf_s.eo)
 .debug_pubnames
                0x00002b58       0x1c c:/program files/microchip/xc32/v1.33/bin/bin/../../lib/gcc/pic32mx/4.5.2/../../../../pic32mx/lib\libc.a(_fputc_simple.o)
 .debug_pubnames
                0x00002b74       0x2a c:/program files/microchip/xc32/v1.33/bin/bin/../../lib/gcc/pic32mx/4.5.2/../../../../pic32mx/lib\libc.a(doprnt_cdnopsuxX.eo)
 .debug_pubnames
                0x00002b9e       0x21 c:/program files/microchip/xc32/v1.33/bin/bin/../../lib/gcc/pic32mx/4.5.2/../../../../pic32mx/lib\libc.a(doscan_s.eo)
 .debug_pubnames
                0x00002bbf       0x1e c:/program files/microchip/xc32/v1.33/bin/bin/../../lib/gcc/pic32mx/4.5.2/../../../../pic32mx/lib\libc.a(_flsbuf_simple.o)
 .debug_pubnames
                0x00002bdd       0x1c c:/program files/microchip/xc32/v1.33/bin/bin/../../lib/gcc/pic32mx/4.5.2/../../../../pic32mx/lib\libc.a(fgetc.o)
 .debug_pubnames
                0x00002bf9       0x1b c:/program files/microchip/xc32/v1.33/bin/bin/../../lib/gcc/pic32mx/4.5.2/../../../../pic32mx/lib\libc.a(atoi.o)
 .debug_pubnames
                0x00002c14       0xe1 c:/program files/microchip/xc32/v1.33/bin/bin/../../lib/gcc/pic32mx/4.5.2/../../../../pic32mx/lib\libc.a(ctypef.o)
 .debug_pubnames
                0x00002cf5       0x1d c:/program files/microchip/xc32/v1.33/bin/bin/../../lib/gcc/pic32mx/4.5.2/../../../../pic32mx/lib\libc.a(ungetc.o)
 .debug_pubnames
                0x00002d12       0x1e c:/program files/microchip/xc32/v1.33/bin/bin/../../lib/gcc/pic32mx/4.5.2/../../../../pic32mx/lib\libc.a(filbuf.o)
 .debug_pubnames
                0x00002d30       0x1d c:/program files/microchip/xc32/v1.33/bin/bin/../../lib/gcc/pic32mx/4.5.2/../../../../pic32mx/lib\libc.a(fflush.o)
 .debug_pubnames
                0x00002d4d       0x1b c:/program files/microchip/xc32/v1.33/bin/bin/../../lib/gcc/pic32mx/4.5.2/../../../../pic32mx/lib\libpic32.a(read.o)
 .debug_pubnames
                0x00002d68       0x1c c:/program files/microchip/xc32/v1.33/bin/bin/../../lib/gcc/pic32mx/4.5.2/../../../../pic32mx/lib\libpic32.a(write.o)
 .debug_pubnames
                0x00002d84       0x20 c:/program files/microchip/xc32/v1.33/bin/bin/../../lib/gcc/pic32mx/4.5.2\libgcc.a(_udivdi3.o)
 .debug_pubnames
                0x00002da4       0x20 c:/program files/microchip/xc32/v1.33/bin/bin/../../lib/gcc/pic32mx/4.5.2\libgcc.a(_umoddi3.o)

.debug_info     0x00000000    0x430c2
 *(.debug_info .gnu.linkonce.wi.*)
 .debug_info    0x00000000       0xd2 c:/program files/microchip/xc32/v1.33/bin/bin/../../lib/gcc/pic32mx/4.5.2/../../../../pic32mx/lib\software-debug-break.o
 .debug_info    0x000000d2     0x2fb5 build/ChaletDuinoV2_795F512H_/debug/Source/ChaletduinoV2Board.o
 .debug_info    0x00003087     0x182e build/ChaletDuinoV2_795F512H_/debug/Source/winc3400_142/common/source/nm_common.o
 .debug_info    0x000048b5     0x1c93 build/ChaletDuinoV2_795F512H_/debug/Source/winc3400_142/driver/source/m2m_flash.o
 .debug_info    0x00006548     0x2782 build/ChaletDuinoV2_795F512H_/debug/Source/winc3400_142/driver/source/m2m_hif.o
 .debug_info    0x00008cca     0x1774 build/ChaletDuinoV2_795F512H_/debug/Source/winc3400_142/driver/source/m2m_ota.o
 .debug_info    0x0000a43e     0x14b9 build/ChaletDuinoV2_795F512H_/debug/Source/winc3400_142/driver/source/m2m_periph.o
 .debug_info    0x0000b8f7     0x1dd2 build/ChaletDuinoV2_795F512H_/debug/Source/winc3400_142/driver/source/m2m_ssl.o
 .debug_info    0x0000d6c9     0x637c build/ChaletDuinoV2_795F512H_/debug/Source/winc3400_142/driver/source/m2m_wifi.o
 .debug_info    0x00013a45     0x1afb build/ChaletDuinoV2_795F512H_/debug/Source/winc3400_142/driver/source/nmasic.o
 .debug_info    0x00015540     0x15e5 build/ChaletDuinoV2_795F512H_/debug/Source/winc3400_142/driver/source/nmbus.o
 .debug_info    0x00016b25     0x174c build/ChaletDuinoV2_795F512H_/debug/Source/winc3400_142/driver/source/nmdrv.o
 .debug_info    0x00018271     0x1c33 build/ChaletDuinoV2_795F512H_/debug/Source/winc3400_142/driver/source/nmspi.o
 .debug_info    0x00019ea4     0x1211 build/ChaletDuinoV2_795F512H_/debug/Source/winc3400_142/socket/source/inet_addr.o
 .debug_info    0x0001b0b5     0x127f build/ChaletDuinoV2_795F512H_/debug/Source/winc3400_142/socket/source/inet_ntop.o
 .debug_info    0x0001c334     0x33fd build/ChaletDuinoV2_795F512H_/debug/Source/winc3400_142/socket/source/socket.o
 .debug_info    0x0001f731     0x19f9 build/ChaletDuinoV2_795F512H_/debug/Source/winc3400_142/spi_flash/source/spi_flash.o
 .debug_info    0x0002112a     0x1161 build/ChaletDuinoV2_795F512H_/debug/Source/DigitalIO.o
 .debug_info    0x0002228b     0x1a43 build/ChaletDuinoV2_795F512H_/debug/Source/NetworkProtocol.o
 .debug_info    0x00023cce     0x195c build/ChaletDuinoV2_795F512H_/debug/Source/Terminal.o
 .debug_info    0x0002562a     0x1521 build/ChaletDuinoV2_795F512H_/debug/Source/Util.o
 .debug_info    0x00026b4b     0x1282 build/ChaletDuinoV2_795F512H_/debug/Source/exceptions.o
 .debug_info    0x00027dcd     0x1143 build/ChaletDuinoV2_795F512H_/debug/Source/interrupts.o
 .debug_info    0x00028f10     0x2285 build/ChaletDuinoV2_795F512H_/debug/Source/main.o
 .debug_info    0x0002b195     0x113f build/ChaletDuinoV2_795F512H_/debug/Source/system.o
 .debug_info    0x0002c2d4     0x1141 build/ChaletDuinoV2_795F512H_/debug/Source/template.o
 .debug_info    0x0002d415     0x213b build/ChaletDuinoV2_795F512H_/debug/Source/timer.o
 .debug_info    0x0002f550     0x350c build/ChaletDuinoV2_795F512H_/debug/Source/WiFiCtrl.o
 .debug_info    0x00032a5c     0x1320 build/ChaletDuinoV2_795F512H_/debug/Source/SPI.o
 .debug_info    0x00033d7c     0x18a5 build/ChaletDuinoV2_795F512H_/debug/Source/SPI_Flash.o
 .debug_info    0x00035621     0x167c build/ChaletDuinoV2_795F512H_/debug/Source/Syslog.o
 .debug_info    0x00036c9d     0x1334 build/ChaletDuinoV2_795F512H_/debug/Source/Watchdog.o
 .debug_info    0x00037fd1     0x2e8c build/ChaletDuinoV2_795F512H_/debug/Source/BootloaderInterface.o
 .debug_info    0x0003ae5d     0x21b9 build/ChaletDuinoV2_795F512H_/debug/Source/BootloaderProtocol.o
 .debug_info    0x0003d016      0x2e8 build/ChaletDuinoV2_795F512H_/debug/Source/crc32.o
 .debug_info    0x0003d2fe     0x20fa build/ChaletDuinoV2_795F512H_/debug/Source/VolumeTransducer.o
 .debug_info    0x0003f3f8     0x17ca build/ChaletDuinoV2_795F512H_/debug/Source/DACInterface.o
 .debug_info    0x00040bc2       0xae c:/program files/microchip/xc32/v1.33/bin/bin/../../lib/gcc/pic32mx/4.5.2/../../../../pic32mx/lib\libmchp_peripheral_32MX795F512H.a(soft_reset_lib.o)
 .debug_info    0x00040c70       0xbb c:/program files/microchip/xc32/v1.33/bin/bin/../../lib/gcc/pic32mx/4.5.2/../../../../pic32mx/lib\libmchp_peripheral_32MX795F512H.a(pcache.o)
 .debug_info    0x00040d2b       0xae c:/program files/microchip/xc32/v1.33/bin/bin/../../lib/gcc/pic32mx/4.5.2/../../../../pic32mx/lib\libmchp_peripheral_32MX795F512H.a(int_configure_system_lib.o)
 .debug_info    0x00040dd9       0xb0 c:/program files/microchip/xc32/v1.33/bin/bin/../../lib/gcc/pic32mx/4.5.2/../../../../pic32mx/lib\libmchp_peripheral_32MX795F512H.a(int_enable_interrupts_lib.o)
 .debug_info    0x00040e89       0xb2 c:/program files/microchip/xc32/v1.33/bin/bin/../../lib/gcc/pic32mx/4.5.2/../../../../pic32mx/lib\libmchp_peripheral_32MX795F512H.a(int_disable_interrupts_lib.o)
 .debug_info    0x00040f3b       0xb2 c:/program files/microchip/xc32/v1.33/bin/bin/../../lib/gcc/pic32mx/4.5.2/../../../../pic32mx/lib\libmchp_peripheral_32MX795F512H.a(int_restore_interrupts_lib.o)
 .debug_info    0x00040fed       0xe2 c:/program files/microchip/xc32/v1.33/bin/bin/../../lib/gcc/pic32mx/4.5.2/../../../../pic32mx/lib\libpic32.a(default-bootstrap-exception-handler.o)
 .debug_info    0x000410cf       0xbc c:/program files/microchip/xc32/v1.33/bin/bin/../../lib/gcc/pic32mx/4.5.2/../../../../pic32mx/lib\libpic32.a(default-on-reset.o)
 .debug_info    0x0004118b       0xc4 c:/program files/microchip/xc32/v1.33/bin/bin/../../lib/gcc/pic32mx/4.5.2/../../../../pic32mx/lib\libpic32.a(default-on-bootstrap.o)
 .debug_info    0x0004124f       0xad c:/program files/microchip/xc32/v1.33/bin/bin/../../lib/gcc/pic32mx/4.5.2/../../../../pic32mx/lib\libpic32.a(close.o)
 .debug_info    0x000412fc       0xd6 c:/program files/microchip/xc32/v1.33/bin/bin/../../lib/gcc/pic32mx/4.5.2/../../../../pic32mx/lib\libpic32.a(defaultinterrupt.o)
 .debug_info    0x000413d2       0xc5 c:/program files/microchip/xc32/v1.33/bin/bin/../../lib/gcc/pic32mx/4.5.2/../../../../pic32mx/lib\libc.a(puts.o)
 .debug_info    0x00041497       0xb7 c:/program files/microchip/xc32/v1.33/bin/bin/../../lib/gcc/pic32mx/4.5.2/../../../../pic32mx/lib\libc.a(strncmp.o)
 .debug_info    0x0004154e       0xc0 c:/program files/microchip/xc32/v1.33/bin/bin/../../lib/gcc/pic32mx/4.5.2/../../../../pic32mx/lib\libc.a(printf_cdnopsuxX.eo)
 .debug_info    0x0004160e       0xc1 c:/program files/microchip/xc32/v1.33/bin/bin/../../lib/gcc/pic32mx/4.5.2/../../../../pic32mx/lib\libc.a(sprintf_cdnopuxX.eo)
 .debug_info    0x000416cf       0xb8 c:/program files/microchip/xc32/v1.33/bin/bin/../../lib/gcc/pic32mx/4.5.2/../../../../pic32mx/lib\libc.a(sscanf_s.eo)
 .debug_info    0x00041787        0x0 c:/program files/microchip/xc32/v1.33/bin/bin/../../lib/gcc/pic32mx/4.5.2/../../../../pic32mx/lib\libc.a(_iob.o)
 .debug_info    0x00041787       0xb3 c:/program files/microchip/xc32/v1.33/bin/bin/../../lib/gcc/pic32mx/4.5.2/../../../../pic32mx/lib\libc.a(_fputc_simple.o)
 .debug_info    0x0004183a       0xc3 c:/program files/microchip/xc32/v1.33/bin/bin/../../lib/gcc/pic32mx/4.5.2/../../../../pic32mx/lib\libc.a(doprnt_cdnopsuxX.eo)
 .debug_info    0x000418fd       0xe0 c:/program files/microchip/xc32/v1.33/bin/bin/../../lib/gcc/pic32mx/4.5.2/../../../../pic32mx/lib\libc.a(doscan_s.eo)
 .debug_info    0x000419dd       0xb6 c:/program files/microchip/xc32/v1.33/bin/bin/../../lib/gcc/pic32mx/4.5.2/../../../../pic32mx/lib\libc.a(_flsbuf_simple.o)
 .debug_info    0x00041a93       0xb3 c:/program files/microchip/xc32/v1.33/bin/bin/../../lib/gcc/pic32mx/4.5.2/../../../../pic32mx/lib\libc.a(fgetc.o)
 .debug_info    0x00041b46       0xb1 c:/program files/microchip/xc32/v1.33/bin/bin/../../lib/gcc/pic32mx/4.5.2/../../../../pic32mx/lib\libc.a(atoi.o)
 .debug_info    0x00041bf7        0x0 c:/program files/microchip/xc32/v1.33/bin/bin/../../lib/gcc/pic32mx/4.5.2/../../../../pic32mx/lib\libc.a(ctype.o)
 .debug_info    0x00041bf7      0x219 c:/program files/microchip/xc32/v1.33/bin/bin/../../lib/gcc/pic32mx/4.5.2/../../../../pic32mx/lib\libc.a(ctypef.o)
 .debug_info    0x00041e10       0xb5 c:/program files/microchip/xc32/v1.33/bin/bin/../../lib/gcc/pic32mx/4.5.2/../../../../pic32mx/lib\libc.a(ungetc.o)
 .debug_info    0x00041ec5       0xb6 c:/program files/microchip/xc32/v1.33/bin/bin/../../lib/gcc/pic32mx/4.5.2/../../../../pic32mx/lib\libc.a(filbuf.o)
 .debug_info    0x00041f7b       0xb5 c:/program files/microchip/xc32/v1.33/bin/bin/../../lib/gcc/pic32mx/4.5.2/../../../../pic32mx/lib\libc.a(fflush.o)
 .debug_info    0x00042030       0xab c:/program files/microchip/xc32/v1.33/bin/bin/../../lib/gcc/pic32mx/4.5.2/../../../../pic32mx/lib\libpic32.a(read.o)
 .debug_info    0x000420db       0xad c:/program files/microchip/xc32/v1.33/bin/bin/../../lib/gcc/pic32mx/4.5.2/../../../../pic32mx/lib\libpic32.a(write.o)
 .debug_info    0x00042188        0x0 c:/program files/microchip/xc32/v1.33/bin/bin/../../lib/gcc/pic32mx/4.5.2/../../../../pic32mx/lib\libpic32.a(xc32_uart.o)
 .debug_info    0x00042188      0x782 c:/program files/microchip/xc32/v1.33/bin/bin/../../lib/gcc/pic32mx/4.5.2\libgcc.a(_udivdi3.o)
 .debug_info    0x0004290a      0x7b8 c:/program files/microchip/xc32/v1.33/bin/bin/../../lib/gcc/pic32mx/4.5.2\libgcc.a(_umoddi3.o)

.debug_abbrev   0x00000000     0x5944
 *(.debug_abbrev)
 .debug_abbrev  0x00000000       0x25 c:/program files/microchip/xc32/v1.33/bin/bin/../../lib/gcc/pic32mx/4.5.2/../../../../pic32mx/lib\software-debug-break.o
 .debug_abbrev  0x00000025      0x1d0 build/ChaletDuinoV2_795F512H_/debug/Source/ChaletduinoV2Board.o
 .debug_abbrev  0x000001f5      0x1e9 build/ChaletDuinoV2_795F512H_/debug/Source/winc3400_142/common/source/nm_common.o
 .debug_abbrev  0x000003de      0x2bb build/ChaletDuinoV2_795F512H_/debug/Source/winc3400_142/driver/source/m2m_flash.o
 .debug_abbrev  0x00000699      0x32d build/ChaletDuinoV2_795F512H_/debug/Source/winc3400_142/driver/source/m2m_hif.o
 .debug_abbrev  0x000009c6      0x208 build/ChaletDuinoV2_795F512H_/debug/Source/winc3400_142/driver/source/m2m_ota.o
 .debug_abbrev  0x00000bce      0x20b build/ChaletDuinoV2_795F512H_/debug/Source/winc3400_142/driver/source/m2m_periph.o
 .debug_abbrev  0x00000dd9      0x310 build/ChaletDuinoV2_795F512H_/debug/Source/winc3400_142/driver/source/m2m_ssl.o
 .debug_abbrev  0x000010e9      0x320 build/ChaletDuinoV2_795F512H_/debug/Source/winc3400_142/driver/source/m2m_wifi.o
 .debug_abbrev  0x00001409      0x2b9 build/ChaletDuinoV2_795F512H_/debug/Source/winc3400_142/driver/source/nmasic.o
 .debug_abbrev  0x000016c2      0x234 build/ChaletDuinoV2_795F512H_/debug/Source/winc3400_142/driver/source/nmbus.o
 .debug_abbrev  0x000018f6      0x247 build/ChaletDuinoV2_795F512H_/debug/Source/winc3400_142/driver/source/nmdrv.o
 .debug_abbrev  0x00001b3d      0x313 build/ChaletDuinoV2_795F512H_/debug/Source/winc3400_142/driver/source/nmspi.o
 .debug_abbrev  0x00001e50      0x19d build/ChaletDuinoV2_795F512H_/debug/Source/winc3400_142/socket/source/inet_addr.o
 .debug_abbrev  0x00001fed      0x1cf build/ChaletDuinoV2_795F512H_/debug/Source/winc3400_142/socket/source/inet_ntop.o
 .debug_abbrev  0x000021bc      0x39d build/ChaletDuinoV2_795F512H_/debug/Source/winc3400_142/socket/source/socket.o
 .debug_abbrev  0x00002559      0x27e build/ChaletDuinoV2_795F512H_/debug/Source/winc3400_142/spi_flash/source/spi_flash.o
 .debug_abbrev  0x000027d7      0x17b build/ChaletDuinoV2_795F512H_/debug/Source/DigitalIO.o
 .debug_abbrev  0x00002952      0x2aa build/ChaletDuinoV2_795F512H_/debug/Source/NetworkProtocol.o
 .debug_abbrev  0x00002bfc      0x27e build/ChaletDuinoV2_795F512H_/debug/Source/Terminal.o
 .debug_abbrev  0x00002e7a      0x26e build/ChaletDuinoV2_795F512H_/debug/Source/Util.o
 .debug_abbrev  0x000030e8      0x1b1 build/ChaletDuinoV2_795F512H_/debug/Source/exceptions.o
 .debug_abbrev  0x00003299      0x166 build/ChaletDuinoV2_795F512H_/debug/Source/interrupts.o
 .debug_abbrev  0x000033ff      0x361 build/ChaletDuinoV2_795F512H_/debug/Source/main.o
 .debug_abbrev  0x00003760      0x166 build/ChaletDuinoV2_795F512H_/debug/Source/system.o
 .debug_abbrev  0x000038c6      0x166 build/ChaletDuinoV2_795F512H_/debug/Source/template.o
 .debug_abbrev  0x00003a2c      0x226 build/ChaletDuinoV2_795F512H_/debug/Source/timer.o
 .debug_abbrev  0x00003c52      0x3dd build/ChaletDuinoV2_795F512H_/debug/Source/WiFiCtrl.o
 .debug_abbrev  0x0000402f      0x19d build/ChaletDuinoV2_795F512H_/debug/Source/SPI.o
 .debug_abbrev  0x000041cc      0x298 build/ChaletDuinoV2_795F512H_/debug/Source/SPI_Flash.o
 .debug_abbrev  0x00004464      0x26b build/ChaletDuinoV2_795F512H_/debug/Source/Syslog.o
 .debug_abbrev  0x000046cf      0x18c build/ChaletDuinoV2_795F512H_/debug/Source/Watchdog.o
 .debug_abbrev  0x0000485b      0x300 build/ChaletDuinoV2_795F512H_/debug/Source/BootloaderInterface.o
 .debug_abbrev  0x00004b5b      0x2be build/ChaletDuinoV2_795F512H_/debug/Source/BootloaderProtocol.o
 .debug_abbrev  0x00004e19       0xa9 build/ChaletDuinoV2_795F512H_/debug/Source/crc32.o
 .debug_abbrev  0x00004ec2      0x1c0 build/ChaletDuinoV2_795F512H_/debug/Source/VolumeTransducer.o
 .debug_abbrev  0x00005082      0x22e build/ChaletDuinoV2_795F512H_/debug/Source/DACInterface.o
 .debug_abbrev  0x000052b0       0x32 c:/program files/microchip/xc32/v1.33/bin/bin/../../lib/gcc/pic32mx/4.5.2/../../../../pic32mx/lib\libmchp_peripheral_32MX795F512H.a(soft_reset_lib.o)
 .debug_abbrev  0x000052e2       0x23 c:/program files/microchip/xc32/v1.33/bin/bin/../../lib/gcc/pic32mx/4.5.2/../../../../pic32mx/lib\libmchp_peripheral_32MX795F512H.a(pcache.o)
 .debug_abbrev  0x00005305       0x23 c:/program files/microchip/xc32/v1.33/bin/bin/../../lib/gcc/pic32mx/4.5.2/../../../../pic32mx/lib\libmchp_peripheral_32MX795F512H.a(int_configure_system_lib.o)
 .debug_abbrev  0x00005328       0x23 c:/program files/microchip/xc32/v1.33/bin/bin/../../lib/gcc/pic32mx/4.5.2/../../../../pic32mx/lib\libmchp_peripheral_32MX795F512H.a(int_enable_interrupts_lib.o)
 .debug_abbrev  0x0000534b       0x23 c:/program files/microchip/xc32/v1.33/bin/bin/../../lib/gcc/pic32mx/4.5.2/../../../../pic32mx/lib\libmchp_peripheral_32MX795F512H.a(int_disable_interrupts_lib.o)
 .debug_abbrev  0x0000536e       0x23 c:/program files/microchip/xc32/v1.33/bin/bin/../../lib/gcc/pic32mx/4.5.2/../../../../pic32mx/lib\libmchp_peripheral_32MX795F512H.a(int_restore_interrupts_lib.o)
 .debug_abbrev  0x00005391       0x25 c:/program files/microchip/xc32/v1.33/bin/bin/../../lib/gcc/pic32mx/4.5.2/../../../../pic32mx/lib\libpic32.a(default-bootstrap-exception-handler.o)
 .debug_abbrev  0x000053b6       0x25 c:/program files/microchip/xc32/v1.33/bin/bin/../../lib/gcc/pic32mx/4.5.2/../../../../pic32mx/lib\libpic32.a(default-on-reset.o)
 .debug_abbrev  0x000053db       0x25 c:/program files/microchip/xc32/v1.33/bin/bin/../../lib/gcc/pic32mx/4.5.2/../../../../pic32mx/lib\libpic32.a(default-on-bootstrap.o)
 .debug_abbrev  0x00005400       0x25 c:/program files/microchip/xc32/v1.33/bin/bin/../../lib/gcc/pic32mx/4.5.2/../../../../pic32mx/lib\libpic32.a(close.o)
 .debug_abbrev  0x00005425       0x25 c:/program files/microchip/xc32/v1.33/bin/bin/../../lib/gcc/pic32mx/4.5.2/../../../../pic32mx/lib\libpic32.a(defaultinterrupt.o)
 .debug_abbrev  0x0000544a       0x25 c:/program files/microchip/xc32/v1.33/bin/bin/../../lib/gcc/pic32mx/4.5.2/../../../../pic32mx/lib\libc.a(puts.o)
 .debug_abbrev  0x0000546f       0x25 c:/program files/microchip/xc32/v1.33/bin/bin/../../lib/gcc/pic32mx/4.5.2/../../../../pic32mx/lib\libc.a(strncmp.o)
 .debug_abbrev  0x00005494       0x25 c:/program files/microchip/xc32/v1.33/bin/bin/../../lib/gcc/pic32mx/4.5.2/../../../../pic32mx/lib\libc.a(printf_cdnopsuxX.eo)
 .debug_abbrev  0x000054b9       0x25 c:/program files/microchip/xc32/v1.33/bin/bin/../../lib/gcc/pic32mx/4.5.2/../../../../pic32mx/lib\libc.a(sprintf_cdnopuxX.eo)
 .debug_abbrev  0x000054de       0x25 c:/program files/microchip/xc32/v1.33/bin/bin/../../lib/gcc/pic32mx/4.5.2/../../../../pic32mx/lib\libc.a(sscanf_s.eo)
 .debug_abbrev  0x00005503        0x1 c:/program files/microchip/xc32/v1.33/bin/bin/../../lib/gcc/pic32mx/4.5.2/../../../../pic32mx/lib\libc.a(_iob.o)
 .debug_abbrev  0x00005504       0x25 c:/program files/microchip/xc32/v1.33/bin/bin/../../lib/gcc/pic32mx/4.5.2/../../../../pic32mx/lib\libc.a(_fputc_simple.o)
 .debug_abbrev  0x00005529       0x25 c:/program files/microchip/xc32/v1.33/bin/bin/../../lib/gcc/pic32mx/4.5.2/../../../../pic32mx/lib\libc.a(doprnt_cdnopsuxX.eo)
 .debug_abbrev  0x0000554e       0x36 c:/program files/microchip/xc32/v1.33/bin/bin/../../lib/gcc/pic32mx/4.5.2/../../../../pic32mx/lib\libc.a(doscan_s.eo)
 .debug_abbrev  0x00005584       0x25 c:/program files/microchip/xc32/v1.33/bin/bin/../../lib/gcc/pic32mx/4.5.2/../../../../pic32mx/lib\libc.a(_flsbuf_simple.o)
 .debug_abbrev  0x000055a9       0x25 c:/program files/microchip/xc32/v1.33/bin/bin/../../lib/gcc/pic32mx/4.5.2/../../../../pic32mx/lib\libc.a(fgetc.o)
 .debug_abbrev  0x000055ce       0x25 c:/program files/microchip/xc32/v1.33/bin/bin/../../lib/gcc/pic32mx/4.5.2/../../../../pic32mx/lib\libc.a(atoi.o)
 .debug_abbrev  0x000055f3        0x1 c:/program files/microchip/xc32/v1.33/bin/bin/../../lib/gcc/pic32mx/4.5.2/../../../../pic32mx/lib\libc.a(ctype.o)
 .debug_abbrev  0x000055f4       0x25 c:/program files/microchip/xc32/v1.33/bin/bin/../../lib/gcc/pic32mx/4.5.2/../../../../pic32mx/lib\libc.a(ctypef.o)
 .debug_abbrev  0x00005619       0x25 c:/program files/microchip/xc32/v1.33/bin/bin/../../lib/gcc/pic32mx/4.5.2/../../../../pic32mx/lib\libc.a(ungetc.o)
 .debug_abbrev  0x0000563e       0x25 c:/program files/microchip/xc32/v1.33/bin/bin/../../lib/gcc/pic32mx/4.5.2/../../../../pic32mx/lib\libc.a(filbuf.o)
 .debug_abbrev  0x00005663       0x25 c:/program files/microchip/xc32/v1.33/bin/bin/../../lib/gcc/pic32mx/4.5.2/../../../../pic32mx/lib\libc.a(fflush.o)
 .debug_abbrev  0x00005688       0x25 c:/program files/microchip/xc32/v1.33/bin/bin/../../lib/gcc/pic32mx/4.5.2/../../../../pic32mx/lib\libpic32.a(read.o)
 .debug_abbrev  0x000056ad       0x25 c:/program files/microchip/xc32/v1.33/bin/bin/../../lib/gcc/pic32mx/4.5.2/../../../../pic32mx/lib\libpic32.a(write.o)
 .debug_abbrev  0x000056d2        0x1 c:/program files/microchip/xc32/v1.33/bin/bin/../../lib/gcc/pic32mx/4.5.2/../../../../pic32mx/lib\libpic32.a(xc32_uart.o)
 .debug_abbrev  0x000056d3      0x132 c:/program files/microchip/xc32/v1.33/bin/bin/../../lib/gcc/pic32mx/4.5.2\libgcc.a(_udivdi3.o)
 .debug_abbrev  0x00005805      0x13f c:/program files/microchip/xc32/v1.33/bin/bin/../../lib/gcc/pic32mx/4.5.2\libgcc.a(_umoddi3.o)

.debug_line     0x00000000     0x7510
 *(.debug_line)
 .debug_line    0x00000000       0x8a c:/program files/microchip/xc32/v1.33/bin/bin/../../lib/gcc/pic32mx/4.5.2/../../../../pic32mx/lib\software-debug-break.o
 .debug_line    0x0000008a      0x1f9 build/ChaletDuinoV2_795F512H_/debug/Source/ChaletduinoV2Board.o
 .debug_line    0x00000283      0x200 build/ChaletDuinoV2_795F512H_/debug/Source/winc3400_142/common/source/nm_common.o
 .debug_line    0x00000483      0x336 build/ChaletDuinoV2_795F512H_/debug/Source/winc3400_142/driver/source/m2m_flash.o
 .debug_line    0x000007b9      0x415 build/ChaletDuinoV2_795F512H_/debug/Source/winc3400_142/driver/source/m2m_hif.o
 .debug_line    0x00000bce      0x287 build/ChaletDuinoV2_795F512H_/debug/Source/winc3400_142/driver/source/m2m_ota.o
 .debug_line    0x00000e55      0x275 build/ChaletDuinoV2_795F512H_/debug/Source/winc3400_142/driver/source/m2m_periph.o
 .debug_line    0x000010ca      0x381 build/ChaletDuinoV2_795F512H_/debug/Source/winc3400_142/driver/source/m2m_ssl.o
 .debug_line    0x0000144b      0x81c build/ChaletDuinoV2_795F512H_/debug/Source/winc3400_142/driver/source/m2m_wifi.o
 .debug_line    0x00001c67      0x44b build/ChaletDuinoV2_795F512H_/debug/Source/winc3400_142/driver/source/nmasic.o
 .debug_line    0x000020b2      0x231 build/ChaletDuinoV2_795F512H_/debug/Source/winc3400_142/driver/source/nmbus.o
 .debug_line    0x000022e3      0x301 build/ChaletDuinoV2_795F512H_/debug/Source/winc3400_142/driver/source/nmdrv.o
 .debug_line    0x000025e4      0x3f5 build/ChaletDuinoV2_795F512H_/debug/Source/winc3400_142/driver/source/nmspi.o
 .debug_line    0x000029d9      0x1f6 build/ChaletDuinoV2_795F512H_/debug/Source/winc3400_142/socket/source/inet_addr.o
 .debug_line    0x00002bcf      0x25e build/ChaletDuinoV2_795F512H_/debug/Source/winc3400_142/socket/source/inet_ntop.o
 .debug_line    0x00002e2d      0x635 build/ChaletDuinoV2_795F512H_/debug/Source/winc3400_142/socket/source/socket.o
 .debug_line    0x00003462      0x36d build/ChaletDuinoV2_795F512H_/debug/Source/winc3400_142/spi_flash/source/spi_flash.o
 .debug_line    0x000037cf      0x15a build/ChaletDuinoV2_795F512H_/debug/Source/DigitalIO.o
 .debug_line    0x00003929      0x290 build/ChaletDuinoV2_795F512H_/debug/Source/NetworkProtocol.o
 .debug_line    0x00003bb9      0x342 build/ChaletDuinoV2_795F512H_/debug/Source/Terminal.o
 .debug_line    0x00003efb      0x25f build/ChaletDuinoV2_795F512H_/debug/Source/Util.o
 .debug_line    0x0000415a      0x165 build/ChaletDuinoV2_795F512H_/debug/Source/exceptions.o
 .debug_line    0x000042bf      0x101 build/ChaletDuinoV2_795F512H_/debug/Source/interrupts.o
 .debug_line    0x000043c0      0x368 build/ChaletDuinoV2_795F512H_/debug/Source/main.o
 .debug_line    0x00004728      0x101 build/ChaletDuinoV2_795F512H_/debug/Source/system.o
 .debug_line    0x00004829      0x101 build/ChaletDuinoV2_795F512H_/debug/Source/template.o
 .debug_line    0x0000492a      0x233 build/ChaletDuinoV2_795F512H_/debug/Source/timer.o
 .debug_line    0x00004b5d      0x508 build/ChaletDuinoV2_795F512H_/debug/Source/WiFiCtrl.o
 .debug_line    0x00005065      0x159 build/ChaletDuinoV2_795F512H_/debug/Source/SPI.o
 .debug_line    0x000051be      0x2a5 build/ChaletDuinoV2_795F512H_/debug/Source/SPI_Flash.o
 .debug_line    0x00005463      0x269 build/ChaletDuinoV2_795F512H_/debug/Source/Syslog.o
 .debug_line    0x000056cc      0x169 build/ChaletDuinoV2_795F512H_/debug/Source/Watchdog.o
 .debug_line    0x00005835      0x4c1 build/ChaletDuinoV2_795F512H_/debug/Source/BootloaderInterface.o
 .debug_line    0x00005cf6      0x388 build/ChaletDuinoV2_795F512H_/debug/Source/BootloaderProtocol.o
 .debug_line    0x0000607e      0x13b build/ChaletDuinoV2_795F512H_/debug/Source/crc32.o
 .debug_line    0x000061b9      0x1d9 build/ChaletDuinoV2_795F512H_/debug/Source/VolumeTransducer.o
 .debug_line    0x00006392      0x1b6 build/ChaletDuinoV2_795F512H_/debug/Source/DACInterface.o
 .debug_line    0x00006548       0xb1 c:/program files/microchip/xc32/v1.33/bin/bin/../../lib/gcc/pic32mx/4.5.2/../../../../pic32mx/lib\libmchp_peripheral_32MX795F512H.a(soft_reset_lib.o)
 .debug_line    0x000065f9       0x62 c:/program files/microchip/xc32/v1.33/bin/bin/../../lib/gcc/pic32mx/4.5.2/../../../../pic32mx/lib\libmchp_peripheral_32MX795F512H.a(pcache.o)
 .debug_line    0x0000665b       0x71 c:/program files/microchip/xc32/v1.33/bin/bin/../../lib/gcc/pic32mx/4.5.2/../../../../pic32mx/lib\libmchp_peripheral_32MX795F512H.a(int_configure_system_lib.o)
 .debug_line    0x000066cc       0x72 c:/program files/microchip/xc32/v1.33/bin/bin/../../lib/gcc/pic32mx/4.5.2/../../../../pic32mx/lib\libmchp_peripheral_32MX795F512H.a(int_enable_interrupts_lib.o)
 .debug_line    0x0000673e       0x73 c:/program files/microchip/xc32/v1.33/bin/bin/../../lib/gcc/pic32mx/4.5.2/../../../../pic32mx/lib\libmchp_peripheral_32MX795F512H.a(int_disable_interrupts_lib.o)
 .debug_line    0x000067b1       0x73 c:/program files/microchip/xc32/v1.33/bin/bin/../../lib/gcc/pic32mx/4.5.2/../../../../pic32mx/lib\libmchp_peripheral_32MX795F512H.a(int_restore_interrupts_lib.o)
 .debug_line    0x00006824       0x97 c:/program files/microchip/xc32/v1.33/bin/bin/../../lib/gcc/pic32mx/4.5.2/../../../../pic32mx/lib\libpic32.a(default-bootstrap-exception-handler.o)
 .debug_line    0x000068bb       0x84 c:/program files/microchip/xc32/v1.33/bin/bin/../../lib/gcc/pic32mx/4.5.2/../../../../pic32mx/lib\libpic32.a(default-on-reset.o)
 .debug_line    0x0000693f       0x88 c:/program files/microchip/xc32/v1.33/bin/bin/../../lib/gcc/pic32mx/4.5.2/../../../../pic32mx/lib\libpic32.a(default-on-bootstrap.o)
 .debug_line    0x000069c7       0x79 c:/program files/microchip/xc32/v1.33/bin/bin/../../lib/gcc/pic32mx/4.5.2/../../../../pic32mx/lib\libpic32.a(close.o)
 .debug_line    0x00006a40       0x96 c:/program files/microchip/xc32/v1.33/bin/bin/../../lib/gcc/pic32mx/4.5.2/../../../../pic32mx/lib\libpic32.a(defaultinterrupt.o)
 .debug_line    0x00006ad6       0x6e c:/program files/microchip/xc32/v1.33/bin/bin/../../lib/gcc/pic32mx/4.5.2/../../../../pic32mx/lib\libc.a(puts.o)
 .debug_line    0x00006b44       0x71 c:/program files/microchip/xc32/v1.33/bin/bin/../../lib/gcc/pic32mx/4.5.2/../../../../pic32mx/lib\libc.a(strncmp.o)
 .debug_line    0x00006bb5       0x70 c:/program files/microchip/xc32/v1.33/bin/bin/../../lib/gcc/pic32mx/4.5.2/../../../../pic32mx/lib\libc.a(printf_cdnopsuxX.eo)
 .debug_line    0x00006c25       0x71 c:/program files/microchip/xc32/v1.33/bin/bin/../../lib/gcc/pic32mx/4.5.2/../../../../pic32mx/lib\libc.a(sprintf_cdnopuxX.eo)
 .debug_line    0x00006c96       0x70 c:/program files/microchip/xc32/v1.33/bin/bin/../../lib/gcc/pic32mx/4.5.2/../../../../pic32mx/lib\libc.a(sscanf_s.eo)
 .debug_line    0x00006d06        0x0 c:/program files/microchip/xc32/v1.33/bin/bin/../../lib/gcc/pic32mx/4.5.2/../../../../pic32mx/lib\libc.a(_iob.o)
 .debug_line    0x00006d06       0x6f c:/program files/microchip/xc32/v1.33/bin/bin/../../lib/gcc/pic32mx/4.5.2/../../../../pic32mx/lib\libc.a(_fputc_simple.o)
 .debug_line    0x00006d75       0x70 c:/program files/microchip/xc32/v1.33/bin/bin/../../lib/gcc/pic32mx/4.5.2/../../../../pic32mx/lib\libc.a(doprnt_cdnopsuxX.eo)
 .debug_line    0x00006de5       0x70 c:/program files/microchip/xc32/v1.33/bin/bin/../../lib/gcc/pic32mx/4.5.2/../../../../pic32mx/lib\libc.a(doscan_s.eo)
 .debug_line    0x00006e55       0x70 c:/program files/microchip/xc32/v1.33/bin/bin/../../lib/gcc/pic32mx/4.5.2/../../../../pic32mx/lib\libc.a(_flsbuf_simple.o)
 .debug_line    0x00006ec5       0x6f c:/program files/microchip/xc32/v1.33/bin/bin/../../lib/gcc/pic32mx/4.5.2/../../../../pic32mx/lib\libc.a(fgetc.o)
 .debug_line    0x00006f34       0x6e c:/program files/microchip/xc32/v1.33/bin/bin/../../lib/gcc/pic32mx/4.5.2/../../../../pic32mx/lib\libc.a(atoi.o)
 .debug_line    0x00006fa2        0x0 c:/program files/microchip/xc32/v1.33/bin/bin/../../lib/gcc/pic32mx/4.5.2/../../../../pic32mx/lib\libc.a(ctype.o)
 .debug_line    0x00006fa2       0x70 c:/program files/microchip/xc32/v1.33/bin/bin/../../lib/gcc/pic32mx/4.5.2/../../../../pic32mx/lib\libc.a(ctypef.o)
 .debug_line    0x00007012       0x70 c:/program files/microchip/xc32/v1.33/bin/bin/../../lib/gcc/pic32mx/4.5.2/../../../../pic32mx/lib\libc.a(ungetc.o)
 .debug_line    0x00007082       0x70 c:/program files/microchip/xc32/v1.33/bin/bin/../../lib/gcc/pic32mx/4.5.2/../../../../pic32mx/lib\libc.a(filbuf.o)
 .debug_line    0x000070f2       0x70 c:/program files/microchip/xc32/v1.33/bin/bin/../../lib/gcc/pic32mx/4.5.2/../../../../pic32mx/lib\libc.a(fflush.o)
 .debug_line    0x00007162       0x78 c:/program files/microchip/xc32/v1.33/bin/bin/../../lib/gcc/pic32mx/4.5.2/../../../../pic32mx/lib\libpic32.a(read.o)
 .debug_line    0x000071da       0x79 c:/program files/microchip/xc32/v1.33/bin/bin/../../lib/gcc/pic32mx/4.5.2/../../../../pic32mx/lib\libpic32.a(write.o)
 .debug_line    0x00007253        0x0 c:/program files/microchip/xc32/v1.33/bin/bin/../../lib/gcc/pic32mx/4.5.2/../../../../pic32mx/lib\libpic32.a(xc32_uart.o)
 .debug_line    0x00007253      0x168 c:/program files/microchip/xc32/v1.33/bin/bin/../../lib/gcc/pic32mx/4.5.2\libgcc.a(_udivdi3.o)
 .debug_line    0x000073bb      0x155 c:/program files/microchip/xc32/v1.33/bin/bin/../../lib/gcc/pic32mx/4.5.2\libgcc.a(_umoddi3.o)

.debug_frame    0x00000000     0x3268
 *(.debug_frame)
 .debug_frame   0x00000000       0x20 c:/program files/microchip/xc32/v1.33/bin/bin/../../lib/gcc/pic32mx/4.5.2/../../../../pic32mx/lib\software-debug-break.o
 .debug_frame   0x00000020       0x2c build/ChaletDuinoV2_795F512H_/debug/Source/ChaletduinoV2Board.o
 .debug_frame   0x0000004c       0xa0 build/ChaletDuinoV2_795F512H_/debug/Source/winc3400_142/common/source/nm_common.o
 .debug_frame   0x000000ec      0x148 build/ChaletDuinoV2_795F512H_/debug/Source/winc3400_142/driver/source/m2m_flash.o
 .debug_frame   0x00000234      0x1ec build/ChaletDuinoV2_795F512H_/debug/Source/winc3400_142/driver/source/m2m_hif.o
 .debug_frame   0x00000420       0xb8 build/ChaletDuinoV2_795F512H_/debug/Source/winc3400_142/driver/source/m2m_ota.o
 .debug_frame   0x000004d8       0xd4 build/ChaletDuinoV2_795F512H_/debug/Source/winc3400_142/driver/source/m2m_periph.o
 .debug_frame   0x000005ac      0x144 build/ChaletDuinoV2_795F512H_/debug/Source/winc3400_142/driver/source/m2m_ssl.o
 .debug_frame   0x000006f0      0x8d0 build/ChaletDuinoV2_795F512H_/debug/Source/winc3400_142/driver/source/m2m_wifi.o
 .debug_frame   0x00000fc0      0x294 build/ChaletDuinoV2_795F512H_/debug/Source/winc3400_142/driver/source/nmasic.o
 .debug_frame   0x00001254      0x17c build/ChaletDuinoV2_795F512H_/debug/Source/winc3400_142/driver/source/nmbus.o
 .debug_frame   0x000013d0      0x128 build/ChaletDuinoV2_795F512H_/debug/Source/winc3400_142/driver/source/nmdrv.o
 .debug_frame   0x000014f8      0x298 build/ChaletDuinoV2_795F512H_/debug/Source/winc3400_142/driver/source/nmspi.o
 .debug_frame   0x00001790       0x2c build/ChaletDuinoV2_795F512H_/debug/Source/winc3400_142/socket/source/inet_addr.o
 .debug_frame   0x000017bc       0x2c build/ChaletDuinoV2_795F512H_/debug/Source/winc3400_142/socket/source/inet_ntop.o
 .debug_frame   0x000017e8      0x320 build/ChaletDuinoV2_795F512H_/debug/Source/winc3400_142/socket/source/socket.o
 .debug_frame   0x00001b08      0x17c build/ChaletDuinoV2_795F512H_/debug/Source/winc3400_142/spi_flash/source/spi_flash.o
 .debug_frame   0x00001c84       0x2c build/ChaletDuinoV2_795F512H_/debug/Source/DigitalIO.o
 .debug_frame   0x00001cb0      0x12c build/ChaletDuinoV2_795F512H_/debug/Source/NetworkProtocol.o
 .debug_frame   0x00001ddc       0xf4 build/ChaletDuinoV2_795F512H_/debug/Source/Terminal.o
 .debug_frame   0x00001ed0      0x10c build/ChaletDuinoV2_795F512H_/debug/Source/Util.o
 .debug_frame   0x00001fdc       0x2c build/ChaletDuinoV2_795F512H_/debug/Source/exceptions.o
 .debug_frame   0x00002008       0x64 build/ChaletDuinoV2_795F512H_/debug/Source/main.o
 .debug_frame   0x0000206c      0x148 build/ChaletDuinoV2_795F512H_/debug/Source/timer.o
 .debug_frame   0x000021b4      0x2d0 build/ChaletDuinoV2_795F512H_/debug/Source/WiFiCtrl.o
 .debug_frame   0x00002484       0x2c build/ChaletDuinoV2_795F512H_/debug/Source/SPI.o
 .debug_frame   0x000024b0      0x17c build/ChaletDuinoV2_795F512H_/debug/Source/SPI_Flash.o
 .debug_frame   0x0000262c       0xd8 build/ChaletDuinoV2_795F512H_/debug/Source/Syslog.o
 .debug_frame   0x00002704       0x80 build/ChaletDuinoV2_795F512H_/debug/Source/Watchdog.o
 .debug_frame   0x00002784      0x1d0 build/ChaletDuinoV2_795F512H_/debug/Source/BootloaderInterface.o
 .debug_frame   0x00002954      0x1b4 build/ChaletDuinoV2_795F512H_/debug/Source/BootloaderProtocol.o
 .debug_frame   0x00002b08       0x64 build/ChaletDuinoV2_795F512H_/debug/Source/crc32.o
 .debug_frame   0x00002b6c       0xd0 build/ChaletDuinoV2_795F512H_/debug/Source/VolumeTransducer.o
 .debug_frame   0x00002c3c       0x48 build/ChaletDuinoV2_795F512H_/debug/Source/DACInterface.o
 .debug_frame   0x00002c84       0x28 c:/program files/microchip/xc32/v1.33/bin/bin/../../lib/gcc/pic32mx/4.5.2/../../../../pic32mx/lib\libmchp_peripheral_32MX795F512H.a(soft_reset_lib.o)
 .debug_frame   0x00002cac       0x30 c:/program files/microchip/xc32/v1.33/bin/bin/../../lib/gcc/pic32mx/4.5.2/../../../../pic32mx/lib\libmchp_peripheral_32MX795F512H.a(pcache.o)
 .debug_frame   0x00002cdc       0x20 c:/program files/microchip/xc32/v1.33/bin/bin/../../lib/gcc/pic32mx/4.5.2/../../../../pic32mx/lib\libmchp_peripheral_32MX795F512H.a(int_configure_system_lib.o)
 .debug_frame   0x00002cfc       0x20 c:/program files/microchip/xc32/v1.33/bin/bin/../../lib/gcc/pic32mx/4.5.2/../../../../pic32mx/lib\libmchp_peripheral_32MX795F512H.a(int_enable_interrupts_lib.o)
 .debug_frame   0x00002d1c       0x20 c:/program files/microchip/xc32/v1.33/bin/bin/../../lib/gcc/pic32mx/4.5.2/../../../../pic32mx/lib\libmchp_peripheral_32MX795F512H.a(int_disable_interrupts_lib.o)
 .debug_frame   0x00002d3c       0x20 c:/program files/microchip/xc32/v1.33/bin/bin/../../lib/gcc/pic32mx/4.5.2/../../../../pic32mx/lib\libmchp_peripheral_32MX795F512H.a(int_restore_interrupts_lib.o)
 .debug_frame   0x00002d5c       0x28 c:/program files/microchip/xc32/v1.33/bin/bin/../../lib/gcc/pic32mx/4.5.2/../../../../pic32mx/lib\libpic32.a(default-bootstrap-exception-handler.o)
 .debug_frame   0x00002d84       0x20 c:/program files/microchip/xc32/v1.33/bin/bin/../../lib/gcc/pic32mx/4.5.2/../../../../pic32mx/lib\libpic32.a(default-on-reset.o)
 .debug_frame   0x00002da4       0x20 c:/program files/microchip/xc32/v1.33/bin/bin/../../lib/gcc/pic32mx/4.5.2/../../../../pic32mx/lib\libpic32.a(default-on-bootstrap.o)
 .debug_frame   0x00002dc4       0x20 c:/program files/microchip/xc32/v1.33/bin/bin/../../lib/gcc/pic32mx/4.5.2/../../../../pic32mx/lib\libpic32.a(close.o)
 .debug_frame   0x00002de4       0x20 c:/program files/microchip/xc32/v1.33/bin/bin/../../lib/gcc/pic32mx/4.5.2/../../../../pic32mx/lib\libpic32.a(defaultinterrupt.o)
 .debug_frame   0x00002e04       0x48 c:/program files/microchip/xc32/v1.33/bin/bin/../../lib/gcc/pic32mx/4.5.2/../../../../pic32mx/lib\libc.a(puts.o)
 .debug_frame   0x00002e4c       0x20 c:/program files/microchip/xc32/v1.33/bin/bin/../../lib/gcc/pic32mx/4.5.2/../../../../pic32mx/lib\libc.a(strncmp.o)
 .debug_frame   0x00002e6c       0x28 c:/program files/microchip/xc32/v1.33/bin/bin/../../lib/gcc/pic32mx/4.5.2/../../../../pic32mx/lib\libc.a(printf_cdnopsuxX.eo)
 .debug_frame   0x00002e94       0x2c c:/program files/microchip/xc32/v1.33/bin/bin/../../lib/gcc/pic32mx/4.5.2/../../../../pic32mx/lib\libc.a(sprintf_cdnopuxX.eo)
 .debug_frame   0x00002ec0       0x28 c:/program files/microchip/xc32/v1.33/bin/bin/../../lib/gcc/pic32mx/4.5.2/../../../../pic32mx/lib\libc.a(sscanf_s.eo)
 .debug_frame   0x00002ee8       0x2c c:/program files/microchip/xc32/v1.33/bin/bin/../../lib/gcc/pic32mx/4.5.2/../../../../pic32mx/lib\libc.a(_fputc_simple.o)
 .debug_frame   0x00002f14       0x38 c:/program files/microchip/xc32/v1.33/bin/bin/../../lib/gcc/pic32mx/4.5.2/../../../../pic32mx/lib\libc.a(doprnt_cdnopsuxX.eo)
 .debug_frame   0x00002f4c       0x74 c:/program files/microchip/xc32/v1.33/bin/bin/../../lib/gcc/pic32mx/4.5.2/../../../../pic32mx/lib\libc.a(doscan_s.eo)
 .debug_frame   0x00002fc0       0x28 c:/program files/microchip/xc32/v1.33/bin/bin/../../lib/gcc/pic32mx/4.5.2/../../../../pic32mx/lib\libc.a(_flsbuf_simple.o)
 .debug_frame   0x00002fe8       0x30 c:/program files/microchip/xc32/v1.33/bin/bin/../../lib/gcc/pic32mx/4.5.2/../../../../pic32mx/lib\libc.a(fgetc.o)
 .debug_frame   0x00003018       0x20 c:/program files/microchip/xc32/v1.33/bin/bin/../../lib/gcc/pic32mx/4.5.2/../../../../pic32mx/lib\libc.a(atoi.o)
 .debug_frame   0x00003038      0x120 c:/program files/microchip/xc32/v1.33/bin/bin/../../lib/gcc/pic32mx/4.5.2/../../../../pic32mx/lib\libc.a(ctypef.o)
 .debug_frame   0x00003158       0x20 c:/program files/microchip/xc32/v1.33/bin/bin/../../lib/gcc/pic32mx/4.5.2/../../../../pic32mx/lib\libc.a(ungetc.o)
 .debug_frame   0x00003178       0x30 c:/program files/microchip/xc32/v1.33/bin/bin/../../lib/gcc/pic32mx/4.5.2/../../../../pic32mx/lib\libc.a(filbuf.o)
 .debug_frame   0x000031a8       0x2c c:/program files/microchip/xc32/v1.33/bin/bin/../../lib/gcc/pic32mx/4.5.2/../../../../pic32mx/lib\libc.a(fflush.o)
 .debug_frame   0x000031d4       0x2c c:/program files/microchip/xc32/v1.33/bin/bin/../../lib/gcc/pic32mx/4.5.2/../../../../pic32mx/lib\libpic32.a(read.o)
 .debug_frame   0x00003200       0x28 c:/program files/microchip/xc32/v1.33/bin/bin/../../lib/gcc/pic32mx/4.5.2/../../../../pic32mx/lib\libpic32.a(write.o)
 .debug_frame   0x00003228       0x20 c:/program files/microchip/xc32/v1.33/bin/bin/../../lib/gcc/pic32mx/4.5.2\libgcc.a(_udivdi3.o)
 .debug_frame   0x00003248       0x20 c:/program files/microchip/xc32/v1.33/bin/bin/../../lib/gcc/pic32mx/4.5.2\libgcc.a(_umoddi3.o)

.debug_str      0x00000000     0x37d1
 *(.debug_str)
 .debug_str     0x00000000        0x0 c:/program files/microchip/xc32/v1.33/bin/bin/../../lib/gcc/pic32mx/4.5.2/../../../../pic32mx/lib\software-debug-break.o
 .debug_str     0x00000000      0x1f3 build/ChaletDuinoV2_795F512H_/debug/Source/ChaletduinoV2Board.o
 .debug_str     0x000001f3      0x141 build/ChaletDuinoV2_795F512H_/debug/Source/winc3400_142/common/source/nm_common.o
 .debug_str     0x00000334      0x1ba build/ChaletDuinoV2_795F512H_/debug/Source/winc3400_142/driver/source/m2m_flash.o
 .debug_str     0x000004ee      0x158 build/ChaletDuinoV2_795F512H_/debug/Source/winc3400_142/driver/source/m2m_hif.o
 .debug_str     0x00000646      0x12f build/ChaletDuinoV2_795F512H_/debug/Source/winc3400_142/driver/source/m2m_ota.o
 .debug_str     0x00000775      0x139 build/ChaletDuinoV2_795F512H_/debug/Source/winc3400_142/driver/source/m2m_periph.o
 .debug_str     0x000008ae      0x166 build/ChaletDuinoV2_795F512H_/debug/Source/winc3400_142/driver/source/m2m_ssl.o
 .debug_str     0x00000a14      0x406 build/ChaletDuinoV2_795F512H_/debug/Source/winc3400_142/driver/source/m2m_wifi.o
 .debug_str     0x00000e1a      0x15c build/ChaletDuinoV2_795F512H_/debug/Source/winc3400_142/driver/source/nmasic.o
 .debug_str     0x00000f76      0x160 build/ChaletDuinoV2_795F512H_/debug/Source/winc3400_142/driver/source/nmbus.o
 .debug_str     0x000010d6      0x12f build/ChaletDuinoV2_795F512H_/debug/Source/winc3400_142/driver/source/nmdrv.o
 .debug_str     0x00001205      0x17f build/ChaletDuinoV2_795F512H_/debug/Source/winc3400_142/driver/source/nmspi.o
 .debug_str     0x00001384      0x12f build/ChaletDuinoV2_795F512H_/debug/Source/winc3400_142/socket/source/inet_addr.o
 .debug_str     0x000014b3      0x12f build/ChaletDuinoV2_795F512H_/debug/Source/winc3400_142/socket/source/inet_ntop.o
 .debug_str     0x000015e2      0x2e5 build/ChaletDuinoV2_795F512H_/debug/Source/winc3400_142/socket/source/socket.o
 .debug_str     0x000018c7      0x18a build/ChaletDuinoV2_795F512H_/debug/Source/winc3400_142/spi_flash/source/spi_flash.o
 .debug_str     0x00001a51      0x12f build/ChaletDuinoV2_795F512H_/debug/Source/DigitalIO.o
 .debug_str     0x00001b80      0x175 build/ChaletDuinoV2_795F512H_/debug/Source/NetworkProtocol.o
 .debug_str     0x00001cf5      0x1a2 build/ChaletDuinoV2_795F512H_/debug/Source/Terminal.o
 .debug_str     0x00001e97      0x145 build/ChaletDuinoV2_795F512H_/debug/Source/Util.o
 .debug_str     0x00001fdc      0x12f build/ChaletDuinoV2_795F512H_/debug/Source/exceptions.o
 .debug_str     0x0000210b      0x12f build/ChaletDuinoV2_795F512H_/debug/Source/interrupts.o
 .debug_str     0x0000223a      0x186 build/ChaletDuinoV2_795F512H_/debug/Source/main.o
 .debug_str     0x000023c0      0x12f build/ChaletDuinoV2_795F512H_/debug/Source/system.o
 .debug_str     0x000024ef      0x12f build/ChaletDuinoV2_795F512H_/debug/Source/template.o
 .debug_str     0x0000261e      0x17f build/ChaletDuinoV2_795F512H_/debug/Source/timer.o
 .debug_str     0x0000279d      0x29e build/ChaletDuinoV2_795F512H_/debug/Source/WiFiCtrl.o
 .debug_str     0x00002a3b      0x146 build/ChaletDuinoV2_795F512H_/debug/Source/SPI.o
 .debug_str     0x00002b81      0x19f build/ChaletDuinoV2_795F512H_/debug/Source/SPI_Flash.o
 .debug_str     0x00002d20      0x168 build/ChaletDuinoV2_795F512H_/debug/Source/Syslog.o
 .debug_str     0x00002e88      0x15e build/ChaletDuinoV2_795F512H_/debug/Source/Watchdog.o
 .debug_str     0x00002fe6      0x2cb build/ChaletDuinoV2_795F512H_/debug/Source/BootloaderInterface.o
 .debug_str     0x000032b1      0x1fe build/ChaletDuinoV2_795F512H_/debug/Source/BootloaderProtocol.o
 .debug_str     0x000034af        0x0 build/ChaletDuinoV2_795F512H_/debug/Source/crc32.o
 .debug_str     0x000034af      0x1b3 build/ChaletDuinoV2_795F512H_/debug/Source/VolumeTransducer.o
 .debug_str     0x00003662      0x16f build/ChaletDuinoV2_795F512H_/debug/Source/DACInterface.o
 .debug_str     0x000037d1        0x0 c:/program files/microchip/xc32/v1.33/bin/bin/../../lib/gcc/pic32mx/4.5.2/../../../../pic32mx/lib\libmchp_peripheral_32MX795F512H.a(soft_reset_lib.o)
 .debug_str     0x000037d1        0x0 c:/program files/microchip/xc32/v1.33/bin/bin/../../lib/gcc/pic32mx/4.5.2/../../../../pic32mx/lib\libmchp_peripheral_32MX795F512H.a(pcache.o)
 .debug_str     0x000037d1        0x0 c:/program files/microchip/xc32/v1.33/bin/bin/../../lib/gcc/pic32mx/4.5.2/../../../../pic32mx/lib\libmchp_peripheral_32MX795F512H.a(int_configure_system_lib.o)
 .debug_str     0x000037d1        0x0 c:/program files/microchip/xc32/v1.33/bin/bin/../../lib/gcc/pic32mx/4.5.2/../../../../pic32mx/lib\libmchp_peripheral_32MX795F512H.a(int_enable_interrupts_lib.o)
 .debug_str     0x000037d1        0x0 c:/program files/microchip/xc32/v1.33/bin/bin/../../lib/gcc/pic32mx/4.5.2/../../../../pic32mx/lib\libmchp_peripheral_32MX795F512H.a(int_disable_interrupts_lib.o)
 .debug_str     0x000037d1        0x0 c:/program files/microchip/xc32/v1.33/bin/bin/../../lib/gcc/pic32mx/4.5.2/../../../../pic32mx/lib\libmchp_peripheral_32MX795F512H.a(int_restore_interrupts_lib.o)
 .debug_str     0x000037d1        0x0 c:/program files/microchip/xc32/v1.33/bin/bin/../../lib/gcc/pic32mx/4.5.2/../../../../pic32mx/lib\libpic32.a(default-bootstrap-exception-handler.o)
 .debug_str     0x000037d1        0x0 c:/program files/microchip/xc32/v1.33/bin/bin/../../lib/gcc/pic32mx/4.5.2/../../../../pic32mx/lib\libpic32.a(default-on-reset.o)
 .debug_str     0x000037d1        0x0 c:/program files/microchip/xc32/v1.33/bin/bin/../../lib/gcc/pic32mx/4.5.2/../../../../pic32mx/lib\libpic32.a(default-on-bootstrap.o)
 .debug_str     0x000037d1        0x0 c:/program files/microchip/xc32/v1.33/bin/bin/../../lib/gcc/pic32mx/4.5.2/../../../../pic32mx/lib\libpic32.a(close.o)
 .debug_str     0x000037d1        0x0 c:/program files/microchip/xc32/v1.33/bin/bin/../../lib/gcc/pic32mx/4.5.2/../../../../pic32mx/lib\libpic32.a(defaultinterrupt.o)
 .debug_str     0x000037d1        0x0 c:/program files/microchip/xc32/v1.33/bin/bin/../../lib/gcc/pic32mx/4.5.2/../../../../pic32mx/lib\libc.a(puts.o)
 .debug_str     0x000037d1        0x0 c:/program files/microchip/xc32/v1.33/bin/bin/../../lib/gcc/pic32mx/4.5.2/../../../../pic32mx/lib\libc.a(strncmp.o)
 .debug_str     0x000037d1        0x0 c:/program files/microchip/xc32/v1.33/bin/bin/../../lib/gcc/pic32mx/4.5.2/../../../../pic32mx/lib\libc.a(printf_cdnopsuxX.eo)
 .debug_str     0x000037d1        0x0 c:/program files/microchip/xc32/v1.33/bin/bin/../../lib/gcc/pic32mx/4.5.2/../../../../pic32mx/lib\libc.a(sprintf_cdnopuxX.eo)
 .debug_str     0x000037d1        0x0 c:/program files/microchip/xc32/v1.33/bin/bin/../../lib/gcc/pic32mx/4.5.2/../../../../pic32mx/lib\libc.a(sscanf_s.eo)
 .debug_str     0x000037d1        0x0 c:/program files/microchip/xc32/v1.33/bin/bin/../../lib/gcc/pic32mx/4.5.2/../../../../pic32mx/lib\libc.a(_iob.o)
 .debug_str     0x000037d1        0x0 c:/program files/microchip/xc32/v1.33/bin/bin/../../lib/gcc/pic32mx/4.5.2/../../../../pic32mx/lib\libc.a(_fputc_simple.o)
 .debug_str     0x000037d1        0x0 c:/program files/microchip/xc32/v1.33/bin/bin/../../lib/gcc/pic32mx/4.5.2/../../../../pic32mx/lib\libc.a(doprnt_cdnopsuxX.eo)
 .debug_str     0x000037d1        0x0 c:/program files/microchip/xc32/v1.33/bin/bin/../../lib/gcc/pic32mx/4.5.2/../../../../pic32mx/lib\libc.a(doscan_s.eo)
 .debug_str     0x000037d1        0x0 c:/program files/microchip/xc32/v1.33/bin/bin/../../lib/gcc/pic32mx/4.5.2/../../../../pic32mx/lib\libc.a(_flsbuf_simple.o)
 .debug_str     0x000037d1        0x0 c:/program files/microchip/xc32/v1.33/bin/bin/../../lib/gcc/pic32mx/4.5.2/../../../../pic32mx/lib\libc.a(fgetc.o)
 .debug_str     0x000037d1        0x0 c:/program files/microchip/xc32/v1.33/bin/bin/../../lib/gcc/pic32mx/4.5.2/../../../../pic32mx/lib\libc.a(atoi.o)
 .debug_str     0x000037d1        0x0 c:/program files/microchip/xc32/v1.33/bin/bin/../../lib/gcc/pic32mx/4.5.2/../../../../pic32mx/lib\libc.a(ctype.o)
 .debug_str     0x000037d1        0x0 c:/program files/microchip/xc32/v1.33/bin/bin/../../lib/gcc/pic32mx/4.5.2/../../../../pic32mx/lib\libc.a(ctypef.o)
 .debug_str     0x000037d1        0x0 c:/program files/microchip/xc32/v1.33/bin/bin/../../lib/gcc/pic32mx/4.5.2/../../../../pic32mx/lib\libc.a(ungetc.o)
 .debug_str     0x000037d1        0x0 c:/program files/microchip/xc32/v1.33/bin/bin/../../lib/gcc/pic32mx/4.5.2/../../../../pic32mx/lib\libc.a(filbuf.o)
 .debug_str     0x000037d1        0x0 c:/program files/microchip/xc32/v1.33/bin/bin/../../lib/gcc/pic32mx/4.5.2/../../../../pic32mx/lib\libc.a(fflush.o)
 .debug_str     0x000037d1        0x0 c:/program files/microchip/xc32/v1.33/bin/bin/../../lib/gcc/pic32mx/4.5.2/../../../../pic32mx/lib\libpic32.a(read.o)
 .debug_str     0x000037d1        0x0 c:/program files/microchip/xc32/v1.33/bin/bin/../../lib/gcc/pic32mx/4.5.2/../../../../pic32mx/lib\libpic32.a(write.o)
 .debug_str     0x000037d1        0x0 c:/program files/microchip/xc32/v1.33/bin/bin/../../lib/gcc/pic32mx/4.5.2/../../../../pic32mx/lib\libpic32.a(xc32_uart.o)
 .debug_str     0x000037d1        0x0 c:/program files/microchip/xc32/v1.33/bin/bin/../../lib/gcc/pic32mx/4.5.2\libgcc.a(_udivdi3.o)
 .debug_str     0x000037d1        0x0 c:/program files/microchip/xc32/v1.33/bin/bin/../../lib/gcc/pic32mx/4.5.2\libgcc.a(_umoddi3.o)

.debug_loc      0x00000000     0xfce0
 *(.debug_loc)
 .debug_loc     0x00000000       0xba build/ChaletDuinoV2_795F512H_/debug/Source/ChaletduinoV2Board.o
 .debug_loc     0x000000ba      0x24e build/ChaletDuinoV2_795F512H_/debug/Source/winc3400_142/common/source/nm_common.o
 .debug_loc     0x00000308      0x850 build/ChaletDuinoV2_795F512H_/debug/Source/winc3400_142/driver/source/m2m_flash.o
 .debug_loc     0x00000b58      0xbda build/ChaletDuinoV2_795F512H_/debug/Source/winc3400_142/driver/source/m2m_hif.o
 .debug_loc     0x00001732      0x2e1 build/ChaletDuinoV2_795F512H_/debug/Source/winc3400_142/driver/source/m2m_ota.o
 .debug_loc     0x00001a13      0x2e2 build/ChaletDuinoV2_795F512H_/debug/Source/winc3400_142/driver/source/m2m_periph.o
 .debug_loc     0x00001cf5      0x86e build/ChaletDuinoV2_795F512H_/debug/Source/winc3400_142/driver/source/m2m_ssl.o
 .debug_loc     0x00002563     0x2ab6 build/ChaletDuinoV2_795F512H_/debug/Source/winc3400_142/driver/source/m2m_wifi.o
 .debug_loc     0x00005019     0x108c build/ChaletDuinoV2_795F512H_/debug/Source/winc3400_142/driver/source/nmasic.o
 .debug_loc     0x000060a5      0x667 build/ChaletDuinoV2_795F512H_/debug/Source/winc3400_142/driver/source/nmbus.o
 .debug_loc     0x0000670c      0x633 build/ChaletDuinoV2_795F512H_/debug/Source/winc3400_142/driver/source/nmdrv.o
 .debug_loc     0x00006d3f      0xf4b build/ChaletDuinoV2_795F512H_/debug/Source/winc3400_142/driver/source/nmspi.o
 .debug_loc     0x00007c8a      0x1c9 build/ChaletDuinoV2_795F512H_/debug/Source/winc3400_142/socket/source/inet_addr.o
 .debug_loc     0x00007e53      0x1eb build/ChaletDuinoV2_795F512H_/debug/Source/winc3400_142/socket/source/inet_ntop.o
 .debug_loc     0x0000803e     0x16c9 build/ChaletDuinoV2_795F512H_/debug/Source/winc3400_142/socket/source/socket.o
 .debug_loc     0x00009707      0xe22 build/ChaletDuinoV2_795F512H_/debug/Source/winc3400_142/spi_flash/source/spi_flash.o
 .debug_loc     0x0000a529       0x2c build/ChaletDuinoV2_795F512H_/debug/Source/DigitalIO.o
 .debug_loc     0x0000a555      0x432 build/ChaletDuinoV2_795F512H_/debug/Source/NetworkProtocol.o
 .debug_loc     0x0000a987      0x25f build/ChaletDuinoV2_795F512H_/debug/Source/Terminal.o
 .debug_loc     0x0000abe6      0x6a1 build/ChaletDuinoV2_795F512H_/debug/Source/Util.o
 .debug_loc     0x0000b287       0x4b build/ChaletDuinoV2_795F512H_/debug/Source/exceptions.o
 .debug_loc     0x0000b2d2      0x349 build/ChaletDuinoV2_795F512H_/debug/Source/main.o
 .debug_loc     0x0000b61b      0x484 build/ChaletDuinoV2_795F512H_/debug/Source/timer.o
 .debug_loc     0x0000ba9f      0xb6f build/ChaletDuinoV2_795F512H_/debug/Source/WiFiCtrl.o
 .debug_loc     0x0000c60e       0x56 build/ChaletDuinoV2_795F512H_/debug/Source/SPI.o
 .debug_loc     0x0000c664      0x8d1 build/ChaletDuinoV2_795F512H_/debug/Source/SPI_Flash.o
 .debug_loc     0x0000cf35      0x1bb build/ChaletDuinoV2_795F512H_/debug/Source/Syslog.o
 .debug_loc     0x0000d0f0       0xb0 build/ChaletDuinoV2_795F512H_/debug/Source/Watchdog.o
 .debug_loc     0x0000d1a0      0x8d5 build/ChaletDuinoV2_795F512H_/debug/Source/BootloaderInterface.o
 .debug_loc     0x0000da75      0x9c9 build/ChaletDuinoV2_795F512H_/debug/Source/BootloaderProtocol.o
 .debug_loc     0x0000e43e      0x2d1 build/ChaletDuinoV2_795F512H_/debug/Source/crc32.o
 .debug_loc     0x0000e70f       0xb4 build/ChaletDuinoV2_795F512H_/debug/Source/VolumeTransducer.o
 .debug_loc     0x0000e7c3      0x1c5 build/ChaletDuinoV2_795F512H_/debug/Source/DACInterface.o
 .debug_loc     0x0000e988      0x9c3 c:/program files/microchip/xc32/v1.33/bin/bin/../../lib/gcc/pic32mx/4.5.2\libgcc.a(_udivdi3.o)
 .debug_loc     0x0000f34b      0x995 c:/program files/microchip/xc32/v1.33/bin/bin/../../lib/gcc/pic32mx/4.5.2\libgcc.a(_umoddi3.o)

.debug_macinfo
 *(.debug_macinfo)

.debug_weaknames
 *(.debug_weaknames)

.debug_funcnames
 *(.debug_funcnames)

.debug_typenames
 *(.debug_typenames)

.debug_varnames
 *(.debug_varnames)

.debug_pubtypes
                0x00000000     0x38de
 *(.debug_pubtypes)
 .debug_pubtypes
                0x00000000      0x229 build/ChaletDuinoV2_795F512H_/debug/Source/ChaletduinoV2Board.o
 .debug_pubtypes
                0x00000229      0x133 build/ChaletDuinoV2_795F512H_/debug/Source/winc3400_142/common/source/nm_common.o
 .debug_pubtypes
                0x0000035c      0x164 build/ChaletDuinoV2_795F512H_/debug/Source/winc3400_142/driver/source/m2m_flash.o
 .debug_pubtypes
                0x000004c0      0x155 build/ChaletDuinoV2_795F512H_/debug/Source/winc3400_142/driver/source/m2m_hif.o
 .debug_pubtypes
                0x00000615      0x15e build/ChaletDuinoV2_795F512H_/debug/Source/winc3400_142/driver/source/m2m_ota.o
 .debug_pubtypes
                0x00000773      0x128 build/ChaletDuinoV2_795F512H_/debug/Source/winc3400_142/driver/source/m2m_periph.o
 .debug_pubtypes
                0x0000089b      0x216 build/ChaletDuinoV2_795F512H_/debug/Source/winc3400_142/driver/source/m2m_ssl.o
 .debug_pubtypes
                0x00000ab1      0x756 build/ChaletDuinoV2_795F512H_/debug/Source/winc3400_142/driver/source/m2m_wifi.o
 .debug_pubtypes
                0x00001207      0x120 build/ChaletDuinoV2_795F512H_/debug/Source/winc3400_142/driver/source/nmasic.o
 .debug_pubtypes
                0x00001327      0x13a build/ChaletDuinoV2_795F512H_/debug/Source/winc3400_142/driver/source/nmbus.o
 .debug_pubtypes
                0x00001461      0x14e build/ChaletDuinoV2_795F512H_/debug/Source/winc3400_142/driver/source/nmdrv.o
 .debug_pubtypes
                0x000015af      0x13f build/ChaletDuinoV2_795F512H_/debug/Source/winc3400_142/driver/source/nmspi.o
 .debug_pubtypes
                0x000016ee      0x113 build/ChaletDuinoV2_795F512H_/debug/Source/winc3400_142/socket/source/inet_addr.o
 .debug_pubtypes
                0x00001801      0x11b build/ChaletDuinoV2_795F512H_/debug/Source/winc3400_142/socket/source/inet_ntop.o
 .debug_pubtypes
                0x0000191c      0x3c3 build/ChaletDuinoV2_795F512H_/debug/Source/winc3400_142/socket/source/socket.o
 .debug_pubtypes
                0x00001cdf      0x120 build/ChaletDuinoV2_795F512H_/debug/Source/winc3400_142/spi_flash/source/spi_flash.o
 .debug_pubtypes
                0x00001dff       0xe7 build/ChaletDuinoV2_795F512H_/debug/Source/DigitalIO.o
 .debug_pubtypes
                0x00001ee6      0x15b build/ChaletDuinoV2_795F512H_/debug/Source/NetworkProtocol.o
 .debug_pubtypes
                0x00002041      0x1a3 build/ChaletDuinoV2_795F512H_/debug/Source/Terminal.o
 .debug_pubtypes
                0x000021e4       0xe7 build/ChaletDuinoV2_795F512H_/debug/Source/Util.o
 .debug_pubtypes
                0x000022cb       0xe7 build/ChaletDuinoV2_795F512H_/debug/Source/exceptions.o
 .debug_pubtypes
                0x000023b2       0xe7 build/ChaletDuinoV2_795F512H_/debug/Source/interrupts.o
 .debug_pubtypes
                0x00002499      0x1dd build/ChaletDuinoV2_795F512H_/debug/Source/main.o
 .debug_pubtypes
                0x00002676       0xe7 build/ChaletDuinoV2_795F512H_/debug/Source/system.o
 .debug_pubtypes
                0x0000275d       0xe7 build/ChaletDuinoV2_795F512H_/debug/Source/template.o
 .debug_pubtypes
                0x00002844      0x145 build/ChaletDuinoV2_795F512H_/debug/Source/timer.o
 .debug_pubtypes
                0x00002989      0x2f4 build/ChaletDuinoV2_795F512H_/debug/Source/WiFiCtrl.o
 .debug_pubtypes
                0x00002c7d       0xfc build/ChaletDuinoV2_795F512H_/debug/Source/SPI.o
 .debug_pubtypes
                0x00002d79       0xf8 build/ChaletDuinoV2_795F512H_/debug/Source/SPI_Flash.o
 .debug_pubtypes
                0x00002e71      0x139 build/ChaletDuinoV2_795F512H_/debug/Source/Syslog.o
 .debug_pubtypes
                0x00002faa       0xf8 build/ChaletDuinoV2_795F512H_/debug/Source/Watchdog.o
 .debug_pubtypes
                0x000030a2      0x344 build/ChaletDuinoV2_795F512H_/debug/Source/BootloaderInterface.o
 .debug_pubtypes
                0x000033e6      0x183 build/ChaletDuinoV2_795F512H_/debug/Source/BootloaderProtocol.o
 .debug_pubtypes
                0x00003569       0x2c build/ChaletDuinoV2_795F512H_/debug/Source/crc32.o
 .debug_pubtypes
                0x00003595      0x150 build/ChaletDuinoV2_795F512H_/debug/Source/VolumeTransducer.o
 .debug_pubtypes
                0x000036e5      0x147 build/ChaletDuinoV2_795F512H_/debug/Source/DACInterface.o
 .debug_pubtypes
                0x0000382c       0x59 c:/program files/microchip/xc32/v1.33/bin/bin/../../lib/gcc/pic32mx/4.5.2\libgcc.a(_udivdi3.o)
 .debug_pubtypes
                0x00003885       0x59 c:/program files/microchip/xc32/v1.33/bin/bin/../../lib/gcc/pic32mx/4.5.2\libgcc.a(_umoddi3.o)

.debug_ranges   0x00000000      0x208
 *(.debug_ranges)
 .debug_ranges  0x00000000       0x10 c:/program files/microchip/xc32/v1.33/bin/bin/../../lib/gcc/pic32mx/4.5.2/../../../../pic32mx/lib\software-debug-break.o
 .debug_ranges  0x00000010       0x10 c:/program files/microchip/xc32/v1.33/bin/bin/../../lib/gcc/pic32mx/4.5.2/../../../../pic32mx/lib\libpic32.a(default-bootstrap-exception-handler.o)
 .debug_ranges  0x00000020       0x10 c:/program files/microchip/xc32/v1.33/bin/bin/../../lib/gcc/pic32mx/4.5.2/../../../../pic32mx/lib\libpic32.a(default-on-reset.o)
 .debug_ranges  0x00000030       0x10 c:/program files/microchip/xc32/v1.33/bin/bin/../../lib/gcc/pic32mx/4.5.2/../../../../pic32mx/lib\libpic32.a(default-on-bootstrap.o)
 .debug_ranges  0x00000040       0x10 c:/program files/microchip/xc32/v1.33/bin/bin/../../lib/gcc/pic32mx/4.5.2/../../../../pic32mx/lib\libpic32.a(close.o)
 .debug_ranges  0x00000050       0x10 c:/program files/microchip/xc32/v1.33/bin/bin/../../lib/gcc/pic32mx/4.5.2/../../../../pic32mx/lib\libpic32.a(defaultinterrupt.o)
 .debug_ranges  0x00000060       0x18 c:/program files/microchip/xc32/v1.33/bin/bin/../../lib/gcc/pic32mx/4.5.2/../../../../pic32mx/lib\libc.a(puts.o)
 .debug_ranges  0x00000078       0x10 c:/program files/microchip/xc32/v1.33/bin/bin/../../lib/gcc/pic32mx/4.5.2/../../../../pic32mx/lib\libc.a(strncmp.o)
 .debug_ranges  0x00000088       0x10 c:/program files/microchip/xc32/v1.33/bin/bin/../../lib/gcc/pic32mx/4.5.2/../../../../pic32mx/lib\libc.a(printf_cdnopsuxX.eo)
 .debug_ranges  0x00000098       0x10 c:/program files/microchip/xc32/v1.33/bin/bin/../../lib/gcc/pic32mx/4.5.2/../../../../pic32mx/lib\libc.a(sprintf_cdnopuxX.eo)
 .debug_ranges  0x000000a8       0x10 c:/program files/microchip/xc32/v1.33/bin/bin/../../lib/gcc/pic32mx/4.5.2/../../../../pic32mx/lib\libc.a(sscanf_s.eo)
 .debug_ranges  0x000000b8       0x10 c:/program files/microchip/xc32/v1.33/bin/bin/../../lib/gcc/pic32mx/4.5.2/../../../../pic32mx/lib\libc.a(_fputc_simple.o)
 .debug_ranges  0x000000c8       0x10 c:/program files/microchip/xc32/v1.33/bin/bin/../../lib/gcc/pic32mx/4.5.2/../../../../pic32mx/lib\libc.a(doprnt_cdnopsuxX.eo)
 .debug_ranges  0x000000d8       0x20 c:/program files/microchip/xc32/v1.33/bin/bin/../../lib/gcc/pic32mx/4.5.2/../../../../pic32mx/lib\libc.a(doscan_s.eo)
 .debug_ranges  0x000000f8       0x10 c:/program files/microchip/xc32/v1.33/bin/bin/../../lib/gcc/pic32mx/4.5.2/../../../../pic32mx/lib\libc.a(_flsbuf_simple.o)
 .debug_ranges  0x00000108       0x10 c:/program files/microchip/xc32/v1.33/bin/bin/../../lib/gcc/pic32mx/4.5.2/../../../../pic32mx/lib\libc.a(fgetc.o)
 .debug_ranges  0x00000118       0x10 c:/program files/microchip/xc32/v1.33/bin/bin/../../lib/gcc/pic32mx/4.5.2/../../../../pic32mx/lib\libc.a(atoi.o)
 .debug_ranges  0x00000128       0x90 c:/program files/microchip/xc32/v1.33/bin/bin/../../lib/gcc/pic32mx/4.5.2/../../../../pic32mx/lib\libc.a(ctypef.o)
 .debug_ranges  0x000001b8       0x10 c:/program files/microchip/xc32/v1.33/bin/bin/../../lib/gcc/pic32mx/4.5.2/../../../../pic32mx/lib\libc.a(ungetc.o)
 .debug_ranges  0x000001c8       0x10 c:/program files/microchip/xc32/v1.33/bin/bin/../../lib/gcc/pic32mx/4.5.2/../../../../pic32mx/lib\libc.a(filbuf.o)
 .debug_ranges  0x000001d8       0x10 c:/program files/microchip/xc32/v1.33/bin/bin/../../lib/gcc/pic32mx/4.5.2/../../../../pic32mx/lib\libc.a(fflush.o)
 .debug_ranges  0x000001e8       0x10 c:/program files/microchip/xc32/v1.33/bin/bin/../../lib/gcc/pic32mx/4.5.2/../../../../pic32mx/lib\libpic32.a(read.o)
 .debug_ranges  0x000001f8       0x10 c:/program files/microchip/xc32/v1.33/bin/bin/../../lib/gcc/pic32mx/4.5.2/../../../../pic32mx/lib\libpic32.a(write.o)

.gnu.attributes
                0x00000000       0x10
 *(.gnu.attributes)
 .gnu.attributes
                0x00000000       0x10 c:/program files/microchip/xc32/v1.33/bin/bin/../../lib/gcc/pic32mx/4.5.2/../../../../pic32mx/lib\software-debug-break.o
 .gnu.attributes
                0x00000010       0x10 build/ChaletDuinoV2_795F512H_/debug/Source/ChaletduinoV2Board.o
 .gnu.attributes
                0x00000020       0x10 build/ChaletDuinoV2_795F512H_/debug/Source/winc3400_142/common/source/nm_common.o
 .gnu.attributes
                0x00000030       0x10 build/ChaletDuinoV2_795F512H_/debug/Source/winc3400_142/driver/source/m2m_flash.o
 .gnu.attributes
                0x00000040       0x10 build/ChaletDuinoV2_795F512H_/debug/Source/winc3400_142/driver/source/m2m_hif.o
 .gnu.attributes
                0x00000050       0x10 build/ChaletDuinoV2_795F512H_/debug/Source/winc3400_142/driver/source/m2m_ota.o
 .gnu.attributes
                0x00000060       0x10 build/ChaletDuinoV2_795F512H_/debug/Source/winc3400_142/driver/source/m2m_periph.o
 .gnu.attributes
                0x00000070       0x10 build/ChaletDuinoV2_795F512H_/debug/Source/winc3400_142/driver/source/m2m_ssl.o
 .gnu.attributes
                0x00000080       0x10 build/ChaletDuinoV2_795F512H_/debug/Source/winc3400_142/driver/source/m2m_wifi.o
 .gnu.attributes
                0x00000090       0x10 build/ChaletDuinoV2_795F512H_/debug/Source/winc3400_142/driver/source/nmasic.o
 .gnu.attributes
                0x000000a0       0x10 build/ChaletDuinoV2_795F512H_/debug/Source/winc3400_142/driver/source/nmbus.o
 .gnu.attributes
                0x000000b0       0x10 build/ChaletDuinoV2_795F512H_/debug/Source/winc3400_142/driver/source/nmdrv.o
 .gnu.attributes
                0x000000c0       0x10 build/ChaletDuinoV2_795F512H_/debug/Source/winc3400_142/driver/source/nmspi.o
 .gnu.attributes
                0x000000d0       0x10 build/ChaletDuinoV2_795F512H_/debug/Source/winc3400_142/socket/source/inet_addr.o
 .gnu.attributes
                0x000000e0       0x10 build/ChaletDuinoV2_795F512H_/debug/Source/winc3400_142/socket/source/inet_ntop.o
 .gnu.attributes
                0x000000f0       0x10 build/ChaletDuinoV2_795F512H_/debug/Source/winc3400_142/socket/source/socket.o
 .gnu.attributes
                0x00000100       0x10 build/ChaletDuinoV2_795F512H_/debug/Source/winc3400_142/spi_flash/source/spi_flash.o
 .gnu.attributes
                0x00000110       0x10 build/ChaletDuinoV2_795F512H_/debug/Source/DigitalIO.o
 .gnu.attributes
                0x00000120       0x10 build/ChaletDuinoV2_795F512H_/debug/Source/NetworkProtocol.o
 .gnu.attributes
                0x00000130       0x10 build/ChaletDuinoV2_795F512H_/debug/Source/Terminal.o
 .gnu.attributes
                0x00000140       0x10 build/ChaletDuinoV2_795F512H_/debug/Source/Util.o
 .gnu.attributes
                0x00000150       0x10 build/ChaletDuinoV2_795F512H_/debug/Source/exceptions.o
 .gnu.attributes
                0x00000160       0x10 build/ChaletDuinoV2_795F512H_/debug/Source/interrupts.o
 .gnu.attributes
                0x00000170       0x10 build/ChaletDuinoV2_795F512H_/debug/Source/main.o
 .gnu.attributes
                0x00000180       0x10 build/ChaletDuinoV2_795F512H_/debug/Source/system.o
 .gnu.attributes
                0x00000190       0x10 build/ChaletDuinoV2_795F512H_/debug/Source/template.o
 .gnu.attributes
                0x000001a0       0x10 build/ChaletDuinoV2_795F512H_/debug/Source/timer.o
 .gnu.attributes
                0x000001b0       0x10 build/ChaletDuinoV2_795F512H_/debug/Source/WiFiCtrl.o
 .gnu.attributes
                0x000001c0       0x10 build/ChaletDuinoV2_795F512H_/debug/Source/SPI.o
 .gnu.attributes
                0x000001d0       0x10 build/ChaletDuinoV2_795F512H_/debug/Source/SPI_Flash.o
 .gnu.attributes
                0x000001e0       0x10 build/ChaletDuinoV2_795F512H_/debug/Source/Syslog.o
 .gnu.attributes
                0x000001f0       0x10 build/ChaletDuinoV2_795F512H_/debug/Source/Watchdog.o
 .gnu.attributes
                0x00000200       0x10 build/ChaletDuinoV2_795F512H_/debug/Source/BootloaderInterface.o
 .gnu.attributes
                0x00000210       0x10 build/ChaletDuinoV2_795F512H_/debug/Source/BootloaderProtocol.o
 .gnu.attributes
                0x00000220       0x10 build/ChaletDuinoV2_795F512H_/debug/Source/crc32.o
 .gnu.attributes
                0x00000230       0x10 build/ChaletDuinoV2_795F512H_/debug/Source/VolumeTransducer.o
 .gnu.attributes
                0x00000240       0x10 build/ChaletDuinoV2_795F512H_/debug/Source/DACInterface.o
 .gnu.attributes
                0x00000250       0x10 c:/program files/microchip/xc32/v1.33/bin/bin/../../lib/gcc/pic32mx/4.5.2/../../../../pic32mx/lib\libmchp_peripheral_32MX795F512H.a(soft_reset_lib.o)
 .gnu.attributes
                0x00000260       0x10 c:/program files/microchip/xc32/v1.33/bin/bin/../../lib/gcc/pic32mx/4.5.2/../../../../pic32mx/lib\libmchp_peripheral_32MX795F512H.a(pcache.o)
 .gnu.attributes
                0x00000270       0x10 c:/program files/microchip/xc32/v1.33/bin/bin/../../lib/gcc/pic32mx/4.5.2/../../../../pic32mx/lib\libmchp_peripheral_32MX795F512H.a(int_configure_system_lib.o)
 .gnu.attributes
                0x00000280       0x10 c:/program files/microchip/xc32/v1.33/bin/bin/../../lib/gcc/pic32mx/4.5.2/../../../../pic32mx/lib\libmchp_peripheral_32MX795F512H.a(int_enable_interrupts_lib.o)
 .gnu.attributes
                0x00000290       0x10 c:/program files/microchip/xc32/v1.33/bin/bin/../../lib/gcc/pic32mx/4.5.2/../../../../pic32mx/lib\libmchp_peripheral_32MX795F512H.a(int_disable_interrupts_lib.o)
 .gnu.attributes
                0x000002a0       0x10 c:/program files/microchip/xc32/v1.33/bin/bin/../../lib/gcc/pic32mx/4.5.2/../../../../pic32mx/lib\libmchp_peripheral_32MX795F512H.a(int_restore_interrupts_lib.o)
 .gnu.attributes
                0x000002b0       0x10 c:/program files/microchip/xc32/v1.33/bin/bin/../../lib/gcc/pic32mx/4.5.2/../../../../pic32mx/lib\libpic32.a(default-bootstrap-exception-handler.o)
 .gnu.attributes
                0x000002c0       0x10 c:/program files/microchip/xc32/v1.33/bin/bin/../../lib/gcc/pic32mx/4.5.2/../../../../pic32mx/lib\libpic32.a(default-on-reset.o)
 .gnu.attributes
                0x000002d0       0x10 c:/program files/microchip/xc32/v1.33/bin/bin/../../lib/gcc/pic32mx/4.5.2/../../../../pic32mx/lib\libpic32.a(default-on-bootstrap.o)
 .gnu.attributes
                0x000002e0       0x10 c:/program files/microchip/xc32/v1.33/bin/bin/../../lib/gcc/pic32mx/4.5.2/../../../../pic32mx/lib\libpic32.a(close.o)
 .gnu.attributes
                0x000002f0       0x10 c:/program files/microchip/xc32/v1.33/bin/bin/../../lib/gcc/pic32mx/4.5.2/../../../../pic32mx/lib\libpic32.a(defaultinterrupt.o)
 .gnu.attributes
                0x00000300       0x10 c:/program files/microchip/xc32/v1.33/bin/bin/../../lib/gcc/pic32mx/4.5.2/../../../../pic32mx/lib\libc.a(puts.o)
 .gnu.attributes
                0x00000310       0x10 c:/program files/microchip/xc32/v1.33/bin/bin/../../lib/gcc/pic32mx/4.5.2/../../../../pic32mx/lib\libc.a(strncmp.o)
 .gnu.attributes
                0x00000320       0x10 c:/program files/microchip/xc32/v1.33/bin/bin/../../lib/gcc/pic32mx/4.5.2/../../../../pic32mx/lib\libc.a(printf_cdnopsuxX.eo)
 .gnu.attributes
                0x00000330       0x10 c:/program files/microchip/xc32/v1.33/bin/bin/../../lib/gcc/pic32mx/4.5.2/../../../../pic32mx/lib\libc.a(sprintf_cdnopuxX.eo)
 .gnu.attributes
                0x00000340       0x10 c:/program files/microchip/xc32/v1.33/bin/bin/../../lib/gcc/pic32mx/4.5.2/../../../../pic32mx/lib\libc.a(sscanf_s.eo)
 .gnu.attributes
                0x00000350       0x10 c:/program files/microchip/xc32/v1.33/bin/bin/../../lib/gcc/pic32mx/4.5.2/../../../../pic32mx/lib\libc.a(_iob.o)
 .gnu.attributes
                0x00000360       0x10 c:/program files/microchip/xc32/v1.33/bin/bin/../../lib/gcc/pic32mx/4.5.2/../../../../pic32mx/lib\libc.a(_fputc_simple.o)
 .gnu.attributes
                0x00000370       0x10 c:/program files/microchip/xc32/v1.33/bin/bin/../../lib/gcc/pic32mx/4.5.2/../../../../pic32mx/lib\libc.a(doprnt_cdnopsuxX.eo)
 .gnu.attributes
                0x00000380       0x10 c:/program files/microchip/xc32/v1.33/bin/bin/../../lib/gcc/pic32mx/4.5.2/../../../../pic32mx/lib\libc.a(doscan_s.eo)
 .gnu.attributes
                0x00000390       0x10 c:/program files/microchip/xc32/v1.33/bin/bin/../../lib/gcc/pic32mx/4.5.2/../../../../pic32mx/lib\libc.a(_flsbuf_simple.o)
 .gnu.attributes
                0x000003a0       0x10 c:/program files/microchip/xc32/v1.33/bin/bin/../../lib/gcc/pic32mx/4.5.2/../../../../pic32mx/lib\libc.a(fgetc.o)
 .gnu.attributes
                0x000003b0       0x10 c:/program files/microchip/xc32/v1.33/bin/bin/../../lib/gcc/pic32mx/4.5.2/../../../../pic32mx/lib\libc.a(atoi.o)
 .gnu.attributes
                0x000003c0       0x10 c:/program files/microchip/xc32/v1.33/bin/bin/../../lib/gcc/pic32mx/4.5.2/../../../../pic32mx/lib\libc.a(ctype.o)
 .gnu.attributes
                0x000003d0       0x10 c:/program files/microchip/xc32/v1.33/bin/bin/../../lib/gcc/pic32mx/4.5.2/../../../../pic32mx/lib\libc.a(ctypef.o)
 .gnu.attributes
                0x000003e0       0x10 c:/program files/microchip/xc32/v1.33/bin/bin/../../lib/gcc/pic32mx/4.5.2/../../../../pic32mx/lib\libc.a(ungetc.o)
 .gnu.attributes
                0x000003f0       0x10 c:/program files/microchip/xc32/v1.33/bin/bin/../../lib/gcc/pic32mx/4.5.2/../../../../pic32mx/lib\libc.a(filbuf.o)
 .gnu.attributes
                0x00000400       0x10 c:/program files/microchip/xc32/v1.33/bin/bin/../../lib/gcc/pic32mx/4.5.2/../../../../pic32mx/lib\libc.a(fflush.o)
 .gnu.attributes
                0x00000410       0x10 c:/program files/microchip/xc32/v1.33/bin/bin/../../lib/gcc/pic32mx/4.5.2/../../../../pic32mx/lib\libpic32.a(read.o)
 .gnu.attributes
                0x00000420       0x10 c:/program files/microchip/xc32/v1.33/bin/bin/../../lib/gcc/pic32mx/4.5.2/../../../../pic32mx/lib\libpic32.a(write.o)
 .gnu.attributes
                0x00000430       0x10 c:/program files/microchip/xc32/v1.33/bin/bin/../../lib/gcc/pic32mx/4.5.2/../../../../pic32mx/lib\libpic32.a(xc32_uart.o)
 .gnu.attributes
                0x00000440       0x10 c:/program files/microchip/xc32/v1.33/bin/bin/../../lib/gcc/pic32mx/4.5.2\libgcc.a(_udivdi3.o)
 .gnu.attributes
                0x00000450       0x10 c:/program files/microchip/xc32/v1.33/bin/bin/../../lib/gcc/pic32mx/4.5.2\libgcc.a(_umoddi3.o)
                0x00000001                __MPLAB_DEBUG = 0x1
                0x00000001                __DEBUG = 0x1
                0x00000001                __MPLAB_DEBUGGER_ICD3 = 0x1
                0x00000080                _min_heap_size = 0x80
LOAD c:/program files/microchip/xc32/v1.33/bin/bin/../../lib/gcc/pic32mx/4.5.2/../../../../pic32mx/lib/./proc/32MX795F512H\default_isr_vectors.o
LOAD c:/program files/microchip/xc32/v1.33/bin/bin/../../lib/gcc/pic32mx/4.5.2/../../../../pic32mx/lib\pic32_software_reset.o
LOAD c:/program files/microchip/xc32/v1.33/bin/bin/../../lib/gcc/pic32mx/4.5.2\libgcc.a
START GROUP
LOAD c:/program files/microchip/xc32/v1.33/bin/bin/../../lib/gcc/pic32mx/4.5.2/../../../../pic32mx/lib\libpic32.a
LOAD c:/program files/microchip/xc32/v1.33/bin/bin/../../lib/gcc/pic32mx/4.5.2/../../../../pic32mx/lib\libdebug.a
LOAD c:/program files/microchip/xc32/v1.33/bin/bin/../../lib/gcc/pic32mx/4.5.2/../../../../pic32mx/lib\libpic32.a
LOAD c:/program files/microchip/xc32/v1.33/bin/bin/../../lib/gcc/pic32mx/4.5.2/../../../../pic32mx/lib\libm.a
LOAD c:/program files/microchip/xc32/v1.33/bin/bin/../../lib/gcc/pic32mx/4.5.2/../../../../pic32mx/lib\libe.a
LOAD c:/program files/microchip/xc32/v1.33/bin/bin/../../lib/gcc/pic32mx/4.5.2/../../../../pic32mx/lib\libdsp.a
LOAD c:/program files/microchip/xc32/v1.33/bin/bin/../../lib/gcc/pic32mx/4.5.2\libgcc.a
LOAD c:/program files/microchip/xc32/v1.33/bin/bin/../../lib/gcc/pic32mx/4.5.2/../../../../pic32mx/lib\libc.a
LOAD c:/program files/microchip/xc32/v1.33/bin/bin/../../lib/gcc/pic32mx/4.5.2/../../../../pic32mx/lib\libpic32.a
END GROUP
LOAD c:/program files/microchip/xc32/v1.33/bin/bin/../../lib/gcc/pic32mx/4.5.2\libgcc.a
OUTPUT(dist/ChaletDuinoV2_795F512H_/debug/AudioConsole.X.debug.elf elf32-tradlittlemips)
LOAD stack
LOAD data_init

.reginfo        0x00000000       0x18
 .reginfo       0x00000000       0x18 c:/program files/microchip/xc32/v1.33/bin/bin/../../lib/gcc/pic32mx/4.5.2/../../../../pic32mx/lib/./proc/32MX795F512H/crt0_mips32r2.o

.stack          0xa0004360      0x400
 .stack         0xa0004360      0x400 stack

.data           0xa000303c      0x7a8
 .data          0xa000303c      0x7a8 build/ChaletDuinoV2_795F512H_/debug/Source/Terminal.o

.bss            0xa00037e4      0x800
 .bss           0xa00037e4      0x400 build/ChaletDuinoV2_795F512H_/debug/Source/WiFiCtrl.o
 .bss           0xa0003be4      0x400 build/ChaletDuinoV2_795F512H_/debug/Source/crc32.o

.data           0xa0003fe4      0x26c
 .data          0xa0003fe4       0xa0 c:/program files/microchip/xc32/v1.33/bin/bin/../../lib/gcc/pic32mx/4.5.2/../../../../pic32mx/lib\libc.a(_iob.o)
                0xa0003fe4                _iob
 .data          0xa0004084       0x6c build/ChaletDuinoV2_795F512H_/debug/Source/WiFiCtrl.o
 .data          0xa00040f0       0x58 build/ChaletDuinoV2_795F512H_/debug/Source/main.o
 .data          0xa0004148       0x58 build/ChaletDuinoV2_795F512H_/debug/Source/Syslog.o
 .data          0xa00041a0       0x58 build/ChaletDuinoV2_795F512H_/debug/Source/BootloaderInterface.o
 .data          0xa00041f8       0x58 build/ChaletDuinoV2_795F512H_/debug/Source/BootloaderProtocol.o

.bss            0xa0004250       0x40
 .bss           0xa0004250       0x40 c:/program files/microchip/xc32/v1.33/bin/bin/../../lib/gcc/pic32mx/4.5.2/../../../../pic32mx/lib\libc.a(_iob.o)
                0xa0004250                _sibuf
                0xa0004270                _sobuf

.data           0xa0004290       0x1c
 .data          0xa0004290       0x1c build/ChaletDuinoV2_795F512H_/debug/Source/winc3400_142/driver/source/m2m_hif.o

.bss            0xa00042ac       0x18
 .bss           0xa00042ac       0x14 build/ChaletDuinoV2_795F512H_/debug/Source/winc3400_142/driver/source/m2m_wifi.o
 .bss           0xa00042c0        0x4 c:/program files/microchip/xc32/v1.33/bin/bin/../../lib/gcc/pic32mx/4.5.2/../../../../pic32mx/lib\libc.a(doscan_s.eo)

.bss%z1         0x00000000        0x0
 .bss           0x00000000        0x0 c:/program files/microchip/xc32/v1.33/bin/bin/../../lib/gcc/pic32mx/4.5.2\libgcc.a(_umoddi3.o)

.data%z2        0x00000000        0x0
 .data          0x00000000        0x0 c:/program files/microchip/xc32/v1.33/bin/bin/../../lib/gcc/pic32mx/4.5.2\libgcc.a(_umoddi3.o)

.bss%z3         0x00000000        0x0
 .bss           0x00000000        0x0 c:/program files/microchip/xc32/v1.33/bin/bin/../../lib/gcc/pic32mx/4.5.2\libgcc.a(_udivdi3.o)

.data%z4        0x00000000        0x0
 .data          0x00000000        0x0 c:/program files/microchip/xc32/v1.33/bin/bin/../../lib/gcc/pic32mx/4.5.2\libgcc.a(_udivdi3.o)

.bss%z5         0x00000000        0x0
 .bss           0x00000000        0x0 c:/program files/microchip/xc32/v1.33/bin/bin/../../lib/gcc/pic32mx/4.5.2/../../../../pic32mx/lib\libpic32.a(xc32_uart.o)

.data%z6        0x00000000        0x0
 .data          0x00000000        0x0 c:/program files/microchip/xc32/v1.33/bin/bin/../../lib/gcc/pic32mx/4.5.2/../../../../pic32mx/lib\libpic32.a(xc32_uart.o)

.bss%z7         0x00000000        0x0
 .bss           0x00000000        0x0 c:/program files/microchip/xc32/v1.33/bin/bin/../../lib/gcc/pic32mx/4.5.2/../../../../pic32mx/lib\libpic32.a(write.o)

.data%z8        0x00000000        0x0
 .data          0x00000000        0x0 c:/program files/microchip/xc32/v1.33/bin/bin/../../lib/gcc/pic32mx/4.5.2/../../../../pic32mx/lib\libpic32.a(write.o)

.bss%z9         0x00000000        0x0
 .bss           0x00000000        0x0 c:/program files/microchip/xc32/v1.33/bin/bin/../../lib/gcc/pic32mx/4.5.2/../../../../pic32mx/lib\libpic32.a(read.o)

.data%z10       0x00000000        0x0
 .data          0x00000000        0x0 c:/program files/microchip/xc32/v1.33/bin/bin/../../lib/gcc/pic32mx/4.5.2/../../../../pic32mx/lib\libpic32.a(read.o)

.bss%z11        0x00000000        0x0
 .bss           0x00000000        0x0 c:/program files/microchip/xc32/v1.33/bin/bin/../../lib/gcc/pic32mx/4.5.2/../../../../pic32mx/lib\libc.a(fflush.o)

.data%z12       0x00000000        0x0
 .data          0x00000000        0x0 c:/program files/microchip/xc32/v1.33/bin/bin/../../lib/gcc/pic32mx/4.5.2/../../../../pic32mx/lib\libc.a(fflush.o)

.bss%z13        0x00000000        0x0
 .bss           0x00000000        0x0 c:/program files/microchip/xc32/v1.33/bin/bin/../../lib/gcc/pic32mx/4.5.2/../../../../pic32mx/lib\libc.a(filbuf.o)

.data%z14       0x00000000        0x0
 .data          0x00000000        0x0 c:/program files/microchip/xc32/v1.33/bin/bin/../../lib/gcc/pic32mx/4.5.2/../../../../pic32mx/lib\libc.a(filbuf.o)

.bss%z15        0x00000000        0x0
 .bss           0x00000000        0x0 c:/program files/microchip/xc32/v1.33/bin/bin/../../lib/gcc/pic32mx/4.5.2/../../../../pic32mx/lib\libc.a(ungetc.o)

.data%z16       0x00000000        0x0
 .data          0x00000000        0x0 c:/program files/microchip/xc32/v1.33/bin/bin/../../lib/gcc/pic32mx/4.5.2/../../../../pic32mx/lib\libc.a(ungetc.o)

.bss%z17        0x00000000        0x0
 .bss           0x00000000        0x0 c:/program files/microchip/xc32/v1.33/bin/bin/../../lib/gcc/pic32mx/4.5.2/../../../../pic32mx/lib\libc.a(ctypef.o)

.data%z18       0x00000000        0x0
 .data          0x00000000        0x0 c:/program files/microchip/xc32/v1.33/bin/bin/../../lib/gcc/pic32mx/4.5.2/../../../../pic32mx/lib\libc.a(ctypef.o)

.bss%z19        0x00000000        0x0
 .bss           0x00000000        0x0 c:/program files/microchip/xc32/v1.33/bin/bin/../../lib/gcc/pic32mx/4.5.2/../../../../pic32mx/lib\libc.a(ctype.o)

.data%z20       0x00000000        0x0
 .data          0x00000000        0x0 c:/program files/microchip/xc32/v1.33/bin/bin/../../lib/gcc/pic32mx/4.5.2/../../../../pic32mx/lib\libc.a(ctype.o)

.bss%z21        0x00000000        0x0
 .bss           0x00000000        0x0 c:/program files/microchip/xc32/v1.33/bin/bin/../../lib/gcc/pic32mx/4.5.2/../../../../pic32mx/lib\libc.a(atoi.o)

.data%z22       0x00000000        0x0
 .data          0x00000000        0x0 c:/program files/microchip/xc32/v1.33/bin/bin/../../lib/gcc/pic32mx/4.5.2/../../../../pic32mx/lib\libc.a(atoi.o)

.bss%z23        0x00000000        0x0
 .bss           0x00000000        0x0 c:/program files/microchip/xc32/v1.33/bin/bin/../../lib/gcc/pic32mx/4.5.2/../../../../pic32mx/lib\libc.a(fgetc.o)

.data%z24       0x00000000        0x0
 .data          0x00000000        0x0 c:/program files/microchip/xc32/v1.33/bin/bin/../../lib/gcc/pic32mx/4.5.2/../../../../pic32mx/lib\libc.a(fgetc.o)

.bss%z25        0x00000000        0x0
 .bss           0x00000000        0x0 c:/program files/microchip/xc32/v1.33/bin/bin/../../lib/gcc/pic32mx/4.5.2/../../../../pic32mx/lib\libc.a(_flsbuf_simple.o)

.data%z26       0x00000000        0x0
 .data          0x00000000        0x0 c:/program files/microchip/xc32/v1.33/bin/bin/../../lib/gcc/pic32mx/4.5.2/../../../../pic32mx/lib\libc.a(_flsbuf_simple.o)

.data%z27       0x00000000        0x0
 .data          0x00000000        0x0 c:/program files/microchip/xc32/v1.33/bin/bin/../../lib/gcc/pic32mx/4.5.2/../../../../pic32mx/lib\libc.a(doscan_s.eo)

.bss%z28        0x00000000        0x0
 .bss           0x00000000        0x0 c:/program files/microchip/xc32/v1.33/bin/bin/../../lib/gcc/pic32mx/4.5.2/../../../../pic32mx/lib\libc.a(doprnt_cdnopsuxX.eo)

.data%z29       0x00000000        0x0
 .data          0x00000000        0x0 c:/program files/microchip/xc32/v1.33/bin/bin/../../lib/gcc/pic32mx/4.5.2/../../../../pic32mx/lib\libc.a(doprnt_cdnopsuxX.eo)

.bss%z30        0x00000000        0x0
 .bss           0x00000000        0x0 c:/program files/microchip/xc32/v1.33/bin/bin/../../lib/gcc/pic32mx/4.5.2/../../../../pic32mx/lib\libc.a(_fputc_simple.o)

.data%z31       0x00000000        0x0
 .data          0x00000000        0x0 c:/program files/microchip/xc32/v1.33/bin/bin/../../lib/gcc/pic32mx/4.5.2/../../../../pic32mx/lib\libc.a(_fputc_simple.o)

.bss%z32        0x00000000        0x0
 .bss           0x00000000        0x0 c:/program files/microchip/xc32/v1.33/bin/bin/../../lib/gcc/pic32mx/4.5.2/../../../../pic32mx/lib\libc.a(sscanf_s.eo)

.data%z33       0x00000000        0x0
 .data          0x00000000        0x0 c:/program files/microchip/xc32/v1.33/bin/bin/../../lib/gcc/pic32mx/4.5.2/../../../../pic32mx/lib\libc.a(sscanf_s.eo)

.bss%z34        0x00000000        0x0
 .bss           0x00000000        0x0 c:/program files/microchip/xc32/v1.33/bin/bin/../../lib/gcc/pic32mx/4.5.2/../../../../pic32mx/lib\libc.a(sprintf_cdnopuxX.eo)

.data%z35       0x00000000        0x0
 .data          0x00000000        0x0 c:/program files/microchip/xc32/v1.33/bin/bin/../../lib/gcc/pic32mx/4.5.2/../../../../pic32mx/lib\libc.a(sprintf_cdnopuxX.eo)

.bss%z36        0x00000000        0x0
 .bss           0x00000000        0x0 c:/program files/microchip/xc32/v1.33/bin/bin/../../lib/gcc/pic32mx/4.5.2/../../../../pic32mx/lib\libc.a(printf_cdnopsuxX.eo)

.data%z37       0x00000000        0x0
 .data          0x00000000        0x0 c:/program files/microchip/xc32/v1.33/bin/bin/../../lib/gcc/pic32mx/4.5.2/../../../../pic32mx/lib\libc.a(printf_cdnopsuxX.eo)

.bss%z38        0x00000000        0x0
 .bss           0x00000000        0x0 c:/program files/microchip/xc32/v1.33/bin/bin/../../lib/gcc/pic32mx/4.5.2/../../../../pic32mx/lib\libc.a(strncmp.o)

.data%z39       0x00000000        0x0
 .data          0x00000000        0x0 c:/program files/microchip/xc32/v1.33/bin/bin/../../lib/gcc/pic32mx/4.5.2/../../../../pic32mx/lib\libc.a(strncmp.o)

.bss%z40        0x00000000        0x0
 .bss           0x00000000        0x0 c:/program files/microchip/xc32/v1.33/bin/bin/../../lib/gcc/pic32mx/4.5.2/../../../../pic32mx/lib\libc.a(puts.o)

.data%z41       0x00000000        0x0
 .data          0x00000000        0x0 c:/program files/microchip/xc32/v1.33/bin/bin/../../lib/gcc/pic32mx/4.5.2/../../../../pic32mx/lib\libc.a(puts.o)

.bss%z42        0x00000000        0x0
 .bss           0x00000000        0x0 c:/program files/microchip/xc32/v1.33/bin/bin/../../lib/gcc/pic32mx/4.5.2/../../../../pic32mx/lib\libpic32.a(defaultinterrupt.o)

.data%z43       0x00000000        0x0
 .data          0x00000000        0x0 c:/program files/microchip/xc32/v1.33/bin/bin/../../lib/gcc/pic32mx/4.5.2/../../../../pic32mx/lib\libpic32.a(defaultinterrupt.o)

.bss%z44        0x00000000        0x0
 .bss           0x00000000        0x0 c:/program files/microchip/xc32/v1.33/bin/bin/../../lib/gcc/pic32mx/4.5.2/../../../../pic32mx/lib\libpic32.a(vector63.o)

.data%z45       0x00000000        0x0
 .data          0x00000000        0x0 c:/program files/microchip/xc32/v1.33/bin/bin/../../lib/gcc/pic32mx/4.5.2/../../../../pic32mx/lib\libpic32.a(vector63.o)

.bss%z46        0x00000000        0x0
 .bss           0x00000000        0x0 c:/program files/microchip/xc32/v1.33/bin/bin/../../lib/gcc/pic32mx/4.5.2/../../../../pic32mx/lib\libpic32.a(vector62.o)

.data%z47       0x00000000        0x0
 .data          0x00000000        0x0 c:/program files/microchip/xc32/v1.33/bin/bin/../../lib/gcc/pic32mx/4.5.2/../../../../pic32mx/lib\libpic32.a(vector62.o)

.bss%z48        0x00000000        0x0
 .bss           0x00000000        0x0 c:/program files/microchip/xc32/v1.33/bin/bin/../../lib/gcc/pic32mx/4.5.2/../../../../pic32mx/lib\libpic32.a(vector61.o)

.data%z49       0x00000000        0x0
 .data          0x00000000        0x0 c:/program files/microchip/xc32/v1.33/bin/bin/../../lib/gcc/pic32mx/4.5.2/../../../../pic32mx/lib\libpic32.a(vector61.o)

.bss%z50        0x00000000        0x0
 .bss           0x00000000        0x0 c:/program files/microchip/xc32/v1.33/bin/bin/../../lib/gcc/pic32mx/4.5.2/../../../../pic32mx/lib\libpic32.a(vector60.o)

.data%z51       0x00000000        0x0
 .data          0x00000000        0x0 c:/program files/microchip/xc32/v1.33/bin/bin/../../lib/gcc/pic32mx/4.5.2/../../../../pic32mx/lib\libpic32.a(vector60.o)

.bss%z52        0x00000000        0x0
 .bss           0x00000000        0x0 c:/program files/microchip/xc32/v1.33/bin/bin/../../lib/gcc/pic32mx/4.5.2/../../../../pic32mx/lib\libpic32.a(vector59.o)

.data%z53       0x00000000        0x0
 .data          0x00000000        0x0 c:/program files/microchip/xc32/v1.33/bin/bin/../../lib/gcc/pic32mx/4.5.2/../../../../pic32mx/lib\libpic32.a(vector59.o)

.bss%z54        0x00000000        0x0
 .bss           0x00000000        0x0 c:/program files/microchip/xc32/v1.33/bin/bin/../../lib/gcc/pic32mx/4.5.2/../../../../pic32mx/lib\libpic32.a(vector58.o)

.data%z55       0x00000000        0x0
 .data          0x00000000        0x0 c:/program files/microchip/xc32/v1.33/bin/bin/../../lib/gcc/pic32mx/4.5.2/../../../../pic32mx/lib\libpic32.a(vector58.o)

.bss%z56        0x00000000        0x0
 .bss           0x00000000        0x0 c:/program files/microchip/xc32/v1.33/bin/bin/../../lib/gcc/pic32mx/4.5.2/../../../../pic32mx/lib\libpic32.a(vector57.o)

.data%z57       0x00000000        0x0
 .data          0x00000000        0x0 c:/program files/microchip/xc32/v1.33/bin/bin/../../lib/gcc/pic32mx/4.5.2/../../../../pic32mx/lib\libpic32.a(vector57.o)

.bss%z58        0x00000000        0x0
 .bss           0x00000000        0x0 c:/program files/microchip/xc32/v1.33/bin/bin/../../lib/gcc/pic32mx/4.5.2/../../../../pic32mx/lib\libpic32.a(vector56.o)

.data%z59       0x00000000        0x0
 .data          0x00000000        0x0 c:/program files/microchip/xc32/v1.33/bin/bin/../../lib/gcc/pic32mx/4.5.2/../../../../pic32mx/lib\libpic32.a(vector56.o)

.bss%z60        0x00000000        0x0
 .bss           0x00000000        0x0 c:/program files/microchip/xc32/v1.33/bin/bin/../../lib/gcc/pic32mx/4.5.2/../../../../pic32mx/lib\libpic32.a(vector55.o)

.data%z61       0x00000000        0x0
 .data          0x00000000        0x0 c:/program files/microchip/xc32/v1.33/bin/bin/../../lib/gcc/pic32mx/4.5.2/../../../../pic32mx/lib\libpic32.a(vector55.o)

.bss%z62        0x00000000        0x0
 .bss           0x00000000        0x0 c:/program files/microchip/xc32/v1.33/bin/bin/../../lib/gcc/pic32mx/4.5.2/../../../../pic32mx/lib\libpic32.a(vector54.o)

.data%z63       0x00000000        0x0
 .data          0x00000000        0x0 c:/program files/microchip/xc32/v1.33/bin/bin/../../lib/gcc/pic32mx/4.5.2/../../../../pic32mx/lib\libpic32.a(vector54.o)

.bss%z64        0x00000000        0x0
 .bss           0x00000000        0x0 c:/program files/microchip/xc32/v1.33/bin/bin/../../lib/gcc/pic32mx/4.5.2/../../../../pic32mx/lib\libpic32.a(vector53.o)

.data%z65       0x00000000        0x0
 .data          0x00000000        0x0 c:/program files/microchip/xc32/v1.33/bin/bin/../../lib/gcc/pic32mx/4.5.2/../../../../pic32mx/lib\libpic32.a(vector53.o)

.bss%z66        0x00000000        0x0
 .bss           0x00000000        0x0 c:/program files/microchip/xc32/v1.33/bin/bin/../../lib/gcc/pic32mx/4.5.2/../../../../pic32mx/lib\libpic32.a(vector52.o)

.data%z67       0x00000000        0x0
 .data          0x00000000        0x0 c:/program files/microchip/xc32/v1.33/bin/bin/../../lib/gcc/pic32mx/4.5.2/../../../../pic32mx/lib\libpic32.a(vector52.o)

.bss%z68        0x00000000        0x0
 .bss           0x00000000        0x0 c:/program files/microchip/xc32/v1.33/bin/bin/../../lib/gcc/pic32mx/4.5.2/../../../../pic32mx/lib\libpic32.a(vector51.o)

.data%z69       0x00000000        0x0
 .data          0x00000000        0x0 c:/program files/microchip/xc32/v1.33/bin/bin/../../lib/gcc/pic32mx/4.5.2/../../../../pic32mx/lib\libpic32.a(vector51.o)

.bss%z70        0x00000000        0x0
 .bss           0x00000000        0x0 c:/program files/microchip/xc32/v1.33/bin/bin/../../lib/gcc/pic32mx/4.5.2/../../../../pic32mx/lib\libpic32.a(vector50.o)

.data%z71       0x00000000        0x0
 .data          0x00000000        0x0 c:/program files/microchip/xc32/v1.33/bin/bin/../../lib/gcc/pic32mx/4.5.2/../../../../pic32mx/lib\libpic32.a(vector50.o)

.bss%z72        0x00000000        0x0
 .bss           0x00000000        0x0 c:/program files/microchip/xc32/v1.33/bin/bin/../../lib/gcc/pic32mx/4.5.2/../../../../pic32mx/lib\libpic32.a(vector49.o)

.data%z73       0x00000000        0x0
 .data          0x00000000        0x0 c:/program files/microchip/xc32/v1.33/bin/bin/../../lib/gcc/pic32mx/4.5.2/../../../../pic32mx/lib\libpic32.a(vector49.o)

.bss%z74        0x00000000        0x0
 .bss           0x00000000        0x0 c:/program files/microchip/xc32/v1.33/bin/bin/../../lib/gcc/pic32mx/4.5.2/../../../../pic32mx/lib\libpic32.a(vector48.o)

.data%z75       0x00000000        0x0
 .data          0x00000000        0x0 c:/program files/microchip/xc32/v1.33/bin/bin/../../lib/gcc/pic32mx/4.5.2/../../../../pic32mx/lib\libpic32.a(vector48.o)

.bss%z76        0x00000000        0x0
 .bss           0x00000000        0x0 c:/program files/microchip/xc32/v1.33/bin/bin/../../lib/gcc/pic32mx/4.5.2/../../../../pic32mx/lib\libpic32.a(vector47.o)

.data%z77       0x00000000        0x0
 .data          0x00000000        0x0 c:/program files/microchip/xc32/v1.33/bin/bin/../../lib/gcc/pic32mx/4.5.2/../../../../pic32mx/lib\libpic32.a(vector47.o)

.bss%z78        0x00000000        0x0
 .bss           0x00000000        0x0 c:/program files/microchip/xc32/v1.33/bin/bin/../../lib/gcc/pic32mx/4.5.2/../../../../pic32mx/lib\libpic32.a(vector46.o)

.data%z79       0x00000000        0x0
 .data          0x00000000        0x0 c:/program files/microchip/xc32/v1.33/bin/bin/../../lib/gcc/pic32mx/4.5.2/../../../../pic32mx/lib\libpic32.a(vector46.o)

.bss%z80        0x00000000        0x0
 .bss           0x00000000        0x0 c:/program files/microchip/xc32/v1.33/bin/bin/../../lib/gcc/pic32mx/4.5.2/../../../../pic32mx/lib\libpic32.a(vector45.o)

.data%z81       0x00000000        0x0
 .data          0x00000000        0x0 c:/program files/microchip/xc32/v1.33/bin/bin/../../lib/gcc/pic32mx/4.5.2/../../../../pic32mx/lib\libpic32.a(vector45.o)

.bss%z82        0x00000000        0x0
 .bss           0x00000000        0x0 c:/program files/microchip/xc32/v1.33/bin/bin/../../lib/gcc/pic32mx/4.5.2/../../../../pic32mx/lib\libpic32.a(vector44.o)

.data%z83       0x00000000        0x0
 .data          0x00000000        0x0 c:/program files/microchip/xc32/v1.33/bin/bin/../../lib/gcc/pic32mx/4.5.2/../../../../pic32mx/lib\libpic32.a(vector44.o)

.bss%z84        0x00000000        0x0
 .bss           0x00000000        0x0 c:/program files/microchip/xc32/v1.33/bin/bin/../../lib/gcc/pic32mx/4.5.2/../../../../pic32mx/lib\libpic32.a(vector43.o)

.data%z85       0x00000000        0x0
 .data          0x00000000        0x0 c:/program files/microchip/xc32/v1.33/bin/bin/../../lib/gcc/pic32mx/4.5.2/../../../../pic32mx/lib\libpic32.a(vector43.o)

.bss%z86        0x00000000        0x0
 .bss           0x00000000        0x0 c:/program files/microchip/xc32/v1.33/bin/bin/../../lib/gcc/pic32mx/4.5.2/../../../../pic32mx/lib\libpic32.a(vector42.o)

.data%z87       0x00000000        0x0
 .data          0x00000000        0x0 c:/program files/microchip/xc32/v1.33/bin/bin/../../lib/gcc/pic32mx/4.5.2/../../../../pic32mx/lib\libpic32.a(vector42.o)

.bss%z88        0x00000000        0x0
 .bss           0x00000000        0x0 c:/program files/microchip/xc32/v1.33/bin/bin/../../lib/gcc/pic32mx/4.5.2/../../../../pic32mx/lib\libpic32.a(vector41.o)

.data%z89       0x00000000        0x0
 .data          0x00000000        0x0 c:/program files/microchip/xc32/v1.33/bin/bin/../../lib/gcc/pic32mx/4.5.2/../../../../pic32mx/lib\libpic32.a(vector41.o)

.bss%z90        0x00000000        0x0
 .bss           0x00000000        0x0 c:/program files/microchip/xc32/v1.33/bin/bin/../../lib/gcc/pic32mx/4.5.2/../../../../pic32mx/lib\libpic32.a(vector40.o)

.data%z91       0x00000000        0x0
 .data          0x00000000        0x0 c:/program files/microchip/xc32/v1.33/bin/bin/../../lib/gcc/pic32mx/4.5.2/../../../../pic32mx/lib\libpic32.a(vector40.o)

.bss%z92        0x00000000        0x0
 .bss           0x00000000        0x0 c:/program files/microchip/xc32/v1.33/bin/bin/../../lib/gcc/pic32mx/4.5.2/../../../../pic32mx/lib\libpic32.a(vector39.o)

.data%z93       0x00000000        0x0
 .data          0x00000000        0x0 c:/program files/microchip/xc32/v1.33/bin/bin/../../lib/gcc/pic32mx/4.5.2/../../../../pic32mx/lib\libpic32.a(vector39.o)

.bss%z94        0x00000000        0x0
 .bss           0x00000000        0x0 c:/program files/microchip/xc32/v1.33/bin/bin/../../lib/gcc/pic32mx/4.5.2/../../../../pic32mx/lib\libpic32.a(vector38.o)

.data%z95       0x00000000        0x0
 .data          0x00000000        0x0 c:/program files/microchip/xc32/v1.33/bin/bin/../../lib/gcc/pic32mx/4.5.2/../../../../pic32mx/lib\libpic32.a(vector38.o)

.bss%z96        0x00000000        0x0
 .bss           0x00000000        0x0 c:/program files/microchip/xc32/v1.33/bin/bin/../../lib/gcc/pic32mx/4.5.2/../../../../pic32mx/lib\libpic32.a(vector37.o)

.data%z97       0x00000000        0x0
 .data          0x00000000        0x0 c:/program files/microchip/xc32/v1.33/bin/bin/../../lib/gcc/pic32mx/4.5.2/../../../../pic32mx/lib\libpic32.a(vector37.o)

.bss%z98        0x00000000        0x0
 .bss           0x00000000        0x0 c:/program files/microchip/xc32/v1.33/bin/bin/../../lib/gcc/pic32mx/4.5.2/../../../../pic32mx/lib\libpic32.a(vector36.o)

.data%z99       0x00000000        0x0
 .data          0x00000000        0x0 c:/program files/microchip/xc32/v1.33/bin/bin/../../lib/gcc/pic32mx/4.5.2/../../../../pic32mx/lib\libpic32.a(vector36.o)

.bss%z100       0x00000000        0x0
 .bss           0x00000000        0x0 c:/program files/microchip/xc32/v1.33/bin/bin/../../lib/gcc/pic32mx/4.5.2/../../../../pic32mx/lib\libpic32.a(vector35.o)

.data%z101      0x00000000        0x0
 .data          0x00000000        0x0 c:/program files/microchip/xc32/v1.33/bin/bin/../../lib/gcc/pic32mx/4.5.2/../../../../pic32mx/lib\libpic32.a(vector35.o)

.bss%z102       0x00000000        0x0
 .bss           0x00000000        0x0 c:/program files/microchip/xc32/v1.33/bin/bin/../../lib/gcc/pic32mx/4.5.2/../../../../pic32mx/lib\libpic32.a(vector34.o)

.data%z103      0x00000000        0x0
 .data          0x00000000        0x0 c:/program files/microchip/xc32/v1.33/bin/bin/../../lib/gcc/pic32mx/4.5.2/../../../../pic32mx/lib\libpic32.a(vector34.o)

.bss%z104       0x00000000        0x0
 .bss           0x00000000        0x0 c:/program files/microchip/xc32/v1.33/bin/bin/../../lib/gcc/pic32mx/4.5.2/../../../../pic32mx/lib\libpic32.a(vector33.o)

.data%z105      0x00000000        0x0
 .data          0x00000000        0x0 c:/program files/microchip/xc32/v1.33/bin/bin/../../lib/gcc/pic32mx/4.5.2/../../../../pic32mx/lib\libpic32.a(vector33.o)

.bss%z106       0x00000000        0x0
 .bss           0x00000000        0x0 c:/program files/microchip/xc32/v1.33/bin/bin/../../lib/gcc/pic32mx/4.5.2/../../../../pic32mx/lib\libpic32.a(vector32.o)

.data%z107      0x00000000        0x0
 .data          0x00000000        0x0 c:/program files/microchip/xc32/v1.33/bin/bin/../../lib/gcc/pic32mx/4.5.2/../../../../pic32mx/lib\libpic32.a(vector32.o)

.bss%z108       0x00000000        0x0
 .bss           0x00000000        0x0 c:/program files/microchip/xc32/v1.33/bin/bin/../../lib/gcc/pic32mx/4.5.2/../../../../pic32mx/lib\libpic32.a(vector31.o)

.data%z109      0x00000000        0x0
 .data          0x00000000        0x0 c:/program files/microchip/xc32/v1.33/bin/bin/../../lib/gcc/pic32mx/4.5.2/../../../../pic32mx/lib\libpic32.a(vector31.o)

.bss%z110       0x00000000        0x0
 .bss           0x00000000        0x0 c:/program files/microchip/xc32/v1.33/bin/bin/../../lib/gcc/pic32mx/4.5.2/../../../../pic32mx/lib\libpic32.a(vector30.o)

.data%z111      0x00000000        0x0
 .data          0x00000000        0x0 c:/program files/microchip/xc32/v1.33/bin/bin/../../lib/gcc/pic32mx/4.5.2/../../../../pic32mx/lib\libpic32.a(vector30.o)

.bss%z112       0x00000000        0x0
 .bss           0x00000000        0x0 c:/program files/microchip/xc32/v1.33/bin/bin/../../lib/gcc/pic32mx/4.5.2/../../../../pic32mx/lib\libpic32.a(vector29.o)

.data%z113      0x00000000        0x0
 .data          0x00000000        0x0 c:/program files/microchip/xc32/v1.33/bin/bin/../../lib/gcc/pic32mx/4.5.2/../../../../pic32mx/lib\libpic32.a(vector29.o)

.bss%z114       0x00000000        0x0
 .bss           0x00000000        0x0 c:/program files/microchip/xc32/v1.33/bin/bin/../../lib/gcc/pic32mx/4.5.2/../../../../pic32mx/lib\libpic32.a(vector28.o)

.data%z115      0x00000000        0x0
 .data          0x00000000        0x0 c:/program files/microchip/xc32/v1.33/bin/bin/../../lib/gcc/pic32mx/4.5.2/../../../../pic32mx/lib\libpic32.a(vector28.o)

.bss%z116       0x00000000        0x0
 .bss           0x00000000        0x0 c:/program files/microchip/xc32/v1.33/bin/bin/../../lib/gcc/pic32mx/4.5.2/../../../../pic32mx/lib\libpic32.a(vector27.o)

.data%z117      0x00000000        0x0
 .data          0x00000000        0x0 c:/program files/microchip/xc32/v1.33/bin/bin/../../lib/gcc/pic32mx/4.5.2/../../../../pic32mx/lib\libpic32.a(vector27.o)

.bss%z118       0x00000000        0x0
 .bss           0x00000000        0x0 c:/program files/microchip/xc32/v1.33/bin/bin/../../lib/gcc/pic32mx/4.5.2/../../../../pic32mx/lib\libpic32.a(vector26.o)

.data%z119      0x00000000        0x0
 .data          0x00000000        0x0 c:/program files/microchip/xc32/v1.33/bin/bin/../../lib/gcc/pic32mx/4.5.2/../../../../pic32mx/lib\libpic32.a(vector26.o)

.bss%z120       0x00000000        0x0
 .bss           0x00000000        0x0 c:/program files/microchip/xc32/v1.33/bin/bin/../../lib/gcc/pic32mx/4.5.2/../../../../pic32mx/lib\libpic32.a(vector25.o)

.data%z121      0x00000000        0x0
 .data          0x00000000        0x0 c:/program files/microchip/xc32/v1.33/bin/bin/../../lib/gcc/pic32mx/4.5.2/../../../../pic32mx/lib\libpic32.a(vector25.o)

.bss%z122       0x00000000        0x0
 .bss           0x00000000        0x0 c:/program files/microchip/xc32/v1.33/bin/bin/../../lib/gcc/pic32mx/4.5.2/../../../../pic32mx/lib\libpic32.a(vector24.o)

.data%z123      0x00000000        0x0
 .data          0x00000000        0x0 c:/program files/microchip/xc32/v1.33/bin/bin/../../lib/gcc/pic32mx/4.5.2/../../../../pic32mx/lib\libpic32.a(vector24.o)

.bss%z124       0x00000000        0x0
 .bss           0x00000000        0x0 c:/program files/microchip/xc32/v1.33/bin/bin/../../lib/gcc/pic32mx/4.5.2/../../../../pic32mx/lib\libpic32.a(vector23.o)

.data%z125      0x00000000        0x0
 .data          0x00000000        0x0 c:/program files/microchip/xc32/v1.33/bin/bin/../../lib/gcc/pic32mx/4.5.2/../../../../pic32mx/lib\libpic32.a(vector23.o)

.bss%z126       0x00000000        0x0
 .bss           0x00000000        0x0 c:/program files/microchip/xc32/v1.33/bin/bin/../../lib/gcc/pic32mx/4.5.2/../../../../pic32mx/lib\libpic32.a(vector22.o)

.data%z127      0x00000000        0x0
 .data          0x00000000        0x0 c:/program files/microchip/xc32/v1.33/bin/bin/../../lib/gcc/pic32mx/4.5.2/../../../../pic32mx/lib\libpic32.a(vector22.o)

.bss%z128       0x00000000        0x0
 .bss           0x00000000        0x0 c:/program files/microchip/xc32/v1.33/bin/bin/../../lib/gcc/pic32mx/4.5.2/../../../../pic32mx/lib\libpic32.a(vector21.o)

.data%z129      0x00000000        0x0
 .data          0x00000000        0x0 c:/program files/microchip/xc32/v1.33/bin/bin/../../lib/gcc/pic32mx/4.5.2/../../../../pic32mx/lib\libpic32.a(vector21.o)

.bss%z130       0x00000000        0x0
 .bss           0x00000000        0x0 c:/program files/microchip/xc32/v1.33/bin/bin/../../lib/gcc/pic32mx/4.5.2/../../../../pic32mx/lib\libpic32.a(vector20.o)

.data%z131      0x00000000        0x0
 .data          0x00000000        0x0 c:/program files/microchip/xc32/v1.33/bin/bin/../../lib/gcc/pic32mx/4.5.2/../../../../pic32mx/lib\libpic32.a(vector20.o)

.bss%z132       0x00000000        0x0
 .bss           0x00000000        0x0 c:/program files/microchip/xc32/v1.33/bin/bin/../../lib/gcc/pic32mx/4.5.2/../../../../pic32mx/lib\libpic32.a(vector19.o)

.data%z133      0x00000000        0x0
 .data          0x00000000        0x0 c:/program files/microchip/xc32/v1.33/bin/bin/../../lib/gcc/pic32mx/4.5.2/../../../../pic32mx/lib\libpic32.a(vector19.o)

.bss%z134       0x00000000        0x0
 .bss           0x00000000        0x0 c:/program files/microchip/xc32/v1.33/bin/bin/../../lib/gcc/pic32mx/4.5.2/../../../../pic32mx/lib\libpic32.a(vector18.o)

.data%z135      0x00000000        0x0
 .data          0x00000000        0x0 c:/program files/microchip/xc32/v1.33/bin/bin/../../lib/gcc/pic32mx/4.5.2/../../../../pic32mx/lib\libpic32.a(vector18.o)

.bss%z136       0x00000000        0x0
 .bss           0x00000000        0x0 c:/program files/microchip/xc32/v1.33/bin/bin/../../lib/gcc/pic32mx/4.5.2/../../../../pic32mx/lib\libpic32.a(vector17.o)

.data%z137      0x00000000        0x0
 .data          0x00000000        0x0 c:/program files/microchip/xc32/v1.33/bin/bin/../../lib/gcc/pic32mx/4.5.2/../../../../pic32mx/lib\libpic32.a(vector17.o)

.bss%z138       0x00000000        0x0
 .bss           0x00000000        0x0 c:/program files/microchip/xc32/v1.33/bin/bin/../../lib/gcc/pic32mx/4.5.2/../../../../pic32mx/lib\libpic32.a(vector16.o)

.data%z139      0x00000000        0x0
 .data          0x00000000        0x0 c:/program files/microchip/xc32/v1.33/bin/bin/../../lib/gcc/pic32mx/4.5.2/../../../../pic32mx/lib\libpic32.a(vector16.o)

.bss%z140       0x00000000        0x0
 .bss           0x00000000        0x0 c:/program files/microchip/xc32/v1.33/bin/bin/../../lib/gcc/pic32mx/4.5.2/../../../../pic32mx/lib\libpic32.a(vector14.o)

.data%z141      0x00000000        0x0
 .data          0x00000000        0x0 c:/program files/microchip/xc32/v1.33/bin/bin/../../lib/gcc/pic32mx/4.5.2/../../../../pic32mx/lib\libpic32.a(vector14.o)

.bss%z142       0x00000000        0x0
 .bss           0x00000000        0x0 c:/program files/microchip/xc32/v1.33/bin/bin/../../lib/gcc/pic32mx/4.5.2/../../../../pic32mx/lib\libpic32.a(vector13.o)

.data%z143      0x00000000        0x0
 .data          0x00000000        0x0 c:/program files/microchip/xc32/v1.33/bin/bin/../../lib/gcc/pic32mx/4.5.2/../../../../pic32mx/lib\libpic32.a(vector13.o)

.bss%z144       0x00000000        0x0
 .bss           0x00000000        0x0 c:/program files/microchip/xc32/v1.33/bin/bin/../../lib/gcc/pic32mx/4.5.2/../../../../pic32mx/lib\libpic32.a(vector12.o)

.data%z145      0x00000000        0x0
 .data          0x00000000        0x0 c:/program files/microchip/xc32/v1.33/bin/bin/../../lib/gcc/pic32mx/4.5.2/../../../../pic32mx/lib\libpic32.a(vector12.o)

.bss%z146       0x00000000        0x0
 .bss           0x00000000        0x0 c:/program files/microchip/xc32/v1.33/bin/bin/../../lib/gcc/pic32mx/4.5.2/../../../../pic32mx/lib\libpic32.a(vector11.o)

.data%z147      0x00000000        0x0
 .data          0x00000000        0x0 c:/program files/microchip/xc32/v1.33/bin/bin/../../lib/gcc/pic32mx/4.5.2/../../../../pic32mx/lib\libpic32.a(vector11.o)

.bss%z148       0x00000000        0x0
 .bss           0x00000000        0x0 c:/program files/microchip/xc32/v1.33/bin/bin/../../lib/gcc/pic32mx/4.5.2/../../../../pic32mx/lib\libpic32.a(vector10.o)

.data%z149      0x00000000        0x0
 .data          0x00000000        0x0 c:/program files/microchip/xc32/v1.33/bin/bin/../../lib/gcc/pic32mx/4.5.2/../../../../pic32mx/lib\libpic32.a(vector10.o)

.bss%z150       0x00000000        0x0
 .bss           0x00000000        0x0 c:/program files/microchip/xc32/v1.33/bin/bin/../../lib/gcc/pic32mx/4.5.2/../../../../pic32mx/lib\libpic32.a(vector9.o)

.data%z151      0x00000000        0x0
 .data          0x00000000        0x0 c:/program files/microchip/xc32/v1.33/bin/bin/../../lib/gcc/pic32mx/4.5.2/../../../../pic32mx/lib\libpic32.a(vector9.o)

.bss%z152       0x00000000        0x0
 .bss           0x00000000        0x0 c:/program files/microchip/xc32/v1.33/bin/bin/../../lib/gcc/pic32mx/4.5.2/../../../../pic32mx/lib\libpic32.a(vector8.o)

.data%z153      0x00000000        0x0
 .data          0x00000000        0x0 c:/program files/microchip/xc32/v1.33/bin/bin/../../lib/gcc/pic32mx/4.5.2/../../../../pic32mx/lib\libpic32.a(vector8.o)

.bss%z154       0x00000000        0x0
 .bss           0x00000000        0x0 c:/program files/microchip/xc32/v1.33/bin/bin/../../lib/gcc/pic32mx/4.5.2/../../../../pic32mx/lib\libpic32.a(vector6.o)

.data%z155      0x00000000        0x0
 .data          0x00000000        0x0 c:/program files/microchip/xc32/v1.33/bin/bin/../../lib/gcc/pic32mx/4.5.2/../../../../pic32mx/lib\libpic32.a(vector6.o)

.bss%z156       0x00000000        0x0
 .bss           0x00000000        0x0 c:/program files/microchip/xc32/v1.33/bin/bin/../../lib/gcc/pic32mx/4.5.2/../../../../pic32mx/lib\libpic32.a(vector5.o)

.data%z157      0x00000000        0x0
 .data          0x00000000        0x0 c:/program files/microchip/xc32/v1.33/bin/bin/../../lib/gcc/pic32mx/4.5.2/../../../../pic32mx/lib\libpic32.a(vector5.o)

.bss%z158       0x00000000        0x0
 .bss           0x00000000        0x0 c:/program files/microchip/xc32/v1.33/bin/bin/../../lib/gcc/pic32mx/4.5.2/../../../../pic32mx/lib\libpic32.a(vector2.o)

.data%z159      0x00000000        0x0
 .data          0x00000000        0x0 c:/program files/microchip/xc32/v1.33/bin/bin/../../lib/gcc/pic32mx/4.5.2/../../../../pic32mx/lib\libpic32.a(vector2.o)

.bss%z160       0x00000000        0x0
 .bss           0x00000000        0x0 c:/program files/microchip/xc32/v1.33/bin/bin/../../lib/gcc/pic32mx/4.5.2/../../../../pic32mx/lib\libpic32.a(vector1.o)

.data%z161      0x00000000        0x0
 .data          0x00000000        0x0 c:/program files/microchip/xc32/v1.33/bin/bin/../../lib/gcc/pic32mx/4.5.2/../../../../pic32mx/lib\libpic32.a(vector1.o)

.bss%z162       0x00000000        0x0
 .bss           0x00000000        0x0 c:/program files/microchip/xc32/v1.33/bin/bin/../../lib/gcc/pic32mx/4.5.2/../../../../pic32mx/lib\libpic32.a(vector0.o)

.data%z163      0x00000000        0x0
 .data          0x00000000        0x0 c:/program files/microchip/xc32/v1.33/bin/bin/../../lib/gcc/pic32mx/4.5.2/../../../../pic32mx/lib\libpic32.a(vector0.o)

.bss%z164       0x00000000        0x0
 .bss           0x00000000        0x0 c:/program files/microchip/xc32/v1.33/bin/bin/../../lib/gcc/pic32mx/4.5.2/../../../../pic32mx/lib\libpic32.a(general-exception.o)

.data%z165      0x00000000        0x0
 .data          0x00000000        0x0 c:/program files/microchip/xc32/v1.33/bin/bin/../../lib/gcc/pic32mx/4.5.2/../../../../pic32mx/lib\libpic32.a(general-exception.o)

.bss%z166       0x00000000        0x0
 .bss           0x00000000        0x0 c:/program files/microchip/xc32/v1.33/bin/bin/../../lib/gcc/pic32mx/4.5.2/../../../../pic32mx/lib\libpic32.a(close.o)

.data%z167      0x00000000        0x0
 .data          0x00000000        0x0 c:/program files/microchip/xc32/v1.33/bin/bin/../../lib/gcc/pic32mx/4.5.2/../../../../pic32mx/lib\libpic32.a(close.o)

.bss%z168       0x00000000        0x0
 .bss           0x00000000        0x0 c:/program files/microchip/xc32/v1.33/bin/bin/../../lib/gcc/pic32mx/4.5.2/../../../../pic32mx/lib\libpic32.a(default-nmi-handler.o)

.data%z169      0x00000000        0x0
 .data          0x00000000        0x0 c:/program files/microchip/xc32/v1.33/bin/bin/../../lib/gcc/pic32mx/4.5.2/../../../../pic32mx/lib\libpic32.a(default-nmi-handler.o)

.bss%z170       0x00000000        0x0
 .bss           0x00000000        0x0 c:/program files/microchip/xc32/v1.33/bin/bin/../../lib/gcc/pic32mx/4.5.2/../../../../pic32mx/lib\libpic32.a(default-on-bootstrap.o)

.data%z171      0x00000000        0x0
 .data          0x00000000        0x0 c:/program files/microchip/xc32/v1.33/bin/bin/../../lib/gcc/pic32mx/4.5.2/../../../../pic32mx/lib\libpic32.a(default-on-bootstrap.o)

.bss%z172       0x00000000        0x0
 .bss           0x00000000        0x0 c:/program files/microchip/xc32/v1.33/bin/bin/../../lib/gcc/pic32mx/4.5.2/../../../../pic32mx/lib\libpic32.a(default-on-reset.o)

.data%z173      0x00000000        0x0
 .data          0x00000000        0x0 c:/program files/microchip/xc32/v1.33/bin/bin/../../lib/gcc/pic32mx/4.5.2/../../../../pic32mx/lib\libpic32.a(default-on-reset.o)

.bss%z174       0x00000000        0x0
 .bss           0x00000000        0x0 c:/program files/microchip/xc32/v1.33/bin/bin/../../lib/gcc/pic32mx/4.5.2/../../../../pic32mx/lib\libpic32.a(default-bootstrap-exception-handler.o)

.data%z175      0x00000000        0x0
 .data          0x00000000        0x0 c:/program files/microchip/xc32/v1.33/bin/bin/../../lib/gcc/pic32mx/4.5.2/../../../../pic32mx/lib\libpic32.a(default-bootstrap-exception-handler.o)

.bss%z176       0x00000000        0x0
 .bss           0x00000000        0x0 c:/program files/microchip/xc32/v1.33/bin/bin/../../lib/gcc/pic32mx/4.5.2/../../../../pic32mx/lib\libpic32.a(strlen.o)

.data%z177      0x00000000        0x0
 .data          0x00000000        0x0 c:/program files/microchip/xc32/v1.33/bin/bin/../../lib/gcc/pic32mx/4.5.2/../../../../pic32mx/lib\libpic32.a(strlen.o)

.bss%z178       0x00000000        0x0
 .bss           0x00000000        0x0 c:/program files/microchip/xc32/v1.33/bin/bin/../../lib/gcc/pic32mx/4.5.2/../../../../pic32mx/lib\libpic32.a(strcpy.o)

.data%z179      0x00000000        0x0
 .data          0x00000000        0x0 c:/program files/microchip/xc32/v1.33/bin/bin/../../lib/gcc/pic32mx/4.5.2/../../../../pic32mx/lib\libpic32.a(strcpy.o)

.bss%z180       0x00000000        0x0
 .bss           0x00000000        0x0 c:/program files/microchip/xc32/v1.33/bin/bin/../../lib/gcc/pic32mx/4.5.2/../../../../pic32mx/lib\libpic32.a(memset.o)

.data%z181      0x00000000        0x0
 .data          0x00000000        0x0 c:/program files/microchip/xc32/v1.33/bin/bin/../../lib/gcc/pic32mx/4.5.2/../../../../pic32mx/lib\libpic32.a(memset.o)

.bss%z182       0x00000000        0x0
 .bss           0x00000000        0x0 c:/program files/microchip/xc32/v1.33/bin/bin/../../lib/gcc/pic32mx/4.5.2/../../../../pic32mx/lib\libpic32.a(memcpy.o)

.data%z183      0x00000000        0x0
 .data          0x00000000        0x0 c:/program files/microchip/xc32/v1.33/bin/bin/../../lib/gcc/pic32mx/4.5.2/../../../../pic32mx/lib\libpic32.a(memcpy.o)

.bss%z184       0x00000000        0x0
 .bss           0x00000000        0x0 c:/program files/microchip/xc32/v1.33/bin/bin/../../lib/gcc/pic32mx/4.5.2/../../../../pic32mx/lib\libpic32.a(memcmp.o)

.data%z185      0x00000000        0x0
 .data          0x00000000        0x0 c:/program files/microchip/xc32/v1.33/bin/bin/../../lib/gcc/pic32mx/4.5.2/../../../../pic32mx/lib\libpic32.a(memcmp.o)

.bss%z186       0x00000000        0x0
 .bss           0x00000000        0x0 c:/program files/microchip/xc32/v1.33/bin/bin/../../lib/gcc/pic32mx/4.5.2/../../../../pic32mx/lib\pic32_software_reset.o

.data%z187      0x00000000        0x0
 .data          0x00000000        0x0 c:/program files/microchip/xc32/v1.33/bin/bin/../../lib/gcc/pic32mx/4.5.2/../../../../pic32mx/lib\pic32_software_reset.o

.bss%z188       0x00000000        0x0
 .bss           0x00000000        0x0 c:/program files/microchip/xc32/v1.33/bin/bin/../../lib/gcc/pic32mx/4.5.2/../../../../pic32mx/lib/./proc/32MX795F512H\default_isr_vectors.o

.data%z189      0x00000000        0x0
 .data          0x00000000        0x0 c:/program files/microchip/xc32/v1.33/bin/bin/../../lib/gcc/pic32mx/4.5.2/../../../../pic32mx/lib/./proc/32MX795F512H\default_isr_vectors.o

.bss%z190       0x00000000        0x0
 .bss           0x00000000        0x0 c:/program files/microchip/xc32/v1.33/bin/bin/../../lib/gcc/pic32mx/4.5.2/../../../../pic32mx/lib\libmchp_peripheral_32MX795F512H.a(int_restore_interrupts_lib.o)

.data%z191      0x00000000        0x0
 .data          0x00000000        0x0 c:/program files/microchip/xc32/v1.33/bin/bin/../../lib/gcc/pic32mx/4.5.2/../../../../pic32mx/lib\libmchp_peripheral_32MX795F512H.a(int_restore_interrupts_lib.o)

.bss%z192       0x00000000        0x0
 .bss           0x00000000        0x0 c:/program files/microchip/xc32/v1.33/bin/bin/../../lib/gcc/pic32mx/4.5.2/../../../../pic32mx/lib\libmchp_peripheral_32MX795F512H.a(int_disable_interrupts_lib.o)

.data%z193      0x00000000        0x0
 .data          0x00000000        0x0 c:/program files/microchip/xc32/v1.33/bin/bin/../../lib/gcc/pic32mx/4.5.2/../../../../pic32mx/lib\libmchp_peripheral_32MX795F512H.a(int_disable_interrupts_lib.o)

.bss%z194       0x00000000        0x0
 .bss           0x00000000        0x0 c:/program files/microchip/xc32/v1.33/bin/bin/../../lib/gcc/pic32mx/4.5.2/../../../../pic32mx/lib\libmchp_peripheral_32MX795F512H.a(int_enable_interrupts_lib.o)

.data%z195      0x00000000        0x0
 .data          0x00000000        0x0 c:/program files/microchip/xc32/v1.33/bin/bin/../../lib/gcc/pic32mx/4.5.2/../../../../pic32mx/lib\libmchp_peripheral_32MX795F512H.a(int_enable_interrupts_lib.o)

.bss%z196       0x00000000        0x0
 .bss           0x00000000        0x0 c:/program files/microchip/xc32/v1.33/bin/bin/../../lib/gcc/pic32mx/4.5.2/../../../../pic32mx/lib\libmchp_peripheral_32MX795F512H.a(int_configure_system_lib.o)

.data%z197      0x00000000        0x0
 .data          0x00000000        0x0 c:/program files/microchip/xc32/v1.33/bin/bin/../../lib/gcc/pic32mx/4.5.2/../../../../pic32mx/lib\libmchp_peripheral_32MX795F512H.a(int_configure_system_lib.o)

.bss%z198       0x00000000        0x0
 .bss           0x00000000        0x0 c:/program files/microchip/xc32/v1.33/bin/bin/../../lib/gcc/pic32mx/4.5.2/../../../../pic32mx/lib\libmchp_peripheral_32MX795F512H.a(pcache.o)

.data%z199      0x00000000        0x0
 .data          0x00000000        0x0 c:/program files/microchip/xc32/v1.33/bin/bin/../../lib/gcc/pic32mx/4.5.2/../../../../pic32mx/lib\libmchp_peripheral_32MX795F512H.a(pcache.o)

.bss%z200       0x00000000        0x0
 .bss           0x00000000        0x0 c:/program files/microchip/xc32/v1.33/bin/bin/../../lib/gcc/pic32mx/4.5.2/../../../../pic32mx/lib\libmchp_peripheral_32MX795F512H.a(soft_reset_lib.o)

.data%z201      0x00000000        0x0
 .data          0x00000000        0x0 c:/program files/microchip/xc32/v1.33/bin/bin/../../lib/gcc/pic32mx/4.5.2/../../../../pic32mx/lib\libmchp_peripheral_32MX795F512H.a(soft_reset_lib.o)

.bss%z202       0x00000000        0x0
 .bss           0x00000000        0x0 c:/program files/microchip/xc32/v1.33/bin/bin/../../lib/gcc/pic32mx/4.5.2/../../../../pic32mx/lib/./proc/32MX795F512H\processor.o

.data%z203      0x00000000        0x0
 .data          0x00000000        0x0 c:/program files/microchip/xc32/v1.33/bin/bin/../../lib/gcc/pic32mx/4.5.2/../../../../pic32mx/lib/./proc/32MX795F512H\processor.o

.bss%z204       0x00000000        0x0
 .bss           0x00000000        0x0 build/ChaletDuinoV2_795F512H_/debug/Source/DACInterface.o

.data%z205      0x00000000        0x0
 .data          0x00000000        0x0 build/ChaletDuinoV2_795F512H_/debug/Source/DACInterface.o

.bss%z206       0x00000000        0x0
 .bss           0x00000000        0x0 build/ChaletDuinoV2_795F512H_/debug/Source/VolumeTransducer.o

.data%z207      0x00000000        0x0
 .data          0x00000000        0x0 build/ChaletDuinoV2_795F512H_/debug/Source/VolumeTransducer.o

.data%z208      0x00000000        0x0
 .data          0x00000000        0x0 build/ChaletDuinoV2_795F512H_/debug/Source/crc32.o

.bss%z209       0x00000000        0x0
 .bss           0x00000000        0x0 build/ChaletDuinoV2_795F512H_/debug/Source/BootloaderProtocol.o

.bss%z210       0x00000000        0x0
 .bss           0x00000000        0x0 build/ChaletDuinoV2_795F512H_/debug/Source/BootloaderInterface.o

.bss%z211       0x00000000        0x0
 .bss           0x00000000        0x0 build/ChaletDuinoV2_795F512H_/debug/Source/Watchdog.o

.data%z212      0x00000000        0x0
 .data          0x00000000        0x0 build/ChaletDuinoV2_795F512H_/debug/Source/Watchdog.o

.bss%z213       0x00000000        0x0
 .bss           0x00000000        0x0 build/ChaletDuinoV2_795F512H_/debug/Source/Syslog.o

.bss%z214       0x00000000        0x0
 .bss           0x00000000        0x0 build/ChaletDuinoV2_795F512H_/debug/Source/SPI_Flash.o

.data%z215      0x00000000        0x0
 .data          0x00000000        0x0 build/ChaletDuinoV2_795F512H_/debug/Source/SPI_Flash.o

.bss%z216       0x00000000        0x0
 .bss           0x00000000        0x0 build/ChaletDuinoV2_795F512H_/debug/Source/SPI.o

.data%z217      0x00000000        0x0
 .data          0x00000000        0x0 build/ChaletDuinoV2_795F512H_/debug/Source/SPI.o

.bss%z218       0x00000000        0x0
 .bss           0x00000000        0x0 build/ChaletDuinoV2_795F512H_/debug/Source/timer.o

.data%z219      0x00000000        0x0
 .data          0x00000000        0x0 build/ChaletDuinoV2_795F512H_/debug/Source/timer.o

.bss%z220       0x00000000        0x0
 .bss           0x00000000        0x0 build/ChaletDuinoV2_795F512H_/debug/Source/template.o

.data%z221      0x00000000        0x0
 .data          0x00000000        0x0 build/ChaletDuinoV2_795F512H_/debug/Source/template.o

.bss%z222       0x00000000        0x0
 .bss           0x00000000        0x0 build/ChaletDuinoV2_795F512H_/debug/Source/system.o

.data%z223      0x00000000        0x0
 .data          0x00000000        0x0 build/ChaletDuinoV2_795F512H_/debug/Source/system.o

.bss%z224       0x00000000        0x0
 .bss           0x00000000        0x0 build/ChaletDuinoV2_795F512H_/debug/Source/main.o

.bss%z225       0x00000000        0x0
 .bss           0x00000000        0x0 build/ChaletDuinoV2_795F512H_/debug/Source/interrupts.o

.data%z226      0x00000000        0x0
 .data          0x00000000        0x0 build/ChaletDuinoV2_795F512H_/debug/Source/interrupts.o

.bss%z227       0x00000000        0x0
 .bss           0x00000000        0x0 build/ChaletDuinoV2_795F512H_/debug/Source/exceptions.o

.data%z228      0x00000000        0x0
 .data          0x00000000        0x0 build/ChaletDuinoV2_795F512H_/debug/Source/exceptions.o

.bss%z229       0x00000000        0x0
 .bss           0x00000000        0x0 build/ChaletDuinoV2_795F512H_/debug/Source/Util.o

.data%z230      0x00000000        0x0
 .data          0x00000000        0x0 build/ChaletDuinoV2_795F512H_/debug/Source/Util.o

.bss%z231       0x00000000        0x0
 .bss           0x00000000        0x0 build/ChaletDuinoV2_795F512H_/debug/Source/Terminal.o

.bss%z232       0x00000000        0x0
 .bss           0x00000000        0x0 build/ChaletDuinoV2_795F512H_/debug/Source/NetworkProtocol.o

.data%z233      0x00000000        0x0
 .data          0x00000000        0x0 build/ChaletDuinoV2_795F512H_/debug/Source/NetworkProtocol.o

.bss%z234       0x00000000        0x0
 .bss           0x00000000        0x0 build/ChaletDuinoV2_795F512H_/debug/Source/DigitalIO.o

.data%z235      0x00000000        0x0
 .data          0x00000000        0x0 build/ChaletDuinoV2_795F512H_/debug/Source/DigitalIO.o

.bss%z236       0x00000000        0x0
 .bss           0x00000000        0x0 build/ChaletDuinoV2_795F512H_/debug/Source/winc3400_142/spi_flash/source/spi_flash.o

.data%z237      0x00000000        0x0
 .data          0x00000000        0x0 build/ChaletDuinoV2_795F512H_/debug/Source/winc3400_142/spi_flash/source/spi_flash.o

.bss%z238       0x00000000        0x0
 .bss           0x00000000        0x0 build/ChaletDuinoV2_795F512H_/debug/Source/winc3400_142/socket/source/socket.o

.data%z239      0x00000000        0x0
 .data          0x00000000        0x0 build/ChaletDuinoV2_795F512H_/debug/Source/winc3400_142/socket/source/socket.o

.bss%z240       0x00000000        0x0
 .bss           0x00000000        0x0 build/ChaletDuinoV2_795F512H_/debug/Source/winc3400_142/socket/source/inet_ntop.o

.data%z241      0x00000000        0x0
 .data          0x00000000        0x0 build/ChaletDuinoV2_795F512H_/debug/Source/winc3400_142/socket/source/inet_ntop.o

.bss%z242       0x00000000        0x0
 .bss           0x00000000        0x0 build/ChaletDuinoV2_795F512H_/debug/Source/winc3400_142/socket/source/inet_addr.o

.data%z243      0x00000000        0x0
 .data          0x00000000        0x0 build/ChaletDuinoV2_795F512H_/debug/Source/winc3400_142/socket/source/inet_addr.o

.bss%z244       0x00000000        0x0
 .bss           0x00000000        0x0 build/ChaletDuinoV2_795F512H_/debug/Source/winc3400_142/driver/source/nmspi.o

.data%z245      0x00000000        0x0
 .data          0x00000000        0x0 build/ChaletDuinoV2_795F512H_/debug/Source/winc3400_142/driver/source/nmspi.o

.bss%z246       0x00000000        0x0
 .bss           0x00000000        0x0 build/ChaletDuinoV2_795F512H_/debug/Source/winc3400_142/driver/source/nmdrv.o

.data%z247      0x00000000        0x0
 .data          0x00000000        0x0 build/ChaletDuinoV2_795F512H_/debug/Source/winc3400_142/driver/source/nmdrv.o

.bss%z248       0x00000000        0x0
 .bss           0x00000000        0x0 build/ChaletDuinoV2_795F512H_/debug/Source/winc3400_142/driver/source/nmbus.o

.data%z249      0x00000000        0x0
 .data          0x00000000        0x0 build/ChaletDuinoV2_795F512H_/debug/Source/winc3400_142/driver/source/nmbus.o

.bss%z250       0x00000000        0x0
 .bss           0x00000000        0x0 build/ChaletDuinoV2_795F512H_/debug/Source/winc3400_142/driver/source/nmasic.o

.data%z251      0x00000000        0x0
 .data          0x00000000        0x0 build/ChaletDuinoV2_795F512H_/debug/Source/winc3400_142/driver/source/nmasic.o

.data%z252      0x00000000        0x0
 .data          0x00000000        0x0 build/ChaletDuinoV2_795F512H_/debug/Source/winc3400_142/driver/source/m2m_wifi.o

.bss%z253       0x00000000        0x0
 .bss           0x00000000        0x0 build/ChaletDuinoV2_795F512H_/debug/Source/winc3400_142/driver/source/m2m_ssl.o

.data%z254      0x00000000        0x0
 .data          0x00000000        0x0 build/ChaletDuinoV2_795F512H_/debug/Source/winc3400_142/driver/source/m2m_ssl.o

.bss%z255       0x00000000        0x0
 .bss           0x00000000        0x0 build/ChaletDuinoV2_795F512H_/debug/Source/winc3400_142/driver/source/m2m_periph.o

.data%z256      0x00000000        0x0
 .data          0x00000000        0x0 build/ChaletDuinoV2_795F512H_/debug/Source/winc3400_142/driver/source/m2m_periph.o

.bss%z257       0x00000000        0x0
 .bss           0x00000000        0x0 build/ChaletDuinoV2_795F512H_/debug/Source/winc3400_142/driver/source/m2m_ota.o

.data%z258      0x00000000        0x0
 .data          0x00000000        0x0 build/ChaletDuinoV2_795F512H_/debug/Source/winc3400_142/driver/source/m2m_ota.o

.bss%z259       0x00000000        0x0
 .bss           0x00000000        0x0 build/ChaletDuinoV2_795F512H_/debug/Source/winc3400_142/driver/source/m2m_hif.o

.bss%z260       0x00000000        0x0
 .bss           0x00000000        0x0 build/ChaletDuinoV2_795F512H_/debug/Source/winc3400_142/driver/source/m2m_flash.o

.data%z261      0x00000000        0x0
 .data          0x00000000        0x0 build/ChaletDuinoV2_795F512H_/debug/Source/winc3400_142/driver/source/m2m_flash.o

.bss%z262       0x00000000        0x0
 .bss           0x00000000        0x0 build/ChaletDuinoV2_795F512H_/debug/Source/winc3400_142/common/source/nm_common.o

.data%z263      0x00000000        0x0
 .data          0x00000000        0x0 build/ChaletDuinoV2_795F512H_/debug/Source/winc3400_142/common/source/nm_common.o

.bss%z264       0x00000000        0x0
 .bss           0x00000000        0x0 build/ChaletDuinoV2_795F512H_/debug/Source/ChaletduinoV2Board.o

.data%z265      0x00000000        0x0
 .data          0x00000000        0x0 build/ChaletDuinoV2_795F512H_/debug/Source/ChaletduinoV2Board.o

.bss%z266       0x00000000        0x0
 .bss           0x00000000        0x0 c:/program files/microchip/xc32/v1.33/bin/bin/../../lib/gcc/pic32mx/4.5.2/../../../../pic32mx/lib\software-debug-break.o

.data%z267      0x00000000        0x0
 .data          0x00000000        0x0 c:/program files/microchip/xc32/v1.33/bin/bin/../../lib/gcc/pic32mx/4.5.2/../../../../pic32mx/lib\software-debug-break.o

.bss%z268       0x00000000        0x0
 .bss           0x00000000        0x0 c:/program files/microchip/xc32/v1.33/bin/bin/../../lib/gcc/pic32mx/4.5.2/../../../../pic32mx/lib/./proc/32MX795F512H/crt0_mips32r2.o

.data%z269      0x00000000        0x0
 .data          0x00000000        0x0 c:/program files/microchip/xc32/v1.33/bin/bin/../../lib/gcc/pic32mx/4.5.2/../../../../pic32mx/lib/./proc/32MX795F512H/crt0_mips32r2.o

.text           0x9d005800    0x108e4
 .text          0x9d005800     0x4174 build/ChaletDuinoV2_795F512H_/debug/Source/winc3400_142/driver/source/m2m_wifi.o
                0x9d006008                m2m_wifi_download_mode
                0x9d006334                m2m_wifi_ble_set_gain_table
                0x9d0063a8                m2m_wifi_init_hold
                0x9d0063e8                m2m_wifi_init_start
                0x9d00657c                m2m_wifi_init
                0x9d0065d8                m2m_wifi_deinit
                0x9d006620                m2m_wifi_reinit_hold
                0x9d00665c                m2m_wifi_reinit_start
                0x9d006694                m2m_wifi_reinit
                0x9d0066f4                m2m_wifi_get_state
                0x9d006778                m2m_wifi_handle_events
                0x9d0067cc                m2m_wifi_delete_sc
                0x9d006848                m2m_wifi_default_connect
                0x9d006bd0                m2m_wifi_connect_open
                0x9d006cc8                m2m_wifi_connect_wep
                0x9d006edc                m2m_wifi_connect_psk
                0x9d007154                m2m_wifi_1x_set_option
                0x9d007430                m2m_wifi_1x_get_option
                0x9d007648                m2m_wifi_connect_1x_mschap2
                0x9d00792c                m2m_wifi_connect_1x_tls
                0x9d007d4c                m2m_wifi_connect
                0x9d007dc0                m2m_wifi_connect_sc
                0x9d008000                m2m_wifi_disconnect
                0x9d00804c                m2m_wifi_set_mac_address
                0x9d0080b8                m2m_wifi_set_static_ip
                0x9d00814c                m2m_wifi_enable_dhcp
                0x9d0081c4                m2m_wifi_set_lsn_int
                0x9d008218                m2m_wifi_set_cust_InfoElement
                0x9d008278                m2m_wifi_set_scan_options
                0x9d0082f0                m2m_wifi_set_stop_scan_on_first
                0x9d008384                m2m_wifi_set_scan_region
                0x9d0083f4                m2m_wifi_request_scan
                0x9d00849c                m2m_wifi_request_scan_passive
                0x9d008544                m2m_wifi_request_scan_ssid_list
                0x9d0086a0                m2m_wifi_wps
                0x9d008728                m2m_wifi_wps_disable
                0x9d008780                m2m_wifi_p2p
                0x9d00882c                m2m_wifi_p2p_disconnect
                0x9d008884                m2m_wifi_enable_ap
                0x9d00891c                m2m_wifi_enable_ap_ext
                0x9d0089d0                m2m_wifi_disable_ap
                0x9d008a28                m2m_wifi_req_curr_rssi
                0x9d008a80                m2m_wifi_req_restrict_ble
                0x9d008ad8                m2m_wifi_req_unrestrict_ble
                0x9d008b30                m2m_wifi_send_ethernet_pkt
                0x9d008bd0                m2m_wifi_get_otp_mac_address
                0x9d008c3c                m2m_wifi_get_mac_address
                0x9d008ca0                m2m_wifi_req_scan_result
                0x9d008d0c                m2m_wifi_get_num_ap_found
                0x9d008d34                m2m_wifi_get_sleep_mode
                0x9d008d64                m2m_wifi_set_sleep_mode
                0x9d008df0                m2m_wifi_request_sleep
                0x9d008e74                m2m_wifi_set_device_name
                0x9d008f10                m2m_wifi_configure_sntp
                0x9d008fc0                m2m_wifi_get_chipId
                0x9d008ff0                m2m_wifi_get_firmware_version
                0x9d009054                m2m_wifi_check_ota_rb
                0x9d0090c0                m2m_ota_get_firmware_version
                0x9d009124                m2m_wifi_start_provision_mode
                0x9d0091d4                m2m_wifi_start_provision_mode_ext
                0x9d009320                m2m_wifi_stop_provision_mode
                0x9d00936c                m2m_wifi_get_connection_info
                0x9d0093b8                m2m_wifi_set_system_time
                0x9d00940c                m2m_wifi_get_system_time
                0x9d009458                m2m_wifi_enable_sntp
                0x9d0094d0                m2m_wifi_set_power_profile
                0x9d00953c                m2m_wifi_set_tx_power
                0x9d0095a8                m2m_wifi_enable_firmware_logs
                0x9d009614                m2m_wifi_set_battery_voltage
                0x9d009684                m2m_wifi_prng_get_random_bytes
                0x9d009724                m2m_wifi_enable_mac_mcast
                0x9d0097bc                m2m_wifi_set_receive_buffer
                0x9d00981c                m2m_wifi_enable_roaming
                0x9d0098ac                m2m_wifi_disable_roaming
                0x9d009900                m2m_wifi_ble_api_send
 .text          0x9d009974     0x28ec build/ChaletDuinoV2_795F512H_/debug/Source/winc3400_142/socket/source/socket.o
                0x9d00a3f0                socketInit
                0x9d00a460                socketDeinit
                0x9d00a4bc                registerSocketCallback
                0x9d00a4f4                registerSocketEventCallback
                0x9d00a520                registerSocketResolveCallback
                0x9d00a54c                socket
                0x9d00a878                bind
                0x9d00a9b4                listen
                0x9d00aaac                accept
                0x9d00ab30                connect
                0x9d00acb4                secure
                0x9d00ae7c                send
                0x9d00b058                sendto
                0x9d00b220                recv
                0x9d00b440                shutdown
                0x9d00b590                recvfrom
                0x9d00b790                gethostbyname
                0x9d00bc18                setsockopt
                0x9d00bde0                getsockopt
                0x9d00be1c                m2m_ping_req
                0x9d00bed8                set_alpn_list
                0x9d00c090                get_alpn_index
                0x9d00c158                IsSocketReady
                0x9d00c180                get_error_detail
 .text          0x9d00c260     0x1a28 build/ChaletDuinoV2_795F512H_/debug/Source/WiFiCtrl.o
                0x9d00ce34                InitWiFi
                0x9d00d200                TurnOFFWiFi
                0x9d00d298                CloseSockets
                0x9d00d384                GetWiFiSate
                0x9d00d3a8                GetCurIPAddress
                0x9d00d3cc                TickWiFi
                0x9d00d4c0                OpenTerminalServer
                0x9d00d57c                SendTerminalData
                0x9d00d604                SentTerminalByte
                0x9d00d680                OpenNetworkServer
                0x9d00d73c                SendNetworkData
                0x9d00d7c4                SentNetworkByte
                0x9d00d840                OpenSyslogServer
                0x9d00d8fc                SendSyslogData
                0x9d00d974                SendSyslogByte
                0x9d00d9f0                IsSyslogClientConnected
                0x9d00da30                OpenBootloaderServer
                0x9d00daec                CloseBootloaderServer
                0x9d00db54                SendBootloaderData
                0x9d00dbcc                SendSBootloaderByte
                0x9d00dc48                IsBootloaderClientConnected
 .text          0x9d00dc88     0x1808 build/ChaletDuinoV2_795F512H_/debug/Source/BootloaderInterface.o
                0x9d00dc88                BootloaderInterfaceInit
                0x9d00dcdc                BootloaderInterfaceTick
                0x9d00dd14                BootloaderExecuteCmd
                0x9d00dfb8                BootloaderCRCError
                0x9d00e020                BootloaderInterfaceStateMachine
                0x9d00ea34                BootloaderResetStateMachine
                0x9d00ea90                BootloaderActivateBootloader
                0x9d00ead0                BootloaderDeactivateBootloader
                0x9d00eb00                BootloaderFlashEraseStateMachine
                0x9d00ed34                ResetBootloaderFlashEraseStateMachine
                0x9d00ed68                BootloaderFlashWriteStateMachine
                0x9d00ef94                BootloaderPrintFlashData
                0x9d00efb4                BootloaderCheckFlashBootloaderData
                0x9d00f2d8                ResetBootloaderFlashWriteStateMachine
                0x9d00f318                BootloaderBytesToInt
                0x9d00f3d0                BootloaderIntToBytes
 .text          0x9d00f490     0x167c build/ChaletDuinoV2_795F512H_/debug/Source/winc3400_142/driver/source/nmasic.o
                0x9d00f490                chip_apply_conf
                0x9d00f544                chip_idle
                0x9d00f5b8                enable_rf_blocks
                0x9d00f658                enable_interrupts
                0x9d00f768                cpu_start
                0x9d00f934                nmi_get_chipid
                0x9d00fb4c                nmi_get_rfrevid
                0x9d00fb98                restore_pmu_settings_after_global_reset
                0x9d00fbec                nmi_update_pll
                0x9d00fc60                nmi_set_sys_clk_src_to_xo
                0x9d00fcbc                chip_sleep
                0x9d00fe24                chip_wake
                0x9d00ffe4                chip_reset_and_cpu_halt
                0x9d010178                chip_reset
                0x9d0101d8                wait_for_bootrom
                0x9d010388                wait_for_firmware_start
                0x9d0104a8                chip_deinit
                0x9d0105c4                set_gpio_dir
                0x9d010698                set_gpio_val
                0x9d01076c                get_gpio_val
                0x9d0107f8                pullup_ctrl
                0x9d0108b0                nmi_get_otp_mac_address
                0x9d010a10                nmi_get_mac_address
 .text          0x9d010b0c     0x14b8 build/ChaletDuinoV2_795F512H_/debug/Source/winc3400_142/driver/source/nmspi.o
                0x9d011a54                nm_spi_reset
                0x9d011aa8                nm_spi_lock_init
                0x9d011ac8                nm_spi_init
                0x9d011c80                nm_spi_deinit
                0x9d011ca8                nm_spi_read_reg
                0x9d011cec                nm_spi_read_reg_with_ret
                0x9d011d7c                nm_spi_write_reg
                0x9d011e0c                nm_spi_read_block
                0x9d011f00                nm_spi_write_block
 .text          0x9d011fc4     0x1384 build/ChaletDuinoV2_795F512H_/debug/Source/winc3400_142/driver/source/m2m_hif.o
                0x9d0120c8                hif_chip_wake
                0x9d012190                hif_set_sleep_mode
                0x9d0121c4                hif_get_sleep_mode
                0x9d012250                hif_chip_sleep
                0x9d0122f4                hif_init
                0x9d012354                hif_deinit
                0x9d0123ac                hif_check_compatibility
                0x9d012424                hif_enable_access
                0x9d01255c                hif_check_code
                0x9d012650                hif_send
                0x9d013048                hif_handle_isr
                0x9d013084                hif_receive
                0x9d013230                hif_register_cb
 .text          0x9d013348     0x1228 build/ChaletDuinoV2_795F512H_/debug/Source/winc3400_142/spi_flash/source/spi_flash.o
                0x9d0140ac                spi_flash_read
                0x9d014184                spi_flash_write
                0x9d01435c                spi_flash_erase
                0x9d0144f0                spi_flash_get_size
 .text          0x9d014570      0xddc build/ChaletDuinoV2_795F512H_/debug/Source/SPI_Flash.o
                0x9d014570                InitSPIFlash
                0x9d0146e8                SPIFlashCheckAndConfigure
                0x9d0147c4                SPIFlashIsPresent
                0x9d0147e8                SPIFlashWriteEnable
                0x9d01484c                SPIFlashReadStatusReg
                0x9d0148f4                SPIFlashCheckBusy
                0x9d014950                SPIFlashCheckChipID
                0x9d014a8c                SPIFlashReadBuffer
                0x9d014c0c                SPIFlashEraseSector
                0x9d014d34                SPIFlashErase64KSector
                0x9d014e88                SPIFlashWriteSectorWorkingBuffer
                0x9d015044                SPIFlashWriteByte
                0x9d015198                SPIFlashWriteBuffer
 .text          0x9d01534c      0xd98 build/ChaletDuinoV2_795F512H_/debug/Source/winc3400_142/driver/source/m2m_ssl.o
                0x9d015658                m2m_ssl_init
                0x9d0156b8                m2m_ssl_handshake_rsp
                0x9d015730                m2m_ssl_send_certs_to_winc
                0x9d015a78                m2m_ssl_retrieve_next_for_verifying
                0x9d015eac                m2m_ssl_retrieve_cert
                0x9d015f24                m2m_ssl_retrieve_hash
                0x9d015fe8                m2m_ssl_stop_retrieving
                0x9d016028                m2m_ssl_stop_processing_certs
                0x9d016058                m2m_ssl_ecc_process_done
                0x9d01607c                m2m_ssl_set_active_ciphersuites

.dinit          0x9d0160e4      0xd60
 .dinit         0x9d0160e4      0xd60 data_init

.text           0x9d016e44     0x4844
 .text          0x9d016e44      0xd54 build/ChaletDuinoV2_795F512H_/debug/Source/BootloaderProtocol.o
                0x9d016e44                BootloaderProtocolInit
                0x9d016e74                BootloaderProtocolStateMachine
                0x9d0173c4                BootloaderProtocolProtocolAnalyzeNewData
                0x9d017440                BootloaderProtocolResetStateMachine
                0x9d017494                BootloaderProtocolSendFrame
                0x9d017660                BootloaderProtocolGetDataBufferPtr
                0x9d017684                BootloaderProtocolSendHeartbeat
                0x9d0176cc                BootloaderProtocolSendACK
                0x9d017720                BootloaderProtocolSendNACK
                0x9d017770                BootloaderProtocolSendInitUploadResponse
                0x9d0178d0                BootloaderProtocolSendDataChunkResult
                0x9d0179c4                BootloaderProtocolSendBootloaderState
                0x9d017a28                BootloaderProtocolSendFirmwareUploadResult
                0x9d017a8c                BootloaderProtocolSendFlashCheckResult
                0x9d017af0                BootloaderProtocolSendStoredFirmwareInfoResponse
 .text          0x9d017b98      0xce8 build/ChaletDuinoV2_795F512H_/debug/Source/Util.o
                0x9d017b98                SwapEndianShort
                0x9d017be4                SwapEndianInt
                0x9d017c40                ConvertIntToStrLeadingZero
                0x9d018064                ConvertIntToStr
                0x9d0183b8                ConvertCharToStrLeadingZero
                0x9d018520                ConvertStrToValue
                0x9d01870c                ConvertCharToStr
                0x9d0187c4                Crc8
                0x9d01885c                Delay
 .text          0x9d018880      0xbac build/ChaletDuinoV2_795F512H_/debug/Source/winc3400_142/driver/source/m2m_flash.o
                0x9d018fc4                m2m_flash_erase_sector
                0x9d019100                m2m_flash_write
                0x9d019238                m2m_flash_read
                0x9d019370                m2m_flash_switch_firmware
 .text          0x9d01942c      0xb98 build/ChaletDuinoV2_795F512H_/debug/Source/timer.o
                0x9d01942c                TimerInit
                0x9d0194fc                IsMilliSecTimerExpired
                0x9d019664                IsSecTimerExpired
                0x9d0197c8                IsTimerExpired
                0x9d019b7c                TimerStart
                0x9d019ca4                TimerStartSeconds
                0x9d019d48                TimerReset
                0x9d019dcc                IsTimerRunning
                0x9d019e10                TimerStop
                0x9d019e54                Sleep
                0x9d019eb0                Timer1MilliSecInterrupt
 .text          0x9d019fc4      0xb88 build/ChaletDuinoV2_795F512H_/debug/Source/Terminal.o
                0x9d019fc4                InitTerminal
                0x9d01a044                TickTerminal
                0x9d01a0a0                RxTerminalBuf
                0x9d01a12c                RxTerminalData
                0x9d01a27c                ParseNewBuffer
                0x9d01aa98                TerminalPrintString
                0x9d01aaec                TerminalPrintChar
                0x9d01ab2c                TerminalStateMachine
 .text          0x9d01ab4c      0xb3c build/ChaletDuinoV2_795F512H_/debug/Source/NetworkProtocol.o
                0x9d01ab4c                ProtocolInit
                0x9d01abc8                StateMachine
                0x9d01b280                ProtocolAnalyzeNewData
                0x9d01b30c                ResetStateMachine
                0x9d01b37c                ProtocolExecCmd
                0x9d01b39c                ProtocolAcknowledge
                0x9d01b400                ProtocolCalcCrc
                0x9d01b47c                ProtocolIsReceiving
                0x9d01b49c                ProtocolGetFrame
                0x9d01b65c                ProtocolMsgDataPtr

.text._vfprintf_cdnopsuxX
                0x9d01b688      0xae8
 .text._vfprintf_cdnopsuxX
                0x9d01b688      0xae8 c:/program files/microchip/xc32/v1.33/bin/bin/../../lib/gcc/pic32mx/4.5.2/../../../../pic32mx/lib\libc.a(doprnt_cdnopsuxX.eo)
                0x9d01b688                _vfprintf_cdnopsuxX
                0x9d01b688                _vfprintf_cdnopuxX

.text._vfscanf_s
                0x9d01c170      0x868
 .text._vfscanf_s
                0x9d01c170      0x868 c:/program files/microchip/xc32/v1.33/bin/bin/../../lib/gcc/pic32mx/4.5.2/../../../../pic32mx/lib\libc.a(doscan_s.eo)
                0x9d01c170                _vfscanf_s
                0x9d01c170                _vfscanf_0

.rodata         0x9d01c9d8      0x7b8
 .rodata        0x9d01c9d8      0x7b8 build/ChaletDuinoV2_795F512H_/debug/Source/BootloaderInterface.o

.text           0x9d01d190     0x286c
 .text          0x9d01d190      0x74c build/ChaletDuinoV2_795F512H_/debug/Source/winc3400_142/driver/source/nmdrv.o
                0x9d01d190                nm_get_hif_info
                0x9d01d230                nm_get_firmware_full_info
                0x9d01d3c0                nm_get_ota_firmware_info
                0x9d01d550                nm_drv_init_download_mode
                0x9d01d5d4                nm_drv_init_hold
                0x9d01d650                nm_drv_init_start
                0x9d01d7a0                nm_drv_init
                0x9d01d7fc                nm_drv_deinit
                0x9d01d880                nm_cpu_start
                0x9d01d8b8                nm_get_state
 .text          0x9d01d8dc      0x6c0 build/ChaletDuinoV2_795F512H_/debug/Source/main.o
                0x9d01d8dc                main
                0x9d01df5c                _mon_putc
 .text          0x9d01df9c      0x69c build/ChaletDuinoV2_795F512H_/debug/Source/VolumeTransducer.o
                0x9d01df9c                VolumeTransducerInit
                0x9d01e100                VolumeTransducerTick
                0x9d01e3b8                BureauTransducerInterrupt
                0x9d01e4f8                CuisineTransducerInterrupt
 .text          0x9d01e638      0x638 build/ChaletDuinoV2_795F512H_/debug/Source/ChaletduinoV2Board.o
                0x9d01e638                InitBoard
 .text          0x9d01ec70      0x4e4 build/ChaletDuinoV2_795F512H_/debug/Source/winc3400_142/driver/source/nmbus.o
                0x9d01ecd8                nm_bus_iface_init
                0x9d01ed1c                nm_bus_iface_deinit
                0x9d01ed58                nm_bus_reset
                0x9d01ed88                nm_bus_iface_reconfigure
                0x9d01edb4                nm_read_reg
                0x9d01edec                nm_read_reg_with_ret
                0x9d01ee2c                nm_write_reg
                0x9d01eebc                nm_read_block
                0x9d01f030                nm_write_block
 .text          0x9d01f154      0x45c c:/program files/microchip/xc32/v1.33/bin/bin/../../lib/gcc/pic32mx/4.5.2\libgcc.a(_umoddi3.o)
                0x9d01f154                __umoddi3
 .text          0x9d01f5b0      0x44c c:/program files/microchip/xc32/v1.33/bin/bin/../../lib/gcc/pic32mx/4.5.2\libgcc.a(_udivdi3.o)
                0x9d01f5b0                __udivdi3

.rodata         0x9d01f9fc      0x804
 .rodata        0x9d01f9fc      0x404 build/ChaletDuinoV2_795F512H_/debug/Source/Util.o
                0x9d01fa00                CRC8_TABLE
 .rodata        0x9d01fe00      0x400 build/ChaletDuinoV2_795F512H_/debug/Source/Terminal.o

.text           0x9d020200      0xf50
 .text          0x9d020200      0x380 build/ChaletDuinoV2_795F512H_/debug/Source/winc3400_142/driver/source/m2m_periph.o
                0x9d020410                m2m_periph_init
                0x9d020438                m2m_periph_gpio_set_dir
                0x9d020490                m2m_periph_gpio_set_val
                0x9d0204e8                m2m_periph_gpio_get_val
                0x9d020538                m2m_periph_pullup_ctrl
 .text          0x9d020580      0x340 build/ChaletDuinoV2_795F512H_/debug/Source/Syslog.o
                0x9d020580                InitSyslog
                0x9d0205d8                SyslogTick
                0x9d020674                SyslogNewByte
                0x9d020728                SyslogNewString
                0x9d0207a0                SyslogIsBufferEmpty
                0x9d0207dc                SyslogSetLTEPassthrough
                0x9d020858                RxSyslogBuf
 .text          0x9d0208c0      0x33c build/ChaletDuinoV2_795F512H_/debug/Source/winc3400_142/driver/source/m2m_ota.o
                0x9d02097c                m2m_ota_init
                0x9d0209d8                m2m_ota_start_update
                0x9d020a54                m2m_ota_rollback
                0x9d020afc                m2m_ota_abort
                0x9d020b54                m2m_ota_switch_firmware
 .text          0x9d020bfc      0x2e8 build/ChaletDuinoV2_795F512H_/debug/Source/winc3400_142/common/source/nm_common.o
                0x9d020bfc                chip_isr
                0x9d020c74                nm_sleep
                0x9d020cac                nm_reset
                0x9d020dc4                hexstr_2_bytes
 .text          0x9d020ee4      0x26c build/ChaletDuinoV2_795F512H_/debug/Source/crc32.o
                0x9d020ee4                crc_32
                0x9d020fdc                update_crc_32

.rodata         0x9d021150      0x25c
 .rodata        0x9d021150      0x25c build/ChaletDuinoV2_795F512H_/debug/Source/WiFiCtrl.o

.text           0x9d0213ac      0x810
 .text          0x9d0213ac      0x250 build/ChaletDuinoV2_795F512H_/debug/Source/DACInterface.o
                0x9d0213ac                DACInit
                0x9d02146c                DACSetValue
 .text          0x9d0215fc      0x244 build/ChaletDuinoV2_795F512H_/debug/Source/winc3400_142/socket/source/inet_addr.o
                0x9d0215fc                inet_addr
 .text          0x9d021840      0x1dc build/ChaletDuinoV2_795F512H_/debug/Source/winc3400_142/socket/source/inet_ntop.o
                0x9d021840                inet_ntop
 .text          0x9d021a1c      0x1a0 c:/program files/microchip/xc32/v1.33/bin/bin/../../lib/gcc/pic32mx/4.5.2/../../../../pic32mx/lib\libpic32.a(strcpy.o)
                0x9d021a1c                strcpy

.text._filbuf   0x9d021bbc      0x188
 .text._filbuf  0x9d021bbc      0x188 c:/program files/microchip/xc32/v1.33/bin/bin/../../lib/gcc/pic32mx/4.5.2/../../../../pic32mx/lib\libc.a(filbuf.o)
                0x9d021bbc                _filbuf

.text.read      0x9d021d44      0x174
 .text.read     0x9d021d44      0x174 c:/program files/microchip/xc32/v1.33/bin/bin/../../lib/gcc/pic32mx/4.5.2/../../../../pic32mx/lib\libpic32.a(read.o)
                0x9d021d44                read

.text           0x9d021eb8      0x2d0
 .text          0x9d021eb8      0x168 c:/program files/microchip/xc32/v1.33/bin/bin/../../lib/gcc/pic32mx/4.5.2/../../../../pic32mx/lib\libpic32.a(memcpy.o)
                0x9d021eb8                memcpy
 .text          0x9d022020      0x168 c:/program files/microchip/xc32/v1.33/bin/bin/../../lib/gcc/pic32mx/4.5.2/../../../../pic32mx/lib\libpic32.a(strlen.o)
                0x9d022020                strlen

.text.fputc     0x9d022188      0x15c
 .text.fputc    0x9d022188      0x15c c:/program files/microchip/xc32/v1.33/bin/bin/../../lib/gcc/pic32mx/4.5.2/../../../../pic32mx/lib\libc.a(_fputc_simple.o)
                0x9d022188                fputc

.text._flsbuf   0x9d0222e4      0x12c
 .text._flsbuf  0x9d0222e4      0x12c c:/program files/microchip/xc32/v1.33/bin/bin/../../lib/gcc/pic32mx/4.5.2/../../../../pic32mx/lib\libc.a(_flsbuf_simple.o)
                0x9d0222e4                _flsbuf

.text.fgetc     0x9d022410      0x108
 .text.fgetc    0x9d022410      0x108 c:/program files/microchip/xc32/v1.33/bin/bin/../../lib/gcc/pic32mx/4.5.2/../../../../pic32mx/lib\libc.a(fgetc.o)
                0x9d022410                fgetc

.rodata         0x9d022518      0x204
 .rodata        0x9d022518      0x104 c:/program files/microchip/xc32/v1.33/bin/bin/../../lib/gcc/pic32mx/4.5.2/../../../../pic32mx/lib\libc.a(ctype.o)
                0x9d022518                _ctype
 .rodata        0x9d02261c      0x100 build/ChaletDuinoV2_795F512H_/debug/Source/winc3400_142/driver/source/nmspi.o

.text.general_exception
                0x9d02271c       0xdc
 .text.general_exception
                0x9d02271c       0xdc c:/program files/microchip/xc32/v1.33/bin/bin/../../lib/gcc/pic32mx/4.5.2/../../../../pic32mx/lib\libpic32.a(general-exception.o)
                0x9d02271c                _general_exception_context

.text           0x9d0227f8       0xd8
 .text          0x9d0227f8       0xd8 build/ChaletDuinoV2_795F512H_/debug/Source/Watchdog.o
                0x9d0227f8                InitWatchdog
                0x9d02284c                EnableWatchdog
                0x9d022878                DisableWatchdog
                0x9d0228a4                KickWatchdog

.rodata         0x9d0228d0      0x198
 .rodata        0x9d0228d0       0xd0 c:/program files/microchip/xc32/v1.33/bin/bin/../../lib/gcc/pic32mx/4.5.2/../../../../pic32mx/lib\libc.a(doprnt_cdnopsuxX.eo)
 .rodata        0x9d0229a0       0xc8 build/ChaletDuinoV2_795F512H_/debug/Source/SPI_Flash.o

.text           0x9d022a68       0xa8
 .text          0x9d022a68       0xa8 c:/program files/microchip/xc32/v1.33/bin/bin/../../lib/gcc/pic32mx/4.5.2/../../../../pic32mx/lib\libpic32.a(memset.o)
                0x9d022a68                memset

.text.atoi      0x9d022b10       0xa8
 .text.atoi     0x9d022b10       0xa8 c:/program files/microchip/xc32/v1.33/bin/bin/../../lib/gcc/pic32mx/4.5.2/../../../../pic32mx/lib\libc.a(atoi.o)
                0x9d022b10                atoi

.text.range     0x9d022bb8       0xa0
 .text.range    0x9d022bb8       0xa0 c:/program files/microchip/xc32/v1.33/bin/bin/../../lib/gcc/pic32mx/4.5.2/../../../../pic32mx/lib\libc.a(doscan_s.eo)

.text           0x9d022c58       0x98
 .text          0x9d022c58       0x98 c:/program files/microchip/xc32/v1.33/bin/bin/../../lib/gcc/pic32mx/4.5.2/../../../../pic32mx/lib\libpic32.a(memcmp.o)
                0x9d022c58                memcmp

.text.fflush    0x9d022cf0       0x94
 .text.fflush   0x9d022cf0       0x94 c:/program files/microchip/xc32/v1.33/bin/bin/../../lib/gcc/pic32mx/4.5.2/../../../../pic32mx/lib\libc.a(fflush.o)
                0x9d022cf0                fflush

.text.write     0x9d022d84       0x94
 .text.write    0x9d022d84       0x94 c:/program files/microchip/xc32/v1.33/bin/bin/../../lib/gcc/pic32mx/4.5.2/../../../../pic32mx/lib\libpic32.a(write.o)
                0x9d022d84                write

.text.SoftReset
                0x9d022e18       0x78
 .text.SoftReset
                0x9d022e18       0x78 c:/program files/microchip/xc32/v1.33/bin/bin/../../lib/gcc/pic32mx/4.5.2/../../../../pic32mx/lib\libmchp_peripheral_32MX795F512H.a(soft_reset_lib.o)
                0x9d022e18                SoftReset

.text.fputs     0x9d022e90       0x78
 .text.fputs    0x9d022e90       0x78 c:/program files/microchip/xc32/v1.33/bin/bin/../../lib/gcc/pic32mx/4.5.2/../../../../pic32mx/lib\libc.a(puts.o)
                0x9d022e90                fputs

.text.strncmp   0x9d022f08       0x78
 .text.strncmp  0x9d022f08       0x78 c:/program files/microchip/xc32/v1.33/bin/bin/../../lib/gcc/pic32mx/4.5.2/../../../../pic32mx/lib\libc.a(strncmp.o)
                0x9d022f08                strncmp

.text.ungetc    0x9d022f80       0x74
 .text.ungetc   0x9d022f80       0x74 c:/program files/microchip/xc32/v1.33/bin/bin/../../lib/gcc/pic32mx/4.5.2/../../../../pic32mx/lib\libc.a(ungetc.o)
                0x9d022f80                ungetc

.text           0x9d022ff4       0x70
 .text          0x9d022ff4       0x70 build/ChaletDuinoV2_795F512H_/debug/Source/SPI.o
                0x9d022ff4                SPITransaction

.text._sprintf_cdnopuxX
                0x9d023064       0x68
 .text._sprintf_cdnopuxX
                0x9d023064       0x68 c:/program files/microchip/xc32/v1.33/bin/bin/../../lib/gcc/pic32mx/4.5.2/../../../../pic32mx/lib\libc.a(sprintf_cdnopuxX.eo)
                0x9d023064                _sprintf_cdnopuxX

.text.wspace    0x9d0230cc       0x60
 .text.wspace   0x9d0230cc       0x60 c:/program files/microchip/xc32/v1.33/bin/bin/../../lib/gcc/pic32mx/4.5.2/../../../../pic32mx/lib\libc.a(doscan_s.eo)

.text           0x9d02312c       0x58
 .text          0x9d02312c       0x58 build/ChaletDuinoV2_795F512H_/debug/Source/exceptions.o
                0x9d02312c                _general_exception_handler

.text._sscanf_s
                0x9d023184       0x54
 .text._sscanf_s
                0x9d023184       0x54 c:/program files/microchip/xc32/v1.33/bin/bin/../../lib/gcc/pic32mx/4.5.2/../../../../pic32mx/lib\libc.a(sscanf_s.eo)
                0x9d023184                _sscanf_s
                0x9d023184                _sscanf_0

.rodata         0x9d0231d8       0x50
 .rodata        0x9d0231d8       0x50 build/ChaletDuinoV2_795F512H_/debug/Source/winc3400_142/driver/source/m2m_flash.o

.text.main_entry
                0x9d023228       0x4c
 .text.main_entry
                0x9d023228       0x4c c:/program files/microchip/xc32/v1.33/bin/bin/../../lib/gcc/pic32mx/4.5.2/../../../../pic32mx/lib/./proc/32MX795F512H/crt0_mips32r2.o
                0x9d023254                __crt0_exit

.rodata         0x9d023274       0x48
 .rodata        0x9d023274       0x48 build/ChaletDuinoV2_795F512H_/debug/Source/Syslog.o

.text._bootstrap_exception_handler
                0x9d0232bc       0x48
 .text._bootstrap_exception_handler
                0x9d0232bc       0x48 c:/program files/microchip/xc32/v1.33/bin/bin/../../lib/gcc/pic32mx/4.5.2/../../../../pic32mx/lib\libpic32.a(default-bootstrap-exception-handler.o)
                0x9d0232bc                _bootstrap_exception_handler

.text           0x9d023304       0x44
 .text          0x9d023304       0x44 c:/program files/microchip/xc32/v1.33/bin/bin/../../lib/gcc/pic32mx/4.5.2/../../../../pic32mx/lib\pic32_software_reset.o
                0x9d023304                __pic32_software_reset

.text.puts      0x9d023348       0x44
 .text.puts     0x9d023348       0x44 c:/program files/microchip/xc32/v1.33/bin/bin/../../lib/gcc/pic32mx/4.5.2/../../../../pic32mx/lib\libc.a(puts.o)
                0x9d023348                puts

.text._printf_cdnopsuxX
                0x9d02338c       0x40
 .text._printf_cdnopsuxX
                0x9d02338c       0x40 c:/program files/microchip/xc32/v1.33/bin/bin/../../lib/gcc/pic32mx/4.5.2/../../../../pic32mx/lib\libc.a(printf_cdnopsuxX.eo)
                0x9d02338c                _printf_cdnopuxX
                0x9d02338c                _printf_cdnopsuxX

.vector_default
                0x9d0233cc       0x38
 .vector_default
                0x9d0233cc       0x38 c:/program files/microchip/xc32/v1.33/bin/bin/../../lib/gcc/pic32mx/4.5.2/../../../../pic32mx/lib\libpic32.a(defaultinterrupt.o)
                0x9d0233cc                _DefaultInterrupt

.rodata         0x9d023404       0x30
 .rodata        0x9d023404       0x30 build/ChaletDuinoV2_795F512H_/debug/Source/main.o

.text.INTConfigureSystem
                0x9d023434       0x30
 .text.INTConfigureSystem
                0x9d023434       0x30 c:/program files/microchip/xc32/v1.33/bin/bin/../../lib/gcc/pic32mx/4.5.2/../../../../pic32mx/lib\libmchp_peripheral_32MX795F512H.a(int_configure_system_lib.o)
                0x9d023434                INTConfigureSystem

.text.tolower   0x9d023464       0x24
 .text.tolower  0x9d023464       0x24 c:/program files/microchip/xc32/v1.33/bin/bin/../../lib/gcc/pic32mx/4.5.2/../../../../pic32mx/lib\libc.a(ctypef.o)
                0x9d023464                tolower

.text.toupper   0x9d023488       0x24
 .text.toupper  0x9d023488       0x24 c:/program files/microchip/xc32/v1.33/bin/bin/../../lib/gcc/pic32mx/4.5.2/../../../../pic32mx/lib\libc.a(ctypef.o)
                0x9d023488                toupper

.text           0x9d0234ac       0x20
 .text          0x9d0234ac       0x20 build/ChaletDuinoV2_795F512H_/debug/Source/DigitalIO.o
                0x9d0234ac                InitDigitalIO

.rodata         0x9d0234cc       0x1c
 .rodata        0x9d0234cc       0x1c build/ChaletDuinoV2_795F512H_/debug/Source/VolumeTransducer.o

.text.INTRestoreInterrupts
                0x9d0234e8       0x1c
 .text.INTRestoreInterrupts
                0x9d0234e8       0x1c c:/program files/microchip/xc32/v1.33/bin/bin/../../lib/gcc/pic32mx/4.5.2/../../../../pic32mx/lib\libmchp_peripheral_32MX795F512H.a(int_restore_interrupts_lib.o)
                0x9d0234e8                INTRestoreInterrupts

.rodata         0x9d023504       0x18
 .rodata        0x9d023504       0x18 build/ChaletDuinoV2_795F512H_/debug/Source/Watchdog.o

.text.CheKseg0CacheOff
                0x9d02351c       0x18
 .text.CheKseg0CacheOff
                0x9d02351c       0x18 c:/program files/microchip/xc32/v1.33/bin/bin/../../lib/gcc/pic32mx/4.5.2/../../../../pic32mx/lib\libmchp_peripheral_32MX795F512H.a(pcache.o)
                0x9d02351c                CheKseg0CacheOff

.text.CheKseg0CacheOn
                0x9d023534       0x18
 .text.CheKseg0CacheOn
                0x9d023534       0x18 c:/program files/microchip/xc32/v1.33/bin/bin/../../lib/gcc/pic32mx/4.5.2/../../../../pic32mx/lib\libmchp_peripheral_32MX795F512H.a(pcache.o)
                0x9d023534                CheKseg0CacheOn

.text           0x9d02354c       0x18
 .text          0x9d02354c       0x18 c:/program files/microchip/xc32/v1.33/bin/bin/../../lib/gcc/pic32mx/4.5.2/../../../../pic32mx/lib\libpic32.a(default-nmi-handler.o)
                0x9d02354c                _nmi_handler

.text.isalnum   0x9d023564       0x18
 .text.isalnum  0x9d023564       0x18 c:/program files/microchip/xc32/v1.33/bin/bin/../../lib/gcc/pic32mx/4.5.2/../../../../pic32mx/lib\libc.a(ctypef.o)
                0x9d023564                isalnum

.text.isalpha   0x9d02357c       0x18
 .text.isalpha  0x9d02357c       0x18 c:/program files/microchip/xc32/v1.33/bin/bin/../../lib/gcc/pic32mx/4.5.2/../../../../pic32mx/lib\libc.a(ctypef.o)
                0x9d02357c                isalpha

.text.iscntrl   0x9d023594       0x18
 .text.iscntrl  0x9d023594       0x18 c:/program files/microchip/xc32/v1.33/bin/bin/../../lib/gcc/pic32mx/4.5.2/../../../../pic32mx/lib\libc.a(ctypef.o)
                0x9d023594                iscntrl

.text.isdigit   0x9d0235ac       0x18
 .text.isdigit  0x9d0235ac       0x18 c:/program files/microchip/xc32/v1.33/bin/bin/../../lib/gcc/pic32mx/4.5.2/../../../../pic32mx/lib\libc.a(ctypef.o)
                0x9d0235ac                isdigit

.text.isgraph   0x9d0235c4       0x18
 .text.isgraph  0x9d0235c4       0x18 c:/program files/microchip/xc32/v1.33/bin/bin/../../lib/gcc/pic32mx/4.5.2/../../../../pic32mx/lib\libc.a(ctypef.o)
                0x9d0235c4                isgraph

.text.islower   0x9d0235dc       0x18
 .text.islower  0x9d0235dc       0x18 c:/program files/microchip/xc32/v1.33/bin/bin/../../lib/gcc/pic32mx/4.5.2/../../../../pic32mx/lib\libc.a(ctypef.o)
                0x9d0235dc                islower

.text.isprint   0x9d0235f4       0x18
 .text.isprint  0x9d0235f4       0x18 c:/program files/microchip/xc32/v1.33/bin/bin/../../lib/gcc/pic32mx/4.5.2/../../../../pic32mx/lib\libc.a(ctypef.o)
                0x9d0235f4                isprint

.text.ispunct   0x9d02360c       0x18
 .text.ispunct  0x9d02360c       0x18 c:/program files/microchip/xc32/v1.33/bin/bin/../../lib/gcc/pic32mx/4.5.2/../../../../pic32mx/lib\libc.a(ctypef.o)
                0x9d02360c                ispunct

.text.isspace   0x9d023624       0x18
 .text.isspace  0x9d023624       0x18 c:/program files/microchip/xc32/v1.33/bin/bin/../../lib/gcc/pic32mx/4.5.2/../../../../pic32mx/lib\libc.a(ctypef.o)
                0x9d023624                isspace

.text.isupper   0x9d02363c       0x18
 .text.isupper  0x9d02363c       0x18 c:/program files/microchip/xc32/v1.33/bin/bin/../../lib/gcc/pic32mx/4.5.2/../../../../pic32mx/lib\libc.a(ctypef.o)
                0x9d02363c                isupper

.text.isxdigit  0x9d023654       0x18
 .text.isxdigit
                0x9d023654       0x18 c:/program files/microchip/xc32/v1.33/bin/bin/../../lib/gcc/pic32mx/4.5.2/../../../../pic32mx/lib\libc.a(ctypef.o)
                0x9d023654                isxdigit

.text.__exception_handler_break
                0x9d02366c        0xc
 .text.__exception_handler_break
                0x9d02366c        0xc c:/program files/microchip/xc32/v1.33/bin/bin/../../lib/gcc/pic32mx/4.5.2/../../../../pic32mx/lib\software-debug-break.o
                0x9d02366c                __exception_handler_break

.rodata         0x9d023678        0x8
 .rodata        0x9d023678        0x8 build/ChaletDuinoV2_795F512H_/debug/Source/BootloaderProtocol.o

.text.INTEnableInterrupts
                0x9d023680        0x8
 .text.INTEnableInterrupts
                0x9d023680        0x8 c:/program files/microchip/xc32/v1.33/bin/bin/../../lib/gcc/pic32mx/4.5.2/../../../../pic32mx/lib\libmchp_peripheral_32MX795F512H.a(int_enable_interrupts_lib.o)
                0x9d023680                INTEnableInterrupts

.text.INTDisableInterrupts
                0x9d023688        0x8
 .text.INTDisableInterrupts
                0x9d023688        0x8 c:/program files/microchip/xc32/v1.33/bin/bin/../../lib/gcc/pic32mx/4.5.2/../../../../pic32mx/lib\libmchp_peripheral_32MX795F512H.a(int_disable_interrupts_lib.o)
                0x9d023688                INTDisableInterrupts

.text._on_reset
                0x9d023690        0x8
 .text._on_reset
                0x9d023690        0x8 c:/program files/microchip/xc32/v1.33/bin/bin/../../lib/gcc/pic32mx/4.5.2/../../../../pic32mx/lib\libpic32.a(default-on-reset.o)
                0x9d023690                _on_reset

.text._on_bootstrap
                0x9d023698        0x8
 .text._on_bootstrap
                0x9d023698        0x8 c:/program files/microchip/xc32/v1.33/bin/bin/../../lib/gcc/pic32mx/4.5.2/../../../../pic32mx/lib\libpic32.a(default-on-bootstrap.o)
                0x9d023698                _on_bootstrap

.text.close     0x9d0236a0        0x8
 .text.close    0x9d0236a0        0x8 c:/program files/microchip/xc32/v1.33/bin/bin/../../lib/gcc/pic32mx/4.5.2/../../../../pic32mx/lib\libpic32.a(close.o)
                0x9d0236a0                close

.text.isascii   0x9d0236a8        0x8
 .text.isascii  0x9d0236a8        0x8 c:/program files/microchip/xc32/v1.33/bin/bin/../../lib/gcc/pic32mx/4.5.2/../../../../pic32mx/lib\libc.a(ctypef.o)
                0x9d0236a8                isascii

.text.toascii   0x9d0236b0        0x8
 .text.toascii  0x9d0236b0        0x8 c:/program files/microchip/xc32/v1.33/bin/bin/../../lib/gcc/pic32mx/4.5.2/../../../../pic32mx/lib\libc.a(ctypef.o)
                0x9d0236b0                toascii

.text._tolower  0x9d0236b8        0x8
 .text._tolower
                0x9d0236b8        0x8 c:/program files/microchip/xc32/v1.33/bin/bin/../../lib/gcc/pic32mx/4.5.2/../../../../pic32mx/lib\libc.a(ctypef.o)
                0x9d0236b8                _tolower

.text._toupper  0x9d0236c0        0x8
 .text._toupper
                0x9d0236c0        0x8 c:/program files/microchip/xc32/v1.33/bin/bin/../../lib/gcc/pic32mx/4.5.2/../../../../pic32mx/lib\libc.a(ctypef.o)
                0x9d0236c0                _toupper

.text%z270      0x00000000        0x0
 .text          0x00000000        0x0 c:/program files/microchip/xc32/v1.33/bin/bin/../../lib/gcc/pic32mx/4.5.2/../../../../pic32mx/lib\libpic32.a(xc32_uart.o)

.text%z271      0x00000000        0x0
 .text          0x00000000        0x0 c:/program files/microchip/xc32/v1.33/bin/bin/../../lib/gcc/pic32mx/4.5.2/../../../../pic32mx/lib\libpic32.a(write.o)

.text%z272      0x00000000        0x0
 .text          0x00000000        0x0 c:/program files/microchip/xc32/v1.33/bin/bin/../../lib/gcc/pic32mx/4.5.2/../../../../pic32mx/lib\libpic32.a(read.o)

.text%z273      0x00000000        0x0
 .text          0x00000000        0x0 c:/program files/microchip/xc32/v1.33/bin/bin/../../lib/gcc/pic32mx/4.5.2/../../../../pic32mx/lib\libc.a(fflush.o)

.text%z274      0x00000000        0x0
 .text          0x00000000        0x0 c:/program files/microchip/xc32/v1.33/bin/bin/../../lib/gcc/pic32mx/4.5.2/../../../../pic32mx/lib\libc.a(filbuf.o)

.text%z275      0x00000000        0x0
 .text          0x00000000        0x0 c:/program files/microchip/xc32/v1.33/bin/bin/../../lib/gcc/pic32mx/4.5.2/../../../../pic32mx/lib\libc.a(ungetc.o)

.text%z276      0x00000000        0x0
 .text          0x00000000        0x0 c:/program files/microchip/xc32/v1.33/bin/bin/../../lib/gcc/pic32mx/4.5.2/../../../../pic32mx/lib\libc.a(ctypef.o)

.text%z277      0x00000000        0x0
 .text          0x00000000        0x0 c:/program files/microchip/xc32/v1.33/bin/bin/../../lib/gcc/pic32mx/4.5.2/../../../../pic32mx/lib\libc.a(ctype.o)

.text%z278      0x00000000        0x0
 .text          0x00000000        0x0 c:/program files/microchip/xc32/v1.33/bin/bin/../../lib/gcc/pic32mx/4.5.2/../../../../pic32mx/lib\libc.a(atoi.o)

.text%z279      0x00000000        0x0
 .text          0x00000000        0x0 c:/program files/microchip/xc32/v1.33/bin/bin/../../lib/gcc/pic32mx/4.5.2/../../../../pic32mx/lib\libc.a(fgetc.o)

.text%z280      0x00000000        0x0
 .text          0x00000000        0x0 c:/program files/microchip/xc32/v1.33/bin/bin/../../lib/gcc/pic32mx/4.5.2/../../../../pic32mx/lib\libc.a(_flsbuf_simple.o)

.text%z281      0x00000000        0x0
 .text          0x00000000        0x0 c:/program files/microchip/xc32/v1.33/bin/bin/../../lib/gcc/pic32mx/4.5.2/../../../../pic32mx/lib\libc.a(doscan_s.eo)

.text%z282      0x00000000        0x0
 .text          0x00000000        0x0 c:/program files/microchip/xc32/v1.33/bin/bin/../../lib/gcc/pic32mx/4.5.2/../../../../pic32mx/lib\libc.a(doprnt_cdnopsuxX.eo)

.text%z283      0x00000000        0x0
 .text          0x00000000        0x0 c:/program files/microchip/xc32/v1.33/bin/bin/../../lib/gcc/pic32mx/4.5.2/../../../../pic32mx/lib\libc.a(_fputc_simple.o)

.text%z284      0x00000000        0x0
 .text          0x00000000        0x0 c:/program files/microchip/xc32/v1.33/bin/bin/../../lib/gcc/pic32mx/4.5.2/../../../../pic32mx/lib\libc.a(_iob.o)

.text%z285      0x00000000        0x0
 .text          0x00000000        0x0 c:/program files/microchip/xc32/v1.33/bin/bin/../../lib/gcc/pic32mx/4.5.2/../../../../pic32mx/lib\libc.a(sscanf_s.eo)

.text%z286      0x00000000        0x0
 .text          0x00000000        0x0 c:/program files/microchip/xc32/v1.33/bin/bin/../../lib/gcc/pic32mx/4.5.2/../../../../pic32mx/lib\libc.a(sprintf_cdnopuxX.eo)

.text%z287      0x00000000        0x0
 .text          0x00000000        0x0 c:/program files/microchip/xc32/v1.33/bin/bin/../../lib/gcc/pic32mx/4.5.2/../../../../pic32mx/lib\libc.a(printf_cdnopsuxX.eo)

.text%z288      0x00000000        0x0
 .text          0x00000000        0x0 c:/program files/microchip/xc32/v1.33/bin/bin/../../lib/gcc/pic32mx/4.5.2/../../../../pic32mx/lib\libc.a(strncmp.o)

.text%z289      0x00000000        0x0
 .text          0x00000000        0x0 c:/program files/microchip/xc32/v1.33/bin/bin/../../lib/gcc/pic32mx/4.5.2/../../../../pic32mx/lib\libc.a(puts.o)

.text%z290      0x00000000        0x0
 .text          0x00000000        0x0 c:/program files/microchip/xc32/v1.33/bin/bin/../../lib/gcc/pic32mx/4.5.2/../../../../pic32mx/lib\libpic32.a(defaultinterrupt.o)

.text%z291      0x00000000        0x0
 .text          0x00000000        0x0 c:/program files/microchip/xc32/v1.33/bin/bin/../../lib/gcc/pic32mx/4.5.2/../../../../pic32mx/lib\libpic32.a(vector63.o)

.text%z292      0x00000000        0x0
 .text          0x00000000        0x0 c:/program files/microchip/xc32/v1.33/bin/bin/../../lib/gcc/pic32mx/4.5.2/../../../../pic32mx/lib\libpic32.a(vector62.o)

.text%z293      0x00000000        0x0
 .text          0x00000000        0x0 c:/program files/microchip/xc32/v1.33/bin/bin/../../lib/gcc/pic32mx/4.5.2/../../../../pic32mx/lib\libpic32.a(vector61.o)

.text%z294      0x00000000        0x0
 .text          0x00000000        0x0 c:/program files/microchip/xc32/v1.33/bin/bin/../../lib/gcc/pic32mx/4.5.2/../../../../pic32mx/lib\libpic32.a(vector60.o)

.text%z295      0x00000000        0x0
 .text          0x00000000        0x0 c:/program files/microchip/xc32/v1.33/bin/bin/../../lib/gcc/pic32mx/4.5.2/../../../../pic32mx/lib\libpic32.a(vector59.o)

.text%z296      0x00000000        0x0
 .text          0x00000000        0x0 c:/program files/microchip/xc32/v1.33/bin/bin/../../lib/gcc/pic32mx/4.5.2/../../../../pic32mx/lib\libpic32.a(vector58.o)

.text%z297      0x00000000        0x0
 .text          0x00000000        0x0 c:/program files/microchip/xc32/v1.33/bin/bin/../../lib/gcc/pic32mx/4.5.2/../../../../pic32mx/lib\libpic32.a(vector57.o)

.text%z298      0x00000000        0x0
 .text          0x00000000        0x0 c:/program files/microchip/xc32/v1.33/bin/bin/../../lib/gcc/pic32mx/4.5.2/../../../../pic32mx/lib\libpic32.a(vector56.o)

.text%z299      0x00000000        0x0
 .text          0x00000000        0x0 c:/program files/microchip/xc32/v1.33/bin/bin/../../lib/gcc/pic32mx/4.5.2/../../../../pic32mx/lib\libpic32.a(vector55.o)

.text%z300      0x00000000        0x0
 .text          0x00000000        0x0 c:/program files/microchip/xc32/v1.33/bin/bin/../../lib/gcc/pic32mx/4.5.2/../../../../pic32mx/lib\libpic32.a(vector54.o)

.text%z301      0x00000000        0x0
 .text          0x00000000        0x0 c:/program files/microchip/xc32/v1.33/bin/bin/../../lib/gcc/pic32mx/4.5.2/../../../../pic32mx/lib\libpic32.a(vector53.o)

.text%z302      0x00000000        0x0
 .text          0x00000000        0x0 c:/program files/microchip/xc32/v1.33/bin/bin/../../lib/gcc/pic32mx/4.5.2/../../../../pic32mx/lib\libpic32.a(vector52.o)

.text%z303      0x00000000        0x0
 .text          0x00000000        0x0 c:/program files/microchip/xc32/v1.33/bin/bin/../../lib/gcc/pic32mx/4.5.2/../../../../pic32mx/lib\libpic32.a(vector51.o)

.text%z304      0x00000000        0x0
 .text          0x00000000        0x0 c:/program files/microchip/xc32/v1.33/bin/bin/../../lib/gcc/pic32mx/4.5.2/../../../../pic32mx/lib\libpic32.a(vector50.o)

.text%z305      0x00000000        0x0
 .text          0x00000000        0x0 c:/program files/microchip/xc32/v1.33/bin/bin/../../lib/gcc/pic32mx/4.5.2/../../../../pic32mx/lib\libpic32.a(vector49.o)

.text%z306      0x00000000        0x0
 .text          0x00000000        0x0 c:/program files/microchip/xc32/v1.33/bin/bin/../../lib/gcc/pic32mx/4.5.2/../../../../pic32mx/lib\libpic32.a(vector48.o)

.text%z307      0x00000000        0x0
 .text          0x00000000        0x0 c:/program files/microchip/xc32/v1.33/bin/bin/../../lib/gcc/pic32mx/4.5.2/../../../../pic32mx/lib\libpic32.a(vector47.o)

.text%z308      0x00000000        0x0
 .text          0x00000000        0x0 c:/program files/microchip/xc32/v1.33/bin/bin/../../lib/gcc/pic32mx/4.5.2/../../../../pic32mx/lib\libpic32.a(vector46.o)

.text%z309      0x00000000        0x0
 .text          0x00000000        0x0 c:/program files/microchip/xc32/v1.33/bin/bin/../../lib/gcc/pic32mx/4.5.2/../../../../pic32mx/lib\libpic32.a(vector45.o)

.text%z310      0x00000000        0x0
 .text          0x00000000        0x0 c:/program files/microchip/xc32/v1.33/bin/bin/../../lib/gcc/pic32mx/4.5.2/../../../../pic32mx/lib\libpic32.a(vector44.o)

.text%z311      0x00000000        0x0
 .text          0x00000000        0x0 c:/program files/microchip/xc32/v1.33/bin/bin/../../lib/gcc/pic32mx/4.5.2/../../../../pic32mx/lib\libpic32.a(vector43.o)

.text%z312      0x00000000        0x0
 .text          0x00000000        0x0 c:/program files/microchip/xc32/v1.33/bin/bin/../../lib/gcc/pic32mx/4.5.2/../../../../pic32mx/lib\libpic32.a(vector42.o)

.text%z313      0x00000000        0x0
 .text          0x00000000        0x0 c:/program files/microchip/xc32/v1.33/bin/bin/../../lib/gcc/pic32mx/4.5.2/../../../../pic32mx/lib\libpic32.a(vector41.o)

.text%z314      0x00000000        0x0
 .text          0x00000000        0x0 c:/program files/microchip/xc32/v1.33/bin/bin/../../lib/gcc/pic32mx/4.5.2/../../../../pic32mx/lib\libpic32.a(vector40.o)

.text%z315      0x00000000        0x0
 .text          0x00000000        0x0 c:/program files/microchip/xc32/v1.33/bin/bin/../../lib/gcc/pic32mx/4.5.2/../../../../pic32mx/lib\libpic32.a(vector39.o)

.text%z316      0x00000000        0x0
 .text          0x00000000        0x0 c:/program files/microchip/xc32/v1.33/bin/bin/../../lib/gcc/pic32mx/4.5.2/../../../../pic32mx/lib\libpic32.a(vector38.o)

.text%z317      0x00000000        0x0
 .text          0x00000000        0x0 c:/program files/microchip/xc32/v1.33/bin/bin/../../lib/gcc/pic32mx/4.5.2/../../../../pic32mx/lib\libpic32.a(vector37.o)

.text%z318      0x00000000        0x0
 .text          0x00000000        0x0 c:/program files/microchip/xc32/v1.33/bin/bin/../../lib/gcc/pic32mx/4.5.2/../../../../pic32mx/lib\libpic32.a(vector36.o)

.text%z319      0x00000000        0x0
 .text          0x00000000        0x0 c:/program files/microchip/xc32/v1.33/bin/bin/../../lib/gcc/pic32mx/4.5.2/../../../../pic32mx/lib\libpic32.a(vector35.o)

.text%z320      0x00000000        0x0
 .text          0x00000000        0x0 c:/program files/microchip/xc32/v1.33/bin/bin/../../lib/gcc/pic32mx/4.5.2/../../../../pic32mx/lib\libpic32.a(vector34.o)

.text%z321      0x00000000        0x0
 .text          0x00000000        0x0 c:/program files/microchip/xc32/v1.33/bin/bin/../../lib/gcc/pic32mx/4.5.2/../../../../pic32mx/lib\libpic32.a(vector33.o)

.text%z322      0x00000000        0x0
 .text          0x00000000        0x0 c:/program files/microchip/xc32/v1.33/bin/bin/../../lib/gcc/pic32mx/4.5.2/../../../../pic32mx/lib\libpic32.a(vector32.o)

.text%z323      0x00000000        0x0
 .text          0x00000000        0x0 c:/program files/microchip/xc32/v1.33/bin/bin/../../lib/gcc/pic32mx/4.5.2/../../../../pic32mx/lib\libpic32.a(vector31.o)

.text%z324      0x00000000        0x0
 .text          0x00000000        0x0 c:/program files/microchip/xc32/v1.33/bin/bin/../../lib/gcc/pic32mx/4.5.2/../../../../pic32mx/lib\libpic32.a(vector30.o)

.text%z325      0x00000000        0x0
 .text          0x00000000        0x0 c:/program files/microchip/xc32/v1.33/bin/bin/../../lib/gcc/pic32mx/4.5.2/../../../../pic32mx/lib\libpic32.a(vector29.o)

.text%z326      0x00000000        0x0
 .text          0x00000000        0x0 c:/program files/microchip/xc32/v1.33/bin/bin/../../lib/gcc/pic32mx/4.5.2/../../../../pic32mx/lib\libpic32.a(vector28.o)

.text%z327      0x00000000        0x0
 .text          0x00000000        0x0 c:/program files/microchip/xc32/v1.33/bin/bin/../../lib/gcc/pic32mx/4.5.2/../../../../pic32mx/lib\libpic32.a(vector27.o)

.text%z328      0x00000000        0x0
 .text          0x00000000        0x0 c:/program files/microchip/xc32/v1.33/bin/bin/../../lib/gcc/pic32mx/4.5.2/../../../../pic32mx/lib\libpic32.a(vector26.o)

.text%z329      0x00000000        0x0
 .text          0x00000000        0x0 c:/program files/microchip/xc32/v1.33/bin/bin/../../lib/gcc/pic32mx/4.5.2/../../../../pic32mx/lib\libpic32.a(vector25.o)

.text%z330      0x00000000        0x0
 .text          0x00000000        0x0 c:/program files/microchip/xc32/v1.33/bin/bin/../../lib/gcc/pic32mx/4.5.2/../../../../pic32mx/lib\libpic32.a(vector24.o)

.text%z331      0x00000000        0x0
 .text          0x00000000        0x0 c:/program files/microchip/xc32/v1.33/bin/bin/../../lib/gcc/pic32mx/4.5.2/../../../../pic32mx/lib\libpic32.a(vector23.o)

.text%z332      0x00000000        0x0
 .text          0x00000000        0x0 c:/program files/microchip/xc32/v1.33/bin/bin/../../lib/gcc/pic32mx/4.5.2/../../../../pic32mx/lib\libpic32.a(vector22.o)

.text%z333      0x00000000        0x0
 .text          0x00000000        0x0 c:/program files/microchip/xc32/v1.33/bin/bin/../../lib/gcc/pic32mx/4.5.2/../../../../pic32mx/lib\libpic32.a(vector21.o)

.text%z334      0x00000000        0x0
 .text          0x00000000        0x0 c:/program files/microchip/xc32/v1.33/bin/bin/../../lib/gcc/pic32mx/4.5.2/../../../../pic32mx/lib\libpic32.a(vector20.o)

.text%z335      0x00000000        0x0
 .text          0x00000000        0x0 c:/program files/microchip/xc32/v1.33/bin/bin/../../lib/gcc/pic32mx/4.5.2/../../../../pic32mx/lib\libpic32.a(vector19.o)

.text%z336      0x00000000        0x0
 .text          0x00000000        0x0 c:/program files/microchip/xc32/v1.33/bin/bin/../../lib/gcc/pic32mx/4.5.2/../../../../pic32mx/lib\libpic32.a(vector18.o)

.text%z337      0x00000000        0x0
 .text          0x00000000        0x0 c:/program files/microchip/xc32/v1.33/bin/bin/../../lib/gcc/pic32mx/4.5.2/../../../../pic32mx/lib\libpic32.a(vector17.o)

.text%z338      0x00000000        0x0
 .text          0x00000000        0x0 c:/program files/microchip/xc32/v1.33/bin/bin/../../lib/gcc/pic32mx/4.5.2/../../../../pic32mx/lib\libpic32.a(vector16.o)

.text%z339      0x00000000        0x0
 .text          0x00000000        0x0 c:/program files/microchip/xc32/v1.33/bin/bin/../../lib/gcc/pic32mx/4.5.2/../../../../pic32mx/lib\libpic32.a(vector14.o)

.text%z340      0x00000000        0x0
 .text          0x00000000        0x0 c:/program files/microchip/xc32/v1.33/bin/bin/../../lib/gcc/pic32mx/4.5.2/../../../../pic32mx/lib\libpic32.a(vector13.o)

.text%z341      0x00000000        0x0
 .text          0x00000000        0x0 c:/program files/microchip/xc32/v1.33/bin/bin/../../lib/gcc/pic32mx/4.5.2/../../../../pic32mx/lib\libpic32.a(vector12.o)

.text%z342      0x00000000        0x0
 .text          0x00000000        0x0 c:/program files/microchip/xc32/v1.33/bin/bin/../../lib/gcc/pic32mx/4.5.2/../../../../pic32mx/lib\libpic32.a(vector11.o)

.text%z343      0x00000000        0x0
 .text          0x00000000        0x0 c:/program files/microchip/xc32/v1.33/bin/bin/../../lib/gcc/pic32mx/4.5.2/../../../../pic32mx/lib\libpic32.a(vector10.o)

.text%z344      0x00000000        0x0
 .text          0x00000000        0x0 c:/program files/microchip/xc32/v1.33/bin/bin/../../lib/gcc/pic32mx/4.5.2/../../../../pic32mx/lib\libpic32.a(vector9.o)

.text%z345      0x00000000        0x0
 .text          0x00000000        0x0 c:/program files/microchip/xc32/v1.33/bin/bin/../../lib/gcc/pic32mx/4.5.2/../../../../pic32mx/lib\libpic32.a(vector8.o)

.text%z346      0x00000000        0x0
 .text          0x00000000        0x0 c:/program files/microchip/xc32/v1.33/bin/bin/../../lib/gcc/pic32mx/4.5.2/../../../../pic32mx/lib\libpic32.a(vector6.o)

.text%z347      0x00000000        0x0
 .text          0x00000000        0x0 c:/program files/microchip/xc32/v1.33/bin/bin/../../lib/gcc/pic32mx/4.5.2/../../../../pic32mx/lib\libpic32.a(vector5.o)

.text%z348      0x00000000        0x0
 .text          0x00000000        0x0 c:/program files/microchip/xc32/v1.33/bin/bin/../../lib/gcc/pic32mx/4.5.2/../../../../pic32mx/lib\libpic32.a(vector2.o)

.text%z349      0x00000000        0x0
 .text          0x00000000        0x0 c:/program files/microchip/xc32/v1.33/bin/bin/../../lib/gcc/pic32mx/4.5.2/../../../../pic32mx/lib\libpic32.a(vector1.o)

.text%z350      0x00000000        0x0
 .text          0x00000000        0x0 c:/program files/microchip/xc32/v1.33/bin/bin/../../lib/gcc/pic32mx/4.5.2/../../../../pic32mx/lib\libpic32.a(vector0.o)

.text%z351      0x00000000        0x0
 .text          0x00000000        0x0 c:/program files/microchip/xc32/v1.33/bin/bin/../../lib/gcc/pic32mx/4.5.2/../../../../pic32mx/lib\libpic32.a(general-exception.o)

.text%z352      0x00000000        0x0
 .text          0x00000000        0x0 c:/program files/microchip/xc32/v1.33/bin/bin/../../lib/gcc/pic32mx/4.5.2/../../../../pic32mx/lib\libpic32.a(close.o)

.text%z353      0x00000000        0x0
 .text          0x00000000        0x0 c:/program files/microchip/xc32/v1.33/bin/bin/../../lib/gcc/pic32mx/4.5.2/../../../../pic32mx/lib\libpic32.a(default-on-bootstrap.o)

.text%z354      0x00000000        0x0
 .text          0x00000000        0x0 c:/program files/microchip/xc32/v1.33/bin/bin/../../lib/gcc/pic32mx/4.5.2/../../../../pic32mx/lib\libpic32.a(default-on-reset.o)

.text%z355      0x00000000        0x0
 .text          0x00000000        0x0 c:/program files/microchip/xc32/v1.33/bin/bin/../../lib/gcc/pic32mx/4.5.2/../../../../pic32mx/lib\libpic32.a(default-bootstrap-exception-handler.o)

.text%z356      0x00000000        0x0
 .text          0x00000000        0x0 c:/program files/microchip/xc32/v1.33/bin/bin/../../lib/gcc/pic32mx/4.5.2/../../../../pic32mx/lib/./proc/32MX795F512H\default_isr_vectors.o

.text%z357      0x00000000        0x0
 .text          0x00000000        0x0 c:/program files/microchip/xc32/v1.33/bin/bin/../../lib/gcc/pic32mx/4.5.2/../../../../pic32mx/lib\libmchp_peripheral_32MX795F512H.a(int_restore_interrupts_lib.o)

.text%z358      0x00000000        0x0
 .text          0x00000000        0x0 c:/program files/microchip/xc32/v1.33/bin/bin/../../lib/gcc/pic32mx/4.5.2/../../../../pic32mx/lib\libmchp_peripheral_32MX795F512H.a(int_disable_interrupts_lib.o)

.text%z359      0x00000000        0x0
 .text          0x00000000        0x0 c:/program files/microchip/xc32/v1.33/bin/bin/../../lib/gcc/pic32mx/4.5.2/../../../../pic32mx/lib\libmchp_peripheral_32MX795F512H.a(int_enable_interrupts_lib.o)

.text%z360      0x00000000        0x0
 .text          0x00000000        0x0 c:/program files/microchip/xc32/v1.33/bin/bin/../../lib/gcc/pic32mx/4.5.2/../../../../pic32mx/lib\libmchp_peripheral_32MX795F512H.a(int_configure_system_lib.o)

.text%z361      0x00000000        0x0
 .text          0x00000000        0x0 c:/program files/microchip/xc32/v1.33/bin/bin/../../lib/gcc/pic32mx/4.5.2/../../../../pic32mx/lib\libmchp_peripheral_32MX795F512H.a(pcache.o)

.text%z362      0x00000000        0x0
 .text          0x00000000        0x0 c:/program files/microchip/xc32/v1.33/bin/bin/../../lib/gcc/pic32mx/4.5.2/../../../../pic32mx/lib\libmchp_peripheral_32MX795F512H.a(soft_reset_lib.o)

.text%z363      0x00000000        0x0
 .text          0x00000000        0x0 c:/program files/microchip/xc32/v1.33/bin/bin/../../lib/gcc/pic32mx/4.5.2/../../../../pic32mx/lib/./proc/32MX795F512H\processor.o

.text%z364      0x00000000        0x0
 .text          0x00000000        0x0 build/ChaletDuinoV2_795F512H_/debug/Source/template.o

.text%z365      0x00000000        0x0
 .text          0x00000000        0x0 build/ChaletDuinoV2_795F512H_/debug/Source/system.o

.text%z366      0x00000000        0x0
 .text          0x00000000        0x0 build/ChaletDuinoV2_795F512H_/debug/Source/interrupts.o

.text%z367      0x00000000        0x0
 .text          0x00000000        0x0 c:/program files/microchip/xc32/v1.33/bin/bin/../../lib/gcc/pic32mx/4.5.2/../../../../pic32mx/lib\software-debug-break.o

.text%z368      0x00000000        0x0
 .text          0x00000000        0x0 c:/program files/microchip/xc32/v1.33/bin/bin/../../lib/gcc/pic32mx/4.5.2/../../../../pic32mx/lib/./proc/32MX795F512H/crt0_mips32r2.o
